 Effect_p

 Timestamp is 56cd4c28 (Wed Feb 24 15:22:32 2016)

 Preferred load address is 10000000

 Start         Length     Name                   Class
 0001:00000000 00042782H .text                   CODE
 0001:00042790 00001486H .text$x                 CODE
 0001:00043c20 000000ccH .text$yc                CODE
 0001:00043cf0 0000007aH .text$yd                CODE
 0002:00000000 000001a4H .idata$5                DATA
 0002:000001a4 00000004H .CRT$XCA                DATA
 0002:000001a8 00000020H .CRT$XCU                DATA
 0002:000001c8 00000004H .CRT$XCZ                DATA
 0002:000001cc 00000004H .CRT$XIA                DATA
 0002:000001d0 00000014H .CRT$XIC                DATA
 0002:000001e4 00000004H .CRT$XIZ                DATA
 0002:000001e8 00000004H .CRT$XPA                DATA
 0002:000001ec 00000004H .CRT$XPX                DATA
 0002:000001f0 00000004H .CRT$XPXA               DATA
 0002:000001f4 00000004H .CRT$XPZ                DATA
 0002:000001f8 00000004H .CRT$XTA                DATA
 0002:000001fc 00000004H .CRT$XTZ                DATA
 0002:00000200 00007828H .rdata                  DATA
 0002:00007a28 0000006cH .rdata$debug            DATA
 0002:00007a94 00000718H .rdata$r                DATA
 0002:000081b0 00000198H .rdata$sxdata           DATA
 0002:00008348 00000004H .rtc$IAA                DATA
 0002:0000834c 00000004H .rtc$IZZ                DATA
 0002:00008350 00000004H .rtc$TAA                DATA
 0002:00008354 00000004H .rtc$TZZ                DATA
 0002:00008358 00001f88H .xdata$x                DATA
 0002:0000a2e0 0000003cH .idata$2                DATA
 0002:0000a31c 00000014H .idata$3                DATA
 0002:0000a330 000001a4H .idata$4                DATA
 0002:0000a4d4 00000814H .idata$6                DATA
 0002:0000acf0 00000b9dH .edata                  DATA
 0003:00000000 00001a10H .data                   DATA
 0003:00001a20 00004120H .bss                    DATA
 0004:00000000 00000058H .rsrc$01                DATA
 0004:00000060 000002f0H .rsrc$02                DATA

  Address         Publics by Value              Rva+Base       Lib:Object

 0000:00000000       __except_list              00000000     <absolute>
 0000:00000066       ___safe_se_handler_count   00000066     <absolute>
 0000:00000000       ___ImageBase               10000000     <linker-defined>
 0001:00000000       ?GetEffectBodyMap@CEffectManager@@QAEAAV?$hash_map@PAXPAVCEffectBody@@V?$hash_compare@PAXU?$less@PAX@std@@@stdext@@V?$allocator@U?$pair@QAXPAVCEffectBody@@@std@@@std@@@stdext@@XZ 10001000 f i dllaccess.obj
 0001:00000011       ?DeleteEleInfo@CEffectManager@@QAEXPAUSt_Ele_Node@@@Z 10001011 f i dllaccess.obj
 0001:00000036       ?CreateEffect@CEffectManager@@QAEPAXKABUWzVector@@H@Z 10001036 f i dllaccess.obj
 0001:0000005c       ?CreateEffect@CEffectManager@@QAEPAXKABUWzVector@@0H@Z 1000105c f i dllaccess.obj
 0001:00000080       ?SetRenderEffect@CEffectManager@@QAEX_N@Z 10001080 f i dllaccess.obj
 0001:00000097       ?IsRenderEffect@CEffectManager@@QAE_NXZ 10001097 f i dllaccess.obj
 0001:000000a9       _Func_ContactEffect        100010a9 f   dllaccess.obj
 0001:0000015d       _DllMain@12                1000115d f   dllentry.obj
 0001:00000191       ??0CEffectManager@@QAE@XZ  10001191 f   effectmanager.obj
 0001:00000332       ??1CEffectManager@@UAE@XZ  10001332 f   effectmanager.obj
 0001:000004dd       ?Create@CEffectManager@@QAE_NPAVCDrawBase@@PAVCWorldBase@@@Z 100014dd f   effectmanager.obj
 0001:00000616       ?Destroy@CEffectManager@@QAEXXZ 10001616 f   effectmanager.obj
 0001:00000759       ?GetEffectTexture@CEffectManager@@QAEPAXK@Z 10001759 f   effectmanager.obj
 0001:0000087e       ?ReleaseEffectTexture@CEffectManager@@QAEXXZ 1000187e f   effectmanager.obj
 0001:00000b74       ?LoadTextureFiles@CEffectManager@@QAE_NPBD0W4EENUM_LOAD_TYPE@@@Z 10001b74 f   effectmanager.obj
 0001:00000e22       ?RemoveTextureFiles@CEffectManager@@AAEXXZ 10001e22 f   effectmanager.obj
 0001:00000ea4       ?LoadMeshFiles@CEffectManager@@QAE_NPBD0W4EENUM_LOAD_TYPE@@@Z 10001ea4 f   effectmanager.obj
 0001:0000111b       ?RemoveMeshFiles@CEffectManager@@AAEXXZ 1000211b f   effectmanager.obj
 0001:000011bc       ?RegisterEffectInfo@CEffectManager@@QAEXPBUSt_BodyCreate@@@Z 100021bc f   effectmanager.obj
 0001:00001229       ?AddEffectInfo@CEffectManager@@QAE_NK@Z 10002229 f   effectmanager.obj
 0001:000012e3       ?GetEffectInfo@CEffectManager@@QAEPAUSt_BodyCreate@@K@Z 100022e3 f   effectmanager.obj
 0001:00001344       ?ReleaseAllEffectInfo@CEffectManager@@QAEXXZ 10002344 f   effectmanager.obj
 0001:000013fe       ?ReleaseAtEffectInfo@CEffectManager@@QAEXK@Z 100023fe f   effectmanager.obj
 0001:0000156a       ?CreateEffect@CEffectManager@@QAEPAXKABUWzVector@@00H@Z 1000256a f   effectmanager.obj
 0001:000018e3       ?CreateElement@CEffectManager@@AAE_NPAVCEffectBody@@PBUSt_BodyCreate@@H@Z 100028e3 f   effectmanager.obj
 0001:00001ad8       ?CreateSelectedElements@CEffectManager@@QAEPAXKABUWzVector@@PAV?$list@HV?$allocator@H@std@@@std@@@Z 10002ad8 f   effectmanager.obj
 0001:00001f78       ?GetEffectPtrHandle@CEffectManager@@QAEPAVCEffectBody@@PAX@Z 10002f78 f   effectmanager.obj
 0001:00001fdf       ?DestroyAllEffect@CEffectManager@@QAEXXZ 10002fdf f   effectmanager.obj
 0001:0000209f       ?RemoveEffectPtr@CEffectManager@@QAEXPAX@Z 1000309f f   effectmanager.obj
 0001:00002182       ?Move@CEffectManager@@QAEXK@Z 10003182 f   effectmanager.obj
 0001:00002739       ?Render@CEffectManager@@QAEXXZ 10003739 f   effectmanager.obj
 0001:00002833       ?ShrinkMemoryPool@CEffectManager@@QAEXXZ 10003833 f   effectmanager.obj
 0001:00002850       ?ClearSoundInfos@CEffectManager@@QAEXXZ 10003850 f   effectmanager.obj
 0001:0000286e       ?AdjustCreateEffectLevel@CEffectManager@@AAEXXZ 1000386e f   effectmanager.obj
 0001:0000294e       ?AdjustEffectRate@CEffectManager@@AAEXXZ 1000394e f   effectmanager.obj
 0001:00002a29       ?ClearAutoLvlCtlParams@CEffectManager@@QAEXXZ 10003a29 f   effectmanager.obj
 0001:00002a42       ?AddAutoLvlCtlParam@CEffectManager@@QAEXHH@Z 10003a42 f   effectmanager.obj
 0001:00002b44       ?ClearAutoRateCtlParams@CEffectManager@@QAEXXZ 10003b44 f   effectmanager.obj
 0001:00002b5d       ?AddAutoRateCtlParam@CEffectManager@@QAEXHH@Z 10003b5d f   effectmanager.obj
 0001:00002c5f       ?ClearEffectLODParams@CEffectManager@@QAEXXZ 10003c5f f   effectmanager.obj
 0001:00002c78       ?AddEffectLODParam@CEffectManager@@QAEXMH@Z 10003c78 f   effectmanager.obj
 0001:00002d5d       ?Initialize@CEffectManager@@AAEXXZ 10003d5d f   effectmanager.obj
 0001:00002f87       ??_GCEffectManager@@UAEPAXI@Z 10003f87 f i effectmanager.obj
 0001:00002f87       ??_ECEffectManager@@UAEPAXI@Z 10003f87 f i effectmanager.obj
 0001:00002fae       ??1?$hash_map@PAXPAVCEffectBody@@V?$hash_compare@PAXU?$less@PAX@std@@@stdext@@V?$allocator@U?$pair@QAXPAVCEffectBody@@@std@@@std@@@stdext@@QAE@XZ 10003fae f i effectmanager.obj
 0001:00002fae       ??1?$hash_map@KPAUSt_BodyCreate@@V?$hash_compare@KU?$less@K@std@@@stdext@@V?$allocator@U?$pair@$$CBKPAUSt_BodyCreate@@@std@@@std@@@stdext@@QAE@XZ 10003fae f i effectmanager.obj
 0001:00002fc1       ?Create@CSoundInfoManager@@QAE_NXZ 10003fc1 f i effectmanager.obj
 0001:0000306a       ?Destroy@CSoundInfoManager@@QAEXXZ 1000406a f i effectmanager.obj
 0001:000030d8       ?Initialize@CSoundInfoManager@@QAEXXZ 100040d8 f i effectmanager.obj
 0001:0000313b       ??4St_BodyCreate@@QAEAAU0@ABU0@@Z 1000413b f i effectmanager.obj
 0001:000037d8       ??0St_Create_Info@@QAE@XZ  100047d8 f i effectmanager.obj
 0001:000038a9       ?Initialize@St_Create_Info@@QAEXXZ 100048a9 f i effectmanager.obj
 0001:00003a1d       ??4St_Create_Info@@QAEAAU0@ABU0@@Z 10004a1d f i effectmanager.obj
 0001:00003c3d       ??1?$map@JUWzVector@@U?$less@J@std@@V?$allocator@U?$pair@$$CBJUWzVector@@@std@@@3@@std@@QAE@XZ 10004c3d f i effectmanager.obj
 0001:00003c92       ??0St_Move_Info@@QAE@XZ    10004c92 f i effectmanager.obj
 0001:00003d97       ?Initialize@St_Move_Info@@QAEXXZ 10004d97 f i effectmanager.obj
 0001:00003f6e       ??4St_Move_Info@@QAEAAU0@ABU0@@Z 10004f6e f i effectmanager.obj
 0001:00004185       ??0St_Change_Info@@QAE@XZ  10005185 f i effectmanager.obj
 0001:000043e7       ?Initialize@St_Change_Info@@QAEXXZ 100053e7 f i effectmanager.obj
 0001:000044d2       ?Release@St_Change_Info@@QAEXXZ 100054d2 f i effectmanager.obj
 0001:000045ae       ??4St_Change_Info@@QAEAAU0@ABU0@@Z 100055ae f i effectmanager.obj
 0001:00004921       ??1?$map@JMU?$less@J@std@@V?$allocator@U?$pair@$$CBJM@std@@@2@@std@@QAE@XZ 10005921 f i effectmanager.obj
 0001:00004976       ??0St_Visual_Info@@QAE@XZ  10005976 f i effectmanager.obj
 0001:000049a0       ?Initialize@St_Visual_Info@@QAEXXZ 100059a0 f i effectmanager.obj
 0001:00004b49       ??4St_Visual_Info@@QAEAAU0@ABU0@@Z 10005b49 f i effectmanager.obj
 0001:00004b6e       ?ReleaseAll@St_BodyCreate@@QAEXXZ 10005b6e f i effectmanager.obj
 0001:00004ff2       ?SetupAllElementCreates@St_BodyCreate@@QAEXXZ 10005ff2 f i effectmanager.obj
 0001:0000517d       ?CreateSpline@St_BodyCreate@@QAEXPAUSt_ElementCreate@@@Z 1000617d f i effectmanager.obj
 0001:00006ef6       ?DestroySpline@St_BodyCreate@@QAEXPAUSt_ElementCreate@@@Z 10007ef6 f i effectmanager.obj
 0001:000076ba       ??1St_Change_Info@@QAE@XZ  100086ba f i effectmanager.obj
 0001:00007a2c       ??1St_Move_Info@@QAE@XZ    10008a2c f i effectmanager.obj
 0001:00007ac0       ??1St_Create_Info@@QAE@XZ  10008ac0 f i effectmanager.obj
 0001:00007b54       ??HWzVector@@QBE?AU0@ABU0@@Z 10008b54 f i effectmanager.obj
 0001:00007b9c       ??GWzVector@@QBE?AU0@ABU0@@Z 10008b9c f i effectmanager.obj
 0001:00007be4       ??DWzVector@@QBE?AU0@M@Z   10008be4 f i effectmanager.obj
 0001:00007c24       ?VectorLength2@@YAMPBUWzVector@@@Z 10008c24 f i effectmanager.obj
 0001:00007c56       ?VectorDotProduct@@YAMPBUWzVector@@0@Z 10008c56 f i effectmanager.obj
 0001:00007c88       ?Outside_Frustum_AABB@@YAGPBUWzFrustum@@PBUBvAABB@@@Z 10008c88 f i effectmanager.obj
 0001:00007d89       ?Distance_Plane_Vertex@@YAMPBUWzPlane@@ABUWzVector@@@Z 10008d89 f i effectmanager.obj
 0001:00007dc1       ?ClearRenderInfo@St_EffDbgInfo@@QAEXXZ 10008dc1 f i effectmanager.obj
 0001:00007dfb       ?IncNumRenderedEffect@St_EffDbgInfo@@QAEXXZ 10008dfb f i effectmanager.obj
 0001:00007e2b       ??4?$_Tree@V?$_Tmap_traits@JUWzVector@@U?$less@J@std@@V?$allocator@U?$pair@$$CBJUWzVector@@@std@@@3@$0A@@std@@@std@@QAEAAV01@ABV01@@Z 10008e2b f i effectmanager.obj
 0001:00007ede       ?begin@?$_Tree@V?$_Tmap_traits@JUWzVector@@U?$less@J@std@@V?$allocator@U?$pair@$$CBJUWzVector@@@std@@@3@$0A@@std@@@std@@QAE?AViterator@12@XZ 10008ede f i effectmanager.obj
 0001:00007f27       ?clear@?$_Tree@V?$_Tmap_traits@JUWzVector@@U?$less@J@std@@V?$allocator@U?$pair@$$CBJUWzVector@@@std@@@3@$0A@@std@@@std@@QAEXXZ 10008f27 f i effectmanager.obj
 0001:00007f7c       ??0?$list@PAVCEElementSprite@@V?$allocator@PAVCEElementSprite@@@std@@@std@@QAE@XZ 10008f7c f i eelementweather.obj
 0001:00007f7c       ??0?$list@PAVCEElementBase@@V?$allocator@PAVCEElementBase@@@std@@@std@@QAE@XZ 10008f7c f i effectbody.obj
 0001:00007f7c       ??0?$list@KV?$allocator@K@std@@@std@@QAE@XZ 10008f7c f i effectmanager.obj
 0001:00007ff1       ??4?$list@KV?$allocator@K@std@@@std@@QAEAAV01@ABV01@@Z 10008ff1 f i effectmanager.obj
 0001:00008083       ??4?$_Tree@V?$_Tmap_traits@JMU?$less@J@std@@V?$allocator@U?$pair@$$CBJM@std@@@2@$0A@@std@@@std@@QAEAAV01@ABV01@@Z 10009083 f i effectmanager.obj
 0001:00008136       ?clear@?$_Tree@V?$_Tmap_traits@JMU?$less@J@std@@V?$allocator@U?$pair@$$CBJM@std@@@2@$0A@@std@@@std@@QAEXXZ 10009136 f i effectmanager.obj
 0001:0000818b       ??1?$vector@PAUsEffectTexture@CEffectManager@@V?$allocator@PAUsEffectTexture@CEffectManager@@@std@@@std@@QAE@XZ 1000918b f i effectmanager.obj
 0001:0000818b       ??1?$vector@PAXV?$allocator@PAX@std@@@std@@QAE@XZ 1000918b f i effectmanager.obj
 0001:000081e1       ?clear@?$vector@PAXV?$allocator@PAX@std@@@std@@QAEXXZ 100091e1 f i effectmanager.obj
 0001:000081e1       ?clear@?$vector@PAUsEffectTexture@CEffectManager@@V?$allocator@PAUsEffectTexture@CEffectManager@@@std@@@std@@QAEXXZ 100091e1 f i effectmanager.obj
 0001:000081e1       ?clear@?$vector@PAUSt_SoundInfo@@V?$allocator@PAUSt_SoundInfo@@@std@@@std@@QAEXXZ 100091e1 f i effectbody.obj
 0001:00008232       ??D?$_Vector_const_iterator@PAUSt_SoundInfo@@V?$allocator@PAUSt_SoundInfo@@@std@@@std@@QBEABQAUSt_SoundInfo@@XZ 10009232 f i effectbody.obj
 0001:00008232       ??D?$_Vector_const_iterator@USt_AutoCtlParam@@V?$allocator@USt_AutoCtlParam@@@std@@@std@@QBEABUSt_AutoCtlParam@@XZ 10009232 f i effectmanager.obj
 0001:00008232       ??D?$_Vector_const_iterator@PAXV?$allocator@PAX@std@@@std@@QBEABQAXXZ 10009232 f i effectmanager.obj
 0001:00008232       ??D?$_Vector_const_iterator@USt_EffLODParam@@V?$allocator@USt_EffLODParam@@@std@@@std@@QBEABUSt_EffLODParam@@XZ 10009232 f i effectmanager.obj
 0001:00008299       ??8?$_Vector_const_iterator@PAUsEffectTexture@CEffectManager@@V?$allocator@PAUsEffectTexture@CEffectManager@@@std@@@std@@QBE_NABV01@@Z 10009299 f i effectmanager.obj
 0001:00008299       ??8?$_Vector_const_iterator@U_List_position@?$_Hash@V?$_Hmap_traits@KPAUSt_BodyCreate@@V?$hash_compare@KU?$less@K@std@@@stdext@@V?$allocator@U?$pair@$$CBKPAUSt_BodyCreate@@@std@@@std@@$0A@@stdext@@@stdext@@V?$allocator@U_List_position@?$_Hash@V?$_Hmap_traits@KPAUSt_BodyCreate@@V?$hash_compare@KU?$less@K@std@@@stdext@@V?$allocator@U?$pair@$$CBKPAUSt_BodyCreate@@@std@@@std@@$0A@@stdext@@@stdext@@@std@@@std@@QBE_NABV01@@Z 10009299 f i effectmanager.obj
 0001:00008299       ??8?$_Vector_const_iterator@U_List_position@?$_Hash@V?$_Hmap_traits@KV?$basic_string@DU?$char_traits@D@std@@V?$allocator@D@2@@std@@V?$hash_compare@KU?$less@K@std@@@stdext@@V?$allocator@U?$pair@$$CBKV?$basic_string@DU?$char_traits@D@std@@V?$allocator@D@2@@std@@@std@@@2@$0A@@stdext@@@stdext@@V?$allocator@U_List_position@?$_Hash@V?$_Hmap_traits@KV?$basic_string@DU?$char_traits@D@std@@V?$allocator@D@2@@std@@V?$hash_compare@KU?$less@K@std@@@stdext@@V?$allocator@U?$pair@$$CBKV?$basic_string@DU?$char_traits@D@std@@V?$allocator@D@2@@std@@@std@@@2@$0A@@stdext@@@stdext@@@std@@@std@@QBE_NABV01@@Z 10009299 f i effectmanager.obj
 0001:00008299       ??8?$_Vector_const_iterator@USt_AutoCtlParam@@V?$allocator@USt_AutoCtlParam@@@std@@@std@@QBE_NABV01@@Z 10009299 f i effectmanager.obj
 0001:00008299       ??8const_iterator@?$_Tree@V?$_Tmap_traits@JUWzVector@@U?$less@J@std@@V?$allocator@U?$pair@$$CBJUWzVector@@@std@@@3@$0A@@std@@@std@@QBE_NABV012@@Z 10009299 f i effectmanager.obj
 0001:00008299       ??8?$_Vector_const_iterator@U_WZNCSPT@WzNaturalCubicSplineDyn@@V?$allocator@U_WZNCSPT@WzNaturalCubicSplineDyn@@@std@@@std@@QBE_NABV01@@Z 10009299 f i Common_p:wznaturalcubicsplinedyn.obj
 0001:00008299       ??8?$_Vector_const_iterator@PAUSt_SoundInfo@@V?$allocator@PAUSt_SoundInfo@@@std@@@std@@QBE_NABV01@@Z 10009299 f i effectbody.obj
 0001:00008299       ??8const_iterator@?$_Tree@V?$_Tmap_traits@JMU?$less@J@std@@V?$allocator@U?$pair@$$CBJM@std@@@2@$0A@@std@@@std@@QBE_NABV012@@Z 10009299 f i effectmanager.obj
 0001:00008299       ??8?$_Vector_const_iterator@U_List_position@?$_Hash@V?$_Hmap_traits@PAXPAVCEffectBody@@V?$hash_compare@PAXU?$less@PAX@std@@@stdext@@V?$allocator@U?$pair@QAXPAVCEffectBody@@@std@@@std@@$0A@@stdext@@@stdext@@V?$allocator@U_List_position@?$_Hash@V?$_Hmap_traits@PAXPAVCEffectBody@@V?$hash_compare@PAXU?$less@PAX@std@@@stdext@@V?$allocator@U?$pair@QAXPAVCEffectBody@@@std@@@std@@$0A@@stdext@@@stdext@@@std@@@std@@QBE_NABV01@@Z 10009299 f i effectmanager.obj
 0001:00008299       ??8?$_Vector_const_iterator@USt_EffLODParam@@V?$allocator@USt_EffLODParam@@@std@@@std@@QBE_NABV01@@Z 10009299 f i effectmanager.obj
 0001:00008299       ??8?$_Vector_const_iterator@PAXV?$allocator@PAX@std@@@std@@QBE_NABV01@@Z 10009299 f i effectmanager.obj
 0001:000082e6       ??1?$CWzSingleton@VCEffectManager@@@@UAE@XZ 100092e6 f i effectmanager.obj
 0001:000082ff       ??0?$vector@PAXV?$allocator@PAX@std@@@std@@QAE@XZ 100092ff f i effectmanager.obj
 0001:000082ff       ??0?$vector@PAUSt_SoundInfo@@V?$allocator@PAUSt_SoundInfo@@@std@@@std@@QAE@XZ 100092ff f i effectbody.obj
 0001:000082ff       ??0?$vector@PAUsEffectTexture@CEffectManager@@V?$allocator@PAUsEffectTexture@CEffectManager@@@std@@@std@@QAE@XZ 100092ff f i effectmanager.obj
 0001:00008381       ?end@?$_Hash@V?$_Hmap_traits@PAXPAVCEffectBody@@V?$hash_compare@PAXU?$less@PAX@std@@@stdext@@V?$allocator@U?$pair@QAXPAVCEffectBody@@@std@@@std@@$0A@@stdext@@@stdext@@QAE?AV?$_Iterator@$00@?$list@U?$pair@QAXPAVCEffectBody@@@std@@V?$allocator@U?$pair@QAXPAVCEffectBody@@@std@@@2@@std@@XZ 10009381 f i effectmanager.obj
 0001:00008381       ?end@?$_Hash@V?$_Hmap_traits@KV?$basic_string@DU?$char_traits@D@std@@V?$allocator@D@2@@std@@V?$hash_compare@KU?$less@K@std@@@stdext@@V?$allocator@U?$pair@$$CBKV?$basic_string@DU?$char_traits@D@std@@V?$allocator@D@2@@std@@@std@@@2@$0A@@stdext@@@stdext@@QAE?AV?$_Iterator@$00@?$list@U?$pair@$$CBKV?$basic_string@DU?$char_traits@D@std@@V?$allocator@D@2@@std@@@std@@V?$allocator@U?$pair@$$CBKV?$basic_string@DU?$char_traits@D@std@@V?$allocator@D@2@@std@@@std@@@2@@std@@XZ 10009381 f i effectmanager.obj
 0001:00008381       ?end@?$_Hash@V?$_Hmap_traits@KPAUSt_BodyCreate@@V?$hash_compare@KU?$less@K@std@@@stdext@@V?$allocator@U?$pair@$$CBKPAUSt_BodyCreate@@@std@@@std@@$0A@@stdext@@@stdext@@QAE?AV?$_Iterator@$00@?$list@U?$pair@$$CBKPAUSt_BodyCreate@@@std@@V?$allocator@U?$pair@$$CBKPAUSt_BodyCreate@@@std@@@2@@std@@XZ 10009381 f i effectmanager.obj
 0001:00008381       ?end@?$_Hash@V?$_Hmap_traits@KV?$basic_string@DU?$char_traits@D@std@@V?$allocator@D@2@@std@@V?$hash_compare@KU?$less@K@std@@@stdext@@V?$allocator@U?$pair@$$CBKV?$basic_string@DU?$char_traits@D@std@@V?$allocator@D@2@@std@@@std@@@2@$0A@@stdext@@@stdext@@QBE?AV?$_Const_iterator@$00@?$list@U?$pair@$$CBKV?$basic_string@DU?$char_traits@D@std@@V?$allocator@D@2@@std@@@std@@V?$allocator@U?$pair@$$CBKV?$basic_string@DU?$char_traits@D@std@@V?$allocator@D@2@@std@@@std@@@2@@std@@XZ 10009381 f i effectmanager.obj
 0001:000083d0       ??1?$_Hash@V?$_Hmap_traits@PAXPAVCEffectBody@@V?$hash_compare@PAXU?$less@PAX@std@@@stdext@@V?$allocator@U?$pair@QAXPAVCEffectBody@@@std@@@std@@$0A@@stdext@@@stdext@@QAE@XZ 100093d0 f i effectmanager.obj
 0001:000083d0       ??1?$_Hash@V?$_Hmap_traits@KPAUSt_BodyCreate@@V?$hash_compare@KU?$less@K@std@@@stdext@@V?$allocator@U?$pair@$$CBKPAUSt_BodyCreate@@@std@@@std@@$0A@@stdext@@@stdext@@QAE@XZ 100093d0 f i effectmanager.obj
 0001:00008468       ?erase@?$_Hash@V?$_Hmap_traits@PAXPAVCEffectBody@@V?$hash_compare@PAXU?$less@PAX@std@@@stdext@@V?$allocator@U?$pair@QAXPAVCEffectBody@@@std@@@std@@$0A@@stdext@@@stdext@@QAE?AV?$_Iterator@$00@?$list@U?$pair@QAXPAVCEffectBody@@@std@@V?$allocator@U?$pair@QAXPAVCEffectBody@@@std@@@2@@std@@V?$_Const_iterator@$00@45@@Z 10009468 f i effectmanager.obj
 0001:00008468       ?erase@?$_Hash@V?$_Hmap_traits@KPAUSt_BodyCreate@@V?$hash_compare@KU?$less@K@std@@@stdext@@V?$allocator@U?$pair@$$CBKPAUSt_BodyCreate@@@std@@@std@@$0A@@stdext@@@stdext@@QAE?AV?$_Iterator@$00@?$list@U?$pair@$$CBKPAUSt_BodyCreate@@@std@@V?$allocator@U?$pair@$$CBKPAUSt_BodyCreate@@@std@@@2@@std@@V?$_Const_iterator@$00@45@@Z 10009468 f i effectmanager.obj
 0001:000085af       ??1?$vector@U_List_position@?$_Hash@V?$_Hmap_traits@PAXPAVCEffectBody@@V?$hash_compare@PAXU?$less@PAX@std@@@stdext@@V?$allocator@U?$pair@QAXPAVCEffectBody@@@std@@@std@@$0A@@stdext@@@stdext@@V?$allocator@U_List_position@?$_Hash@V?$_Hmap_traits@PAXPAVCEffectBody@@V?$hash_compare@PAXU?$less@PAX@std@@@stdext@@V?$allocator@U?$pair@QAXPAVCEffectBody@@@std@@@std@@$0A@@stdext@@@stdext@@@std@@@std@@QAE@XZ 100095af f i effectmanager.obj
 0001:000085af       ??1?$vector@U_List_position@?$_Hash@V?$_Hmap_traits@KPAUSt_BodyCreate@@V?$hash_compare@KU?$less@K@std@@@stdext@@V?$allocator@U?$pair@$$CBKPAUSt_BodyCreate@@@std@@@std@@$0A@@stdext@@@stdext@@V?$allocator@U_List_position@?$_Hash@V?$_Hmap_traits@KPAUSt_BodyCreate@@V?$hash_compare@KU?$less@K@std@@@stdext@@V?$allocator@U?$pair@$$CBKPAUSt_BodyCreate@@@std@@@std@@$0A@@stdext@@@stdext@@@std@@@std@@QAE@XZ 100095af f i effectmanager.obj
 0001:000085af       ??1?$vector@U_WZNCSPT@WzNaturalCubicSplineDyn@@V?$allocator@U_WZNCSPT@WzNaturalCubicSplineDyn@@@std@@@std@@QAE@XZ 100095af f i Common_p:wznaturalcubicsplinedyn.obj
 0001:000085af       ??1?$vector@USt_EffLODParam@@V?$allocator@USt_EffLODParam@@@std@@@std@@QAE@XZ 100095af f i effectmanager.obj
 0001:000085af       ??1?$vector@USt_AutoCtlParam@@V?$allocator@USt_AutoCtlParam@@@std@@@std@@QAE@XZ 100095af f i effectmanager.obj
 0001:000085af       ??1?$vector@U_List_position@?$_Hash@V?$_Hmap_traits@KV?$basic_string@DU?$char_traits@D@std@@V?$allocator@D@2@@std@@V?$hash_compare@KU?$less@K@std@@@stdext@@V?$allocator@U?$pair@$$CBKV?$basic_string@DU?$char_traits@D@std@@V?$allocator@D@2@@std@@@std@@@2@$0A@@stdext@@@stdext@@V?$allocator@U_List_position@?$_Hash@V?$_Hmap_traits@KV?$basic_string@DU?$char_traits@D@std@@V?$allocator@D@2@@std@@V?$hash_compare@KU?$less@K@std@@@stdext@@V?$allocator@U?$pair@$$CBKV?$basic_string@DU?$char_traits@D@std@@V?$allocator@D@2@@std@@@std@@@2@$0A@@stdext@@@stdext@@@std@@@std@@QAE@XZ 100095af f i loadmanager.obj
 0001:00008605       ?clear@?$vector@USt_AutoCtlParam@@V?$allocator@USt_AutoCtlParam@@@std@@@std@@QAEXXZ 10009605 f i effectmanager.obj
 0001:00008605       ?clear@?$vector@USt_EffLODParam@@V?$allocator@USt_EffLODParam@@@std@@@std@@QAEXXZ 10009605 f i effectmanager.obj
 0001:00008605       ?clear@?$vector@U_WZNCSPT@WzNaturalCubicSplineDyn@@V?$allocator@U_WZNCSPT@WzNaturalCubicSplineDyn@@@std@@@std@@QAEXXZ 10009605 f i Common_p:wznaturalcubicsplinedyn.obj
 0001:00008656       ?end@?$vector@U_List_position@?$_Hash@V?$_Hmap_traits@PAXPAVCEffectBody@@V?$hash_compare@PAXU?$less@PAX@std@@@stdext@@V?$allocator@U?$pair@QAXPAVCEffectBody@@@std@@@std@@$0A@@stdext@@@stdext@@V?$allocator@U_List_position@?$_Hash@V?$_Hmap_traits@PAXPAVCEffectBody@@V?$hash_compare@PAXU?$less@PAX@std@@@stdext@@V?$allocator@U?$pair@QAXPAVCEffectBody@@@std@@@std@@$0A@@stdext@@@stdext@@@std@@@std@@QAE?AV?$_Vector_iterator@U_List_position@?$_Hash@V?$_Hmap_traits@PAXPAVCEffectBody@@V?$hash_compare@PAXU?$less@PAX@std@@@stdext@@V?$allocator@U?$pair@QAXPAVCEffectBody@@@std@@@std@@$0A@@stdext@@@stdext@@V?$allocator@U_List_position@?$_Hash@V?$_Hmap_traits@PAXPAVCEffectBody@@V?$hash_compare@PAXU?$less@PAX@std@@@stdext@@V?$allocator@U?$pair@QAXPAVCEffectBody@@@std@@@std@@$0A@@stdext@@@stdext@@@std@@@2@XZ 10009656 f i effectmanager.obj
 0001:00008656       ?end@?$vector@PAUSt_SoundInfo@@V?$allocator@PAUSt_SoundInfo@@@std@@@std@@QAE?AV?$_Vector_iterator@PAUSt_SoundInfo@@V?$allocator@PAUSt_SoundInfo@@@std@@@2@XZ 10009656 f i effectbody.obj
 0001:00008656       ?end@?$vector@U_WZNCSPT@WzNaturalCubicSplineDyn@@V?$allocator@U_WZNCSPT@WzNaturalCubicSplineDyn@@@std@@@std@@QAE?AV?$_Vector_iterator@U_WZNCSPT@WzNaturalCubicSplineDyn@@V?$allocator@U_WZNCSPT@WzNaturalCubicSplineDyn@@@std@@@2@XZ 10009656 f i Common_p:wznaturalcubicsplinedyn.obj
 0001:00008656       ?end@?$vector@USt_AutoCtlParam@@V?$allocator@USt_AutoCtlParam@@@std@@@std@@QAE?AV?$_Vector_iterator@USt_AutoCtlParam@@V?$allocator@USt_AutoCtlParam@@@std@@@2@XZ 10009656 f i effectmanager.obj
 0001:00008656       ?end@?$vector@U_List_position@?$_Hash@V?$_Hmap_traits@KV?$basic_string@DU?$char_traits@D@std@@V?$allocator@D@2@@std@@V?$hash_compare@KU?$less@K@std@@@stdext@@V?$allocator@U?$pair@$$CBKV?$basic_string@DU?$char_traits@D@std@@V?$allocator@D@2@@std@@@std@@@2@$0A@@stdext@@@stdext@@V?$allocator@U_List_position@?$_Hash@V?$_Hmap_traits@KV?$basic_string@DU?$char_traits@D@std@@V?$allocator@D@2@@std@@V?$hash_compare@KU?$less@K@std@@@stdext@@V?$allocator@U?$pair@$$CBKV?$basic_string@DU?$char_traits@D@std@@V?$allocator@D@2@@std@@@std@@@2@$0A@@stdext@@@stdext@@@std@@@std@@QAE?AV?$_Vector_iterator@U_List_position@?$_Hash@V?$_Hmap_traits@KV?$basic_string@DU?$char_traits@D@std@@V?$allocator@D@2@@std@@V?$hash_compare@KU?$less@K@std@@@stdext@@V?$allocator@U?$pair@$$CBKV?$basic_string@DU?$char_traits@D@std@@V?$allocator@D@2@@std@@@std@@@2@$0A@@stdext@@@stdext@@V?$allocator@U_List_position@?$_Hash@V?$_Hmap_traits@KV?$basic_string@DU?$char_traits@D@std@@V?$allocator@D@2@@std@@V?$hash_compare@KU?$less@K@std@@@stdext@@V?$allocator@U?$pair@$$CBKV?$basic_string@DU?$char_traits@D@std@@V?$allocator@D@2@@std@@@std@@@2@$0A@@stdext@@@stdext@@@std@@@2@XZ 10009656 f i effectmanager.obj
 0001:00008656       ?end@?$vector@USt_EffLODParam@@V?$allocator@USt_EffLODParam@@@std@@@std@@QAE?AV?$_Vector_iterator@USt_EffLODParam@@V?$allocator@USt_EffLODParam@@@std@@@2@XZ 10009656 f i effectmanager.obj
 0001:00008656       ?end@?$vector@PAUsEffectTexture@CEffectManager@@V?$allocator@PAUsEffectTexture@CEffectManager@@@std@@@std@@QAE?AV?$_Vector_iterator@PAUsEffectTexture@CEffectManager@@V?$allocator@PAUsEffectTexture@CEffectManager@@@std@@@2@XZ 10009656 f i effectmanager.obj
 0001:00008656       ?end@?$vector@PAXV?$allocator@PAX@std@@@std@@QBE?AV?$_Vector_const_iterator@PAXV?$allocator@PAX@std@@@2@XZ 10009656 f i effectmanager.obj
 0001:00008656       ?end@?$vector@PAXV?$allocator@PAX@std@@@std@@QAE?AV?$_Vector_iterator@PAXV?$allocator@PAX@std@@@2@XZ 10009656 f i effectmanager.obj
 0001:00008656       ?end@?$vector@U_List_position@?$_Hash@V?$_Hmap_traits@KPAUSt_BodyCreate@@V?$hash_compare@KU?$less@K@std@@@stdext@@V?$allocator@U?$pair@$$CBKPAUSt_BodyCreate@@@std@@@std@@$0A@@stdext@@@stdext@@V?$allocator@U_List_position@?$_Hash@V?$_Hmap_traits@KPAUSt_BodyCreate@@V?$hash_compare@KU?$less@K@std@@@stdext@@V?$allocator@U?$pair@$$CBKPAUSt_BodyCreate@@@std@@@std@@$0A@@stdext@@@stdext@@@std@@@std@@QAE?AV?$_Vector_iterator@U_List_position@?$_Hash@V?$_Hmap_traits@KPAUSt_BodyCreate@@V?$hash_compare@KU?$less@K@std@@@stdext@@V?$allocator@U?$pair@$$CBKPAUSt_BodyCreate@@@std@@@std@@$0A@@stdext@@@stdext@@V?$allocator@U_List_position@?$_Hash@V?$_Hmap_traits@KPAUSt_BodyCreate@@V?$hash_compare@KU?$less@K@std@@@stdext@@V?$allocator@U?$pair@$$CBKPAUSt_BodyCreate@@@std@@@std@@$0A@@stdext@@@stdext@@@std@@@2@XZ 10009656 f i effectmanager.obj
 0001:000086ac       ?push_back@?$vector@USt_EffLODParam@@V?$allocator@USt_EffLODParam@@@std@@@std@@QAEXABUSt_EffLODParam@@@Z 100096ac f i effectmanager.obj
 0001:000086ac       ?push_back@?$vector@U_WZNCSPT@WzNaturalCubicSplineDyn@@V?$allocator@U_WZNCSPT@WzNaturalCubicSplineDyn@@@std@@@std@@QAEXABU_WZNCSPT@WzNaturalCubicSplineDyn@@@Z 100096ac f i Common_p:wznaturalcubicsplinedyn.obj
 0001:000086ac       ?push_back@?$vector@USt_AutoCtlParam@@V?$allocator@USt_AutoCtlParam@@@std@@@std@@QAEXABUSt_AutoCtlParam@@@Z 100096ac f i effectmanager.obj
 0001:0000876b       ?insert@?$vector@USt_EffLODParam@@V?$allocator@USt_EffLODParam@@@std@@@std@@QAE?AV?$_Vector_iterator@USt_EffLODParam@@V?$allocator@USt_EffLODParam@@@std@@@2@V?$_Vector_const_iterator@USt_EffLODParam@@V?$allocator@USt_EffLODParam@@@std@@@2@ABUSt_EffLODParam@@@Z 1000976b f i effectmanager.obj
 0001:0000876b       ?insert@?$vector@USt_AutoCtlParam@@V?$allocator@USt_AutoCtlParam@@@std@@@std@@QAE?AV?$_Vector_iterator@USt_AutoCtlParam@@V?$allocator@USt_AutoCtlParam@@@std@@@2@V?$_Vector_const_iterator@USt_AutoCtlParam@@V?$allocator@USt_AutoCtlParam@@@std@@@2@ABUSt_AutoCtlParam@@@Z 1000976b f i effectmanager.obj
 0001:0000876b       ?insert@?$vector@U_WZNCSPT@WzNaturalCubicSplineDyn@@V?$allocator@U_WZNCSPT@WzNaturalCubicSplineDyn@@@std@@@std@@QAE?AV?$_Vector_iterator@U_WZNCSPT@WzNaturalCubicSplineDyn@@V?$allocator@U_WZNCSPT@WzNaturalCubicSplineDyn@@@std@@@2@V?$_Vector_const_iterator@U_WZNCSPT@WzNaturalCubicSplineDyn@@V?$allocator@U_WZNCSPT@WzNaturalCubicSplineDyn@@@std@@@2@ABU_WZNCSPT@WzNaturalCubicSplineDyn@@@Z 1000976b f i Common_p:wznaturalcubicsplinedyn.obj
 0001:000087fb       ?Alloc@?$CWzMemoryPool@VCEffectBody@@@@QAEPAVCEffectBody@@XZ 100097fb f i effectmanager.obj
 0001:000088b3       ??_G?$CWzSingleton@VCEffectManager@@@@UAEPAXI@Z 100098b3 f i effectmanager.obj
 0001:000088b3       ??_E?$CWzSingleton@VCEffectManager@@@@UAEPAXI@Z 100098b3 f i effectmanager.obj
 0001:000088e2       ??1?$_List_val@U?$pair@$$CBKPAUSt_BodyCreate@@@std@@V?$allocator@U?$pair@$$CBKPAUSt_BodyCreate@@@std@@@2@@std@@QAE@XZ 100098e2 f i effectmanager.obj
 0001:000088e2       ??1?$_Vector_val@PAUSt_SoundInfo@@V?$allocator@PAUSt_SoundInfo@@@std@@@std@@QAE@XZ 100098e2 f i effectbody.obj
 0001:000088e2       ??1?$_Vector_val@U_WZNCSPT@WzNaturalCubicSplineDyn@@V?$allocator@U_WZNCSPT@WzNaturalCubicSplineDyn@@@std@@@std@@QAE@XZ 100098e2 f i Common_p:wznaturalcubicsplinedyn.obj
 0001:000088e2       ??1?$_Vector_val@U_List_position@?$_Hash@V?$_Hmap_traits@PAXPAVCEffectBody@@V?$hash_compare@PAXU?$less@PAX@std@@@stdext@@V?$allocator@U?$pair@QAXPAVCEffectBody@@@std@@@std@@$0A@@stdext@@@stdext@@V?$allocator@U_List_position@?$_Hash@V?$_Hmap_traits@PAXPAVCEffectBody@@V?$hash_compare@PAXU?$less@PAX@std@@@stdext@@V?$allocator@U?$pair@QAXPAVCEffectBody@@@std@@@std@@$0A@@stdext@@@stdext@@@std@@@std@@QAE@XZ 100098e2 f i effectmanager.obj
 0001:000088e2       ??1?$_Vector_val@USt_EffLODParam@@V?$allocator@USt_EffLODParam@@@std@@@std@@QAE@XZ 100098e2 f i effectmanager.obj
 0001:000088e2       ??1?$_Container_base_aux_alloc_real@V?$allocator@USt_AutoCtlParam@@@std@@@std@@IAE@XZ 100098e2 f i effectmanager.obj
 0001:000088e2       ??1?$_Container_base_aux_alloc_real@V?$allocator@USt_EffLODParam@@@std@@@std@@IAE@XZ 100098e2 f i effectmanager.obj
 0001:000088e2       ??1?$_Vector_val@U_List_position@?$_Hash@V?$_Hmap_traits@KPAUSt_BodyCreate@@V?$hash_compare@KU?$less@K@std@@@stdext@@V?$allocator@U?$pair@$$CBKPAUSt_BodyCreate@@@std@@@std@@$0A@@stdext@@@stdext@@V?$allocator@U_List_position@?$_Hash@V?$_Hmap_traits@KPAUSt_BodyCreate@@V?$hash_compare@KU?$less@K@std@@@stdext@@V?$allocator@U?$pair@$$CBKPAUSt_BodyCreate@@@std@@@std@@$0A@@stdext@@@stdext@@@std@@@std@@QAE@XZ 100098e2 f i effectmanager.obj
 0001:000088e2       ??1?$_List_val@PAVCEElementBase@@V?$allocator@PAVCEElementBase@@@std@@@std@@QAE@XZ 100098e2 f i effectbody.obj
 0001:000088e2       ??1?$_Vector_val@U_List_position@?$_Hash@V?$_Hmap_traits@KV?$basic_string@DU?$char_traits@D@std@@V?$allocator@D@2@@std@@V?$hash_compare@KU?$less@K@std@@@stdext@@V?$allocator@U?$pair@$$CBKV?$basic_string@DU?$char_traits@D@std@@V?$allocator@D@2@@std@@@std@@@2@$0A@@stdext@@@stdext@@V?$allocator@U_List_position@?$_Hash@V?$_Hmap_traits@KV?$basic_string@DU?$char_traits@D@std@@V?$allocator@D@2@@std@@V?$hash_compare@KU?$less@K@std@@@stdext@@V?$allocator@U?$pair@$$CBKV?$basic_string@DU?$char_traits@D@std@@V?$allocator@D@2@@std@@@std@@@2@$0A@@stdext@@@stdext@@@std@@@std@@QAE@XZ 100098e2 f i loadmanager.obj
 0001:000088e2       ??1?$_Vector_val@PAXV?$allocator@PAX@std@@@std@@QAE@XZ 100098e2 f i effectmanager.obj
 0001:000088e2       ??1?$_List_val@U?$pair@$$CBKV?$basic_string@DU?$char_traits@D@std@@V?$allocator@D@2@@std@@@std@@V?$allocator@U?$pair@$$CBKV?$basic_string@DU?$char_traits@D@std@@V?$allocator@D@2@@std@@@std@@@2@@std@@QAE@XZ 100098e2 f i loadmanager.obj
 0001:000088e2       ??1?$_List_val@U?$pair@QAXPAVCEffectBody@@@std@@V?$allocator@U?$pair@QAXPAVCEffectBody@@@std@@@2@@std@@QAE@XZ 100098e2 f i effectmanager.obj
 0001:000088e2       ??1?$_Tree_val@V?$_Tmap_traits@JUWzVector@@U?$less@J@std@@V?$allocator@U?$pair@$$CBJUWzVector@@@std@@@3@$0A@@std@@@std@@QAE@XZ 100098e2 f i effectmanager.obj
 0001:000088e2       ??1?$_Tree_val@V?$_Tmap_traits@JMU?$less@J@std@@V?$allocator@U?$pair@$$CBJM@std@@@2@$0A@@std@@@std@@QAE@XZ 100098e2 f i effectmanager.obj
 0001:000088e2       ??1?$_Vector_val@USt_AutoCtlParam@@V?$allocator@USt_AutoCtlParam@@@std@@@std@@QAE@XZ 100098e2 f i effectmanager.obj
 0001:000088e2       ??1?$_List_val@KV?$allocator@K@std@@@std@@QAE@XZ 100098e2 f i effectmanager.obj
 0001:000088e2       ??1?$_Vector_val@PAUsEffectTexture@CEffectManager@@V?$allocator@PAUsEffectTexture@CEffectManager@@@std@@@std@@QAE@XZ 100098e2 f i effectmanager.obj
 0001:000088e2       ??1?$_List_val@PAVCEElementSprite@@V?$allocator@PAVCEElementSprite@@@std@@@std@@QAE@XZ 100098e2 f i eelementweather.obj
 0001:000088fd       ??0?$_Tree@V?$_Tmap_traits@JUWzVector@@U?$less@J@std@@V?$allocator@U?$pair@$$CBJUWzVector@@@std@@@3@$0A@@std@@@std@@QAE@ABU?$less@J@1@ABV?$allocator@U?$pair@$$CBJUWzVector@@@std@@@1@@Z 100098fd f i effectmanager.obj
 0001:0000895e       ?erase@?$_Tree@V?$_Tmap_traits@JUWzVector@@U?$less@J@std@@V?$allocator@U?$pair@$$CBJUWzVector@@@std@@@3@$0A@@std@@@std@@QAE?AViterator@12@Vconst_iterator@12@0@Z 1000995e f i effectmanager.obj
 0001:00008b18       ?erase@?$_Tree@V?$_Tmap_traits@JUWzVector@@U?$less@J@std@@V?$allocator@U?$pair@$$CBJUWzVector@@@std@@@3@$0A@@std@@@std@@QAE?AViterator@12@Vconst_iterator@12@@Z 10009b18 f i effectmanager.obj
 0001:000090f3       ??0logic_error@std@@QAE@ABV?$basic_string@DU?$char_traits@D@std@@V?$allocator@D@2@@1@@Z 1000a0f3 f i effectmanager.obj
 0001:0000916e       ?what@logic_error@std@@UBEPBDXZ 1000a16e f i effectmanager.obj
 0001:000091a2       ??_Glogic_error@std@@UAEPAXI@Z 1000a1a2 f i effectmanager.obj
 0001:000091a2       ??_Elogic_error@std@@UAEPAXI@Z 1000a1a2 f i effectmanager.obj
 0001:000091cb       ??1logic_error@std@@UAE@XZ 1000a1cb f i effectmanager.obj
 0001:000091f6       ??1out_of_range@std@@UAE@XZ 1000a1f6 f i effectmanager.obj
 0001:00009212       ??_Eout_of_range@std@@UAEPAXI@Z 1000a212 f i effectmanager.obj
 0001:00009212       ??_Gout_of_range@std@@UAEPAXI@Z 1000a212 f i effectmanager.obj
 0001:00009244       ??1?$basic_string@DU?$char_traits@D@std@@V?$allocator@D@2@@std@@QAE@XZ 1000a244 f i effectmanager.obj
 0001:0000925b       ?assign@?$basic_string@DU?$char_traits@D@std@@V?$allocator@D@2@@std@@QAEAAV12@ABV12@II@Z 1000a25b f i effectmanager.obj
 0001:0000937e       ?_Tidy@?$basic_string@DU?$char_traits@D@std@@V?$allocator@D@2@@std@@IAEX_NI@Z 1000a37e f i effectmanager.obj
 0001:00009421       ?erase@?$basic_string@DU?$char_traits@D@std@@V?$allocator@D@2@@std@@QAEAAV12@II@Z 1000a421 f i effectmanager.obj
 0001:00009525       ?_Grow@?$basic_string@DU?$char_traits@D@std@@V?$allocator@D@2@@std@@IAE_NI_N@Z 1000a525 f i effectmanager.obj
 0001:00009606       ?_Copy@?$basic_string@DU?$char_traits@D@std@@V?$allocator@D@2@@std@@IAEXII@Z 1000a606 f i effectmanager.obj
 0001:00009832       ??$_Allocate@D@std@@YAPADIPAD@Z 1000a832 f i effectmanager.obj
 0001:00009881       ??1bad_alloc@std@@UAE@XZ   1000a881 f i effectmanager.obj
 0001:0000989b       ??_Ebad_alloc@std@@UAEPAXI@Z 1000a89b f i effectmanager.obj
 0001:0000989b       ??_Gbad_alloc@std@@UAEPAXI@Z 1000a89b f i effectmanager.obj
 0001:000098cb       ??0bad_alloc@std@@QAE@ABV01@@Z 1000a8cb f i effectmanager.obj
 0001:000098ed       ??0out_of_range@std@@QAE@ABV01@@Z 1000a8ed f i effectmanager.obj
 0001:00009911       ??0logic_error@std@@QAE@ABV01@@Z 1000a911 f i effectmanager.obj
 0001:00009993       ??0?$basic_string@DU?$char_traits@D@std@@V?$allocator@D@2@@std@@QAE@PBD@Z 1000a993 f i effectmanager.obj
 0001:000099ea       ?_Copy@?$_Tree@V?$_Tmap_traits@JUWzVector@@U?$less@J@std@@V?$allocator@U?$pair@$$CBJUWzVector@@@std@@@3@$0A@@std@@@std@@IAEXABV12@@Z 1000a9ea f i effectmanager.obj
 0001:00009aec       ?_Erase@?$_Tree@V?$_Tmap_traits@JUWzVector@@U?$less@J@std@@V?$allocator@U?$pair@$$CBJUWzVector@@@std@@@3@$0A@@std@@@std@@IAEXPAU_Node@?$_Tree_nod@V?$_Tmap_traits@JUWzVector@@U?$less@J@std@@V?$allocator@U?$pair@$$CBJUWzVector@@@std@@@3@$0A@@std@@@2@@Z 1000aaec f i effectmanager.obj
 0001:00009b32       ?_Lrotate@?$_Tree@V?$_Tmap_traits@JUWzVector@@U?$less@J@std@@V?$allocator@U?$pair@$$CBJUWzVector@@@std@@@3@$0A@@std@@@std@@IAEXPAU_Node@?$_Tree_nod@V?$_Tmap_traits@JUWzVector@@U?$less@J@std@@V?$allocator@U?$pair@$$CBJUWzVector@@@std@@@3@$0A@@std@@@2@@Z 1000ab32 f i effectmanager.obj
 0001:00009bd6       ?_Rrotate@?$_Tree@V?$_Tmap_traits@JUWzVector@@U?$less@J@std@@V?$allocator@U?$pair@$$CBJUWzVector@@@std@@@3@$0A@@std@@@std@@IAEXPAU_Node@?$_Tree_nod@V?$_Tmap_traits@JUWzVector@@U?$less@J@std@@V?$allocator@U?$pair@$$CBJUWzVector@@@std@@@3@$0A@@std@@@2@@Z 1000abd6 f i effectmanager.obj
 0001:00009c77       ?_Tidy@?$_Tree@V?$_Tmap_traits@JUWzVector@@U?$less@J@std@@V?$allocator@U?$pair@$$CBJUWzVector@@@std@@@3@$0A@@std@@@std@@IAEXXZ 1000ac77 f i effectmanager.obj
 0001:00009d37       ?_Buynode@?$list@PAVCEElementSprite@@V?$allocator@PAVCEElementSprite@@@std@@@std@@IAEPAU_Node@?$_List_nod@PAVCEElementSprite@@V?$allocator@PAVCEElementSprite@@@std@@@2@XZ 1000ad37 f i eelementweather.obj
 0001:00009d37       ?_Buynode@?$list@KV?$allocator@K@std@@@std@@IAEPAU_Node@?$_List_nod@KV?$allocator@K@std@@@2@XZ 1000ad37 f i effectmanager.obj
 0001:00009d37       ?_Buynode@?$list@PAVCEElementBase@@V?$allocator@PAVCEElementBase@@@std@@@std@@IAEPAU_Node@?$_List_nod@PAVCEElementBase@@V?$allocator@PAVCEElementBase@@@std@@@2@XZ 1000ad37 f i effectbody.obj
 0001:00009e19       ??0?$_Tree@V?$_Tmap_traits@JMU?$less@J@std@@V?$allocator@U?$pair@$$CBJM@std@@@2@$0A@@std@@@std@@QAE@ABU?$less@J@1@ABV?$allocator@U?$pair@$$CBJM@std@@@1@@Z 1000ae19 f i effectmanager.obj
 0001:00009e7a       ?erase@?$_Tree@V?$_Tmap_traits@JMU?$less@J@std@@V?$allocator@U?$pair@$$CBJM@std@@@2@$0A@@std@@@std@@QAE?AViterator@12@Vconst_iterator@12@0@Z 1000ae7a f i effectmanager.obj
 0001:0000a034       ?erase@?$_Tree@V?$_Tmap_traits@JMU?$less@J@std@@V?$allocator@U?$pair@$$CBJM@std@@@2@$0A@@std@@@std@@QAE?AViterator@12@Vconst_iterator@12@@Z 1000b034 f i effectmanager.obj
 0001:0000a60f       ??9const_iterator@?$_Tree@V?$_Tmap_traits@JUWzVector@@U?$less@J@std@@V?$allocator@U?$pair@$$CBJUWzVector@@@std@@@3@$0A@@std@@@std@@QBE_NABV012@@Z 1000b60f f i effectmanager.obj
 0001:0000a60f       ??9const_iterator@?$_Tree@V?$_Tmap_traits@JMU?$less@J@std@@V?$allocator@U?$pair@$$CBJM@std@@@2@$0A@@std@@@std@@QBE_NABV012@@Z 1000b60f f i effectmanager.obj
 0001:0000a664       ?_Copy@?$_Tree@V?$_Tmap_traits@JMU?$less@J@std@@V?$allocator@U?$pair@$$CBJM@std@@@2@$0A@@std@@@std@@IAEXABV12@@Z 1000b664 f i effectmanager.obj
 0001:0000a766       ?_Erase@?$_Tree@V?$_Tmap_traits@JMU?$less@J@std@@V?$allocator@U?$pair@$$CBJM@std@@@2@$0A@@std@@@std@@IAEXPAU_Node@?$_Tree_nod@V?$_Tmap_traits@JMU?$less@J@std@@V?$allocator@U?$pair@$$CBJM@std@@@2@$0A@@std@@@2@@Z 1000b766 f i effectmanager.obj
 0001:0000a7ac       ?_Lrotate@?$_Tree@V?$_Tmap_traits@JMU?$less@J@std@@V?$allocator@U?$pair@$$CBJM@std@@@2@$0A@@std@@@std@@IAEXPAU_Node@?$_Tree_nod@V?$_Tmap_traits@JMU?$less@J@std@@V?$allocator@U?$pair@$$CBJM@std@@@2@$0A@@std@@@2@@Z 1000b7ac f i effectmanager.obj
 0001:0000a850       ?_Rrotate@?$_Tree@V?$_Tmap_traits@JMU?$less@J@std@@V?$allocator@U?$pair@$$CBJM@std@@@2@$0A@@std@@@std@@IAEXPAU_Node@?$_Tree_nod@V?$_Tmap_traits@JMU?$less@J@std@@V?$allocator@U?$pair@$$CBJM@std@@@2@$0A@@std@@@2@@Z 1000b850 f i effectmanager.obj
 0001:0000a8f1       ?_Tidy@?$_Tree@V?$_Tmap_traits@JMU?$less@J@std@@V?$allocator@U?$pair@$$CBJM@std@@@2@$0A@@std@@@std@@IAEXXZ 1000b8f1 f i effectmanager.obj
 0001:0000a9b1       ?erase@?$vector@PAXV?$allocator@PAX@std@@@std@@QAE?AV?$_Vector_iterator@PAXV?$allocator@PAX@std@@@2@V?$_Vector_const_iterator@PAXV?$allocator@PAX@std@@@2@0@Z 1000b9b1 f i effectmanager.obj
 0001:0000a9b1       ?erase@?$vector@PAUSt_SoundInfo@@V?$allocator@PAUSt_SoundInfo@@@std@@@std@@QAE?AV?$_Vector_iterator@PAUSt_SoundInfo@@V?$allocator@PAUSt_SoundInfo@@@std@@@2@V?$_Vector_const_iterator@PAUSt_SoundInfo@@V?$allocator@PAUSt_SoundInfo@@@std@@@2@0@Z 1000b9b1 f i effectbody.obj
 0001:0000a9b1       ?erase@?$vector@PAUsEffectTexture@CEffectManager@@V?$allocator@PAUsEffectTexture@CEffectManager@@@std@@@std@@QAE?AV?$_Vector_iterator@PAUsEffectTexture@CEffectManager@@V?$allocator@PAUsEffectTexture@CEffectManager@@@std@@@2@V?$_Vector_const_iterator@PAUsEffectTexture@CEffectManager@@V?$allocator@PAUsEffectTexture@CEffectManager@@@std@@@2@0@Z 1000b9b1 f i effectmanager.obj
 0001:0000aa41       ??0?$_Vector_const_iterator@USt_AutoCtlParam@@V?$allocator@USt_AutoCtlParam@@@std@@@std@@QAE@PAUSt_AutoCtlParam@@PBV_Container_base_aux@1@@Z 1000ba41 f i effectmanager.obj
 0001:0000aa41       ??0?$_Vector_const_iterator@U_List_position@?$_Hash@V?$_Hmap_traits@PAXPAVCEffectBody@@V?$hash_compare@PAXU?$less@PAX@std@@@stdext@@V?$allocator@U?$pair@QAXPAVCEffectBody@@@std@@@std@@$0A@@stdext@@@stdext@@V?$allocator@U_List_position@?$_Hash@V?$_Hmap_traits@PAXPAVCEffectBody@@V?$hash_compare@PAXU?$less@PAX@std@@@stdext@@V?$allocator@U?$pair@QAXPAVCEffectBody@@@std@@@std@@$0A@@stdext@@@stdext@@@std@@@std@@QAE@PAU_List_position@?$_Hash@V?$_Hmap_traits@PAXPAVCEffectBody@@V?$hash_compare@PAXU?$less@PAX@std@@@stdext@@V?$allocator@U?$pair@QAXPAVCEffectBody@@@std@@@std@@$0A@@stdext@@@stdext@@PBV_Container_base_aux@1@@Z 1000ba41 f i effectmanager.obj
 0001:0000aa41       ??0?$_Vector_const_iterator@PAUsEffectTexture@CEffectManager@@V?$allocator@PAUsEffectTexture@CEffectManager@@@std@@@std@@QAE@PAPAUsEffectTexture@CEffectManager@@PBV_Container_base_aux@1@@Z 1000ba41 f i effectmanager.obj
 0001:0000aa41       ??0?$_Vector_const_iterator@PAUSt_SoundInfo@@V?$allocator@PAUSt_SoundInfo@@@std@@@std@@QAE@PAPAUSt_SoundInfo@@PBV_Container_base_aux@1@@Z 1000ba41 f i effectbody.obj
 0001:0000aa41       ??0?$_Vector_const_iterator@U_List_position@?$_Hash@V?$_Hmap_traits@KV?$basic_string@DU?$char_traits@D@std@@V?$allocator@D@2@@std@@V?$hash_compare@KU?$less@K@std@@@stdext@@V?$allocator@U?$pair@$$CBKV?$basic_string@DU?$char_traits@D@std@@V?$allocator@D@2@@std@@@std@@@2@$0A@@stdext@@@stdext@@V?$allocator@U_List_position@?$_Hash@V?$_Hmap_traits@KV?$basic_string@DU?$char_traits@D@std@@V?$allocator@D@2@@std@@V?$hash_compare@KU?$less@K@std@@@stdext@@V?$allocator@U?$pair@$$CBKV?$basic_string@DU?$char_traits@D@std@@V?$allocator@D@2@@std@@@std@@@2@$0A@@stdext@@@stdext@@@std@@@std@@QAE@PAU_List_position@?$_Hash@V?$_Hmap_traits@KV?$basic_string@DU?$char_traits@D@std@@V?$allocator@D@2@@std@@V?$hash_compare@KU?$less@K@std@@@stdext@@V?$allocator@U?$pair@$$CBKV?$basic_string@DU?$char_traits@D@std@@V?$allocator@D@2@@std@@@std@@@2@$0A@@stdext@@@stdext@@PBV_Container_base_aux@1@@Z 1000ba41 f i effectmanager.obj
 0001:0000aa41       ??0?$_Vector_const_iterator@PAXV?$allocator@PAX@std@@@std@@QAE@PAPAXPBV_Container_base_aux@1@@Z 1000ba41 f i effectmanager.obj
 0001:0000aa41       ??0?$_Vector_const_iterator@U_WZNCSPT@WzNaturalCubicSplineDyn@@V?$allocator@U_WZNCSPT@WzNaturalCubicSplineDyn@@@std@@@std@@QAE@PAU_WZNCSPT@WzNaturalCubicSplineDyn@@PBV_Container_base_aux@1@@Z 1000ba41 f i Common_p:wznaturalcubicsplinedyn.obj
 0001:0000aa41       ??0?$_Vector_const_iterator@USt_EffLODParam@@V?$allocator@USt_EffLODParam@@@std@@@std@@QAE@PAUSt_EffLODParam@@PBV_Container_base_aux@1@@Z 1000ba41 f i effectmanager.obj
 0001:0000aa41       ??0?$_Vector_const_iterator@U_List_position@?$_Hash@V?$_Hmap_traits@KPAUSt_BodyCreate@@V?$hash_compare@KU?$less@K@std@@@stdext@@V?$allocator@U?$pair@$$CBKPAUSt_BodyCreate@@@std@@@std@@$0A@@stdext@@@stdext@@V?$allocator@U_List_position@?$_Hash@V?$_Hmap_traits@KPAUSt_BodyCreate@@V?$hash_compare@KU?$less@K@std@@@stdext@@V?$allocator@U?$pair@$$CBKPAUSt_BodyCreate@@@std@@@std@@$0A@@stdext@@@stdext@@@std@@@std@@QAE@PAU_List_position@?$_Hash@V?$_Hmap_traits@KPAUSt_BodyCreate@@V?$hash_compare@KU?$less@K@std@@@stdext@@V?$allocator@U?$pair@$$CBKPAUSt_BodyCreate@@@std@@@std@@$0A@@stdext@@@stdext@@PBV_Container_base_aux@1@@Z 1000ba41 f i effectmanager.obj
 0001:0000aa8d       ?clear@?$list@U?$pair@$$CBKV?$basic_string@DU?$char_traits@D@std@@V?$allocator@D@2@@std@@@std@@V?$allocator@U?$pair@$$CBKV?$basic_string@DU?$char_traits@D@std@@V?$allocator@D@2@@std@@@std@@@2@@std@@QAEXXZ 1000ba8d f i effectmanager.obj
 0001:0000ab03       ??8?$_Const_iterator@$00@?$list@U?$pair@$$CBKPAUSt_BodyCreate@@@std@@V?$allocator@U?$pair@$$CBKPAUSt_BodyCreate@@@std@@@2@@std@@QBE_NABV012@@Z 1000bb03 f i effectmanager.obj
 0001:0000ab03       ??8?$_Const_iterator@$00@?$list@HV?$allocator@H@std@@@std@@QBE_NABV012@@Z 1000bb03 f i effectmanager.obj
 0001:0000ab03       ??8?$_Const_iterator@$00@?$list@U?$pair@$$CBKV?$basic_string@DU?$char_traits@D@std@@V?$allocator@D@2@@std@@@std@@V?$allocator@U?$pair@$$CBKV?$basic_string@DU?$char_traits@D@std@@V?$allocator@D@2@@std@@@std@@@2@@std@@QBE_NABV012@@Z 1000bb03 f i effectmanager.obj
 0001:0000ab03       ??8?$_Const_iterator@$00@?$list@KV?$allocator@K@std@@@std@@QBE_NABV012@@Z 1000bb03 f i effectmanager.obj
 0001:0000ab03       ??8?$_Const_iterator@$00@?$list@PAVCEElementSprite@@V?$allocator@PAVCEElementSprite@@@std@@@std@@QBE_NABV012@@Z 1000bb03 f i eelementweather.obj
 0001:0000ab03       ??8?$_Const_iterator@$00@?$list@PAVCEElementBase@@V?$allocator@PAVCEElementBase@@@std@@@std@@QBE_NABV012@@Z 1000bb03 f i effectbody.obj
 0001:0000ab03       ??8?$_Const_iterator@$00@?$list@U?$pair@QAXPAVCEffectBody@@@std@@V?$allocator@U?$pair@QAXPAVCEffectBody@@@std@@@2@@std@@QBE_NABV012@@Z 1000bb03 f i effectmanager.obj
 0001:0000ab55       ??0?$_Hash@V?$_Hmap_traits@PAXPAVCEffectBody@@V?$hash_compare@PAXU?$less@PAX@std@@@stdext@@V?$allocator@U?$pair@QAXPAVCEffectBody@@@std@@@std@@$0A@@stdext@@@stdext@@QAE@ABV?$hash_compare@PAXU?$less@PAX@std@@@1@ABV?$allocator@U?$pair@QAXPAVCEffectBody@@@std@@@std@@@Z 1000bb55 f i effectmanager.obj
 0001:0000ab55       ??0?$_Hash@V?$_Hmap_traits@KPAUSt_BodyCreate@@V?$hash_compare@KU?$less@K@std@@@stdext@@V?$allocator@U?$pair@$$CBKPAUSt_BodyCreate@@@std@@@std@@$0A@@stdext@@@stdext@@QAE@ABV?$hash_compare@KU?$less@K@std@@@1@ABV?$allocator@U?$pair@$$CBKPAUSt_BodyCreate@@@std@@@std@@@Z 1000bb55 f i effectmanager.obj
 0001:0000abf9       ?_Hashval@?$_Hash@V?$_Hmap_traits@KV?$basic_string@DU?$char_traits@D@std@@V?$allocator@D@2@@std@@V?$hash_compare@KU?$less@K@std@@@stdext@@V?$allocator@U?$pair@$$CBKV?$basic_string@DU?$char_traits@D@std@@V?$allocator@D@2@@std@@@std@@@2@$0A@@stdext@@@stdext@@IBEIABK@Z 1000bbf9 f i loadmanager.obj
 0001:0000abf9       ?_Hashval@?$_Hash@V?$_Hmap_traits@KPAUSt_BodyCreate@@V?$hash_compare@KU?$less@K@std@@@stdext@@V?$allocator@U?$pair@$$CBKPAUSt_BodyCreate@@@std@@@std@@$0A@@stdext@@@stdext@@IBEIABK@Z 1000bbf9 f i effectmanager.obj
 0001:0000abf9       ?_Hashval@?$_Hash@V?$_Hmap_traits@PAXPAVCEffectBody@@V?$hash_compare@PAXU?$less@PAX@std@@@stdext@@V?$allocator@U?$pair@QAXPAVCEffectBody@@@std@@@std@@$0A@@stdext@@@stdext@@IBEIABQAX@Z 1000bbf9 f i effectmanager.obj
 0001:0000ac3c       ?_Insert@?$_Hash@V?$_Hmap_traits@PAXPAVCEffectBody@@V?$hash_compare@PAXU?$less@PAX@std@@@stdext@@V?$allocator@U?$pair@QAXPAVCEffectBody@@@std@@@std@@$0A@@stdext@@@stdext@@IAE?AU?$pair@V?$_Iterator@$00@?$list@U?$pair@QAXPAVCEffectBody@@@std@@V?$allocator@U?$pair@QAXPAVCEffectBody@@@std@@@2@@std@@_N@std@@ABU?$pair@QAXPAVCEffectBody@@@4@V?$_Iterator@$00@?$list@U?$pair@QAXPAVCEffectBody@@@std@@V?$allocator@U?$pair@QAXPAVCEffectBody@@@std@@@2@@4@@Z 1000bc3c f i effectmanager.obj
 0001:0000ac3c       ?_Insert@?$_Hash@V?$_Hmap_traits@KPAUSt_BodyCreate@@V?$hash_compare@KU?$less@K@std@@@stdext@@V?$allocator@U?$pair@$$CBKPAUSt_BodyCreate@@@std@@@std@@$0A@@stdext@@@stdext@@IAE?AU?$pair@V?$_Iterator@$00@?$list@U?$pair@$$CBKPAUSt_BodyCreate@@@std@@V?$allocator@U?$pair@$$CBKPAUSt_BodyCreate@@@std@@@2@@std@@_N@std@@ABU?$pair@$$CBKPAUSt_BodyCreate@@@4@V?$_Iterator@$00@?$list@U?$pair@$$CBKPAUSt_BodyCreate@@@std@@V?$allocator@U?$pair@$$CBKPAUSt_BodyCreate@@@std@@@2@@4@@Z 1000bc3c f i effectmanager.obj
 0001:0000b16e       ?lower_bound@?$_Hash@V?$_Hmap_traits@KPAUSt_BodyCreate@@V?$hash_compare@KU?$less@K@std@@@stdext@@V?$allocator@U?$pair@$$CBKPAUSt_BodyCreate@@@std@@@std@@$0A@@stdext@@@stdext@@QAE?AV?$_Iterator@$00@?$list@U?$pair@$$CBKPAUSt_BodyCreate@@@std@@V?$allocator@U?$pair@$$CBKPAUSt_BodyCreate@@@std@@@2@@std@@ABK@Z 1000c16e f i effectmanager.obj
 0001:0000b16e       ?lower_bound@?$_Hash@V?$_Hmap_traits@PAXPAVCEffectBody@@V?$hash_compare@PAXU?$less@PAX@std@@@stdext@@V?$allocator@U?$pair@QAXPAVCEffectBody@@@std@@@std@@$0A@@stdext@@@stdext@@QAE?AV?$_Iterator@$00@?$list@U?$pair@QAXPAVCEffectBody@@@std@@V?$allocator@U?$pair@QAXPAVCEffectBody@@@std@@@2@@std@@ABQAX@Z 1000c16e f i effectmanager.obj
 0001:0000b2e1       ?_Init@?$_Hash@V?$_Hmap_traits@KPAUSt_BodyCreate@@V?$hash_compare@KU?$less@K@std@@@stdext@@V?$allocator@U?$pair@$$CBKPAUSt_BodyCreate@@@std@@@std@@$0A@@stdext@@@stdext@@IAEXI@Z 1000c2e1 f i effectmanager.obj
 0001:0000b2e1       ?_Init@?$_Hash@V?$_Hmap_traits@PAXPAVCEffectBody@@V?$hash_compare@PAXU?$less@PAX@std@@@stdext@@V?$allocator@U?$pair@QAXPAVCEffectBody@@@std@@@std@@$0A@@stdext@@@stdext@@IAEXI@Z 1000c2e1 f i effectmanager.obj
 0001:0000b2e1       ?_Init@?$_Hash@V?$_Hmap_traits@KV?$basic_string@DU?$char_traits@D@std@@V?$allocator@D@2@@std@@V?$hash_compare@KU?$less@K@std@@@stdext@@V?$allocator@U?$pair@$$CBKV?$basic_string@DU?$char_traits@D@std@@V?$allocator@D@2@@std@@@std@@@2@$0A@@stdext@@@stdext@@IAEXI@Z 1000c2e1 f i effectmanager.obj
 0001:0000b32e       ??1?$list@U?$pair@$$CBKPAUSt_BodyCreate@@@std@@V?$allocator@U?$pair@$$CBKPAUSt_BodyCreate@@@std@@@2@@std@@QAE@XZ 1000c32e f i effectmanager.obj
 0001:0000b32e       ??1?$list@U?$pair@QAXPAVCEffectBody@@@std@@V?$allocator@U?$pair@QAXPAVCEffectBody@@@std@@@2@@std@@QAE@XZ 1000c32e f i effectmanager.obj
 0001:0000b32e       ??1?$list@PAVCEElementBase@@V?$allocator@PAVCEElementBase@@@std@@@std@@QAE@XZ 1000c32e f i effectbody.obj
 0001:0000b32e       ??1?$list@KV?$allocator@K@std@@@std@@QAE@XZ 1000c32e f i effectmanager.obj
 0001:0000b384       ?erase@?$vector@U_List_position@?$_Hash@V?$_Hmap_traits@KV?$basic_string@DU?$char_traits@D@std@@V?$allocator@D@2@@std@@V?$hash_compare@KU?$less@K@std@@@stdext@@V?$allocator@U?$pair@$$CBKV?$basic_string@DU?$char_traits@D@std@@V?$allocator@D@2@@std@@@std@@@2@$0A@@stdext@@@stdext@@V?$allocator@U_List_position@?$_Hash@V?$_Hmap_traits@KV?$basic_string@DU?$char_traits@D@std@@V?$allocator@D@2@@std@@V?$hash_compare@KU?$less@K@std@@@stdext@@V?$allocator@U?$pair@$$CBKV?$basic_string@DU?$char_traits@D@std@@V?$allocator@D@2@@std@@@std@@@2@$0A@@stdext@@@stdext@@@std@@@std@@QAE?AV?$_Vector_iterator@U_List_position@?$_Hash@V?$_Hmap_traits@KV?$basic_string@DU?$char_traits@D@std@@V?$allocator@D@2@@std@@V?$hash_compare@KU?$less@K@std@@@stdext@@V?$allocator@U?$pair@$$CBKV?$basic_string@DU?$char_traits@D@std@@V?$allocator@D@2@@std@@@std@@@2@$0A@@stdext@@@stdext@@V?$allocator@U_List_position@?$_Hash@V?$_Hmap_traits@KV?$basic_string@DU?$char_traits@D@std@@V?$allocator@D@2@@std@@V?$hash_compare@KU?$less@K@std@@@stdext@@V?$allocator@U?$pair@$$CBKV?$basic_string@DU?$char_traits@D@std@@V?$allocator@D@2@@std@@@std@@@2@$0A@@stdext@@@stdext@@@std@@@2@V?$_Vector_const_iterator@U_List_position@?$_Hash@V?$_Hmap_traits@KV?$basic_string@DU?$char_traits@D@std@@V?$allocator@D@2@@std@@V?$hash_compare@KU?$less@K@std@@@stdext@@V?$allocator@U?$pair@$$CBKV?$basic_string@DU?$char_traits@D@std@@V?$allocator@D@2@@std@@@std@@@2@$0A@@stdext@@@stdext@@V?$allocator@U_List_position@?$_Hash@V?$_Hmap_traits@KV?$basic_string@DU?$char_traits@D@std@@V?$allocator@D@2@@std@@V?$hash_compare@KU?$less@K@std@@@stdext@@V?$allocator@U?$pair@$$CBKV?$basic_string@DU?$char_traits@D@std@@V?$allocator@D@2@@std@@@std@@@2@$0A@@stdext@@@stdext@@@std@@@2@0@Z 1000c384 f i effectmanager.obj
 0001:0000b384       ?erase@?$vector@USt_AutoCtlParam@@V?$allocator@USt_AutoCtlParam@@@std@@@std@@QAE?AV?$_Vector_iterator@USt_AutoCtlParam@@V?$allocator@USt_AutoCtlParam@@@std@@@2@V?$_Vector_const_iterator@USt_AutoCtlParam@@V?$allocator@USt_AutoCtlParam@@@std@@@2@0@Z 1000c384 f i effectmanager.obj
 0001:0000b384       ?erase@?$vector@U_List_position@?$_Hash@V?$_Hmap_traits@PAXPAVCEffectBody@@V?$hash_compare@PAXU?$less@PAX@std@@@stdext@@V?$allocator@U?$pair@QAXPAVCEffectBody@@@std@@@std@@$0A@@stdext@@@stdext@@V?$allocator@U_List_position@?$_Hash@V?$_Hmap_traits@PAXPAVCEffectBody@@V?$hash_compare@PAXU?$less@PAX@std@@@stdext@@V?$allocator@U?$pair@QAXPAVCEffectBody@@@std@@@std@@$0A@@stdext@@@stdext@@@std@@@std@@QAE?AV?$_Vector_iterator@U_List_position@?$_Hash@V?$_Hmap_traits@PAXPAVCEffectBody@@V?$hash_compare@PAXU?$less@PAX@std@@@stdext@@V?$allocator@U?$pair@QAXPAVCEffectBody@@@std@@@std@@$0A@@stdext@@@stdext@@V?$allocator@U_List_position@?$_Hash@V?$_Hmap_traits@PAXPAVCEffectBody@@V?$hash_compare@PAXU?$less@PAX@std@@@stdext@@V?$allocator@U?$pair@QAXPAVCEffectBody@@@std@@@std@@$0A@@stdext@@@stdext@@@std@@@2@V?$_Vector_const_iterator@U_List_position@?$_Hash@V?$_Hmap_traits@PAXPAVCEffectBody@@V?$hash_compare@PAXU?$less@PAX@std@@@stdext@@V?$allocator@U?$pair@QAXPAVCEffectBody@@@std@@@std@@$0A@@stdext@@@stdext@@V?$allocator@U_List_position@?$_Hash@V?$_Hmap_traits@PAXPAVCEffectBody@@V?$hash_compare@PAXU?$less@PAX@std@@@stdext@@V?$allocator@U?$pair@QAXPAVCEffectBody@@@std@@@std@@$0A@@stdext@@@stdext@@@std@@@2@0@Z 1000c384 f i effectmanager.obj
 0001:0000b384       ?erase@?$vector@USt_EffLODParam@@V?$allocator@USt_EffLODParam@@@std@@@std@@QAE?AV?$_Vector_iterator@USt_EffLODParam@@V?$allocator@USt_EffLODParam@@@std@@@2@V?$_Vector_const_iterator@USt_EffLODParam@@V?$allocator@USt_EffLODParam@@@std@@@2@0@Z 1000c384 f i effectmanager.obj
 0001:0000b384       ?erase@?$vector@U_List_position@?$_Hash@V?$_Hmap_traits@KPAUSt_BodyCreate@@V?$hash_compare@KU?$less@K@std@@@stdext@@V?$allocator@U?$pair@$$CBKPAUSt_BodyCreate@@@std@@@std@@$0A@@stdext@@@stdext@@V?$allocator@U_List_position@?$_Hash@V?$_Hmap_traits@KPAUSt_BodyCreate@@V?$hash_compare@KU?$less@K@std@@@stdext@@V?$allocator@U?$pair@$$CBKPAUSt_BodyCreate@@@std@@@std@@$0A@@stdext@@@stdext@@@std@@@std@@QAE?AV?$_Vector_iterator@U_List_position@?$_Hash@V?$_Hmap_traits@KPAUSt_BodyCreate@@V?$hash_compare@KU?$less@K@std@@@stdext@@V?$allocator@U?$pair@$$CBKPAUSt_BodyCreate@@@std@@@std@@$0A@@stdext@@@stdext@@V?$allocator@U_List_position@?$_Hash@V?$_Hmap_traits@KPAUSt_BodyCreate@@V?$hash_compare@KU?$less@K@std@@@stdext@@V?$allocator@U?$pair@$$CBKPAUSt_BodyCreate@@@std@@@std@@$0A@@stdext@@@stdext@@@std@@@2@V?$_Vector_const_iterator@U_List_position@?$_Hash@V?$_Hmap_traits@KPAUSt_BodyCreate@@V?$hash_compare@KU?$less@K@std@@@stdext@@V?$allocator@U?$pair@$$CBKPAUSt_BodyCreate@@@std@@@std@@$0A@@stdext@@@stdext@@V?$allocator@U_List_position@?$_Hash@V?$_Hmap_traits@KPAUSt_BodyCreate@@V?$hash_compare@KU?$less@K@std@@@stdext@@V?$allocator@U?$pair@$$CBKPAUSt_BodyCreate@@@std@@@std@@$0A@@stdext@@@stdext@@@std@@@2@0@Z 1000c384 f i effectmanager.obj
 0001:0000b384       ?erase@?$vector@U_WZNCSPT@WzNaturalCubicSplineDyn@@V?$allocator@U_WZNCSPT@WzNaturalCubicSplineDyn@@@std@@@std@@QAE?AV?$_Vector_iterator@U_WZNCSPT@WzNaturalCubicSplineDyn@@V?$allocator@U_WZNCSPT@WzNaturalCubicSplineDyn@@@std@@@2@V?$_Vector_const_iterator@U_WZNCSPT@WzNaturalCubicSplineDyn@@V?$allocator@U_WZNCSPT@WzNaturalCubicSplineDyn@@@std@@@2@0@Z 1000c384 f i Common_p:wznaturalcubicsplinedyn.obj
 0001:0000b42f       ?_Tidy@?$vector@USt_AutoCtlParam@@V?$allocator@USt_AutoCtlParam@@@std@@@std@@IAEXXZ 1000c42f f i effectmanager.obj
 0001:0000b42f       ?_Tidy@?$vector@U_WZNCSPT@WzNaturalCubicSplineDyn@@V?$allocator@U_WZNCSPT@WzNaturalCubicSplineDyn@@@std@@@std@@IAEXXZ 1000c42f f i Common_p:wznaturalcubicsplinedyn.obj
 0001:0000b42f       ?_Tidy@?$vector@U_List_position@?$_Hash@V?$_Hmap_traits@KPAUSt_BodyCreate@@V?$hash_compare@KU?$less@K@std@@@stdext@@V?$allocator@U?$pair@$$CBKPAUSt_BodyCreate@@@std@@@std@@$0A@@stdext@@@stdext@@V?$allocator@U_List_position@?$_Hash@V?$_Hmap_traits@KPAUSt_BodyCreate@@V?$hash_compare@KU?$less@K@std@@@stdext@@V?$allocator@U?$pair@$$CBKPAUSt_BodyCreate@@@std@@@std@@$0A@@stdext@@@stdext@@@std@@@std@@IAEXXZ 1000c42f f i effectmanager.obj
 0001:0000b42f       ?_Tidy@?$vector@USt_EffLODParam@@V?$allocator@USt_EffLODParam@@@std@@@std@@IAEXXZ 1000c42f f i effectmanager.obj
 0001:0000b42f       ?_Tidy@?$vector@U_List_position@?$_Hash@V?$_Hmap_traits@PAXPAVCEffectBody@@V?$hash_compare@PAXU?$less@PAX@std@@@stdext@@V?$allocator@U?$pair@QAXPAVCEffectBody@@@std@@@std@@$0A@@stdext@@@stdext@@V?$allocator@U_List_position@?$_Hash@V?$_Hmap_traits@PAXPAVCEffectBody@@V?$hash_compare@PAXU?$less@PAX@std@@@stdext@@V?$allocator@U?$pair@QAXPAVCEffectBody@@@std@@@std@@$0A@@stdext@@@stdext@@@std@@@std@@IAEXXZ 1000c42f f i effectmanager.obj
 0001:0000b42f       ?_Tidy@?$vector@U_List_position@?$_Hash@V?$_Hmap_traits@KV?$basic_string@DU?$char_traits@D@std@@V?$allocator@D@2@@std@@V?$hash_compare@KU?$less@K@std@@@stdext@@V?$allocator@U?$pair@$$CBKV?$basic_string@DU?$char_traits@D@std@@V?$allocator@D@2@@std@@@std@@@2@$0A@@stdext@@@stdext@@V?$allocator@U_List_position@?$_Hash@V?$_Hmap_traits@KV?$basic_string@DU?$char_traits@D@std@@V?$allocator@D@2@@std@@V?$hash_compare@KU?$less@K@std@@@stdext@@V?$allocator@U?$pair@$$CBKV?$basic_string@DU?$char_traits@D@std@@V?$allocator@D@2@@std@@@std@@@2@$0A@@stdext@@@stdext@@@std@@@std@@IAEXXZ 1000c42f f i loadmanager.obj
 0001:0000b4bb       ?AllocBand@?$CWzMemoryPool@VCEffectBody@@@@AAEPAV?$CWzMemoryBand@VCEffectBody@@@@H@Z 1000c4bb f i effectmanager.obj
 0001:0000b596       ??D?$_Const_iterator@$00@?$list@U?$pair@$$CBKV?$basic_string@DU?$char_traits@D@std@@V?$allocator@D@2@@std@@@std@@V?$allocator@U?$pair@$$CBKV?$basic_string@DU?$char_traits@D@std@@V?$allocator@D@2@@std@@@std@@@2@@std@@QBEABU?$pair@$$CBKV?$basic_string@DU?$char_traits@D@std@@V?$allocator@D@2@@std@@@2@XZ 1000c596 f i effectmanager.obj
 0001:0000b596       ??D?$_Const_iterator@$00@?$list@PAVCEElementBase@@V?$allocator@PAVCEElementBase@@@std@@@std@@QBEABQAVCEElementBase@@XZ 1000c596 f i effectbody.obj
 0001:0000b596       ??D?$_Const_iterator@$00@?$list@U?$pair@$$CBKPAUSt_BodyCreate@@@std@@V?$allocator@U?$pair@$$CBKPAUSt_BodyCreate@@@std@@@2@@std@@QBEABU?$pair@$$CBKPAUSt_BodyCreate@@@2@XZ 1000c596 f i effectmanager.obj
 0001:0000b596       ??D?$_Const_iterator@$00@?$list@U?$pair@QAXPAVCEffectBody@@@std@@V?$allocator@U?$pair@QAXPAVCEffectBody@@@std@@@2@@std@@QBEABU?$pair@QAXPAVCEffectBody@@@2@XZ 1000c596 f i effectmanager.obj
 0001:0000b596       ??D?$_Const_iterator@$00@?$list@KV?$allocator@K@std@@@std@@QBEABKXZ 1000c596 f i effectmanager.obj
 0001:0000b596       ??D?$_Const_iterator@$00@?$list@HV?$allocator@H@std@@@std@@QBEABHXZ 1000c596 f i effectmanager.obj
 0001:0000b596       ??D?$_Const_iterator@$00@?$list@PAVCEElementSprite@@V?$allocator@PAVCEElementSprite@@@std@@@std@@QBEABQAVCEElementSprite@@XZ 1000c596 f i eelementweather.obj
 0001:0000b60a       ??E?$_Const_iterator@$00@?$list@U?$pair@$$CBKV?$basic_string@DU?$char_traits@D@std@@V?$allocator@D@2@@std@@@std@@V?$allocator@U?$pair@$$CBKV?$basic_string@DU?$char_traits@D@std@@V?$allocator@D@2@@std@@@std@@@2@@std@@QAEAAV012@XZ 1000c60a f i effectmanager.obj
 0001:0000b60a       ??E?$_Const_iterator@$00@?$list@U?$pair@QAXPAVCEffectBody@@@std@@V?$allocator@U?$pair@QAXPAVCEffectBody@@@std@@@2@@std@@QAEAAV012@XZ 1000c60a f i effectmanager.obj
 0001:0000b60a       ??E?$_Const_iterator@$00@?$list@HV?$allocator@H@std@@@std@@QAEAAV012@XZ 1000c60a f i effectmanager.obj
 0001:0000b60a       ??E?$_Const_iterator@$00@?$list@U?$pair@$$CBKPAUSt_BodyCreate@@@std@@V?$allocator@U?$pair@$$CBKPAUSt_BodyCreate@@@std@@@2@@std@@QAEAAV012@XZ 1000c60a f i effectmanager.obj
 0001:0000b60a       ??E?$_Const_iterator@$00@?$list@KV?$allocator@K@std@@@std@@QAEAAV012@XZ 1000c60a f i effectmanager.obj
 0001:0000b60a       ??E?$_Const_iterator@$00@?$list@PAVCEElementSprite@@V?$allocator@PAVCEElementSprite@@@std@@@std@@QAEAAV012@XZ 1000c60a f i eelementweather.obj
 0001:0000b60a       ??E?$_Const_iterator@$00@?$list@PAVCEElementBase@@V?$allocator@PAVCEElementBase@@@std@@@std@@QAEAAV012@XZ 1000c60a f i effectbody.obj
 0001:0000b68c       ??E?$_Vector_const_iterator@USt_EffLODParam@@V?$allocator@USt_EffLODParam@@@std@@@std@@QAEAAV01@XZ 1000c68c f i effectmanager.obj
 0001:0000b68c       ??E?$_Vector_const_iterator@USt_AutoCtlParam@@V?$allocator@USt_AutoCtlParam@@@std@@@std@@QAEAAV01@XZ 1000c68c f i effectmanager.obj
 0001:0000b6ff       ??G?$_Vector_const_iterator@USt_EffLODParam@@V?$allocator@USt_EffLODParam@@@std@@@std@@QBEHABV01@@Z 1000c6ff f i effectmanager.obj
 0001:0000b6ff       ??G?$_Vector_const_iterator@USt_AutoCtlParam@@V?$allocator@USt_AutoCtlParam@@@std@@@std@@QBEHABV01@@Z 1000c6ff f i effectmanager.obj
 0001:0000b6ff       ??G?$_Vector_const_iterator@U_WZNCSPT@WzNaturalCubicSplineDyn@@V?$allocator@U_WZNCSPT@WzNaturalCubicSplineDyn@@@std@@@std@@QBEHABV01@@Z 1000c6ff f i Common_p:wznaturalcubicsplinedyn.obj
 0001:0000b74a       ?assign@?$basic_string@DU?$char_traits@D@std@@V?$allocator@D@2@@std@@QAEAAV12@PBDI@Z 1000c74a f i effectmanager.obj
 0001:0000b82c       ?_Copy@?$_Tree@V?$_Tmap_traits@JUWzVector@@U?$less@J@std@@V?$allocator@U?$pair@$$CBJUWzVector@@@std@@@3@$0A@@std@@@std@@IAEPAU_Node@?$_Tree_nod@V?$_Tmap_traits@JUWzVector@@U?$less@J@std@@V?$allocator@U?$pair@$$CBJUWzVector@@@std@@@3@$0A@@std@@@2@PAU342@0@Z 1000c82c f i effectmanager.obj
 0001:0000b922       ?_Init@?$_Tree@V?$_Tmap_traits@JUWzVector@@U?$less@J@std@@V?$allocator@U?$pair@$$CBJUWzVector@@@std@@@3@$0A@@std@@@std@@IAEXXZ 1000c922 f i effectmanager.obj
 0001:0000b97d       ?_Inc@const_iterator@?$_Tree@V?$_Tmap_traits@JUWzVector@@U?$less@J@std@@V?$allocator@U?$pair@$$CBJUWzVector@@@std@@@3@$0A@@std@@@std@@QAEXXZ 1000c97d f i effectmanager.obj
 0001:0000ba43       ?_Copy@?$_Tree@V?$_Tmap_traits@JMU?$less@J@std@@V?$allocator@U?$pair@$$CBJM@std@@@2@$0A@@std@@@std@@IAEPAU_Node@?$_Tree_nod@V?$_Tmap_traits@JMU?$less@J@std@@V?$allocator@U?$pair@$$CBJM@std@@@2@$0A@@std@@@2@PAU342@0@Z 1000ca43 f i effectmanager.obj
 0001:0000bb39       ?_Init@?$_Tree@V?$_Tmap_traits@JMU?$less@J@std@@V?$allocator@U?$pair@$$CBJM@std@@@2@$0A@@std@@@std@@IAEXXZ 1000cb39 f i effectmanager.obj
 0001:0000bb94       ??0?$_Tree_val@V?$_Tmap_traits@JMU?$less@J@std@@V?$allocator@U?$pair@$$CBJM@std@@@2@$0A@@std@@@std@@IAE@ABU?$less@J@1@V?$allocator@U?$pair@$$CBJM@std@@@1@@Z 1000cb94 f i effectmanager.obj
 0001:0000bb94       ??0?$_Tree_val@V?$_Tmap_traits@JUWzVector@@U?$less@J@std@@V?$allocator@U?$pair@$$CBJUWzVector@@@std@@@3@$0A@@std@@@std@@IAE@ABU?$less@J@1@V?$allocator@U?$pair@$$CBJUWzVector@@@std@@@1@@Z 1000cb94 f i effectmanager.obj
 0001:0000bbbb       ??0const_iterator@?$_Tree@V?$_Tmap_traits@JMU?$less@J@std@@V?$allocator@U?$pair@$$CBJM@std@@@2@$0A@@std@@@std@@QAE@PAU_Node@?$_Tree_nod@V?$_Tmap_traits@JMU?$less@J@std@@V?$allocator@U?$pair@$$CBJM@std@@@2@$0A@@std@@@2@PBV12@@Z 1000cbbb f i effectmanager.obj
 0001:0000bbbb       ??0const_iterator@?$_Tree@V?$_Tmap_traits@JUWzVector@@U?$less@J@std@@V?$allocator@U?$pair@$$CBJUWzVector@@@std@@@3@$0A@@std@@@std@@QAE@PAU_Node@?$_Tree_nod@V?$_Tmap_traits@JUWzVector@@U?$less@J@std@@V?$allocator@U?$pair@$$CBJUWzVector@@@std@@@3@$0A@@std@@@2@PBV12@@Z 1000cbbb f i effectmanager_load.obj
 0001:0000bbf1       ??Dconst_iterator@?$_Tree@V?$_Tmap_traits@JUWzVector@@U?$less@J@std@@V?$allocator@U?$pair@$$CBJUWzVector@@@std@@@3@$0A@@std@@@std@@QBEABU?$pair@$$CBJUWzVector@@@2@XZ 1000cbf1 f i effectmanager.obj
 0001:0000bbf1       ??Dconst_iterator@?$_Tree@V?$_Tmap_traits@JMU?$less@J@std@@V?$allocator@U?$pair@$$CBJM@std@@@2@$0A@@std@@@std@@QBEABU?$pair@$$CBJM@2@XZ 1000cbf1 f i effectmanager.obj
 0001:0000bc5b       ?_Inc@const_iterator@?$_Tree@V?$_Tmap_traits@JMU?$less@J@std@@V?$allocator@U?$pair@$$CBJM@std@@@2@$0A@@std@@@std@@QAEXXZ 1000cc5b f i effectmanager.obj
 0001:0000bd21       ??1length_error@std@@UAE@XZ 1000cd21 f i effectmanager.obj
 0001:0000bd3d       ??_Elength_error@std@@UAEPAXI@Z 1000cd3d f i effectmanager.obj
 0001:0000bd3d       ??_Glength_error@std@@UAEPAXI@Z 1000cd3d f i effectmanager.obj
 0001:0000bd6f       ?OnBeingBorn@CEElementBase@@MAEXXZ 1000cd6f f i eelementbase.obj
 0001:0000bd6f       ??1?$_Hmap_traits@KPAUSt_BodyCreate@@V?$hash_compare@KU?$less@K@std@@@stdext@@V?$allocator@U?$pair@$$CBKPAUSt_BodyCreate@@@std@@@std@@$0A@@stdext@@QAE@XZ 1000cd6f f i effectmanager.obj
 0001:0000bd6f       ?ReloadTexture@CEElementBase@@UAEXXZ 1000cd6f f i eelementbase.obj
 0001:0000bd6f       ?Render@CEElementBase@@UAEXXZ 1000cd6f f i eelementbase.obj
 0001:0000bd6f       ?OnRelease@WzLogHandler@WzLog@@EAEXXZ 1000cd6f f i ProgramCommonLibForEngine_p:WzFileLogHandler.obj
 0001:0000bd6f       ??1?$_Hmap_traits@KV?$basic_string@DU?$char_traits@D@std@@V?$allocator@D@2@@std@@V?$hash_compare@KU?$less@K@std@@@stdext@@V?$allocator@U?$pair@$$CBKV?$basic_string@DU?$char_traits@D@std@@V?$allocator@D@2@@std@@@std@@@2@$0A@@stdext@@QAE@XZ 1000cd6f f i loadmanager.obj
 0001:0000bd6f       ??1?$CWzFlag@K@@QAE@XZ     1000cd6f f i effectmanager.obj
 0001:0000bd6f       ??1CDivideCube@@QAE@XZ     1000cd6f f i eelementweather.obj
 0001:0000bd6f       ?Destroy@CEElementBase@@UAEXXZ 1000cd6f f i eelementbase.obj
 0001:0000bd6f       ??1?$_Hmap_traits@PAXPAVCEffectBody@@V?$hash_compare@PAXU?$less@PAX@std@@@stdext@@V?$allocator@U?$pair@QAXPAVCEffectBody@@@std@@@std@@$0A@@stdext@@QAE@XZ 1000cd6f f i effectmanager.obj
 0001:0000bd6f       ??1_Container_base_aux@std@@QAE@XZ 1000cd6f f i effectmanager.obj
 0001:0000bd78       ??R?$hash_compare@PAXU?$less@PAX@std@@@stdext@@QBEIABQAX@Z 1000cd78 f i effectmanager.obj
 0001:0000bd78       ??R?$hash_compare@KU?$less@K@std@@@stdext@@QBEIABK@Z 1000cd78 f i effectmanager.obj
 0001:0000bddf       ??0?$_Container_base_aux_alloc_real@V?$allocator@U?$pair@$$CBKPAUSt_BodyCreate@@@std@@@std@@@std@@IAE@V?$allocator@U?$pair@$$CBKPAUSt_BodyCreate@@@std@@@1@@Z 1000cddf f i effectmanager.obj
 0001:0000bddf       ??0?$_Container_base_aux_alloc_real@V?$allocator@PAX@std@@@std@@IAE@V?$allocator@PAX@1@@Z 1000cddf f i effectmanager.obj
 0001:0000bddf       ??0?$_Container_base_aux_alloc_real@V?$allocator@U?$pair@$$CBJUWzVector@@@std@@@std@@@std@@IAE@V?$allocator@U?$pair@$$CBJUWzVector@@@std@@@1@@Z 1000cddf f i effectmanager.obj
 0001:0000bddf       ??0?$_Container_base_aux_alloc_real@V?$allocator@U_List_position@?$_Hash@V?$_Hmap_traits@KPAUSt_BodyCreate@@V?$hash_compare@KU?$less@K@std@@@stdext@@V?$allocator@U?$pair@$$CBKPAUSt_BodyCreate@@@std@@@std@@$0A@@stdext@@@stdext@@@std@@@std@@IAE@V?$allocator@U_List_position@?$_Hash@V?$_Hmap_traits@KPAUSt_BodyCreate@@V?$hash_compare@KU?$less@K@std@@@stdext@@V?$allocator@U?$pair@$$CBKPAUSt_BodyCreate@@@std@@@std@@$0A@@stdext@@@stdext@@@1@@Z 1000cddf f i effectmanager.obj
 0001:0000bddf       ??0?$_Container_base_aux_alloc_real@V?$allocator@U_WZNCSPT@WzNaturalCubicSplineDyn@@@std@@@std@@IAE@V?$allocator@U_WZNCSPT@WzNaturalCubicSplineDyn@@@1@@Z 1000cddf f i Common_p:wznaturalcubicsplinedyn.obj
 0001:0000bddf       ??0?$_Container_base_aux_alloc_real@V?$allocator@PAUSt_SoundInfo@@@std@@@std@@IAE@V?$allocator@PAUSt_SoundInfo@@@1@@Z 1000cddf f i effectbody.obj
 0001:0000bddf       ??0?$_Container_base_aux_alloc_real@V?$allocator@PAUsEffectTexture@CEffectManager@@@std@@@std@@IAE@V?$allocator@PAUsEffectTexture@CEffectManager@@@1@@Z 1000cddf f i effectmanager.obj
 0001:0000bddf       ??0?$_Container_base_aux_alloc_real@V?$allocator@U?$pair@$$CBKV?$basic_string@DU?$char_traits@D@std@@V?$allocator@D@2@@std@@@std@@@std@@@std@@IAE@V?$allocator@U?$pair@$$CBKV?$basic_string@DU?$char_traits@D@std@@V?$allocator@D@2@@std@@@std@@@1@@Z 1000cddf f i loadmanager.obj
 0001:0000bddf       ??0?$_Container_base_aux_alloc_real@V?$allocator@USt_AutoCtlParam@@@std@@@std@@IAE@V?$allocator@USt_AutoCtlParam@@@1@@Z 1000cddf f i effectmanager.obj
 0001:0000bddf       ??0?$_Container_base_aux_alloc_real@V?$allocator@U?$pair@QAXPAVCEffectBody@@@std@@@std@@@std@@IAE@V?$allocator@U?$pair@QAXPAVCEffectBody@@@std@@@1@@Z 1000cddf f i effectmanager.obj
 0001:0000bddf       ??0?$_Container_base_aux_alloc_real@V?$allocator@U_List_position@?$_Hash@V?$_Hmap_traits@KV?$basic_string@DU?$char_traits@D@std@@V?$allocator@D@2@@std@@V?$hash_compare@KU?$less@K@std@@@stdext@@V?$allocator@U?$pair@$$CBKV?$basic_string@DU?$char_traits@D@std@@V?$allocator@D@2@@std@@@std@@@2@$0A@@stdext@@@stdext@@@std@@@std@@IAE@V?$allocator@U_List_position@?$_Hash@V?$_Hmap_traits@KV?$basic_string@DU?$char_traits@D@std@@V?$allocator@D@2@@std@@V?$hash_compare@KU?$less@K@std@@@stdext@@V?$allocator@U?$pair@$$CBKV?$basic_string@DU?$char_traits@D@std@@V?$allocator@D@2@@std@@@std@@@2@$0A@@stdext@@@stdext@@@1@@Z 1000cddf f i loadmanager.obj
 0001:0000bddf       ??0?$_Container_base_aux_alloc_real@V?$allocator@PAVCEElementSprite@@@std@@@std@@IAE@V?$allocator@PAVCEElementSprite@@@1@@Z 1000cddf f i eelementweather.obj
 0001:0000bddf       ??0?$_Container_base_aux_alloc_real@V?$allocator@U?$pair@$$CBJM@std@@@std@@@std@@IAE@V?$allocator@U?$pair@$$CBJM@std@@@1@@Z 1000cddf f i effectmanager.obj
 0001:0000bddf       ??0?$_Container_base_aux_alloc_real@V?$allocator@USt_EffLODParam@@@std@@@std@@IAE@V?$allocator@USt_EffLODParam@@@1@@Z 1000cddf f i effectmanager.obj
 0001:0000bddf       ??0?$_Container_base_aux_alloc_real@V?$allocator@K@std@@@std@@IAE@V?$allocator@K@1@@Z 1000cddf f i effectmanager.obj
 0001:0000bddf       ??0?$_Container_base_aux_alloc_real@V?$allocator@PAVCEElementBase@@@std@@@std@@IAE@V?$allocator@PAVCEElementBase@@@1@@Z 1000cddf f i effectbody.obj
 0001:0000bddf       ??0?$_Container_base_aux_alloc_real@V?$allocator@U_List_position@?$_Hash@V?$_Hmap_traits@PAXPAVCEffectBody@@V?$hash_compare@PAXU?$less@PAX@std@@@stdext@@V?$allocator@U?$pair@QAXPAVCEffectBody@@@std@@@std@@$0A@@stdext@@@stdext@@@std@@@std@@IAE@V?$allocator@U_List_position@?$_Hash@V?$_Hmap_traits@PAXPAVCEffectBody@@V?$hash_compare@PAXU?$less@PAX@std@@@stdext@@V?$allocator@U?$pair@QAXPAVCEffectBody@@@std@@@std@@$0A@@stdext@@@stdext@@@1@@Z 1000cddf f i effectmanager.obj
 0001:0000be5d       ?load_factor@?$_Hash@V?$_Hmap_traits@KPAUSt_BodyCreate@@V?$hash_compare@KU?$less@K@std@@@stdext@@V?$allocator@U?$pair@$$CBKPAUSt_BodyCreate@@@std@@@std@@$0A@@stdext@@@stdext@@QBEMXZ 1000ce5d f i effectmanager.obj
 0001:0000be5d       ?load_factor@?$_Hash@V?$_Hmap_traits@KV?$basic_string@DU?$char_traits@D@std@@V?$allocator@D@2@@std@@V?$hash_compare@KU?$less@K@std@@@stdext@@V?$allocator@U?$pair@$$CBKV?$basic_string@DU?$char_traits@D@std@@V?$allocator@D@2@@std@@@std@@@2@$0A@@stdext@@@stdext@@QBEMXZ 1000ce5d f i loadmanager.obj
 0001:0000be5d       ?load_factor@?$_Hash@V?$_Hmap_traits@PAXPAVCEffectBody@@V?$hash_compare@PAXU?$less@PAX@std@@@stdext@@V?$allocator@U?$pair@QAXPAVCEffectBody@@@std@@@std@@$0A@@stdext@@@stdext@@QBEMXZ 1000ce5d f i effectmanager.obj
 0001:0000be9c       ?_Reinsert@?$_Hash@V?$_Hmap_traits@KPAUSt_BodyCreate@@V?$hash_compare@KU?$less@K@std@@@stdext@@V?$allocator@U?$pair@$$CBKPAUSt_BodyCreate@@@std@@@std@@$0A@@stdext@@@stdext@@IAEXXZ 1000ce9c f i effectmanager.obj
 0001:0000be9c       ?_Reinsert@?$_Hash@V?$_Hmap_traits@PAXPAVCEffectBody@@V?$hash_compare@PAXU?$less@PAX@std@@@stdext@@V?$allocator@U?$pair@QAXPAVCEffectBody@@@std@@@std@@$0A@@stdext@@@stdext@@IAEXXZ 1000ce9c f i effectmanager.obj
 0001:0000bfa6       ??0?$vector@U_List_position@?$_Hash@V?$_Hmap_traits@PAXPAVCEffectBody@@V?$hash_compare@PAXU?$less@PAX@std@@@stdext@@V?$allocator@U?$pair@QAXPAVCEffectBody@@@std@@@std@@$0A@@stdext@@@stdext@@V?$allocator@U_List_position@?$_Hash@V?$_Hmap_traits@PAXPAVCEffectBody@@V?$hash_compare@PAXU?$less@PAX@std@@@stdext@@V?$allocator@U?$pair@QAXPAVCEffectBody@@@std@@@std@@$0A@@stdext@@@stdext@@@std@@@std@@QAE@ABV?$allocator@U_List_position@?$_Hash@V?$_Hmap_traits@PAXPAVCEffectBody@@V?$hash_compare@PAXU?$less@PAX@std@@@stdext@@V?$allocator@U?$pair@QAXPAVCEffectBody@@@std@@@std@@$0A@@stdext@@@stdext@@@1@@Z 1000cfa6 f i effectmanager.obj
 0001:0000bfa6       ??0?$vector@U_List_position@?$_Hash@V?$_Hmap_traits@KPAUSt_BodyCreate@@V?$hash_compare@KU?$less@K@std@@@stdext@@V?$allocator@U?$pair@$$CBKPAUSt_BodyCreate@@@std@@@std@@$0A@@stdext@@@stdext@@V?$allocator@U_List_position@?$_Hash@V?$_Hmap_traits@KPAUSt_BodyCreate@@V?$hash_compare@KU?$less@K@std@@@stdext@@V?$allocator@U?$pair@$$CBKPAUSt_BodyCreate@@@std@@@std@@$0A@@stdext@@@stdext@@@std@@@std@@QAE@ABV?$allocator@U_List_position@?$_Hash@V?$_Hmap_traits@KPAUSt_BodyCreate@@V?$hash_compare@KU?$less@K@std@@@stdext@@V?$allocator@U?$pair@$$CBKPAUSt_BodyCreate@@@std@@@std@@$0A@@stdext@@@stdext@@@1@@Z 1000cfa6 f i effectmanager.obj
 0001:0000bfa6       ??0?$vector@U_List_position@?$_Hash@V?$_Hmap_traits@KV?$basic_string@DU?$char_traits@D@std@@V?$allocator@D@2@@std@@V?$hash_compare@KU?$less@K@std@@@stdext@@V?$allocator@U?$pair@$$CBKV?$basic_string@DU?$char_traits@D@std@@V?$allocator@D@2@@std@@@std@@@2@$0A@@stdext@@@stdext@@V?$allocator@U_List_position@?$_Hash@V?$_Hmap_traits@KV?$basic_string@DU?$char_traits@D@std@@V?$allocator@D@2@@std@@V?$hash_compare@KU?$less@K@std@@@stdext@@V?$allocator@U?$pair@$$CBKV?$basic_string@DU?$char_traits@D@std@@V?$allocator@D@2@@std@@@std@@@2@$0A@@stdext@@@stdext@@@std@@@std@@QAE@ABV?$allocator@U_List_position@?$_Hash@V?$_Hmap_traits@KV?$basic_string@DU?$char_traits@D@std@@V?$allocator@D@2@@std@@V?$hash_compare@KU?$less@K@std@@@stdext@@V?$allocator@U?$pair@$$CBKV?$basic_string@DU?$char_traits@D@std@@V?$allocator@D@2@@std@@@std@@@2@$0A@@stdext@@@stdext@@@1@@Z 1000cfa6 f i loadmanager.obj
 0001:0000c02a       ??0?$list@U?$pair@QAXPAVCEffectBody@@@std@@V?$allocator@U?$pair@QAXPAVCEffectBody@@@std@@@2@@std@@QAE@ABV?$allocator@U?$pair@QAXPAVCEffectBody@@@std@@@1@@Z 1000d02a f i effectmanager.obj
 0001:0000c02a       ??0?$list@U?$pair@$$CBKPAUSt_BodyCreate@@@std@@V?$allocator@U?$pair@$$CBKPAUSt_BodyCreate@@@std@@@2@@std@@QAE@ABV?$allocator@U?$pair@$$CBKPAUSt_BodyCreate@@@std@@@1@@Z 1000d02a f i effectmanager.obj
 0001:0000c0a1       ?splice@?$list@U?$pair@QAXPAVCEffectBody@@@std@@V?$allocator@U?$pair@QAXPAVCEffectBody@@@std@@@2@@std@@QAEXV?$_Const_iterator@$00@12@AAV12@0@Z 1000d0a1 f i effectmanager.obj
 0001:0000c0a1       ?splice@?$list@U?$pair@$$CBKPAUSt_BodyCreate@@@std@@V?$allocator@U?$pair@$$CBKPAUSt_BodyCreate@@@std@@@2@@std@@QAEXV?$_Const_iterator@$00@12@AAV12@0@Z 1000d0a1 f i effectmanager.obj
 0001:0000c16b       ??G?$_Vector_const_iterator@PAUsEffectTexture@CEffectManager@@V?$allocator@PAUsEffectTexture@CEffectManager@@@std@@@std@@QBEHABV01@@Z 1000d16b f i effectmanager.obj
 0001:0000c16b       ??G?$_Vector_const_iterator@PAUSt_SoundInfo@@V?$allocator@PAUSt_SoundInfo@@@std@@@std@@QBEHABV01@@Z 1000d16b f i effectbody.obj
 0001:0000c16b       ??G?$_Vector_const_iterator@PAXV?$allocator@PAX@std@@@std@@QBEHABV01@@Z 1000d16b f i effectmanager.obj
 0001:0000c1b6       ?Create@?$CWzMemoryBand@VCEffectBody@@@@QAE_NH@Z 1000d1b6 f i effectmanager.obj
 0001:0000c33d       ??0_List_position@?$_Hash@V?$_Hmap_traits@KPAUSt_BodyCreate@@V?$hash_compare@KU?$less@K@std@@@stdext@@V?$allocator@U?$pair@$$CBKPAUSt_BodyCreate@@@std@@@std@@$0A@@stdext@@@stdext@@QAE@V?$_Iterator@$00@?$list@U?$pair@$$CBKPAUSt_BodyCreate@@@std@@V?$allocator@U?$pair@$$CBKPAUSt_BodyCreate@@@std@@@2@@std@@@Z 1000d33d f i effectmanager.obj
 0001:0000c33d       ??0_List_position@?$_Hash@V?$_Hmap_traits@KV?$basic_string@DU?$char_traits@D@std@@V?$allocator@D@2@@std@@V?$hash_compare@KU?$less@K@std@@@stdext@@V?$allocator@U?$pair@$$CBKV?$basic_string@DU?$char_traits@D@std@@V?$allocator@D@2@@std@@@std@@@2@$0A@@stdext@@@stdext@@QAE@V?$_Iterator@$00@?$list@U?$pair@$$CBKV?$basic_string@DU?$char_traits@D@std@@V?$allocator@D@2@@std@@@std@@V?$allocator@U?$pair@$$CBKV?$basic_string@DU?$char_traits@D@std@@V?$allocator@D@2@@std@@@std@@@2@@std@@@Z 1000d33d f i effectmanager.obj
 0001:0000c33d       ??0_List_position@?$_Hash@V?$_Hmap_traits@PAXPAVCEffectBody@@V?$hash_compare@PAXU?$less@PAX@std@@@stdext@@V?$allocator@U?$pair@QAXPAVCEffectBody@@@std@@@std@@$0A@@stdext@@@stdext@@QAE@V?$_Iterator@$00@?$list@U?$pair@QAXPAVCEffectBody@@@std@@V?$allocator@U?$pair@QAXPAVCEffectBody@@@std@@@2@@std@@@Z 1000d33d f i effectmanager.obj
 0001:0000c399       ??0length_error@std@@QAE@ABV01@@Z 1000d399 f i effectmanager.obj
 0001:0000c3bd       ??_ECEElementSprite@@UAEPAXI@Z 1000d3bd f i effectmanager.obj
 0001:0000c421       ??_ECEElementMesh@@UAEPAXI@Z 1000d421 f i effectmanager.obj
 0001:0000c485       ??_ECEElementChain@@UAEPAXI@Z 1000d485 f i effectmanager.obj
 0001:0000c4e9       ??_ECEElementFlatChain@@UAEPAXI@Z 1000d4e9 f i effectmanager.obj
 0001:0000c54d       ??_ECEElementDecal@@UAEPAXI@Z 1000d54d f i effectmanager.obj
 0001:0000c5b1       ??_ECEElementWeather@@UAEPAXI@Z 1000d5b1 f i effectmanager.obj
 0001:0000c615       ??_ECEffectBody@@UAEPAXI@Z 1000d615 f i effectmanager.obj
 0001:0000c679       ?_Inside@?$basic_string@DU?$char_traits@D@std@@V?$allocator@D@2@@std@@IAE_NPBD@Z 1000d679 f i effectmanager.obj
 0001:0000c6e4       ?_Buynode@?$_Tree@V?$_Tmap_traits@JUWzVector@@U?$less@J@std@@V?$allocator@U?$pair@$$CBJUWzVector@@@std@@@3@$0A@@std@@@std@@IAEPAU_Node@?$_Tree_nod@V?$_Tmap_traits@JUWzVector@@U?$less@J@std@@V?$allocator@U?$pair@$$CBJUWzVector@@@std@@@3@$0A@@std@@@2@XZ 1000d6e4 f i effectmanager.obj
 0001:0000c7fe       ?_Buynode@?$_Tree@V?$_Tmap_traits@JUWzVector@@U?$less@J@std@@V?$allocator@U?$pair@$$CBJUWzVector@@@std@@@3@$0A@@std@@@std@@IAEPAU_Node@?$_Tree_nod@V?$_Tmap_traits@JUWzVector@@U?$less@J@std@@V?$allocator@U?$pair@$$CBJUWzVector@@@std@@@3@$0A@@std@@@2@PAU342@00ABU?$pair@$$CBJUWzVector@@@2@D@Z 1000d7fe f i effectmanager.obj
 0001:0000c8cb       ?_Buynode@?$_Tree@V?$_Tmap_traits@JMU?$less@J@std@@V?$allocator@U?$pair@$$CBJM@std@@@2@$0A@@std@@@std@@IAEPAU_Node@?$_Tree_nod@V?$_Tmap_traits@JMU?$less@J@std@@V?$allocator@U?$pair@$$CBJM@std@@@2@$0A@@std@@@2@XZ 1000d8cb f i effectmanager.obj
 0001:0000c9e5       ?_Buynode@?$_Tree@V?$_Tmap_traits@JMU?$less@J@std@@V?$allocator@U?$pair@$$CBJM@std@@@2@$0A@@std@@@std@@IAEPAU_Node@?$_Tree_nod@V?$_Tmap_traits@JMU?$less@J@std@@V?$allocator@U?$pair@$$CBJM@std@@@2@$0A@@std@@@2@PAU342@00ABU?$pair@$$CBJM@2@D@Z 1000d9e5 f i effectmanager.obj
 0001:0000cab6       ??0?$_Tree_ptr@V?$_Tmap_traits@JMU?$less@J@std@@V?$allocator@U?$pair@$$CBJM@std@@@2@$0A@@std@@@std@@IAE@ABU?$less@J@1@V?$allocator@U?$pair@$$CBJM@std@@@1@@Z 1000dab6 f i effectmanager.obj
 0001:0000cab6       ??0?$_Tree_ptr@V?$_Tmap_traits@JUWzVector@@U?$less@J@std@@V?$allocator@U?$pair@$$CBJUWzVector@@@std@@@3@$0A@@std@@@std@@IAE@ABU?$less@J@1@V?$allocator@U?$pair@$$CBJUWzVector@@@std@@@1@@Z 1000dab6 f i effectmanager.obj
 0001:0000cafa       ?_Buy@?$vector@USt_AutoCtlParam@@V?$allocator@USt_AutoCtlParam@@@std@@@std@@IAE_NI@Z 1000dafa f i effectmanager.obj
 0001:0000cafa       ?_Buy@?$vector@U_WZNCSPT@WzNaturalCubicSplineDyn@@V?$allocator@U_WZNCSPT@WzNaturalCubicSplineDyn@@@std@@@std@@IAE_NI@Z 1000dafa f i Common_p:wznaturalcubicsplinedyn.obj
 0001:0000cafa       ?_Buy@?$vector@USt_EffLODParam@@V?$allocator@USt_EffLODParam@@@std@@@std@@IAE_NI@Z 1000dafa f i effectmanager.obj
 0001:0000cafa       ?_Buy@?$vector@U_List_position@?$_Hash@V?$_Hmap_traits@KPAUSt_BodyCreate@@V?$hash_compare@KU?$less@K@std@@@stdext@@V?$allocator@U?$pair@$$CBKPAUSt_BodyCreate@@@std@@@std@@$0A@@stdext@@@stdext@@V?$allocator@U_List_position@?$_Hash@V?$_Hmap_traits@KPAUSt_BodyCreate@@V?$hash_compare@KU?$less@K@std@@@stdext@@V?$allocator@U?$pair@$$CBKPAUSt_BodyCreate@@@std@@@std@@$0A@@stdext@@@stdext@@@std@@@std@@IAE_NI@Z 1000dafa f i effectmanager.obj
 0001:0000cafa       ?_Buy@?$vector@U_List_position@?$_Hash@V?$_Hmap_traits@PAXPAVCEffectBody@@V?$hash_compare@PAXU?$less@PAX@std@@@stdext@@V?$allocator@U?$pair@QAXPAVCEffectBody@@@std@@@std@@$0A@@stdext@@@stdext@@V?$allocator@U_List_position@?$_Hash@V?$_Hmap_traits@PAXPAVCEffectBody@@V?$hash_compare@PAXU?$less@PAX@std@@@stdext@@V?$allocator@U?$pair@QAXPAVCEffectBody@@@std@@@std@@$0A@@stdext@@@stdext@@@std@@@std@@IAE_NI@Z 1000dafa f i effectmanager.obj
 0001:0000cafa       ?_Buy@?$vector@U_List_position@?$_Hash@V?$_Hmap_traits@KV?$basic_string@DU?$char_traits@D@std@@V?$allocator@D@2@@std@@V?$hash_compare@KU?$less@K@std@@@stdext@@V?$allocator@U?$pair@$$CBKV?$basic_string@DU?$char_traits@D@std@@V?$allocator@D@2@@std@@@std@@@2@$0A@@stdext@@@stdext@@V?$allocator@U_List_position@?$_Hash@V?$_Hmap_traits@KV?$basic_string@DU?$char_traits@D@std@@V?$allocator@D@2@@std@@V?$hash_compare@KU?$less@K@std@@@stdext@@V?$allocator@U?$pair@$$CBKV?$basic_string@DU?$char_traits@D@std@@V?$allocator@D@2@@std@@@std@@@2@$0A@@stdext@@@stdext@@@std@@@std@@IAE_NI@Z 1000dafa f i loadmanager.obj
 0001:0000cbac       ?_Insert@?$list@U?$pair@QAXPAVCEffectBody@@@std@@V?$allocator@U?$pair@QAXPAVCEffectBody@@@std@@@2@@std@@QAEXV?$_Const_iterator@$00@12@ABU?$pair@QAXPAVCEffectBody@@@2@@Z 1000dbac f i effectmanager.obj
 0001:0000cbac       ?_Insert@?$list@U?$pair@$$CBKPAUSt_BodyCreate@@@std@@V?$allocator@U?$pair@$$CBKPAUSt_BodyCreate@@@std@@@2@@std@@QAEXV?$_Const_iterator@$00@12@ABU?$pair@$$CBKPAUSt_BodyCreate@@@2@@Z 1000dbac f i effectmanager.obj
 0001:0000cbfa       ?_Splice@?$list@U?$pair@$$CBKPAUSt_BodyCreate@@@std@@V?$allocator@U?$pair@$$CBKPAUSt_BodyCreate@@@std@@@2@@std@@QAEXV?$_Const_iterator@$00@12@AAV12@00I_N@Z 1000dbfa f i effectmanager.obj
 0001:0000cbfa       ?_Splice@?$list@U?$pair@QAXPAVCEffectBody@@@std@@V?$allocator@U?$pair@QAXPAVCEffectBody@@@std@@@2@@std@@QAEXV?$_Const_iterator@$00@12@AAV12@00I_N@Z 1000dbfa f i effectmanager.obj
 0001:0000cd83       ?_Buynode@?$list@U?$pair@QAXPAVCEffectBody@@@std@@V?$allocator@U?$pair@QAXPAVCEffectBody@@@std@@@2@@std@@IAEPAU_Node@?$_List_nod@U?$pair@QAXPAVCEffectBody@@@std@@V?$allocator@U?$pair@QAXPAVCEffectBody@@@std@@@2@@2@XZ 1000dd83 f i effectmanager.obj
 0001:0000cd83       ?_Buynode@?$list@U?$pair@$$CBKPAUSt_BodyCreate@@@std@@V?$allocator@U?$pair@$$CBKPAUSt_BodyCreate@@@std@@@2@@std@@IAEPAU_Node@?$_List_nod@U?$pair@$$CBKPAUSt_BodyCreate@@@std@@V?$allocator@U?$pair@$$CBKPAUSt_BodyCreate@@@std@@@2@@2@XZ 1000dd83 f i effectmanager.obj
 0001:0000ce65       ?_Assign_n@?$vector@U_List_position@?$_Hash@V?$_Hmap_traits@PAXPAVCEffectBody@@V?$hash_compare@PAXU?$less@PAX@std@@@stdext@@V?$allocator@U?$pair@QAXPAVCEffectBody@@@std@@@std@@$0A@@stdext@@@stdext@@V?$allocator@U_List_position@?$_Hash@V?$_Hmap_traits@PAXPAVCEffectBody@@V?$hash_compare@PAXU?$less@PAX@std@@@stdext@@V?$allocator@U?$pair@QAXPAVCEffectBody@@@std@@@std@@$0A@@stdext@@@stdext@@@std@@@std@@IAEXIABU_List_position@?$_Hash@V?$_Hmap_traits@PAXPAVCEffectBody@@V?$hash_compare@PAXU?$less@PAX@std@@@stdext@@V?$allocator@U?$pair@QAXPAVCEffectBody@@@std@@@std@@$0A@@stdext@@@stdext@@@Z 1000de65 f i effectmanager.obj
 0001:0000ce65       ?_Assign_n@?$vector@U_List_position@?$_Hash@V?$_Hmap_traits@KV?$basic_string@DU?$char_traits@D@std@@V?$allocator@D@2@@std@@V?$hash_compare@KU?$less@K@std@@@stdext@@V?$allocator@U?$pair@$$CBKV?$basic_string@DU?$char_traits@D@std@@V?$allocator@D@2@@std@@@std@@@2@$0A@@stdext@@@stdext@@V?$allocator@U_List_position@?$_Hash@V?$_Hmap_traits@KV?$basic_string@DU?$char_traits@D@std@@V?$allocator@D@2@@std@@V?$hash_compare@KU?$less@K@std@@@stdext@@V?$allocator@U?$pair@$$CBKV?$basic_string@DU?$char_traits@D@std@@V?$allocator@D@2@@std@@@std@@@2@$0A@@stdext@@@stdext@@@std@@@std@@IAEXIABU_List_position@?$_Hash@V?$_Hmap_traits@KV?$basic_string@DU?$char_traits@D@std@@V?$allocator@D@2@@std@@V?$hash_compare@KU?$less@K@std@@@stdext@@V?$allocator@U?$pair@$$CBKV?$basic_string@DU?$char_traits@D@std@@V?$allocator@D@2@@std@@@std@@@2@$0A@@stdext@@@stdext@@@Z 1000de65 f i effectmanager.obj
 0001:0000ce65       ?_Assign_n@?$vector@U_List_position@?$_Hash@V?$_Hmap_traits@KPAUSt_BodyCreate@@V?$hash_compare@KU?$less@K@std@@@stdext@@V?$allocator@U?$pair@$$CBKPAUSt_BodyCreate@@@std@@@std@@$0A@@stdext@@@stdext@@V?$allocator@U_List_position@?$_Hash@V?$_Hmap_traits@KPAUSt_BodyCreate@@V?$hash_compare@KU?$less@K@std@@@stdext@@V?$allocator@U?$pair@$$CBKPAUSt_BodyCreate@@@std@@@std@@$0A@@stdext@@@stdext@@@std@@@std@@IAEXIABU_List_position@?$_Hash@V?$_Hmap_traits@KPAUSt_BodyCreate@@V?$hash_compare@KU?$less@K@std@@@stdext@@V?$allocator@U?$pair@$$CBKPAUSt_BodyCreate@@@std@@@std@@$0A@@stdext@@@stdext@@@Z 1000de65 f i effectmanager.obj
 0001:0000cef2       ??F?$_Const_iterator@$00@?$list@KV?$allocator@K@std@@@std@@QAEAAV012@XZ 1000def2 f i effectmanager.obj
 0001:0000cef2       ??F?$_Const_iterator@$00@?$list@U?$pair@$$CBKPAUSt_BodyCreate@@@std@@V?$allocator@U?$pair@$$CBKPAUSt_BodyCreate@@@std@@@2@@std@@QAEAAV012@XZ 1000def2 f i effectmanager.obj
 0001:0000cef2       ??F?$_Const_iterator@$00@?$list@U?$pair@QAXPAVCEffectBody@@@std@@V?$allocator@U?$pair@QAXPAVCEffectBody@@@std@@@2@@std@@QAEAAV012@XZ 1000def2 f i effectmanager.obj
 0001:0000cef2       ??F?$_Const_iterator@$00@?$list@U?$pair@$$CBKV?$basic_string@DU?$char_traits@D@std@@V?$allocator@D@2@@std@@@std@@V?$allocator@U?$pair@$$CBKV?$basic_string@DU?$char_traits@D@std@@V?$allocator@D@2@@std@@@std@@@2@@std@@QAEAAV012@XZ 1000def2 f i loadmanager.obj
 0001:0000cf6f       ??Y?$_Vector_const_iterator@USt_EffLODParam@@V?$allocator@USt_EffLODParam@@@std@@@std@@QAEAAV01@H@Z 1000df6f f i effectmanager.obj
 0001:0000cf6f       ??Y?$_Vector_const_iterator@U_WZNCSPT@WzNaturalCubicSplineDyn@@V?$allocator@U_WZNCSPT@WzNaturalCubicSplineDyn@@@std@@@std@@QAEAAV01@H@Z 1000df6f f i Common_p:wznaturalcubicsplinedyn.obj
 0001:0000cf6f       ??Y?$_Vector_const_iterator@USt_AutoCtlParam@@V?$allocator@USt_AutoCtlParam@@@std@@@std@@QAEAAV01@H@Z 1000df6f f i effectmanager.obj
 0001:0000d025       ??Y?$_Vector_const_iterator@PAUsEffectTexture@CEffectManager@@V?$allocator@PAUsEffectTexture@CEffectManager@@@std@@@std@@QAEAAV01@H@Z 1000e025 f i effectmanager.obj
 0001:0000d025       ??Y?$_Vector_const_iterator@PAXV?$allocator@PAX@std@@@std@@QAEAAV01@H@Z 1000e025 f i effectmanager.obj
 0001:0000d025       ??Y?$_Vector_const_iterator@PAUSt_SoundInfo@@V?$allocator@PAUSt_SoundInfo@@@std@@@std@@QAEAAV01@H@Z 1000e025 f i effectbody.obj
 0001:0000d0db       ?erase@?$list@U?$pair@QAXPAVCEffectBody@@@std@@V?$allocator@U?$pair@QAXPAVCEffectBody@@@std@@@2@@std@@QAE?AV?$_Iterator@$00@12@V?$_Const_iterator@$00@12@0@Z 1000e0db f i effectmanager.obj
 0001:0000d0db       ?erase@?$list@U?$pair@$$CBKPAUSt_BodyCreate@@@std@@V?$allocator@U?$pair@$$CBKPAUSt_BodyCreate@@@std@@@2@@std@@QAE?AV?$_Iterator@$00@12@V?$_Const_iterator@$00@12@0@Z 1000e0db f i effectmanager.obj
 0001:0000d233       ?_Buynode@?$list@U?$pair@QAXPAVCEffectBody@@@std@@V?$allocator@U?$pair@QAXPAVCEffectBody@@@std@@@2@@std@@IAEPAU_Node@?$_List_nod@U?$pair@QAXPAVCEffectBody@@@std@@V?$allocator@U?$pair@QAXPAVCEffectBody@@@std@@@2@@2@PAU342@0ABU?$pair@QAXPAVCEffectBody@@@2@@Z 1000e233 f i effectmanager.obj
 0001:0000d233       ?_Buynode@?$list@U?$pair@$$CBKPAUSt_BodyCreate@@@std@@V?$allocator@U?$pair@$$CBKPAUSt_BodyCreate@@@std@@@2@@std@@IAEPAU_Node@?$_List_nod@U?$pair@$$CBKPAUSt_BodyCreate@@@std@@V?$allocator@U?$pair@$$CBKPAUSt_BodyCreate@@@std@@@2@@2@PAU342@0ABU?$pair@$$CBKPAUSt_BodyCreate@@@2@@Z 1000e233 f i effectmanager.obj
 0001:0000d33d       ?_Incsize@?$list@U?$pair@QAXPAVCEffectBody@@@std@@V?$allocator@U?$pair@QAXPAVCEffectBody@@@std@@@2@@std@@IAEXI@Z 1000e33d f i effectmanager.obj
 0001:0000d33d       ?_Incsize@?$list@U?$pair@$$CBKPAUSt_BodyCreate@@@std@@V?$allocator@U?$pair@$$CBKPAUSt_BodyCreate@@@std@@@2@@std@@IAEXI@Z 1000e33d f i effectmanager.obj
 0001:0000d407       ?begin@?$vector@PAUSt_SoundInfo@@V?$allocator@PAUSt_SoundInfo@@@std@@@std@@QAE?AV?$_Vector_iterator@PAUSt_SoundInfo@@V?$allocator@PAUSt_SoundInfo@@@std@@@2@XZ 1000e407 f i effectbody.obj
 0001:0000d407       ?begin@?$vector@PAUsEffectTexture@CEffectManager@@V?$allocator@PAUsEffectTexture@CEffectManager@@@std@@@std@@QAE?AV?$_Vector_iterator@PAUsEffectTexture@CEffectManager@@V?$allocator@PAUsEffectTexture@CEffectManager@@@std@@@2@XZ 1000e407 f i effectmanager.obj
 0001:0000d407       ?begin@?$vector@USt_AutoCtlParam@@V?$allocator@USt_AutoCtlParam@@@std@@@std@@QAE?AV?$_Vector_iterator@USt_AutoCtlParam@@V?$allocator@USt_AutoCtlParam@@@std@@@2@XZ 1000e407 f i effectmanager.obj
 0001:0000d407       ?begin@?$vector@U_List_position@?$_Hash@V?$_Hmap_traits@KV?$basic_string@DU?$char_traits@D@std@@V?$allocator@D@2@@std@@V?$hash_compare@KU?$less@K@std@@@stdext@@V?$allocator@U?$pair@$$CBKV?$basic_string@DU?$char_traits@D@std@@V?$allocator@D@2@@std@@@std@@@2@$0A@@stdext@@@stdext@@V?$allocator@U_List_position@?$_Hash@V?$_Hmap_traits@KV?$basic_string@DU?$char_traits@D@std@@V?$allocator@D@2@@std@@V?$hash_compare@KU?$less@K@std@@@stdext@@V?$allocator@U?$pair@$$CBKV?$basic_string@DU?$char_traits@D@std@@V?$allocator@D@2@@std@@@std@@@2@$0A@@stdext@@@stdext@@@std@@@std@@QAE?AV?$_Vector_iterator@U_List_position@?$_Hash@V?$_Hmap_traits@KV?$basic_string@DU?$char_traits@D@std@@V?$allocator@D@2@@std@@V?$hash_compare@KU?$less@K@std@@@stdext@@V?$allocator@U?$pair@$$CBKV?$basic_string@DU?$char_traits@D@std@@V?$allocator@D@2@@std@@@std@@@2@$0A@@stdext@@@stdext@@V?$allocator@U_List_position@?$_Hash@V?$_Hmap_traits@KV?$basic_string@DU?$char_traits@D@std@@V?$allocator@D@2@@std@@V?$hash_compare@KU?$less@K@std@@@stdext@@V?$allocator@U?$pair@$$CBKV?$basic_string@DU?$char_traits@D@std@@V?$allocator@D@2@@std@@@std@@@2@$0A@@stdext@@@stdext@@@std@@@2@XZ 1000e407 f i effectmanager.obj
 0001:0000d407       ?begin@?$vector@U_WZNCSPT@WzNaturalCubicSplineDyn@@V?$allocator@U_WZNCSPT@WzNaturalCubicSplineDyn@@@std@@@std@@QAE?AV?$_Vector_iterator@U_WZNCSPT@WzNaturalCubicSplineDyn@@V?$allocator@U_WZNCSPT@WzNaturalCubicSplineDyn@@@std@@@2@XZ 1000e407 f i Common_p:wznaturalcubicsplinedyn.obj
 0001:0000d407       ?begin@?$vector@U_List_position@?$_Hash@V?$_Hmap_traits@PAXPAVCEffectBody@@V?$hash_compare@PAXU?$less@PAX@std@@@stdext@@V?$allocator@U?$pair@QAXPAVCEffectBody@@@std@@@std@@$0A@@stdext@@@stdext@@V?$allocator@U_List_position@?$_Hash@V?$_Hmap_traits@PAXPAVCEffectBody@@V?$hash_compare@PAXU?$less@PAX@std@@@stdext@@V?$allocator@U?$pair@QAXPAVCEffectBody@@@std@@@std@@$0A@@stdext@@@stdext@@@std@@@std@@QAE?AV?$_Vector_iterator@U_List_position@?$_Hash@V?$_Hmap_traits@PAXPAVCEffectBody@@V?$hash_compare@PAXU?$less@PAX@std@@@stdext@@V?$allocator@U?$pair@QAXPAVCEffectBody@@@std@@@std@@$0A@@stdext@@@stdext@@V?$allocator@U_List_position@?$_Hash@V?$_Hmap_traits@PAXPAVCEffectBody@@V?$hash_compare@PAXU?$less@PAX@std@@@stdext@@V?$allocator@U?$pair@QAXPAVCEffectBody@@@std@@@std@@$0A@@stdext@@@stdext@@@std@@@2@XZ 1000e407 f i effectmanager.obj
 0001:0000d407       ?begin@?$vector@PAXV?$allocator@PAX@std@@@std@@QBE?AV?$_Vector_const_iterator@PAXV?$allocator@PAX@std@@@2@XZ 1000e407 f i effectmanager.obj
 0001:0000d407       ?begin@?$vector@PAXV?$allocator@PAX@std@@@std@@QAE?AV?$_Vector_iterator@PAXV?$allocator@PAX@std@@@2@XZ 1000e407 f i effectmanager.obj
 0001:0000d407       ?begin@?$vector@U_List_position@?$_Hash@V?$_Hmap_traits@KPAUSt_BodyCreate@@V?$hash_compare@KU?$less@K@std@@@stdext@@V?$allocator@U?$pair@$$CBKPAUSt_BodyCreate@@@std@@@std@@$0A@@stdext@@@stdext@@V?$allocator@U_List_position@?$_Hash@V?$_Hmap_traits@KPAUSt_BodyCreate@@V?$hash_compare@KU?$less@K@std@@@stdext@@V?$allocator@U?$pair@$$CBKPAUSt_BodyCreate@@@std@@@std@@$0A@@stdext@@@stdext@@@std@@@std@@QAE?AV?$_Vector_iterator@U_List_position@?$_Hash@V?$_Hmap_traits@KPAUSt_BodyCreate@@V?$hash_compare@KU?$less@K@std@@@stdext@@V?$allocator@U?$pair@$$CBKPAUSt_BodyCreate@@@std@@@std@@$0A@@stdext@@@stdext@@V?$allocator@U_List_position@?$_Hash@V?$_Hmap_traits@KPAUSt_BodyCreate@@V?$hash_compare@KU?$less@K@std@@@stdext@@V?$allocator@U?$pair@$$CBKPAUSt_BodyCreate@@@std@@@std@@$0A@@stdext@@@stdext@@@std@@@2@XZ 1000e407 f i effectmanager.obj
 0001:0000d407       ?begin@?$vector@USt_EffLODParam@@V?$allocator@USt_EffLODParam@@@std@@@std@@QAE?AV?$_Vector_iterator@USt_EffLODParam@@V?$allocator@USt_EffLODParam@@@std@@@2@XZ 1000e407 f i effectmanager.obj
 0001:0000d45d       ?_Insert_n@?$vector@USt_AutoCtlParam@@V?$allocator@USt_AutoCtlParam@@@std@@@std@@IAEXV?$_Vector_const_iterator@USt_AutoCtlParam@@V?$allocator@USt_AutoCtlParam@@@std@@@2@IABUSt_AutoCtlParam@@@Z 1000e45d f i effectmanager.obj
 0001:0000d45d       ?_Insert_n@?$vector@U_WZNCSPT@WzNaturalCubicSplineDyn@@V?$allocator@U_WZNCSPT@WzNaturalCubicSplineDyn@@@std@@@std@@IAEXV?$_Vector_const_iterator@U_WZNCSPT@WzNaturalCubicSplineDyn@@V?$allocator@U_WZNCSPT@WzNaturalCubicSplineDyn@@@std@@@2@IABU_WZNCSPT@WzNaturalCubicSplineDyn@@@Z 1000e45d f i Common_p:wznaturalcubicsplinedyn.obj
 0001:0000d45d       ?_Insert_n@?$vector@USt_EffLODParam@@V?$allocator@USt_EffLODParam@@@std@@@std@@IAEXV?$_Vector_const_iterator@USt_EffLODParam@@V?$allocator@USt_EffLODParam@@@std@@@2@IABUSt_EffLODParam@@@Z 1000e45d f i effectmanager.obj
 0001:0000d45d       ?_Insert_n@?$vector@U_List_position@?$_Hash@V?$_Hmap_traits@KPAUSt_BodyCreate@@V?$hash_compare@KU?$less@K@std@@@stdext@@V?$allocator@U?$pair@$$CBKPAUSt_BodyCreate@@@std@@@std@@$0A@@stdext@@@stdext@@V?$allocator@U_List_position@?$_Hash@V?$_Hmap_traits@KPAUSt_BodyCreate@@V?$hash_compare@KU?$less@K@std@@@stdext@@V?$allocator@U?$pair@$$CBKPAUSt_BodyCreate@@@std@@@std@@$0A@@stdext@@@stdext@@@std@@@std@@IAEXV?$_Vector_const_iterator@U_List_position@?$_Hash@V?$_Hmap_traits@KPAUSt_BodyCreate@@V?$hash_compare@KU?$less@K@std@@@stdext@@V?$allocator@U?$pair@$$CBKPAUSt_BodyCreate@@@std@@@std@@$0A@@stdext@@@stdext@@V?$allocator@U_List_position@?$_Hash@V?$_Hmap_traits@KPAUSt_BodyCreate@@V?$hash_compare@KU?$less@K@std@@@stdext@@V?$allocator@U?$pair@$$CBKPAUSt_BodyCreate@@@std@@@std@@$0A@@stdext@@@stdext@@@std@@@2@IABU_List_position@?$_Hash@V?$_Hmap_traits@KPAUSt_BodyCreate@@V?$hash_compare@KU?$less@K@std@@@stdext@@V?$allocator@U?$pair@$$CBKPAUSt_BodyCreate@@@std@@@std@@$0A@@stdext@@@stdext@@@Z 1000e45d f i effectmanager.obj
 0001:0000d45d       ?_Insert_n@?$vector@U_List_position@?$_Hash@V?$_Hmap_traits@KV?$basic_string@DU?$char_traits@D@std@@V?$allocator@D@2@@std@@V?$hash_compare@KU?$less@K@std@@@stdext@@V?$allocator@U?$pair@$$CBKV?$basic_string@DU?$char_traits@D@std@@V?$allocator@D@2@@std@@@std@@@2@$0A@@stdext@@@stdext@@V?$allocator@U_List_position@?$_Hash@V?$_Hmap_traits@KV?$basic_string@DU?$char_traits@D@std@@V?$allocator@D@2@@std@@V?$hash_compare@KU?$less@K@std@@@stdext@@V?$allocator@U?$pair@$$CBKV?$basic_string@DU?$char_traits@D@std@@V?$allocator@D@2@@std@@@std@@@2@$0A@@stdext@@@stdext@@@std@@@std@@IAEXV?$_Vector_const_iterator@U_List_position@?$_Hash@V?$_Hmap_traits@KV?$basic_string@DU?$char_traits@D@std@@V?$allocator@D@2@@std@@V?$hash_compare@KU?$less@K@std@@@stdext@@V?$allocator@U?$pair@$$CBKV?$basic_string@DU?$char_traits@D@std@@V?$allocator@D@2@@std@@@std@@@2@$0A@@stdext@@@stdext@@V?$allocator@U_List_position@?$_Hash@V?$_Hmap_traits@KV?$basic_string@DU?$char_traits@D@std@@V?$allocator@D@2@@std@@V?$hash_compare@KU?$less@K@std@@@stdext@@V?$allocator@U?$pair@$$CBKV?$basic_string@DU?$char_traits@D@std@@V?$allocator@D@2@@std@@@std@@@2@$0A@@stdext@@@stdext@@@std@@@2@IABU_List_position@?$_Hash@V?$_Hmap_traits@KV?$basic_string@DU?$char_traits@D@std@@V?$allocator@D@2@@std@@V?$hash_compare@KU?$less@K@std@@@stdext@@V?$allocator@U?$pair@$$CBKV?$basic_string@DU?$char_traits@D@std@@V?$allocator@D@2@@std@@@std@@@2@$0A@@stdext@@@stdext@@@Z 1000e45d f i effectmanager.obj
 0001:0000d45d       ?_Insert_n@?$vector@U_List_position@?$_Hash@V?$_Hmap_traits@PAXPAVCEffectBody@@V?$hash_compare@PAXU?$less@PAX@std@@@stdext@@V?$allocator@U?$pair@QAXPAVCEffectBody@@@std@@@std@@$0A@@stdext@@@stdext@@V?$allocator@U_List_position@?$_Hash@V?$_Hmap_traits@PAXPAVCEffectBody@@V?$hash_compare@PAXU?$less@PAX@std@@@stdext@@V?$allocator@U?$pair@QAXPAVCEffectBody@@@std@@@std@@$0A@@stdext@@@stdext@@@std@@@std@@IAEXV?$_Vector_const_iterator@U_List_position@?$_Hash@V?$_Hmap_traits@PAXPAVCEffectBody@@V?$hash_compare@PAXU?$less@PAX@std@@@stdext@@V?$allocator@U?$pair@QAXPAVCEffectBody@@@std@@@std@@$0A@@stdext@@@stdext@@V?$allocator@U_List_position@?$_Hash@V?$_Hmap_traits@PAXPAVCEffectBody@@V?$hash_compare@PAXU?$less@PAX@std@@@stdext@@V?$allocator@U?$pair@QAXPAVCEffectBody@@@std@@@std@@$0A@@stdext@@@stdext@@@std@@@2@IABU_List_position@?$_Hash@V?$_Hmap_traits@PAXPAVCEffectBody@@V?$hash_compare@PAXU?$less@PAX@std@@@stdext@@V?$allocator@U?$pair@QAXPAVCEffectBody@@@std@@@std@@$0A@@stdext@@@stdext@@@Z 1000e45d f i effectmanager.obj
 0001:0000db4d       ??0?$CWzHandleManager@PAVCEffectBody@@@@QAE@XZ 1000eb4d f i effectmanager.obj
 0001:0000dbd7       ??1?$CWzHandleManager@PAVCEffectBody@@@@UAE@XZ 1000ebd7 f i effectmanager.obj
 0001:0000dc43       ?Clear@?$CWzHandleManager@PAVCEffectBody@@@@QAEXXZ 1000ec43 f i effectmanager.obj
 0001:0000dc89       ?Add@?$CWzHandleManager@PAVCEffectBody@@@@QAEPAXABQAVCEffectBody@@@Z 1000ec89 f i effectmanager.obj
 0001:0000dd5d       ?Release@?$CWzHandleManager@PAVCEffectBody@@@@QAEHPAX@Z 1000ed5d f i effectmanager.obj
 0001:0000de09       ??0St_BodyCreate@@QAE@XZ   1000ee09 f i effectmanager.obj
 0001:0000df49       ??1St_BodyCreate@@QAE@XZ   1000ef49 f i effectmanager.obj
 0001:0000e09f       ??$assign@V?$_Const_iterator@$00@?$list@KV?$allocator@K@std@@@std@@@?$list@KV?$allocator@K@std@@@std@@QAEXV?$_Const_iterator@$00@01@0@Z 1000f09f f i effectmanager.obj
 0001:0000e12c       ??$_Umove@PAU_List_position@?$_Hash@V?$_Hmap_traits@KV?$basic_string@DU?$char_traits@D@std@@V?$allocator@D@2@@std@@V?$hash_compare@KU?$less@K@std@@@stdext@@V?$allocator@U?$pair@$$CBKV?$basic_string@DU?$char_traits@D@std@@V?$allocator@D@2@@std@@@std@@@2@$0A@@stdext@@@stdext@@@?$vector@U_List_position@?$_Hash@V?$_Hmap_traits@KV?$basic_string@DU?$char_traits@D@std@@V?$allocator@D@2@@std@@V?$hash_compare@KU?$less@K@std@@@stdext@@V?$allocator@U?$pair@$$CBKV?$basic_string@DU?$char_traits@D@std@@V?$allocator@D@2@@std@@@std@@@2@$0A@@stdext@@@stdext@@V?$allocator@U_List_position@?$_Hash@V?$_Hmap_traits@KV?$basic_string@DU?$char_traits@D@std@@V?$allocator@D@2@@std@@V?$hash_compare@KU?$less@K@std@@@stdext@@V?$allocator@U?$pair@$$CBKV?$basic_string@DU?$char_traits@D@std@@V?$allocator@D@2@@std@@@std@@@2@$0A@@stdext@@@stdext@@@std@@@std@@IAEPAU_List_position@?$_Hash@V?$_Hmap_traits@KV?$basic_string@DU?$char_traits@D@std@@V?$allocator@D@2@@std@@V?$hash_compare@KU?$less@K@std@@@stdext@@V?$allocator@U?$pair@$$CBKV?$basic_string@DU?$char_traits@D@std@@V?$allocator@D@2@@std@@@std@@@2@$0A@@stdext@@@stdext@@PAU234@00@Z 1000f12c f i effectmanager.obj
 0001:0000e12c       ??$_Umove@PAUSt_EffLODParam@@@?$vector@USt_EffLODParam@@V?$allocator@USt_EffLODParam@@@std@@@std@@IAEPAUSt_EffLODParam@@PAU2@00@Z 1000f12c f i effectmanager.obj
 0001:0000e12c       ??$_Umove@PAU_List_position@?$_Hash@V?$_Hmap_traits@PAXPAVCEffectBody@@V?$hash_compare@PAXU?$less@PAX@std@@@stdext@@V?$allocator@U?$pair@QAXPAVCEffectBody@@@std@@@std@@$0A@@stdext@@@stdext@@@?$vector@U_List_position@?$_Hash@V?$_Hmap_traits@PAXPAVCEffectBody@@V?$hash_compare@PAXU?$less@PAX@std@@@stdext@@V?$allocator@U?$pair@QAXPAVCEffectBody@@@std@@@std@@$0A@@stdext@@@stdext@@V?$allocator@U_List_position@?$_Hash@V?$_Hmap_traits@PAXPAVCEffectBody@@V?$hash_compare@PAXU?$less@PAX@std@@@stdext@@V?$allocator@U?$pair@QAXPAVCEffectBody@@@std@@@std@@$0A@@stdext@@@stdext@@@std@@@std@@IAEPAU_List_position@?$_Hash@V?$_Hmap_traits@PAXPAVCEffectBody@@V?$hash_compare@PAXU?$less@PAX@std@@@stdext@@V?$allocator@U?$pair@QAXPAVCEffectBody@@@std@@@std@@$0A@@stdext@@@stdext@@PAU234@00@Z 1000f12c f i effectmanager.obj
 0001:0000e12c       ??$_Umove@PAU_WZNCSPT@WzNaturalCubicSplineDyn@@@?$vector@U_WZNCSPT@WzNaturalCubicSplineDyn@@V?$allocator@U_WZNCSPT@WzNaturalCubicSplineDyn@@@std@@@std@@IAEPAU_WZNCSPT@WzNaturalCubicSplineDyn@@PAU23@00@Z 1000f12c f i Common_p:wznaturalcubicsplinedyn.obj
 0001:0000e12c       ??$_Umove@PAU_List_position@?$_Hash@V?$_Hmap_traits@KPAUSt_BodyCreate@@V?$hash_compare@KU?$less@K@std@@@stdext@@V?$allocator@U?$pair@$$CBKPAUSt_BodyCreate@@@std@@@std@@$0A@@stdext@@@stdext@@@?$vector@U_List_position@?$_Hash@V?$_Hmap_traits@KPAUSt_BodyCreate@@V?$hash_compare@KU?$less@K@std@@@stdext@@V?$allocator@U?$pair@$$CBKPAUSt_BodyCreate@@@std@@@std@@$0A@@stdext@@@stdext@@V?$allocator@U_List_position@?$_Hash@V?$_Hmap_traits@KPAUSt_BodyCreate@@V?$hash_compare@KU?$less@K@std@@@stdext@@V?$allocator@U?$pair@$$CBKPAUSt_BodyCreate@@@std@@@std@@$0A@@stdext@@@stdext@@@std@@@std@@IAEPAU_List_position@?$_Hash@V?$_Hmap_traits@KPAUSt_BodyCreate@@V?$hash_compare@KU?$less@K@std@@@stdext@@V?$allocator@U?$pair@$$CBKPAUSt_BodyCreate@@@std@@@std@@$0A@@stdext@@@stdext@@PAU234@00@Z 1000f12c f i effectmanager.obj
 0001:0000e12c       ??$_Umove@PAUSt_AutoCtlParam@@@?$vector@USt_AutoCtlParam@@V?$allocator@USt_AutoCtlParam@@@std@@@std@@IAEPAUSt_AutoCtlParam@@PAU2@00@Z 1000f12c f i effectmanager.obj
 0001:0000e151       ??$_Unchecked_move_backward@PAPAUsEffectTexture@CEffectManager@@PAPAU12@@stdext@@YAPAPAUsEffectTexture@CEffectManager@@PAPAU12@00@Z 1000f151 f i effectmanager.obj
 0001:0000e151       ??$_Unchecked_move_backward@PAPAUSt_SoundInfo@@PAPAU1@@stdext@@YAPAPAUSt_SoundInfo@@PAPAU1@00@Z 1000f151 f i effectbody.obj
 0001:0000e151       ??$_Unchecked_move_backward@PAPAXPAPAX@stdext@@YAPAPAXPAPAX00@Z 1000f151 f i effectmanager.obj
 0001:0000e1e8       ??$_Umove@PAPAUsEffectTexture@CEffectManager@@@?$vector@PAUsEffectTexture@CEffectManager@@V?$allocator@PAUsEffectTexture@CEffectManager@@@std@@@std@@IAEPAPAUsEffectTexture@CEffectManager@@PAPAU23@00@Z 1000f1e8 f i effectmanager.obj
 0001:0000e1e8       ??$_Umove@PAPAX@?$vector@PAXV?$allocator@PAX@std@@@std@@IAEPAPAXPAPAX00@Z 1000f1e8 f i effectmanager.obj
 0001:0000e1e8       ??$_Umove@PAPAUSt_SoundInfo@@@?$vector@PAUSt_SoundInfo@@V?$allocator@PAUSt_SoundInfo@@@std@@@std@@IAEPAPAUSt_SoundInfo@@PAPAU2@00@Z 1000f1e8 f i effectbody.obj
 0001:0000e245       ??$_Allocate@U_Node@?$_Tree_nod@V?$_Tmap_traits@JUWzVector@@U?$less@J@std@@V?$allocator@U?$pair@$$CBJUWzVector@@@std@@@3@$0A@@std@@@std@@@std@@YAPAU_Node@?$_Tree_nod@V?$_Tmap_traits@JUWzVector@@U?$less@J@std@@V?$allocator@U?$pair@$$CBJUWzVector@@@std@@@3@$0A@@std@@@0@IPAU120@@Z 1000f245 f i effectmanager.obj
 0001:0000e298       ??$_Allocate@U_Node@?$_Tree_nod@V?$_Tmap_traits@JMU?$less@J@std@@V?$allocator@U?$pair@$$CBJM@std@@@2@$0A@@std@@@std@@@std@@YAPAU_Node@?$_Tree_nod@V?$_Tmap_traits@JMU?$less@J@std@@V?$allocator@U?$pair@$$CBJM@std@@@2@$0A@@std@@@0@IPAU120@@Z 1000f298 f i effectmanager.obj
 0001:0000e2eb       ??$unchecked_copy@PAU_List_position@?$_Hash@V?$_Hmap_traits@PAXPAVCEffectBody@@V?$hash_compare@PAXU?$less@PAX@std@@@stdext@@V?$allocator@U?$pair@QAXPAVCEffectBody@@@std@@@std@@$0A@@stdext@@@stdext@@PAU123@@stdext@@YAPAU_List_position@?$_Hash@V?$_Hmap_traits@PAXPAVCEffectBody@@V?$hash_compare@PAXU?$less@PAX@std@@@stdext@@V?$allocator@U?$pair@QAXPAVCEffectBody@@@std@@@std@@$0A@@stdext@@@0@PAU120@00@Z 1000f2eb f i effectmanager.obj
 0001:0000e2eb       ??$unchecked_copy@PAU_WZNCSPT@WzNaturalCubicSplineDyn@@PAU12@@stdext@@YAPAU_WZNCSPT@WzNaturalCubicSplineDyn@@PAU12@00@Z 1000f2eb f i Common_p:wznaturalcubicsplinedyn.obj
 0001:0000e2eb       ??$unchecked_copy@PAU_List_position@?$_Hash@V?$_Hmap_traits@KV?$basic_string@DU?$char_traits@D@std@@V?$allocator@D@2@@std@@V?$hash_compare@KU?$less@K@std@@@stdext@@V?$allocator@U?$pair@$$CBKV?$basic_string@DU?$char_traits@D@std@@V?$allocator@D@2@@std@@@std@@@2@$0A@@stdext@@@stdext@@PAU123@@stdext@@YAPAU_List_position@?$_Hash@V?$_Hmap_traits@KV?$basic_string@DU?$char_traits@D@std@@V?$allocator@D@2@@std@@V?$hash_compare@KU?$less@K@std@@@stdext@@V?$allocator@U?$pair@$$CBKV?$basic_string@DU?$char_traits@D@std@@V?$allocator@D@2@@std@@@std@@@2@$0A@@stdext@@@0@PAU120@00@Z 1000f2eb f i effectmanager.obj
 0001:0000e2eb       ??$unchecked_copy@PAUSt_AutoCtlParam@@PAU1@@stdext@@YAPAUSt_AutoCtlParam@@PAU1@00@Z 1000f2eb f i effectmanager.obj
 0001:0000e2eb       ??$unchecked_copy@PAUSt_EffLODParam@@PAU1@@stdext@@YAPAUSt_EffLODParam@@PAU1@00@Z 1000f2eb f i effectmanager.obj
 0001:0000e2eb       ??$unchecked_copy@PAU_List_position@?$_Hash@V?$_Hmap_traits@KPAUSt_BodyCreate@@V?$hash_compare@KU?$less@K@std@@@stdext@@V?$allocator@U?$pair@$$CBKPAUSt_BodyCreate@@@std@@@std@@$0A@@stdext@@@stdext@@PAU123@@stdext@@YAPAU_List_position@?$_Hash@V?$_Hmap_traits@KPAUSt_BodyCreate@@V?$hash_compare@KU?$less@K@std@@@stdext@@V?$allocator@U?$pair@$$CBKPAUSt_BodyCreate@@@std@@@std@@$0A@@stdext@@@0@PAU120@00@Z 1000f2eb f i effectmanager.obj
 0001:0000e386       ??$_Allocate@USt_EffLODParam@@@std@@YAPAUSt_EffLODParam@@IPAU1@@Z 1000f386 f i effectmanager.obj
 0001:0000e386       ??$_Allocate@U_List_position@?$_Hash@V?$_Hmap_traits@PAXPAVCEffectBody@@V?$hash_compare@PAXU?$less@PAX@std@@@stdext@@V?$allocator@U?$pair@QAXPAVCEffectBody@@@std@@@std@@$0A@@stdext@@@stdext@@@std@@YAPAU_List_position@?$_Hash@V?$_Hmap_traits@PAXPAVCEffectBody@@V?$hash_compare@PAXU?$less@PAX@std@@@stdext@@V?$allocator@U?$pair@QAXPAVCEffectBody@@@std@@@std@@$0A@@stdext@@@stdext@@IPAU123@@Z 1000f386 f i effectmanager.obj
 0001:0000e386       ??$_Allocate@U_WZNCSPT@WzNaturalCubicSplineDyn@@@std@@YAPAU_WZNCSPT@WzNaturalCubicSplineDyn@@IPAU12@@Z 1000f386 f i Common_p:wznaturalcubicsplinedyn.obj
 0001:0000e386       ??$_Allocate@U_List_position@?$_Hash@V?$_Hmap_traits@KPAUSt_BodyCreate@@V?$hash_compare@KU?$less@K@std@@@stdext@@V?$allocator@U?$pair@$$CBKPAUSt_BodyCreate@@@std@@@std@@$0A@@stdext@@@stdext@@@std@@YAPAU_List_position@?$_Hash@V?$_Hmap_traits@KPAUSt_BodyCreate@@V?$hash_compare@KU?$less@K@std@@@stdext@@V?$allocator@U?$pair@$$CBKPAUSt_BodyCreate@@@std@@@std@@$0A@@stdext@@@stdext@@IPAU123@@Z 1000f386 f i effectmanager.obj
 0001:0000e386       ??$_Allocate@U_List_position@?$_Hash@V?$_Hmap_traits@KV?$basic_string@DU?$char_traits@D@std@@V?$allocator@D@2@@std@@V?$hash_compare@KU?$less@K@std@@@stdext@@V?$allocator@U?$pair@$$CBKV?$basic_string@DU?$char_traits@D@std@@V?$allocator@D@2@@std@@@std@@@2@$0A@@stdext@@@stdext@@@std@@YAPAU_List_position@?$_Hash@V?$_Hmap_traits@KV?$basic_string@DU?$char_traits@D@std@@V?$allocator@D@2@@std@@V?$hash_compare@KU?$less@K@std@@@stdext@@V?$allocator@U?$pair@$$CBKV?$basic_string@DU?$char_traits@D@std@@V?$allocator@D@2@@std@@@std@@@2@$0A@@stdext@@@stdext@@IPAU123@@Z 1000f386 f i effectmanager.obj
 0001:0000e386       ??$_Allocate@USt_AutoCtlParam@@@std@@YAPAUSt_AutoCtlParam@@IPAU1@@Z 1000f386 f i effectmanager.obj
 0001:0000e3d9       ??$_Allocate@U_Node@?$_List_nod@U?$pair@QAXPAVCEffectBody@@@std@@V?$allocator@U?$pair@QAXPAVCEffectBody@@@std@@@2@@std@@@std@@YAPAU_Node@?$_List_nod@U?$pair@QAXPAVCEffectBody@@@std@@V?$allocator@U?$pair@QAXPAVCEffectBody@@@std@@@2@@0@IPAU120@@Z 1000f3d9 f i effectmanager.obj
 0001:0000e3d9       ??$_Allocate@U_Node@?$_List_nod@U?$pair@$$CBKPAUSt_BodyCreate@@@std@@V?$allocator@U?$pair@$$CBKPAUSt_BodyCreate@@@std@@@2@@std@@@std@@YAPAU_Node@?$_List_nod@U?$pair@$$CBKPAUSt_BodyCreate@@@std@@V?$allocator@U?$pair@$$CBKPAUSt_BodyCreate@@@std@@@2@@0@IPAU120@@Z 1000f3d9 f i effectmanager.obj
 0001:0000e42c       ??_G?$CWzHandleManager@PAVCEffectBody@@@@UAEPAXI@Z 1000f42c f i effectmanager.obj
 0001:0000e42c       ??_E?$CWzHandleManager@PAVCEffectBody@@@@UAEPAXI@Z 1000f42c f i effectmanager.obj
 0001:0000e453       ??_G_Node@?$_List_nod@U?$pair@$$CBKV?$basic_string@DU?$char_traits@D@std@@V?$allocator@D@2@@std@@@std@@V?$allocator@U?$pair@$$CBKV?$basic_string@DU?$char_traits@D@std@@V?$allocator@D@2@@std@@@std@@@2@@std@@QAEPAXI@Z 1000f453 f i effectmanager.obj
 0001:0000e48c       ??0?$CWzArray@G@@QAE@XZ    1000f48c f i effectmanager.obj
 0001:0000e4f4       ??1?$CWzArray@USt_DAFileInfo@@@@QAE@XZ 1000f4f4 f i ProgramCommonLibForEngine_p:discaccess.obj
 0001:0000e4f4       ??1?$CWzArray@G@@QAE@XZ    1000f4f4 f i effectmanager.obj
 0001:0000e4f4       ??1?$CWzArray@PAVCEffectBody@@@@QAE@XZ 1000f4f4 f i effectmanager.obj
 0001:0000e505       ?Clear@?$CWzArray@G@@QAEXXZ 1000f505 f i effectmanager.obj
 0001:0000e52d       ?Set@?$CWzArray@G@@QAEXHABG@Z 1000f52d f i effectmanager.obj
 0001:0000e57b       ?Get@?$CWzArray@G@@QBEAAGH@Z 1000f57b f i effectmanager.obj
 0001:0000e5c2       ??0?$CWzArray@PAVCEffectBody@@@@QAE@XZ 1000f5c2 f i effectmanager.obj
 0001:0000e62a       ?Clear@?$CWzArray@PAVCEffectBody@@@@QAEXXZ 1000f62a f i effectmanager.obj
 0001:0000e653       ?Set@?$CWzArray@PAVCEffectBody@@@@QAEXHABQAVCEffectBody@@@Z 1000f653 f i effectmanager.obj
 0001:0000e69f       ??$_Unchecked_uninitialized_move@PAU_WZNCSPT@WzNaturalCubicSplineDyn@@PAU12@V?$allocator@U_WZNCSPT@WzNaturalCubicSplineDyn@@@std@@@stdext@@YAPAU_WZNCSPT@WzNaturalCubicSplineDyn@@PAU12@00AAV?$allocator@U_WZNCSPT@WzNaturalCubicSplineDyn@@@std@@@Z 1000f69f f i Common_p:wznaturalcubicsplinedyn.obj
 0001:0000e69f       ??$_Unchecked_uninitialized_move@PAU_List_position@?$_Hash@V?$_Hmap_traits@KV?$basic_string@DU?$char_traits@D@std@@V?$allocator@D@2@@std@@V?$hash_compare@KU?$less@K@std@@@stdext@@V?$allocator@U?$pair@$$CBKV?$basic_string@DU?$char_traits@D@std@@V?$allocator@D@2@@std@@@std@@@2@$0A@@stdext@@@stdext@@PAU123@V?$allocator@U_List_position@?$_Hash@V?$_Hmap_traits@KV?$basic_string@DU?$char_traits@D@std@@V?$allocator@D@2@@std@@V?$hash_compare@KU?$less@K@std@@@stdext@@V?$allocator@U?$pair@$$CBKV?$basic_string@DU?$char_traits@D@std@@V?$allocator@D@2@@std@@@std@@@2@$0A@@stdext@@@stdext@@@std@@@stdext@@YAPAU_List_position@?$_Hash@V?$_Hmap_traits@KV?$basic_string@DU?$char_traits@D@std@@V?$allocator@D@2@@std@@V?$hash_compare@KU?$less@K@std@@@stdext@@V?$allocator@U?$pair@$$CBKV?$basic_string@DU?$char_traits@D@std@@V?$allocator@D@2@@std@@@std@@@2@$0A@@stdext@@@0@PAU120@00AAV?$allocator@U_List_position@?$_Hash@V?$_Hmap_traits@KV?$basic_string@DU?$char_traits@D@std@@V?$allocator@D@2@@std@@V?$hash_compare@KU?$less@K@std@@@stdext@@V?$allocator@U?$pair@$$CBKV?$basic_string@DU?$char_traits@D@std@@V?$allocator@D@2@@std@@@std@@@2@$0A@@stdext@@@stdext@@@std@@@Z 1000f69f f i effectmanager.obj
 0001:0000e69f       ??$_Unchecked_uninitialized_move@PAUSt_AutoCtlParam@@PAU1@V?$allocator@USt_AutoCtlParam@@@std@@@stdext@@YAPAUSt_AutoCtlParam@@PAU1@00AAV?$allocator@USt_AutoCtlParam@@@std@@@Z 1000f69f f i effectmanager.obj
 0001:0000e69f       ??$_Unchecked_uninitialized_move@PAU_List_position@?$_Hash@V?$_Hmap_traits@PAXPAVCEffectBody@@V?$hash_compare@PAXU?$less@PAX@std@@@stdext@@V?$allocator@U?$pair@QAXPAVCEffectBody@@@std@@@std@@$0A@@stdext@@@stdext@@PAU123@V?$allocator@U_List_position@?$_Hash@V?$_Hmap_traits@PAXPAVCEffectBody@@V?$hash_compare@PAXU?$less@PAX@std@@@stdext@@V?$allocator@U?$pair@QAXPAVCEffectBody@@@std@@@std@@$0A@@stdext@@@stdext@@@std@@@stdext@@YAPAU_List_position@?$_Hash@V?$_Hmap_traits@PAXPAVCEffectBody@@V?$hash_compare@PAXU?$less@PAX@std@@@stdext@@V?$allocator@U?$pair@QAXPAVCEffectBody@@@std@@@std@@$0A@@stdext@@@0@PAU120@00AAV?$allocator@U_List_position@?$_Hash@V?$_Hmap_traits@PAXPAVCEffectBody@@V?$hash_compare@PAXU?$less@PAX@std@@@stdext@@V?$allocator@U?$pair@QAXPAVCEffectBody@@@std@@@std@@$0A@@stdext@@@stdext@@@std@@@Z 1000f69f f i effectmanager.obj
 0001:0000e69f       ??$_Unchecked_uninitialized_move@PAU_List_position@?$_Hash@V?$_Hmap_traits@KPAUSt_BodyCreate@@V?$hash_compare@KU?$less@K@std@@@stdext@@V?$allocator@U?$pair@$$CBKPAUSt_BodyCreate@@@std@@@std@@$0A@@stdext@@@stdext@@PAU123@V?$allocator@U_List_position@?$_Hash@V?$_Hmap_traits@KPAUSt_BodyCreate@@V?$hash_compare@KU?$less@K@std@@@stdext@@V?$allocator@U?$pair@$$CBKPAUSt_BodyCreate@@@std@@@std@@$0A@@stdext@@@stdext@@@std@@@stdext@@YAPAU_List_position@?$_Hash@V?$_Hmap_traits@KPAUSt_BodyCreate@@V?$hash_compare@KU?$less@K@std@@@stdext@@V?$allocator@U?$pair@$$CBKPAUSt_BodyCreate@@@std@@@std@@$0A@@stdext@@@0@PAU120@00AAV?$allocator@U_List_position@?$_Hash@V?$_Hmap_traits@KPAUSt_BodyCreate@@V?$hash_compare@KU?$less@K@std@@@stdext@@V?$allocator@U?$pair@$$CBKPAUSt_BodyCreate@@@std@@@std@@$0A@@stdext@@@stdext@@@std@@@Z 1000f69f f i effectmanager.obj
 0001:0000e69f       ??$_Unchecked_uninitialized_move@PAUSt_EffLODParam@@PAU1@V?$allocator@USt_EffLODParam@@@std@@@stdext@@YAPAUSt_EffLODParam@@PAU1@00AAV?$allocator@USt_EffLODParam@@@std@@@Z 1000f69f f i effectmanager.obj
 0001:0000e711       ??$_Move_backward_opt@PAU_List_position@?$_Hash@V?$_Hmap_traits@PAXPAVCEffectBody@@V?$hash_compare@PAXU?$less@PAX@std@@@stdext@@V?$allocator@U?$pair@QAXPAVCEffectBody@@@std@@@std@@$0A@@stdext@@@stdext@@PAU123@Urandom_access_iterator_tag@std@@U_Undefined_move_tag@5@@std@@YAPAU_List_position@?$_Hash@V?$_Hmap_traits@PAXPAVCEffectBody@@V?$hash_compare@PAXU?$less@PAX@std@@@stdext@@V?$allocator@U?$pair@QAXPAVCEffectBody@@@std@@@std@@$0A@@stdext@@@stdext@@PAU123@00Urandom_access_iterator_tag@0@U_Undefined_move_tag@0@U_Range_checked_iterator_tag@0@@Z 1000f711 f i effectmanager.obj
 0001:0000e711       ??$_Move_backward_opt@PAU_List_position@?$_Hash@V?$_Hmap_traits@KV?$basic_string@DU?$char_traits@D@std@@V?$allocator@D@2@@std@@V?$hash_compare@KU?$less@K@std@@@stdext@@V?$allocator@U?$pair@$$CBKV?$basic_string@DU?$char_traits@D@std@@V?$allocator@D@2@@std@@@std@@@2@$0A@@stdext@@@stdext@@PAU123@Urandom_access_iterator_tag@std@@U_Undefined_move_tag@5@@std@@YAPAU_List_position@?$_Hash@V?$_Hmap_traits@KV?$basic_string@DU?$char_traits@D@std@@V?$allocator@D@2@@std@@V?$hash_compare@KU?$less@K@std@@@stdext@@V?$allocator@U?$pair@$$CBKV?$basic_string@DU?$char_traits@D@std@@V?$allocator@D@2@@std@@@std@@@2@$0A@@stdext@@@stdext@@PAU123@00Urandom_access_iterator_tag@0@U_Undefined_move_tag@0@U_Range_checked_iterator_tag@0@@Z 1000f711 f i effectmanager.obj
 0001:0000e711       ??$_Move_backward_opt@PAUSt_EffLODParam@@PAU1@Urandom_access_iterator_tag@std@@U_Undefined_move_tag@3@@std@@YAPAUSt_EffLODParam@@PAU1@00Urandom_access_iterator_tag@0@U_Undefined_move_tag@0@U_Range_checked_iterator_tag@0@@Z 1000f711 f i effectmanager.obj
 0001:0000e711       ??$_Move_backward_opt@PAUSt_AutoCtlParam@@PAU1@Urandom_access_iterator_tag@std@@U_Undefined_move_tag@3@@std@@YAPAUSt_AutoCtlParam@@PAU1@00Urandom_access_iterator_tag@0@U_Undefined_move_tag@0@U_Range_checked_iterator_tag@0@@Z 1000f711 f i effectmanager.obj
 0001:0000e711       ??$_Move_backward_opt@PAU_WZNCSPT@WzNaturalCubicSplineDyn@@PAU12@Urandom_access_iterator_tag@std@@U_Undefined_move_tag@4@@std@@YAPAU_WZNCSPT@WzNaturalCubicSplineDyn@@PAU12@00Urandom_access_iterator_tag@0@U_Undefined_move_tag@0@U_Range_checked_iterator_tag@0@@Z 1000f711 f i Common_p:wznaturalcubicsplinedyn.obj
 0001:0000e711       ??$_Move_backward_opt@PAU_List_position@?$_Hash@V?$_Hmap_traits@KPAUSt_BodyCreate@@V?$hash_compare@KU?$less@K@std@@@stdext@@V?$allocator@U?$pair@$$CBKPAUSt_BodyCreate@@@std@@@std@@$0A@@stdext@@@stdext@@PAU123@Urandom_access_iterator_tag@std@@U_Undefined_move_tag@5@@std@@YAPAU_List_position@?$_Hash@V?$_Hmap_traits@KPAUSt_BodyCreate@@V?$hash_compare@KU?$less@K@std@@@stdext@@V?$allocator@U?$pair@$$CBKPAUSt_BodyCreate@@@std@@@std@@$0A@@stdext@@@stdext@@PAU123@00Urandom_access_iterator_tag@0@U_Undefined_move_tag@0@U_Range_checked_iterator_tag@0@@Z 1000f711 f i effectmanager.obj
 0001:0000e7a0       ??$_Uninit_fill_n@PAU_List_position@?$_Hash@V?$_Hmap_traits@KPAUSt_BodyCreate@@V?$hash_compare@KU?$less@K@std@@@stdext@@V?$allocator@U?$pair@$$CBKPAUSt_BodyCreate@@@std@@@std@@$0A@@stdext@@@stdext@@IU123@V?$allocator@U_List_position@?$_Hash@V?$_Hmap_traits@KPAUSt_BodyCreate@@V?$hash_compare@KU?$less@K@std@@@stdext@@V?$allocator@U?$pair@$$CBKPAUSt_BodyCreate@@@std@@@std@@$0A@@stdext@@@stdext@@@std@@@std@@YAXPAU_List_position@?$_Hash@V?$_Hmap_traits@KPAUSt_BodyCreate@@V?$hash_compare@KU?$less@K@std@@@stdext@@V?$allocator@U?$pair@$$CBKPAUSt_BodyCreate@@@std@@@std@@$0A@@stdext@@@stdext@@IABU123@AAV?$allocator@U_List_position@?$_Hash@V?$_Hmap_traits@KPAUSt_BodyCreate@@V?$hash_compare@KU?$less@K@std@@@stdext@@V?$allocator@U?$pair@$$CBKPAUSt_BodyCreate@@@std@@@std@@$0A@@stdext@@@stdext@@@0@U_Nonscalar_ptr_iterator_tag@0@U_Range_checked_iterator_tag@0@@Z 1000f7a0 f i effectmanager.obj
 0001:0000e7a0       ??$_Uninit_fill_n@PAUSt_AutoCtlParam@@IU1@V?$allocator@USt_AutoCtlParam@@@std@@@std@@YAXPAUSt_AutoCtlParam@@IABU1@AAV?$allocator@USt_AutoCtlParam@@@0@U_Nonscalar_ptr_iterator_tag@0@U_Range_checked_iterator_tag@0@@Z 1000f7a0 f i effectmanager.obj
 0001:0000e7a0       ??$_Uninit_fill_n@PAUSt_EffLODParam@@IU1@V?$allocator@USt_EffLODParam@@@std@@@std@@YAXPAUSt_EffLODParam@@IABU1@AAV?$allocator@USt_EffLODParam@@@0@U_Nonscalar_ptr_iterator_tag@0@U_Range_checked_iterator_tag@0@@Z 1000f7a0 f i effectmanager.obj
 0001:0000e7a0       ??$_Uninit_fill_n@PAU_WZNCSPT@WzNaturalCubicSplineDyn@@IU12@V?$allocator@U_WZNCSPT@WzNaturalCubicSplineDyn@@@std@@@std@@YAXPAU_WZNCSPT@WzNaturalCubicSplineDyn@@IABU12@AAV?$allocator@U_WZNCSPT@WzNaturalCubicSplineDyn@@@0@U_Nonscalar_ptr_iterator_tag@0@U_Range_checked_iterator_tag@0@@Z 1000f7a0 f i Common_p:wznaturalcubicsplinedyn.obj
 0001:0000e7a0       ??$_Uninit_fill_n@PAU_List_position@?$_Hash@V?$_Hmap_traits@PAXPAVCEffectBody@@V?$hash_compare@PAXU?$less@PAX@std@@@stdext@@V?$allocator@U?$pair@QAXPAVCEffectBody@@@std@@@std@@$0A@@stdext@@@stdext@@IU123@V?$allocator@U_List_position@?$_Hash@V?$_Hmap_traits@PAXPAVCEffectBody@@V?$hash_compare@PAXU?$less@PAX@std@@@stdext@@V?$allocator@U?$pair@QAXPAVCEffectBody@@@std@@@std@@$0A@@stdext@@@stdext@@@std@@@std@@YAXPAU_List_position@?$_Hash@V?$_Hmap_traits@PAXPAVCEffectBody@@V?$hash_compare@PAXU?$less@PAX@std@@@stdext@@V?$allocator@U?$pair@QAXPAVCEffectBody@@@std@@@std@@$0A@@stdext@@@stdext@@IABU123@AAV?$allocator@U_List_position@?$_Hash@V?$_Hmap_traits@PAXPAVCEffectBody@@V?$hash_compare@PAXU?$less@PAX@std@@@stdext@@V?$allocator@U?$pair@QAXPAVCEffectBody@@@std@@@std@@$0A@@stdext@@@stdext@@@0@U_Nonscalar_ptr_iterator_tag@0@U_Range_checked_iterator_tag@0@@Z 1000f7a0 f i effectmanager.obj
 0001:0000e7a0       ??$_Uninit_fill_n@PAU_List_position@?$_Hash@V?$_Hmap_traits@KV?$basic_string@DU?$char_traits@D@std@@V?$allocator@D@2@@std@@V?$hash_compare@KU?$less@K@std@@@stdext@@V?$allocator@U?$pair@$$CBKV?$basic_string@DU?$char_traits@D@std@@V?$allocator@D@2@@std@@@std@@@2@$0A@@stdext@@@stdext@@IU123@V?$allocator@U_List_position@?$_Hash@V?$_Hmap_traits@KV?$basic_string@DU?$char_traits@D@std@@V?$allocator@D@2@@std@@V?$hash_compare@KU?$less@K@std@@@stdext@@V?$allocator@U?$pair@$$CBKV?$basic_string@DU?$char_traits@D@std@@V?$allocator@D@2@@std@@@std@@@2@$0A@@stdext@@@stdext@@@std@@@std@@YAXPAU_List_position@?$_Hash@V?$_Hmap_traits@KV?$basic_string@DU?$char_traits@D@std@@V?$allocator@D@2@@std@@V?$hash_compare@KU?$less@K@std@@@stdext@@V?$allocator@U?$pair@$$CBKV?$basic_string@DU?$char_traits@D@std@@V?$allocator@D@2@@std@@@std@@@2@$0A@@stdext@@@stdext@@IABU123@AAV?$allocator@U_List_position@?$_Hash@V?$_Hmap_traits@KV?$basic_string@DU?$char_traits@D@std@@V?$allocator@D@2@@std@@V?$hash_compare@KU?$less@K@std@@@stdext@@V?$allocator@U?$pair@$$CBKV?$basic_string@DU?$char_traits@D@std@@V?$allocator@D@2@@std@@@std@@@2@$0A@@stdext@@@stdext@@@0@U_Nonscalar_ptr_iterator_tag@0@U_Range_checked_iterator_tag@0@@Z 1000f7a0 f i effectmanager.obj
 0001:0000e85c       ??$_Unchecked_uninitialized_move@PAPAXPAPAXV?$allocator@PAX@std@@@stdext@@YAPAPAXPAPAX00AAV?$allocator@PAX@std@@@Z 1000f85c f i effectmanager.obj
 0001:0000e85c       ??$_Unchecked_uninitialized_move@PAPAUSt_SoundInfo@@PAPAU1@V?$allocator@PAUSt_SoundInfo@@@std@@@stdext@@YAPAPAUSt_SoundInfo@@PAPAU1@00AAV?$allocator@PAUSt_SoundInfo@@@std@@@Z 1000f85c f i effectbody.obj
 0001:0000e85c       ??$_Unchecked_uninitialized_move@PAPAUsEffectTexture@CEffectManager@@PAPAU12@V?$allocator@PAUsEffectTexture@CEffectManager@@@std@@@stdext@@YAPAPAUsEffectTexture@CEffectManager@@PAPAU12@00AAV?$allocator@PAUsEffectTexture@CEffectManager@@@std@@@Z 1000f85c f i effectmanager.obj
 0001:0000e89e       ??$_Insert@V?$_Const_iterator@$00@?$list@U?$pair@$$CBKPAUSt_BodyCreate@@@std@@V?$allocator@U?$pair@$$CBKPAUSt_BodyCreate@@@std@@@2@@std@@@?$list@U?$pair@$$CBKPAUSt_BodyCreate@@@std@@V?$allocator@U?$pair@$$CBKPAUSt_BodyCreate@@@std@@@2@@std@@QAEXV?$_Const_iterator@$00@01@00Uforward_iterator_tag@1@@Z 1000f89e f i effectmanager.obj
 0001:0000e89e       ??$_Insert@V?$_Const_iterator@$00@?$list@U?$pair@QAXPAVCEffectBody@@@std@@V?$allocator@U?$pair@QAXPAVCEffectBody@@@std@@@2@@std@@@?$list@U?$pair@QAXPAVCEffectBody@@@std@@V?$allocator@U?$pair@QAXPAVCEffectBody@@@std@@@2@@std@@QAEXV?$_Const_iterator@$00@01@00Uforward_iterator_tag@1@@Z 1000f89e f i effectmanager.obj
 0001:0000e9b3       ?MakeSureDimensionSize@?$CWzArray@G@@AAEXH@Z 1000f9b3 f i effectmanager.obj
 0001:0000ea7f       ?Release@?$CWzArray@G@@AAEXXZ 1000fa7f f i effectmanager.obj
 0001:0000ea7f       ?Release@?$CWzArray@USt_DAFileInfo@@@@AAEXXZ 1000fa7f f i ProgramCommonLibForEngine_p:discaccess.obj
 0001:0000ea7f       ?Release@?$CWzArray@PAVCEffectBody@@@@AAEXXZ 1000fa7f f i effectmanager.obj
 0001:0000eab8       ?MakeSureDimensionSize@?$CWzArray@PAVCEffectBody@@@@AAEXH@Z 1000fab8 f i effectmanager.obj
 0001:0000eb86       ??$_Insert@V?$_Const_iterator@$00@?$list@KV?$allocator@K@std@@@std@@@?$list@KV?$allocator@K@std@@@std@@QAEXV?$_Const_iterator@$00@01@00Uforward_iterator_tag@1@@Z 1000fb86 f i effectmanager.obj
 0001:0000ec9b       ??$unchecked_uninitialized_copy@PAPAXPAPAXV?$allocator@PAX@std@@@stdext@@YAPAPAXPAPAX00AAV?$allocator@PAX@std@@@Z 1000fc9b f i effectmanager.obj
 0001:0000ec9b       ??$unchecked_uninitialized_copy@PAPAUSt_SoundInfo@@PAPAU1@V?$allocator@PAUSt_SoundInfo@@@std@@@stdext@@YAPAPAUSt_SoundInfo@@PAPAU1@00AAV?$allocator@PAUSt_SoundInfo@@@std@@@Z 1000fc9b f i effectbody.obj
 0001:0000ec9b       ??$unchecked_uninitialized_copy@PAPAUsEffectTexture@CEffectManager@@PAPAU12@V?$allocator@PAUsEffectTexture@CEffectManager@@@std@@@stdext@@YAPAPAUsEffectTexture@CEffectManager@@PAPAU12@00AAV?$allocator@PAUsEffectTexture@CEffectManager@@@std@@@Z 1000fc9b f i effectmanager.obj
 0001:0000ed06       ??$_Uninit_copy@PAUSt_EffLODParam@@PAU1@V?$allocator@USt_EffLODParam@@@std@@@std@@YAPAUSt_EffLODParam@@PAU1@00AAV?$allocator@USt_EffLODParam@@@0@U_Nonscalar_ptr_iterator_tag@0@U_Range_checked_iterator_tag@0@@Z 1000fd06 f i effectmanager.obj
 0001:0000ed06       ??$_Uninit_copy@PAU_List_position@?$_Hash@V?$_Hmap_traits@KV?$basic_string@DU?$char_traits@D@std@@V?$allocator@D@2@@std@@V?$hash_compare@KU?$less@K@std@@@stdext@@V?$allocator@U?$pair@$$CBKV?$basic_string@DU?$char_traits@D@std@@V?$allocator@D@2@@std@@@std@@@2@$0A@@stdext@@@stdext@@PAU123@V?$allocator@U_List_position@?$_Hash@V?$_Hmap_traits@KV?$basic_string@DU?$char_traits@D@std@@V?$allocator@D@2@@std@@V?$hash_compare@KU?$less@K@std@@@stdext@@V?$allocator@U?$pair@$$CBKV?$basic_string@DU?$char_traits@D@std@@V?$allocator@D@2@@std@@@std@@@2@$0A@@stdext@@@stdext@@@std@@@std@@YAPAU_List_position@?$_Hash@V?$_Hmap_traits@KV?$basic_string@DU?$char_traits@D@std@@V?$allocator@D@2@@std@@V?$hash_compare@KU?$less@K@std@@@stdext@@V?$allocator@U?$pair@$$CBKV?$basic_string@DU?$char_traits@D@std@@V?$allocator@D@2@@std@@@std@@@2@$0A@@stdext@@@stdext@@PAU123@00AAV?$allocator@U_List_position@?$_Hash@V?$_Hmap_traits@KV?$basic_string@DU?$char_traits@D@std@@V?$allocator@D@2@@std@@V?$hash_compare@KU?$less@K@std@@@stdext@@V?$allocator@U?$pair@$$CBKV?$basic_string@DU?$char_traits@D@std@@V?$allocator@D@2@@std@@@std@@@2@$0A@@stdext@@@stdext@@@0@U_Nonscalar_ptr_iterator_tag@0@U_Range_checked_iterator_tag@0@@Z 1000fd06 f i effectmanager.obj
 0001:0000ed06       ??$_Uninit_copy@PAU_List_position@?$_Hash@V?$_Hmap_traits@KPAUSt_BodyCreate@@V?$hash_compare@KU?$less@K@std@@@stdext@@V?$allocator@U?$pair@$$CBKPAUSt_BodyCreate@@@std@@@std@@$0A@@stdext@@@stdext@@PAU123@V?$allocator@U_List_position@?$_Hash@V?$_Hmap_traits@KPAUSt_BodyCreate@@V?$hash_compare@KU?$less@K@std@@@stdext@@V?$allocator@U?$pair@$$CBKPAUSt_BodyCreate@@@std@@@std@@$0A@@stdext@@@stdext@@@std@@@std@@YAPAU_List_position@?$_Hash@V?$_Hmap_traits@KPAUSt_BodyCreate@@V?$hash_compare@KU?$less@K@std@@@stdext@@V?$allocator@U?$pair@$$CBKPAUSt_BodyCreate@@@std@@@std@@$0A@@stdext@@@stdext@@PAU123@00AAV?$allocator@U_List_position@?$_Hash@V?$_Hmap_traits@KPAUSt_BodyCreate@@V?$hash_compare@KU?$less@K@std@@@stdext@@V?$allocator@U?$pair@$$CBKPAUSt_BodyCreate@@@std@@@std@@$0A@@stdext@@@stdext@@@0@U_Nonscalar_ptr_iterator_tag@0@U_Range_checked_iterator_tag@0@@Z 1000fd06 f i effectmanager.obj
 0001:0000ed06       ??$_Uninit_copy@PAU_List_position@?$_Hash@V?$_Hmap_traits@PAXPAVCEffectBody@@V?$hash_compare@PAXU?$less@PAX@std@@@stdext@@V?$allocator@U?$pair@QAXPAVCEffectBody@@@std@@@std@@$0A@@stdext@@@stdext@@PAU123@V?$allocator@U_List_position@?$_Hash@V?$_Hmap_traits@PAXPAVCEffectBody@@V?$hash_compare@PAXU?$less@PAX@std@@@stdext@@V?$allocator@U?$pair@QAXPAVCEffectBody@@@std@@@std@@$0A@@stdext@@@stdext@@@std@@@std@@YAPAU_List_position@?$_Hash@V?$_Hmap_traits@PAXPAVCEffectBody@@V?$hash_compare@PAXU?$less@PAX@std@@@stdext@@V?$allocator@U?$pair@QAXPAVCEffectBody@@@std@@@std@@$0A@@stdext@@@stdext@@PAU123@00AAV?$allocator@U_List_position@?$_Hash@V?$_Hmap_traits@PAXPAVCEffectBody@@V?$hash_compare@PAXU?$less@PAX@std@@@stdext@@V?$allocator@U?$pair@QAXPAVCEffectBody@@@std@@@std@@$0A@@stdext@@@stdext@@@0@U_Nonscalar_ptr_iterator_tag@0@U_Range_checked_iterator_tag@0@@Z 1000fd06 f i effectmanager.obj
 0001:0000ed06       ??$_Uninit_copy@PAUSt_AutoCtlParam@@PAU1@V?$allocator@USt_AutoCtlParam@@@std@@@std@@YAPAUSt_AutoCtlParam@@PAU1@00AAV?$allocator@USt_AutoCtlParam@@@0@U_Nonscalar_ptr_iterator_tag@0@U_Range_checked_iterator_tag@0@@Z 1000fd06 f i effectmanager.obj
 0001:0000ed06       ??$_Uninit_copy@PAU_WZNCSPT@WzNaturalCubicSplineDyn@@PAU12@V?$allocator@U_WZNCSPT@WzNaturalCubicSplineDyn@@@std@@@std@@YAPAU_WZNCSPT@WzNaturalCubicSplineDyn@@PAU12@00AAV?$allocator@U_WZNCSPT@WzNaturalCubicSplineDyn@@@0@U_Nonscalar_ptr_iterator_tag@0@U_Range_checked_iterator_tag@0@@Z 1000fd06 f i Common_p:wznaturalcubicsplinedyn.obj
 0001:0000edc9       ?LoadEffectFromFile@CEffectManager@@QAE_NPBD0W4EENUM_LOAD_TYPE@@H@Z 1000fdc9 f   effectmanager_load.obj
 0001:0000f0aa       ?UnLoadEffectFromFile@CEffectManager@@QAEXPBD@Z 100100aa f   effectmanager_load.obj
 0001:0000f247       ?Load@CEffectManager@@QAEPAUSt_BodyCreate@@PAXK@Z 10010247 f   effectmanager_load.obj
 0001:0000f39a       ?Load@CEffectManager@@QAEPAUSt_BodyCreate@@PBDK@Z 1001039a f   effectmanager_load.obj
 0001:0000f416       ?LoadBodyInfoOld@CEffectManager@@AAEXPAXPAUSt_BodyCreate@@@Z 10010416 f   effectmanager_load.obj
 0001:0000f62a       ?LoadBodyInfo@CEffectManager@@AAEXPAXPAUSt_BodyCreate@@@Z 1001062a f   effectmanager_load.obj
 0001:0000fbc3       ?LoadEleInfo@CEffectManager@@QAEPAUSt_Ele_Node@@PAX@Z 10010bc3 f   effectmanager_load.obj
 0001:0000fcc0       ?LoadElementInfo@CEffectManager@@AAEXPAXPAUSt_ElementCreate@@@Z 10010cc0 f   effectmanager_load.obj
 0001:0000ff07       ?LoadCreateInfo@CEffectManager@@AAEXPAXPAUSt_Create_Info@@@Z 10010f07 f   effectmanager_load.obj
 0001:000105cb       ?LoadMoveInfo@CEffectManager@@AAEXPAXPAUSt_Move_Info@@@Z 100115cb f   effectmanager_load.obj
 0001:00010f72       ?LoadChangeInfo@CEffectManager@@AAEXPAXPAUSt_Change_Info@@@Z 10011f72 f   effectmanager_load.obj
 0001:00011c42       ?LoadVisualInfo@CEffectManager@@AAEXPAXPAUSt_Visual_Info@@@Z 10012c42 f   effectmanager_load.obj
 0001:00012867       ?VectorLength@@YAMPBUWzVector@@@Z 10013867 f i effectmanager_load.obj
 0001:00012888       ?Add@St_Change_Info@@QAEXHMW4ENUM_MAP_KIND@@@Z 10013888 f i effectmanager_load.obj
 0001:00012b34       ?insert@?$_Tree@V?$_Tmap_traits@JUWzVector@@U?$less@J@std@@V?$allocator@U?$pair@$$CBJUWzVector@@@std@@@3@$0A@@std@@@std@@QAE?AU?$pair@Viterator@?$_Tree@V?$_Tmap_traits@JUWzVector@@U?$less@J@std@@V?$allocator@U?$pair@$$CBJUWzVector@@@std@@@3@$0A@@std@@@std@@_N@2@ABU?$pair@$$CBJUWzVector@@@2@@Z 10013b34 f i effectmanager_load.obj
 0001:00012d04       ?push_back@?$list@KV?$allocator@K@std@@@std@@QAEXABK@Z 10013d04 f i effectmanager_load.obj
 0001:00012d04       ?push_back@?$list@PAVCEElementSprite@@V?$allocator@PAVCEElementSprite@@@std@@@std@@QAEXABQAVCEElementSprite@@@Z 10013d04 f i eelementweather.obj
 0001:00012d5d       ??A?$map@JMU?$less@J@std@@V?$allocator@U?$pair@$$CBJM@std@@@2@@std@@QAEAAMABJ@Z 10013d5d f i effectmanager_load.obj
 0001:00012e37       ?insert@?$_Tree@V?$_Tmap_traits@JMU?$less@J@std@@V?$allocator@U?$pair@$$CBJM@std@@@2@$0A@@std@@@std@@QAE?AU?$pair@Viterator@?$_Tree@V?$_Tmap_traits@JMU?$less@J@std@@V?$allocator@U?$pair@$$CBJM@std@@@2@$0A@@std@@@std@@_N@2@ABU?$pair@$$CBJM@2@@Z 10013e37 f i effectmanager_load.obj
 0001:00013007       ?_Insert@?$_Tree@V?$_Tmap_traits@JUWzVector@@U?$less@J@std@@V?$allocator@U?$pair@$$CBJUWzVector@@@std@@@3@$0A@@std@@@std@@IAE?AViterator@12@_NPAU_Node@?$_Tree_nod@V?$_Tmap_traits@JUWzVector@@U?$less@J@std@@V?$allocator@U?$pair@$$CBJUWzVector@@@std@@@3@$0A@@std@@@2@ABU?$pair@$$CBJUWzVector@@@2@@Z 10014007 f i effectmanager_load.obj
 0001:000133c2       ?insert@?$_Tree@V?$_Tmap_traits@JMU?$less@J@std@@V?$allocator@U?$pair@$$CBJM@std@@@2@$0A@@std@@@std@@QAE?AViterator@12@Vconst_iterator@12@ABU?$pair@$$CBJM@2@@Z 100143c2 f i effectmanager_load.obj
 0001:00013ac1       ?_Insert@?$_Tree@V?$_Tmap_traits@JMU?$less@J@std@@V?$allocator@U?$pair@$$CBJM@std@@@2@$0A@@std@@@std@@IAE?AViterator@12@_NPAU_Node@?$_Tree_nod@V?$_Tmap_traits@JMU?$less@J@std@@V?$allocator@U?$pair@$$CBJM@std@@@2@$0A@@std@@@2@ABU?$pair@$$CBJM@2@@Z 10014ac1 f i effectmanager_load.obj
 0001:00013e7c       ?_Lbound@?$_Tree@V?$_Tmap_traits@JMU?$less@J@std@@V?$allocator@U?$pair@$$CBJM@std@@@2@$0A@@std@@@std@@IBEPAU_Node@?$_Tree_nod@V?$_Tmap_traits@JMU?$less@J@std@@V?$allocator@U?$pair@$$CBJM@std@@@2@$0A@@std@@@2@ABJ@Z 10014e7c f i effectmanager_load.obj
 0001:00013ede       ?_Dec@const_iterator@?$_Tree@V?$_Tmap_traits@JUWzVector@@U?$less@J@std@@V?$allocator@U?$pair@$$CBJUWzVector@@@std@@@3@$0A@@std@@@std@@QAEXXZ 10014ede f i effectmanager_load.obj
 0001:00013fd1       ?_Dec@const_iterator@?$_Tree@V?$_Tmap_traits@JMU?$less@J@std@@V?$allocator@U?$pair@$$CBJM@std@@@2@$0A@@std@@@std@@QAEXXZ 10014fd1 f i effectmanager_load.obj
 0001:000140c4       ?Save@CEffectManager@@QAE_NPAXK@Z 100150c4 f   effectmanager_save.obj
 0001:00014195       ?Save@CEffectManager@@QAE_NPBDK@Z 10015195 f   effectmanager_save.obj
 0001:00014213       ?SaveBodyInfo@CEffectManager@@AAEXPAXPAUSt_BodyCreate@@@Z 10015213 f   effectmanager_save.obj
 0001:000146fc       ?SaveEleInfo@CEffectManager@@QAEXPAXPAUSt_Ele_Node@@@Z 100156fc f   effectmanager_save.obj
 0001:000147a3       ?SaveElementInfo@CEffectManager@@AAEXPAXPAUSt_ElementCreate@@@Z 100157a3 f   effectmanager_save.obj
 0001:000148ab       ?SaveCreateInfo@CEffectManager@@AAEXPAXPAUSt_Create_Info@@@Z 100158ab f   effectmanager_save.obj
 0001:00014d39       ?SaveMoveInfo@CEffectManager@@AAEXPAXPAUSt_Move_Info@@@Z 10015d39 f   effectmanager_save.obj
 0001:000152c2       ?SaveChangeInfo@CEffectManager@@AAEXPAXPAUSt_Change_Info@@@Z 100162c2 f   effectmanager_save.obj
 0001:00016954       ?SaveVisualInfo@CEffectManager@@AAEXPAXPAUSt_Visual_Info@@@Z 10017954 f   effectmanager_save.obj
 0001:00016dd2       ??0CLoadBaseManager@@QAE@XZ 10017dd2 f   loadmanager.obj
 0001:00016dfc       ??1CLoadBaseManager@@QAE@XZ 10017dfc f   loadmanager.obj
 0001:00016e0f       ?CreateFromFile@CLoadBaseManager@@QAEHPBDPAVCDiscAccess@@W4EENUM_LOAD_TYPE@@@Z 10017e0f f   loadmanager.obj
 0001:0001711e       ?Merge@CLoadBaseManager@@QAEXABV1@@Z 1001811e f   loadmanager.obj
 0001:0001723c       ?Copy@CLoadBaseManager@@QAEXABV1@@Z 1001823c f   loadmanager.obj
 0001:00017278       ??0?$basic_string@DU?$char_traits@D@std@@V?$allocator@D@2@@std@@QAE@ABV01@@Z 10018278 f i loadmanager.obj
 0001:000172a7       ??1?$pair@$$CBKV?$basic_string@DU?$char_traits@D@std@@V?$allocator@D@2@@std@@@std@@QAE@XZ 100182a7 f i loadmanager.obj
 0001:000172c1       ??1?$_Hash@V?$_Hmap_traits@KV?$basic_string@DU?$char_traits@D@std@@V?$allocator@D@2@@std@@V?$hash_compare@KU?$less@K@std@@@stdext@@V?$allocator@U?$pair@$$CBKV?$basic_string@DU?$char_traits@D@std@@V?$allocator@D@2@@std@@@std@@@2@$0A@@stdext@@@stdext@@QAE@XZ 100182c1 f i loadmanager.obj
 0001:00017359       ??0?$_Hash@V?$_Hmap_traits@KV?$basic_string@DU?$char_traits@D@std@@V?$allocator@D@2@@std@@V?$hash_compare@KU?$less@K@std@@@stdext@@V?$allocator@U?$pair@$$CBKV?$basic_string@DU?$char_traits@D@std@@V?$allocator@D@2@@std@@@std@@@2@$0A@@stdext@@@stdext@@QAE@ABV?$hash_compare@KU?$less@K@std@@@1@ABV?$allocator@U?$pair@$$CBKV?$basic_string@DU?$char_traits@D@std@@V?$allocator@D@2@@std@@@std@@@std@@@Z 10018359 f i loadmanager.obj
 0001:000173fd       ?_Insert@?$_Hash@V?$_Hmap_traits@KV?$basic_string@DU?$char_traits@D@std@@V?$allocator@D@2@@std@@V?$hash_compare@KU?$less@K@std@@@stdext@@V?$allocator@U?$pair@$$CBKV?$basic_string@DU?$char_traits@D@std@@V?$allocator@D@2@@std@@@std@@@2@$0A@@stdext@@@stdext@@IAE?AU?$pair@V?$_Iterator@$00@?$list@U?$pair@$$CBKV?$basic_string@DU?$char_traits@D@std@@V?$allocator@D@2@@std@@@std@@V?$allocator@U?$pair@$$CBKV?$basic_string@DU?$char_traits@D@std@@V?$allocator@D@2@@std@@@std@@@2@@std@@_N@std@@ABU?$pair@$$CBKV?$basic_string@DU?$char_traits@D@std@@V?$allocator@D@2@@std@@@4@V?$_Iterator@$00@?$list@U?$pair@$$CBKV?$basic_string@DU?$char_traits@D@std@@V?$allocator@D@2@@std@@@std@@V?$allocator@U?$pair@$$CBKV?$basic_string@DU?$char_traits@D@std@@V?$allocator@D@2@@std@@@std@@@2@@4@@Z 100183fd f i loadmanager.obj
 0001:0001792f       ??1?$list@U?$pair@$$CBKV?$basic_string@DU?$char_traits@D@std@@V?$allocator@D@2@@std@@@std@@V?$allocator@U?$pair@$$CBKV?$basic_string@DU?$char_traits@D@std@@V?$allocator@D@2@@std@@@std@@@2@@std@@QAE@XZ 1001892f f i loadmanager.obj
 0001:00017985       ?_Reinsert@?$_Hash@V?$_Hmap_traits@KV?$basic_string@DU?$char_traits@D@std@@V?$allocator@D@2@@std@@V?$hash_compare@KU?$less@K@std@@@stdext@@V?$allocator@U?$pair@$$CBKV?$basic_string@DU?$char_traits@D@std@@V?$allocator@D@2@@std@@@std@@@2@$0A@@stdext@@@stdext@@IAEXXZ 10018985 f i loadmanager.obj
 0001:00017a8f       ??0?$list@U?$pair@$$CBKV?$basic_string@DU?$char_traits@D@std@@V?$allocator@D@2@@std@@@std@@V?$allocator@U?$pair@$$CBKV?$basic_string@DU?$char_traits@D@std@@V?$allocator@D@2@@std@@@std@@@2@@std@@QAE@ABV?$allocator@U?$pair@$$CBKV?$basic_string@DU?$char_traits@D@std@@V?$allocator@D@2@@std@@@std@@@1@@Z 10018a8f f i loadmanager.obj
 0001:00017b06       ?erase@?$list@U?$pair@$$CBKV?$basic_string@DU?$char_traits@D@std@@V?$allocator@D@2@@std@@@std@@V?$allocator@U?$pair@$$CBKV?$basic_string@DU?$char_traits@D@std@@V?$allocator@D@2@@std@@@std@@@2@@std@@QAE?AV?$_Iterator@$00@12@V?$_Const_iterator@$00@12@@Z 10018b06 f i loadmanager.obj
 0001:00017bc1       ?splice@?$list@U?$pair@$$CBKV?$basic_string@DU?$char_traits@D@std@@V?$allocator@D@2@@std@@@std@@V?$allocator@U?$pair@$$CBKV?$basic_string@DU?$char_traits@D@std@@V?$allocator@D@2@@std@@@std@@@2@@std@@QAEXV?$_Const_iterator@$00@12@AAV12@0@Z 10018bc1 f i loadmanager.obj
 0001:00017c8b       ?_Tidy@?$list@U?$pair@$$CBKV?$basic_string@DU?$char_traits@D@std@@V?$allocator@D@2@@std@@@std@@V?$allocator@U?$pair@$$CBKV?$basic_string@DU?$char_traits@D@std@@V?$allocator@D@2@@std@@@std@@@2@@std@@IAEXXZ 10018c8b f i loadmanager.obj
 0001:00017cc0       ?_Insert@?$list@U?$pair@$$CBKV?$basic_string@DU?$char_traits@D@std@@V?$allocator@D@2@@std@@@std@@V?$allocator@U?$pair@$$CBKV?$basic_string@DU?$char_traits@D@std@@V?$allocator@D@2@@std@@@std@@@2@@std@@QAEXV?$_Const_iterator@$00@12@ABU?$pair@$$CBKV?$basic_string@DU?$char_traits@D@std@@V?$allocator@D@2@@std@@@2@@Z 10018cc0 f i loadmanager.obj
 0001:00017d0e       ?_Splice@?$list@U?$pair@$$CBKV?$basic_string@DU?$char_traits@D@std@@V?$allocator@D@2@@std@@@std@@V?$allocator@U?$pair@$$CBKV?$basic_string@DU?$char_traits@D@std@@V?$allocator@D@2@@std@@@std@@@2@@std@@QAEXV?$_Const_iterator@$00@12@AAV12@00I_N@Z 10018d0e f i loadmanager.obj
 0001:00017e97       ?_Buynode@?$list@U?$pair@$$CBKV?$basic_string@DU?$char_traits@D@std@@V?$allocator@D@2@@std@@@std@@V?$allocator@U?$pair@$$CBKV?$basic_string@DU?$char_traits@D@std@@V?$allocator@D@2@@std@@@std@@@2@@std@@IAEPAU_Node@?$_List_nod@U?$pair@$$CBKV?$basic_string@DU?$char_traits@D@std@@V?$allocator@D@2@@std@@@std@@V?$allocator@U?$pair@$$CBKV?$basic_string@DU?$char_traits@D@std@@V?$allocator@D@2@@std@@@std@@@2@@2@XZ 10018e97 f i loadmanager.obj
 0001:00017f79       ?_Get_iter@_List_position@?$_Hash@V?$_Hmap_traits@KV?$basic_string@DU?$char_traits@D@std@@V?$allocator@D@2@@std@@V?$hash_compare@KU?$less@K@std@@@stdext@@V?$allocator@U?$pair@$$CBKV?$basic_string@DU?$char_traits@D@std@@V?$allocator@D@2@@std@@@std@@@2@$0A@@stdext@@@stdext@@QBE?AV?$_Iterator@$00@?$list@U?$pair@$$CBKV?$basic_string@DU?$char_traits@D@std@@V?$allocator@D@2@@std@@@std@@V?$allocator@U?$pair@$$CBKV?$basic_string@DU?$char_traits@D@std@@V?$allocator@D@2@@std@@@std@@@2@@std@@ABV56@@Z 10018f79 f i loadmanager.obj
 0001:00017f79       ?_Get_iter@_List_position@?$_Hash@V?$_Hmap_traits@KPAUSt_BodyCreate@@V?$hash_compare@KU?$less@K@std@@@stdext@@V?$allocator@U?$pair@$$CBKPAUSt_BodyCreate@@@std@@@std@@$0A@@stdext@@@stdext@@QBE?AV?$_Iterator@$00@?$list@U?$pair@$$CBKPAUSt_BodyCreate@@@std@@V?$allocator@U?$pair@$$CBKPAUSt_BodyCreate@@@std@@@2@@std@@ABV56@@Z 10018f79 f i effectmanager.obj
 0001:00017f79       ?_Get_iter@_List_position@?$_Hash@V?$_Hmap_traits@PAXPAVCEffectBody@@V?$hash_compare@PAXU?$less@PAX@std@@@stdext@@V?$allocator@U?$pair@QAXPAVCEffectBody@@@std@@@std@@$0A@@stdext@@@stdext@@QBE?AV?$_Iterator@$00@?$list@U?$pair@QAXPAVCEffectBody@@@std@@V?$allocator@U?$pair@QAXPAVCEffectBody@@@std@@@2@@std@@ABV56@@Z 10018f79 f i effectmanager.obj
 0001:00017fbe       ?erase@?$list@U?$pair@$$CBKV?$basic_string@DU?$char_traits@D@std@@V?$allocator@D@2@@std@@@std@@V?$allocator@U?$pair@$$CBKV?$basic_string@DU?$char_traits@D@std@@V?$allocator@D@2@@std@@@std@@@2@@std@@QAE?AV?$_Iterator@$00@12@V?$_Const_iterator@$00@12@0@Z 10018fbe f i loadmanager.obj
 0001:00018116       ?_Buynode@?$list@U?$pair@$$CBKV?$basic_string@DU?$char_traits@D@std@@V?$allocator@D@2@@std@@@std@@V?$allocator@U?$pair@$$CBKV?$basic_string@DU?$char_traits@D@std@@V?$allocator@D@2@@std@@@std@@@2@@std@@IAEPAU_Node@?$_List_nod@U?$pair@$$CBKV?$basic_string@DU?$char_traits@D@std@@V?$allocator@D@2@@std@@@std@@V?$allocator@U?$pair@$$CBKV?$basic_string@DU?$char_traits@D@std@@V?$allocator@D@2@@std@@@std@@@2@@2@PAU342@0ABU?$pair@$$CBKV?$basic_string@DU?$char_traits@D@std@@V?$allocator@D@2@@std@@@2@@Z 10019116 f i loadmanager.obj
 0001:00018200       ?_Incsize@?$list@U?$pair@$$CBKV?$basic_string@DU?$char_traits@D@std@@V?$allocator@D@2@@std@@@std@@V?$allocator@U?$pair@$$CBKV?$basic_string@DU?$char_traits@D@std@@V?$allocator@D@2@@std@@@std@@@2@@std@@IAEXI@Z 10019200 f i loadmanager.obj
 0001:000182ca       ??0?$_Const_iterator@$0A@@?$list@U?$pair@$$CBKV?$basic_string@DU?$char_traits@D@std@@V?$allocator@D@2@@std@@@std@@V?$allocator@U?$pair@$$CBKV?$basic_string@DU?$char_traits@D@std@@V?$allocator@D@2@@std@@@std@@@2@@std@@QAE@PAU_Node@?$_List_nod@U?$pair@$$CBKV?$basic_string@DU?$char_traits@D@std@@V?$allocator@D@2@@std@@@std@@V?$allocator@U?$pair@$$CBKV?$basic_string@DU?$char_traits@D@std@@V?$allocator@D@2@@std@@@std@@@2@@2@PBV12@@Z 100192ca f i loadmanager.obj
 0001:000182ca       ??0?$_Const_iterator@$0A@@?$list@U?$pair@$$CBKPAUSt_BodyCreate@@@std@@V?$allocator@U?$pair@$$CBKPAUSt_BodyCreate@@@std@@@2@@std@@QAE@PAU_Node@?$_List_nod@U?$pair@$$CBKPAUSt_BodyCreate@@@std@@V?$allocator@U?$pair@$$CBKPAUSt_BodyCreate@@@std@@@2@@2@PBV12@@Z 100192ca f i effectmanager.obj
 0001:000182ca       ??0?$_Const_iterator@$0A@@?$list@U?$pair@QAXPAVCEffectBody@@@std@@V?$allocator@U?$pair@QAXPAVCEffectBody@@@std@@@2@@std@@QAE@PAU_Node@?$_List_nod@U?$pair@QAXPAVCEffectBody@@@std@@V?$allocator@U?$pair@QAXPAVCEffectBody@@@std@@@2@@2@PBV12@@Z 100192ca f i effectmanager.obj
 0001:00018304       ??$_Allocate@U_Node@?$_List_nod@U?$pair@$$CBKV?$basic_string@DU?$char_traits@D@std@@V?$allocator@D@2@@std@@@std@@V?$allocator@U?$pair@$$CBKV?$basic_string@DU?$char_traits@D@std@@V?$allocator@D@2@@std@@@std@@@2@@std@@@std@@YAPAU_Node@?$_List_nod@U?$pair@$$CBKV?$basic_string@DU?$char_traits@D@std@@V?$allocator@D@2@@std@@@std@@V?$allocator@U?$pair@$$CBKV?$basic_string@DU?$char_traits@D@std@@V?$allocator@D@2@@std@@@std@@@2@@0@IPAU120@@Z 10019304 f i loadmanager.obj
 0001:00018357       ??$_Construct@U?$pair@$$CBKV?$basic_string@DU?$char_traits@D@std@@V?$allocator@D@2@@std@@@std@@U12@@std@@YAXPAU?$pair@$$CBKV?$basic_string@DU?$char_traits@D@std@@V?$allocator@D@2@@std@@@0@ABU10@@Z 10019357 f i loadmanager.obj
 0001:000183bd       ??3@YAXPAX0@Z              100193bd f i loadmanager.obj
 0001:000183c2       ??0?$pair@$$CBKV?$basic_string@DU?$char_traits@D@std@@V?$allocator@D@2@@std@@@std@@QAE@ABU01@@Z 100193c2 f i loadmanager.obj
 0001:00018408       ??$_Insert@V?$_Const_iterator@$00@?$list@U?$pair@$$CBKV?$basic_string@DU?$char_traits@D@std@@V?$allocator@D@2@@std@@@std@@V?$allocator@U?$pair@$$CBKV?$basic_string@DU?$char_traits@D@std@@V?$allocator@D@2@@std@@@std@@@2@@std@@@?$list@U?$pair@$$CBKV?$basic_string@DU?$char_traits@D@std@@V?$allocator@D@2@@std@@@std@@V?$allocator@U?$pair@$$CBKV?$basic_string@DU?$char_traits@D@std@@V?$allocator@D@2@@std@@@std@@@2@@std@@QAEXV?$_Const_iterator@$00@01@00Uforward_iterator_tag@1@@Z 10019408 f i loadmanager.obj
 0001:0001851d       ??0CMemoryManager@@QAE@XZ  1001951d f   memorymanager.obj
 0001:00018559       ??1CMemoryManager@@QAE@XZ  10019559 f   memorymanager.obj
 0001:0001856a       ?Create@CMemoryManager@@QAEHXZ 1001956a f   memorymanager.obj
 0001:000188ed       ?Destroy@CMemoryManager@@QAEXXZ 100198ed f   memorymanager.obj
 0001:00018b6a       ?Shrink@CMemoryManager@@QAEXXZ 10019b6a f   memorymanager.obj
 0001:00018c2f       ?Create@?$CWzMemoryPool@VCEElementSprite@@@@QAE_NHH@Z 10019c2f f i memorymanager.obj
 0001:00018cde       ?Shrink@?$CWzMemoryPool@VCEElementSprite@@@@QAEXXZ 10019cde f i memorymanager.obj
 0001:00018d84       ?Create@?$CWzMemoryPool@VCEElementMesh@@@@QAE_NHH@Z 10019d84 f i memorymanager.obj
 0001:00018e33       ?Shrink@?$CWzMemoryPool@VCEElementMesh@@@@QAEXXZ 10019e33 f i memorymanager.obj
 0001:00018ed9       ?Create@?$CWzMemoryPool@VCEElementChain@@@@QAE_NHH@Z 10019ed9 f i memorymanager.obj
 0001:00018f88       ?Shrink@?$CWzMemoryPool@VCEElementChain@@@@QAEXXZ 10019f88 f i memorymanager.obj
 0001:0001902e       ?Create@?$CWzMemoryPool@VCEElementFlatChain@@@@QAE_NHH@Z 1001a02e f i memorymanager.obj
 0001:000190dd       ?Shrink@?$CWzMemoryPool@VCEElementFlatChain@@@@QAEXXZ 1001a0dd f i memorymanager.obj
 0001:00019183       ?Create@?$CWzMemoryPool@VCEElementDecal@@@@QAE_NHH@Z 1001a183 f i memorymanager.obj
 0001:00019232       ?Shrink@?$CWzMemoryPool@VCEElementDecal@@@@QAEXXZ 1001a232 f i memorymanager.obj
 0001:000192d8       ?Create@?$CWzMemoryPool@VCEElementWeather@@@@QAE_NHH@Z 1001a2d8 f i memorymanager.obj
 0001:00019387       ?Shrink@?$CWzMemoryPool@VCEElementWeather@@@@QAEXXZ 1001a387 f i memorymanager.obj
 0001:0001942d       ?Create@?$CWzMemoryPool@VCEffectBody@@@@QAE_NHH@Z 1001a42d f i memorymanager.obj
 0001:000194dc       ?Shrink@?$CWzMemoryPool@VCEffectBody@@@@QAEXXZ 1001a4dc f i memorymanager.obj
 0001:00019582       ?AllocBand@?$CWzMemoryPool@VCEElementSprite@@@@AAEPAV?$CWzMemoryBand@VCEElementSprite@@@@H@Z 1001a582 f i memorymanager.obj
 0001:0001965d       ?AllocBand@?$CWzMemoryPool@VCEElementMesh@@@@AAEPAV?$CWzMemoryBand@VCEElementMesh@@@@H@Z 1001a65d f i memorymanager.obj
 0001:00019738       ?AllocBand@?$CWzMemoryPool@VCEElementChain@@@@AAEPAV?$CWzMemoryBand@VCEElementChain@@@@H@Z 1001a738 f i memorymanager.obj
 0001:00019813       ?Destroy@?$CWzMemoryPool@VCEElementSprite@@@@QAEXXZ 1001a813 f i memorymanager.obj
 0001:00019813       ?Destroy@?$CWzMemoryPool@VCEElementDecal@@@@QAEXXZ 1001a813 f i memorymanager.obj
 0001:00019813       ?Destroy@?$CWzMemoryPool@VCEElementMesh@@@@QAEXXZ 1001a813 f i memorymanager.obj
 0001:00019813       ?Destroy@?$CWzMemoryPool@VCEElementChain@@@@QAEXXZ 1001a813 f i memorymanager.obj
 0001:00019813       ?Destroy@?$CWzMemoryPool@VCEElementWeather@@@@QAEXXZ 1001a813 f i memorymanager.obj
 0001:00019813       ?Destroy@?$CWzMemoryPool@VCEElementFlatChain@@@@QAEXXZ 1001a813 f i memorymanager.obj
 0001:00019813       ?Destroy@?$CWzMemoryPool@VCEffectBody@@@@QAEXXZ 1001a813 f i memorymanager.obj
 0001:00019889       ?AllocBand@?$CWzMemoryPool@VCEElementFlatChain@@@@AAEPAV?$CWzMemoryBand@VCEElementFlatChain@@@@H@Z 1001a889 f i memorymanager.obj
 0001:00019964       ?AllocBand@?$CWzMemoryPool@VCEElementDecal@@@@AAEPAV?$CWzMemoryBand@VCEElementDecal@@@@H@Z 1001a964 f i memorymanager.obj
 0001:00019a3f       ?AllocBand@?$CWzMemoryPool@VCEElementWeather@@@@AAEPAV?$CWzMemoryBand@VCEElementWeather@@@@H@Z 1001aa3f f i memorymanager.obj
 0001:00019b1a       ?Initialize@?$CWzMemoryBand@VCEElementSprite@@@@QAEXXZ 1001ab1a f i memorymanager.obj
 0001:00019b65       ?Initialize@?$CWzMemoryBand@VCEElementMesh@@@@QAEXXZ 1001ab65 f i memorymanager.obj
 0001:00019bb0       ?Initialize@?$CWzMemoryBand@VCEElementChain@@@@QAEXXZ 1001abb0 f i memorymanager.obj
 0001:00019bfb       ?Initialize@?$CWzMemoryBand@VCEElementFlatChain@@@@QAEXXZ 1001abfb f i memorymanager.obj
 0001:00019c46       ?Initialize@?$CWzMemoryBand@VCEElementDecal@@@@QAEXXZ 1001ac46 f i memorymanager.obj
 0001:00019c91       ?Initialize@?$CWzMemoryBand@VCEElementWeather@@@@QAEXXZ 1001ac91 f i memorymanager.obj
 0001:00019cdc       ?Initialize@?$CWzMemoryBand@VCEffectBody@@@@QAEXXZ 1001acdc f i memorymanager.obj
 0001:00019d27       ?Create@?$CWzMemoryBand@VCEElementSprite@@@@QAE_NH@Z 1001ad27 f i memorymanager.obj
 0001:00019eae       ?Create@?$CWzMemoryBand@VCEElementMesh@@@@QAE_NH@Z 1001aeae f i memorymanager.obj
 0001:0001a035       ?Create@?$CWzMemoryBand@VCEElementChain@@@@QAE_NH@Z 1001b035 f i memorymanager.obj
 0001:0001a1bc       ?Create@?$CWzMemoryBand@VCEElementFlatChain@@@@QAE_NH@Z 1001b1bc f i memorymanager.obj
 0001:0001a343       ?Destroy@?$CWzMemoryBand@VCEElementFlatChain@@@@QAEXXZ 1001b343 f i memorymanager.obj
 0001:0001a343       ?Destroy@?$CWzMemoryBand@VCEElementSprite@@@@QAEXXZ 1001b343 f i memorymanager.obj
 0001:0001a343       ?Destroy@?$CWzMemoryBand@VCEElementWeather@@@@QAEXXZ 1001b343 f i memorymanager.obj
 0001:0001a343       ?Destroy@?$CWzMemoryBand@VCEElementChain@@@@QAEXXZ 1001b343 f i memorymanager.obj
 0001:0001a343       ?Destroy@?$CWzMemoryBand@VCEElementDecal@@@@QAEXXZ 1001b343 f i memorymanager.obj
 0001:0001a343       ?Destroy@?$CWzMemoryBand@VCEElementMesh@@@@QAEXXZ 1001b343 f i memorymanager.obj
 0001:0001a343       ?Destroy@?$CWzMemoryBand@VCEffectBody@@@@QAEXXZ 1001b343 f i effectmanager.obj
 0001:0001a3ed       ?Create@?$CWzMemoryBand@VCEElementDecal@@@@QAE_NH@Z 1001b3ed f i memorymanager.obj
 0001:0001a574       ?Create@?$CWzMemoryBand@VCEElementWeather@@@@QAE_NH@Z 1001b574 f i memorymanager.obj
 0001:0001a6fb       ??0CEElementBase@@QAE@XZ   1001b6fb f   eelementbase.obj
 0001:0001a710       ??1CEElementBase@@UAE@XZ   1001b710 f   eelementbase.obj
 0001:0001a722       ?Clear@CEElementBase@@UAEXXZ 1001b722 f   eelementbase.obj
 0001:0001a78f       ?Create@CEElementBase@@UAE_N_N@Z 1001b78f f   eelementbase.obj
 0001:0001a7bf       ?Move@CEElementBase@@UAE?AW4_ENUM_RESULT_EFFECT_MOVE@@KAA_N@Z 1001b7bf f   eelementbase.obj
 0001:0001a914       ?OnInitialize@WzLogHandler@WzLog@@EAEHXZ 1001b914 f i ProgramCommonLibForEngine_p:WzFileLogHandler.obj
 0001:0001a914       ?GetType@CEElementBase@@UBE?AW4ENUM_EELEMENT_TYPE@@XZ 1001b914 f i eelementbase.obj
 0001:0001a91f       ?SetElementInfo@CEElementBase@@UAEXPAUSt_ElementCreate@@@Z 1001b91f f i eelementbase.obj
 0001:0001a933       ?SetParentPtr@CEElementBase@@UAEXPAVCEffectBody@@@Z 1001b933 f i eelementbase.obj
 0001:0001a947       ?Loop@CEElementBase@@UAEXXZ 1001b947 f i eelementbase.obj
 0001:0001a957       ?Reset@CEElementBase@@MAEXXZ 1001b957 f i eelementbase.obj
 0001:0001a96d       ?Free@CEElementBase@@UAEXXZ 1001b96d f i eelementbase.obj
 0001:0001a981       ?SetResultMatrix@CEElementBase@@UAEXABUWzVector@@00@Z 1001b981 f i eelementbase.obj
 0001:0001a981       ?SetResultMatrix@CEElementBase@@UAEXPBUWzMatrix@@00@Z 1001b981 f i eelementbase.obj
 0001:0001a98c       ?GetTextureHandle@CEElementBase@@UAEXAAV?$vector@PAXV?$allocator@PAX@std@@@std@@@Z 1001b98c f i eelementbase.obj
 0001:0001a98c       ?SetTargetPos@CEElementBase@@UAEXABUWzVector@@@Z 1001b98c f i eelementbase.obj
 0001:0001a997       ??_GCEElementBase@@UAEPAXI@Z 1001b997 f i eelementbase.obj
 0001:0001a997       ??_ECEElementBase@@UAEPAXI@Z 1001b997 f i eelementbase.obj
 0001:0001a9be       ??0CEElementChain@@QAE@XZ  1001b9be f   eelementchain.obj
 0001:0001a9db       ??1CEElementChain@@UAE@XZ  1001b9db f   eelementchain.obj
 0001:0001a9f5       ?Clear@CEElementChain@@UAEXXZ 1001b9f5 f   eelementchain.obj
 0001:0001aa7d       ?SetElementInfo@CEElementChain@@UAEXPAUSt_ElementCreate@@@Z 1001ba7d f   eelementchain.obj
 0001:0001aaa6       ?ReloadTexture@CEElementChain@@UAEXXZ 1001baa6 f   eelementchain.obj
 0001:0001aae2       ?Create@CEElementChain@@UAE_N_N@Z 1001bae2 f   eelementchain.obj
 0001:0001ad5e       ?Destroy@CEElementChain@@UAEXXZ 1001bd5e f   eelementchain.obj
 0001:0001adea       ?Free@CEElementChain@@UAEXXZ 1001bdea f   eelementchain.obj
 0001:0001ae2e       ?Move@CEElementChain@@UAE?AW4_ENUM_RESULT_EFFECT_MOVE@@KAA_N@Z 1001be2e f   eelementchain.obj
 0001:0001ae8a       ?Render@CEElementChain@@UAEXXZ 1001be8a f   eelementchain.obj
 0001:0001b0b5       ?GenerateHead@CEElementChain@@IAEXXZ 1001c0b5 f   eelementchain.obj
 0001:0001b652       ?CheckCollWithTarget@CEElementChain@@IAE_NXZ 1001c652 f   eelementchain.obj
 0001:0001b6a1       ?Loop@CEElementParticle@@UAEXXZ 1001c6a1 f i eelementchain.obj
 0001:0001b6bb       ?GetTextureHandle@CEElementSprite@@UAEXAAV?$vector@PAXV?$allocator@PAX@std@@@std@@@Z 1001c6bb f i eelementsprite.obj
 0001:0001b6bb       ?GetTextureHandle@CEElementChain@@UAEXAAV?$vector@PAXV?$allocator@PAX@std@@@std@@@Z 1001c6bb f i eelementchain.obj
 0001:0001b6dc       ?GetType@CEElementChain@@UBE?AW4ENUM_EELEMENT_TYPE@@XZ 1001c6dc f i eelementchain.obj
 0001:0001b6e8       ?SetTargetPos@CEElementChain@@UAEXABUWzVector@@@Z 1001c6e8 f i eelementchain.obj
 0001:0001b706       ?Math_GetRandomFloatBetween@@YAMMM@Z 1001c706 f i eelementchain.obj
 0001:0001b73c       ?IncNumRenderedChain@St_EffDbgInfo@@QAEXXZ 1001c73c f i eelementchain.obj
 0001:0001b76c       ?VectorTransformCoord@@YAPAUWzVector@@PAU1@PBU1@PBUWzMatrix@@@Z 1001c76c f i eelementchain.obj
 0001:0001b80b       ?VectorCrossProduct@@YAPAUWzVector@@PAU1@PBU1@1@Z 1001c80b f i eelementchain.obj
 0001:0001b86e       ?VectorNormalize@@YAPAUWzVector@@PAU1@PBU1@@Z 1001c86e f i eelementchain.obj
 0001:0001b8c9       ?FreeObject@?$CWzMemoryBand@VCEffectBody@@@@QAE_NPAVCEffectBody@@@Z 1001c8c9 f i effectmanager.obj
 0001:0001b8c9       ?FreeObject@?$CWzMemoryBand@VCEElementSprite@@@@QAE_NPAVCEElementSprite@@@Z 1001c8c9 f i eelementsprite.obj
 0001:0001b8c9       ?FreeObject@?$CWzMemoryBand@VCEElementMesh@@@@QAE_NPAVCEElementMesh@@@Z 1001c8c9 f i eelementmesh.obj
 0001:0001b8c9       ?FreeObject@?$CWzMemoryBand@VCEElementChain@@@@QAE_NPAVCEElementChain@@@Z 1001c8c9 f i eelementchain.obj
 0001:0001b8c9       ?FreeObject@?$CWzMemoryBand@VCEElementDecal@@@@QAE_NPAVCEElementDecal@@@Z 1001c8c9 f i eelementdecal.obj
 0001:0001b8c9       ?FreeObject@?$CWzMemoryBand@VCEElementWeather@@@@QAE_NPAVCEElementWeather@@@Z 1001c8c9 f i eelementweather.obj
 0001:0001b8c9       ?FreeObject@?$CWzMemoryBand@VCEElementFlatChain@@@@QAE_NPAVCEElementFlatChain@@@Z 1001c8c9 f i eelementflatchain.obj
 0001:0001b90d       ??0CEElementDecal@@QAE@XZ  1001c90d f   eelementdecal.obj
 0001:0001b92a       ??1CEElementDecal@@UAE@XZ  1001c92a f   eelementdecal.obj
 0001:0001b944       ?Clear@CEElementDecal@@UAEXXZ 1001c944 f   eelementdecal.obj
 0001:0001b9c7       ?SetElementInfo@CEElementDecal@@UAEXPAUSt_ElementCreate@@@Z 1001c9c7 f   eelementdecal.obj
 0001:0001b9ed       ?Create@CEElementDecal@@UAE_N_N@Z 1001c9ed f   eelementdecal.obj
 0001:0001bbb3       ?Destroy@CEElementDecal@@UAEXXZ 1001cbb3 f   eelementdecal.obj
 0001:0001bbc4       ?DestroyMesh@CEElementDecal@@IAEXXZ 1001cbc4 f   eelementdecal.obj
 0001:0001bc0a       ?Free@CEElementDecal@@UAEXXZ 1001cc0a f   eelementdecal.obj
 0001:0001bc4e       ?OnBeingBorn@CEElementDecal@@MAEXXZ 1001cc4e f   eelementdecal.obj
 0001:0001bce0       ?Move@CEElementDecal@@UAE?AW4_ENUM_RESULT_EFFECT_MOVE@@KAA_N@Z 1001cce0 f   eelementdecal.obj
 0001:0001bd42       ?Render@CEElementDecal@@UAEXXZ 1001cd42 f   eelementdecal.obj
 0001:0001be5b       ?CalculateAll@CEElementDecal@@IAEXK@Z 1001ce5b f   eelementdecal.obj
 0001:0001c086       ?GetTextureHandle@CEElementDecal@@UAEXAAV?$vector@PAXV?$allocator@PAX@std@@@std@@@Z 1001d086 f   eelementdecal.obj
 0001:0001c0af       ?ReloadTexture@CEElementDecal@@UAEXXZ 1001d0af f   eelementdecal.obj
 0001:0001c0e4       ?GenerateMesh@CEElementDecal@@IAE_NXZ 1001d0e4 f   eelementdecal.obj
 0001:0001c25e       ?SetResultMatrix@CEElementDecal@@UAEXABUWzVector@@00@Z 1001d25e f   eelementdecal.obj
 0001:0001c2cf       ?SetResultMatrix@CEElementDecal@@UAEXPBUWzMatrix@@00@Z 1001d2cf f   eelementdecal.obj
 0001:0001c3fd       ?GetType@CEElementDecal@@UBE?AW4ENUM_EELEMENT_TYPE@@XZ 1001d3fd f i eelementdecal.obj
 0001:0001c409       ?MatrixIdentity@@YAPAUWzMatrix@@PAU1@@Z 1001d409 f i eelementdecal.obj
 0001:0001c510       ??YWzVector@@QAEAAU0@ABU0@@Z 1001d510 f i eelementdecal.obj
 0001:0001c551       ??XWzVector@@QAEAAU0@M@Z   1001d551 f i eelementdecal.obj
 0001:0001c58a       ?IncNumRenderedDecal@St_EffDbgInfo@@QAEXXZ 1001d58a f i eelementdecal.obj
 0001:0001c5ba       ?VectorTransformNormal@@YAPAUWzVector@@PAU1@PBU1@PBUWzMatrix@@@Z 1001d5ba f i eelementdecal.obj
 0001:0001c647       ??8WzVector@@QBEHABU0@@Z   1001d647 f i eelementdecal.obj
 0001:0001c6cb       ??0CEElementFlatChain@@QAE@XZ 1001d6cb f   eelementflatchain.obj
 0001:0001c6e8       ??1CEElementFlatChain@@UAE@XZ 1001d6e8 f   eelementflatchain.obj
 0001:0001c702       ?Clear@CEElementFlatChain@@UAEXXZ 1001d702 f   eelementflatchain.obj
 0001:0001c757       ?SetElementInfo@CEElementFlatChain@@UAEXPAUSt_ElementCreate@@@Z 1001d757 f   eelementflatchain.obj
 0001:0001c77d       ?ReloadTexture@CEElementFlatChain@@UAEXXZ 1001d77d f   eelementflatchain.obj
 0001:0001c7a5       ?Create@CEElementFlatChain@@UAE_N_N@Z 1001d7a5 f   eelementflatchain.obj
 0001:0001c8e2       ?Destroy@CEElementFlatChain@@UAEXXZ 1001d8e2 f   eelementflatchain.obj
 0001:0001c8f3       ?DestroyBuffers@CEElementFlatChain@@IAEXXZ 1001d8f3 f   eelementflatchain.obj
 0001:0001c949       ?Free@CEElementFlatChain@@UAEXXZ 1001d949 f   eelementflatchain.obj
 0001:0001c98d       ?SetLifeInfo@CEElementFlatChain@@QAEXKK@Z 1001d98d f   eelementflatchain.obj
 0001:0001c9db       ?SetTailNum@CEElementFlatChain@@QAEXH@Z 1001d9db f   eelementflatchain.obj
 0001:0001caec       ?GenerateHead@CEElementFlatChain@@IAEXXZ 1001daec f   eelementflatchain.obj
 0001:0001d18e       ?Move@CEElementFlatChain@@UAE?AW4_ENUM_RESULT_EFFECT_MOVE@@KAA_N@Z 1001e18e f   eelementflatchain.obj
 0001:0001d1e6       ?Render@CEElementFlatChain@@UAEXXZ 1001e1e6 f   eelementflatchain.obj
 0001:0001d3b4       ?GetTextureHandle@CEElementFlatChain@@UAEXAAV?$vector@PAXV?$allocator@PAX@std@@@std@@@Z 1001e3b4 f i eelementflatchain.obj
 0001:0001d3d3       ?GetType@CEElementFlatChain@@UBE?AW4ENUM_EELEMENT_TYPE@@XZ 1001e3d3 f i eelementflatchain.obj
 0001:0001d3df       ?IncNumRenderedFlatChain@St_EffDbgInfo@@QAEXXZ 1001e3df f i eelementflatchain.obj
 0001:0001d40f       ??0CEElementMesh@@QAE@XZ   1001e40f f   eelementmesh.obj
 0001:0001d42c       ??1CEElementMesh@@UAE@XZ   1001e42c f   eelementmesh.obj
 0001:0001d446       ?Clear@CEElementMesh@@UAEXXZ 1001e446 f   eelementmesh.obj
 0001:0001d47e       ?SetElementInfo@CEElementMesh@@UAEXPAUSt_ElementCreate@@@Z 1001e47e f   eelementmesh.obj
 0001:0001d4a7       ?Create@CEElementMesh@@UAE_N_N@Z 1001e4a7 f   eelementmesh.obj
 0001:0001d6a1       ?Destroy@CEElementMesh@@UAEXXZ 1001e6a1 f   eelementmesh.obj
 0001:0001d6d3       ?Free@CEElementMesh@@UAEXXZ 1001e6d3 f   eelementmesh.obj
 0001:0001d717       ?SetResultMatrix@CEElementMesh@@UAEXABUWzVector@@00@Z 1001e717 f   eelementmesh.obj
 0001:0001d7e5       ?SetResultMatrix@CEElementMesh@@UAEXPBUWzMatrix@@00@Z 1001e7e5 f   eelementmesh.obj
 0001:0001d8a8       ?Move@CEElementMesh@@UAE?AW4_ENUM_RESULT_EFFECT_MOVE@@KAA_N@Z 1001e8a8 f   eelementmesh.obj
 0001:0001d8f3       ?Render@CEElementMesh@@UAEXXZ 1001e8f3 f   eelementmesh.obj
 0001:0001da4e       ?MoveMesh@CEElementMesh@@IAEXK@Z 1001ea4e f   eelementmesh.obj
 0001:0001dcd2       ?GetType@CEElementMesh@@UBE?AW4ENUM_EELEMENT_TYPE@@XZ 1001ecd2 f i eelementmesh.obj
 0001:0001dcde       ?MatrixScaling@@YAPAUWzMatrix@@PAU1@MMM@Z 1001ecde f i eelementmesh.obj
 0001:0001dddc       ?MatrixTranslation@@YAPAUWzMatrix@@PAU1@MMM@Z 1001eddc f i eelementmesh.obj
 0001:0001deda       ?IsEnableSetMatrix@CEElementParticle@@IAE_NXZ 1001eeda f i eelementmesh.obj
 0001:0001df12       ?IncNumRenderedMesh@St_EffDbgInfo@@QAEXXZ 1001ef12 f i eelementmesh.obj
 0001:0001df42       ?SetRotationByMatrix@CWzUnitDraw@@QAEXPBUWzMatrix@@@Z 1001ef42 f i eelementmesh.obj
 0001:0001dfd8       ?Get@?$CWzArray@PAUWzRenderInfo@@@@QBEAAPAUWzRenderInfo@@H@Z 1001efd8 f i eelementmesh.obj
 0001:0001e01f       ?Get@?$CWzArray@PAVWzAnimationInfo@@@@QBEAAPAVWzAnimationInfo@@H@Z 1001f01f f i eelementmesh.obj
 0001:0001e066       ?GetCount@?$CWzArray@PAVWzAnimationInfo@@@@QBEHXZ 1001f066 f i eelementmesh.obj
 0001:0001e066       ?GetCount@?$CWzArray@PAVCWzUnitSubType@@@@QBEHXZ 1001f066 f i eelementmesh.obj
 0001:0001e074       ?Get@?$CWzArray@PAVCWzUnitSubType@@@@QBEAAPAVCWzUnitSubType@@H@Z 1001f074 f i eelementmesh.obj
 0001:0001e0bb       ?Get@?$CWzHashTable@PAUSt_WzUnitContainer@@K@@QBEABQAUSt_WzUnitContainer@@ABK@Z 1001f0bb f i eelementmesh.obj
 0001:0001e11b       ?IsSameKey@?$CWzHashTable@PAUSt_WzUnitContainer@@K@@IBEHABK0@Z 1001f11b f i eelementmesh.obj
 0001:0001e135       ??0CEElementParticle@@QAE@XZ 1001f135 f   eelementparticle.obj
 0001:0001e152       ??1CEElementParticle@@UAE@XZ 1001f152 f   eelementparticle.obj
 0001:0001e16c       ?Clear@CEElementParticle@@UAEXXZ 1001f16c f   eelementparticle.obj
 0001:0001e1f2       ?Create@CEElementParticle@@UAE_N_N@Z 1001f1f2 f   eelementparticle.obj
 0001:0001f3d6       ?OnBeingBorn@CEElementParticle@@MAEXXZ 100203d6 f   eelementparticle.obj
 0001:0001f4f4       ?Move@CEElementParticle@@UAE?AW4_ENUM_RESULT_EFFECT_MOVE@@KAA_N@Z 100204f4 f   eelementparticle.obj
 0001:0001f57d       ?CalculateToColor@CEElementParticle@@IAEXK@Z 1002057d f   eelementparticle.obj
 0001:0001f6a3       ?CalculateToScale@CEElementParticle@@IAEXK@Z 100206a3 f   eelementparticle.obj
 0001:0001f745       ?CalculateToRotation@CEElementParticle@@IAEXK@Z 10020745 f   eelementparticle.obj
 0001:0001f848       ?CalculateToPosRotation@CEElementParticle@@IAEXK@Z 10020848 f   eelementparticle.obj
 0001:0001f963       ?CalculateToPos@CEElementParticle@@IAEXKK@Z 10020963 f   eelementparticle.obj
 0001:00020080       ?SetResultMatrix@CEElementParticle@@UAEXABUWzVector@@00@Z 10021080 f   eelementparticle.obj
 0001:00020158       ?SetResultMatrix@CEElementParticle@@UAEXPBUWzMatrix@@00@Z 10021158 f   eelementparticle.obj
 0001:0002023d       ??_GCEElementParticle@@UAEPAXI@Z 1002123d f i eelementparticle.obj
 0001:0002023d       ??_ECEElementParticle@@UAEPAXI@Z 1002123d f i eelementparticle.obj
 0001:00020264       ?GetValue@WzNaturalCubicSplineDyn@@QAEMH@Z 10021264 f i eelementparticle.obj
 0001:000202cb       ??ZWzVector@@QAEAAU0@ABU0@@Z 100212cb f i eelementparticle.obj
 0001:0002030c       ??0CEElementSprite@@QAE@XZ 1002130c f   eelementsprite.obj
 0001:00020329       ??1CEElementSprite@@UAE@XZ 10021329 f   eelementsprite.obj
 0001:00020343       ?Clear@CEElementSprite@@UAEXXZ 10021343 f   eelementsprite.obj
 0001:000203cb       ?SetElementInfo@CEElementSprite@@UAEXPAUSt_ElementCreate@@@Z 100213cb f   eelementsprite.obj
 0001:000203f4       ?ReloadTexture@CEElementSprite@@UAEXXZ 100213f4 f   eelementsprite.obj
 0001:00020430       ?Create@CEElementSprite@@UAE_N_N@Z 10021430 f   eelementsprite.obj
 0001:000207c1       ?Free@CEElementSprite@@UAEXXZ 100217c1 f   eelementsprite.obj
 0001:00020803       ?Move@CEElementSprite@@UAE?AW4_ENUM_RESULT_EFFECT_MOVE@@KAA_N@Z 10021803 f   eelementsprite.obj
 0001:000208d3       ?Render@CEElementSprite@@UAEXXZ 100218d3 f   eelementsprite.obj
 0001:00020ab7       ?SetSpriteColor@CEElementSprite@@IAEX_N@Z 10021ab7 f   eelementsprite.obj
 0001:00020bf0       ?MoveSprite@CEElementSprite@@IAEX_N@Z 10021bf0 f   eelementsprite.obj
 0001:000218a3       ?UVAnimation@CEElementSprite@@IAEXK@Z 100228a3 f   eelementsprite.obj
 0001:00021b83       ?UVAniInterpolation@CEElementSprite@@IAEXK@Z 10022b83 f   eelementsprite.obj
 0001:00021c55       ?GetType@CEElementSprite@@UBE?AW4ENUM_EELEMENT_TYPE@@XZ 10022c55 f i eelementsprite.obj
 0001:00021c61       ?GetTextureInfo@CManagerTexture@@QAEPAUSt_TextureContainer@@PAX@Z 10022c61 f i eelementsprite.obj
 0001:00021d21       ??1CWzSync@@QAE@XZ         10022d21 f i eelementsprite.obj
 0001:00021d44       ?IncNumRenderedSprite@St_EffDbgInfo@@QAEXXZ 10022d44 f i eelementsprite.obj
 0001:00021d74       ?QuaternionRotation@@YAPAUWzQuaternion@@PAU1@PBUWzVector@@M@Z 10022d74 f i eelementsprite.obj
 0001:00021df7       ?QuaternionToMatrix@@YAPAUWzMatrix@@PAU1@PBUWzQuaternion@@@Z 10022df7 f i eelementsprite.obj
 0001:00021fcb       ?GetData@?$CWzHandleManager@PAUSt_TextureContainer@@@@QBEABQAUSt_TextureContainer@@PAX@Z 10022fcb f i eelementsprite.obj
 0001:00022003       ?IsValidHandle@?$CWzHandleManager@PAVCEffectBody@@@@QBEHPAX@Z 10023003 f i effectmanager.obj
 0001:00022003       ?IsValidHandle@?$CWzHandleManager@USt_DAFileInfo@@@@QBEHPAX@Z 10023003 f i ProgramCommonLibForEngine_p:discaccess.obj
 0001:00022003       ?IsValidHandle@?$CWzHandleManager@PAUSt_TextureContainer@@@@QBEHPAX@Z 10023003 f i eelementsprite.obj
 0001:00022052       ?Get@?$CWzArray@PAUSt_TextureContainer@@@@QBEAAPAUSt_TextureContainer@@H@Z 10023052 f i eelementsprite.obj
 0001:00022099       ?FindCube@CDivideCube@@QAEXHPAUSt_Cube@@PBU2@@Z 10023099 f   eelementweather.obj
 0001:000225ad       ??0CEElementWeather@@QAE@XZ 100235ad f   eelementweather.obj
 0001:00022651       ??1CEElementWeather@@UAE@XZ 10023651 f   eelementweather.obj
 0001:000226d2       ?Clear@CEElementWeather@@UAEXXZ 100236d2 f   eelementweather.obj
 0001:000226fd       ?SetElementInfo@CEElementWeather@@UAEXPAUSt_ElementCreate@@@Z 100236fd f   eelementweather.obj
 0001:0002279b       ?Create@CEElementWeather@@UAE_N_N@Z 1002379b f   eelementweather.obj
 0001:000227be       ?Destroy@CEElementWeather@@UAEXXZ 100237be f   eelementweather.obj
 0001:000227cf       ?DestroyAllElements@CEElementWeather@@IAEXXZ 100237cf f   eelementweather.obj
 0001:0002288f       ?Free@CEElementWeather@@UAEXXZ 1002388f f   eelementweather.obj
 0001:000228d3       ?Move@CEElementWeather@@UAE?AW4_ENUM_RESULT_EFFECT_MOVE@@KAA_N@Z 100238d3 f   eelementweather.obj
 0001:00022a2a       ?MoveElement@CEElementWeather@@IAEXKAA_N@Z 10023a2a f   eelementweather.obj
 0001:00022b9c       ?Render@CEElementWeather@@UAEXXZ 10023b9c f   eelementweather.obj
 0001:00022c68       ?CreateElement@CEElementWeather@@IAEXXZ 10023c68 f   eelementweather.obj
 0001:00022eb3       ?GetType@CEElementWeather@@UBE?AW4ENUM_EELEMENT_TYPE@@XZ 10023eb3 f i eelementweather.obj
 0001:00022ebf       ?Outside_Frustum_Vertex@@YAGPBUWzFrustum@@ABUWzVector@@@Z 10023ebf f i eelementweather.obj
 0001:00022f05       ?IncNumRenderedWeather@St_EffDbgInfo@@QAEXXZ 10023f05 f i eelementweather.obj
 0001:00022f35       ?erase@?$list@PAVCEElementBase@@V?$allocator@PAVCEElementBase@@@std@@@std@@QAE?AV?$_Iterator@$00@12@V?$_Const_iterator@$00@12@@Z 10023f35 f i effectbody.obj
 0001:00022f35       ?erase@?$list@U?$pair@QAXPAVCEffectBody@@@std@@V?$allocator@U?$pair@QAXPAVCEffectBody@@@std@@@2@@std@@QAE?AV?$_Iterator@$00@12@V?$_Const_iterator@$00@12@@Z 10023f35 f i effectmanager.obj
 0001:00022f35       ?erase@?$list@U?$pair@$$CBKPAUSt_BodyCreate@@@std@@V?$allocator@U?$pair@$$CBKPAUSt_BodyCreate@@@std@@@2@@std@@QAE?AV?$_Iterator@$00@12@V?$_Const_iterator@$00@12@@Z 10023f35 f i effectmanager.obj
 0001:00022f35       ?erase@?$list@KV?$allocator@K@std@@@std@@QAE?AV?$_Iterator@$00@12@V?$_Const_iterator@$00@12@@Z 10023f35 f i effectmanager.obj
 0001:00022f35       ?erase@?$list@PAVCEElementSprite@@V?$allocator@PAVCEElementSprite@@@std@@@std@@QAE?AV?$_Iterator@$00@12@V?$_Const_iterator@$00@12@@Z 10023f35 f i eelementweather.obj
 0001:00022fe6       ?clear@?$list@PAVCEElementBase@@V?$allocator@PAVCEElementBase@@@std@@@std@@QAEXXZ 10023fe6 f i effectbody.obj
 0001:00022fe6       ?clear@?$list@U?$pair@QAXPAVCEffectBody@@@std@@V?$allocator@U?$pair@QAXPAVCEffectBody@@@std@@@2@@std@@QAEXXZ 10023fe6 f i effectmanager.obj
 0001:00022fe6       ?clear@?$list@KV?$allocator@K@std@@@std@@QAEXXZ 10023fe6 f i effectmanager.obj
 0001:00022fe6       ?clear@?$list@U?$pair@$$CBKPAUSt_BodyCreate@@@std@@V?$allocator@U?$pair@$$CBKPAUSt_BodyCreate@@@std@@@2@@std@@QAEXXZ 10023fe6 f i effectmanager.obj
 0001:00022fe6       ?clear@?$list@PAVCEElementSprite@@V?$allocator@PAVCEElementSprite@@@std@@@std@@QAEXXZ 10023fe6 f i eelementweather.obj
 0001:00023052       ?Alloc@?$CWzMemoryPool@VCEElementSprite@@@@QAEPAVCEElementSprite@@XZ 10024052 f i eelementweather.obj
 0001:0002310a       ?Free@?$CWzMemoryPool@VCEElementFlatChain@@@@QAEXPAVCEElementFlatChain@@@Z 1002410a f i eelementflatchain.obj
 0001:0002310a       ?Free@?$CWzMemoryPool@VCEElementMesh@@@@QAEXPAVCEElementMesh@@@Z 1002410a f i eelementmesh.obj
 0001:0002310a       ?Free@?$CWzMemoryPool@VCEffectBody@@@@QAEXPAVCEffectBody@@@Z 1002410a f i effectmanager.obj
 0001:0002310a       ?Free@?$CWzMemoryPool@VCEElementSprite@@@@QAEXPAVCEElementSprite@@@Z 1002410a f i eelementsprite.obj
 0001:0002310a       ?Free@?$CWzMemoryPool@VCEElementDecal@@@@QAEXPAVCEElementDecal@@@Z 1002410a f i eelementdecal.obj
 0001:0002310a       ?Free@?$CWzMemoryPool@VCEElementWeather@@@@QAEXPAVCEElementWeather@@@Z 1002410a f i eelementweather.obj
 0001:0002310a       ?Free@?$CWzMemoryPool@VCEElementChain@@@@QAEXPAVCEElementChain@@@Z 1002410a f i eelementchain.obj
 0001:00023161       ?_Insert@?$list@PAVCEElementSprite@@V?$allocator@PAVCEElementSprite@@@std@@@std@@QAEXV?$_Const_iterator@$00@12@ABQAVCEElementSprite@@@Z 10024161 f i eelementweather.obj
 0001:00023161       ?_Insert@?$list@KV?$allocator@K@std@@@std@@QAEXV?$_Const_iterator@$00@12@ABK@Z 10024161 f i effectmanager.obj
 0001:00023161       ?_Insert@?$list@PAVCEElementBase@@V?$allocator@PAVCEElementBase@@@std@@@std@@QAEXV?$_Const_iterator@$00@12@ABQAVCEElementBase@@@Z 10024161 f i effectbody.obj
 0001:000231af       ?_Buynode@?$list@KV?$allocator@K@std@@@std@@IAEPAU_Node@?$_List_nod@KV?$allocator@K@std@@@2@PAU342@0ABK@Z 100241af f i effectmanager.obj
 0001:000231af       ?_Buynode@?$list@PAVCEElementBase@@V?$allocator@PAVCEElementBase@@@std@@@std@@IAEPAU_Node@?$_List_nod@PAVCEElementBase@@V?$allocator@PAVCEElementBase@@@std@@@2@PAU342@0ABQAVCEElementBase@@@Z 100241af f i effectbody.obj
 0001:000231af       ?_Buynode@?$list@PAVCEElementSprite@@V?$allocator@PAVCEElementSprite@@@std@@@std@@IAEPAU_Node@?$_List_nod@PAVCEElementSprite@@V?$allocator@PAVCEElementSprite@@@std@@@2@PAU342@0ABQAVCEElementSprite@@@Z 100241af f i eelementweather.obj
 0001:000232b3       ?_Incsize@?$list@PAVCEElementSprite@@V?$allocator@PAVCEElementSprite@@@std@@@std@@IAEXI@Z 100242b3 f i eelementweather.obj
 0001:000232b3       ?_Incsize@?$list@KV?$allocator@K@std@@@std@@IAEXI@Z 100242b3 f i effectmanager.obj
 0001:000232b3       ?_Incsize@?$list@PAVCEElementBase@@V?$allocator@PAVCEElementBase@@@std@@@std@@IAEXI@Z 100242b3 f i effectbody.obj
 0001:0002337d       ??0?$_List_ptr@U?$pair@$$CBKPAUSt_BodyCreate@@@std@@V?$allocator@U?$pair@$$CBKPAUSt_BodyCreate@@@std@@@2@@std@@IAE@V?$allocator@U?$pair@$$CBKPAUSt_BodyCreate@@@std@@@1@@Z 1002437d f i effectmanager.obj
 0001:0002337d       ??0?$_List_ptr@U?$pair@$$CBKV?$basic_string@DU?$char_traits@D@std@@V?$allocator@D@2@@std@@@std@@V?$allocator@U?$pair@$$CBKV?$basic_string@DU?$char_traits@D@std@@V?$allocator@D@2@@std@@@std@@@2@@std@@IAE@V?$allocator@U?$pair@$$CBKV?$basic_string@DU?$char_traits@D@std@@V?$allocator@D@2@@std@@@std@@@1@@Z 1002437d f i loadmanager.obj
 0001:0002337d       ??0?$_List_ptr@PAVCEElementBase@@V?$allocator@PAVCEElementBase@@@std@@@std@@IAE@V?$allocator@PAVCEElementBase@@@1@@Z 1002437d f i effectbody.obj
 0001:0002337d       ??0?$_List_ptr@PAVCEElementSprite@@V?$allocator@PAVCEElementSprite@@@std@@@std@@IAE@V?$allocator@PAVCEElementSprite@@@1@@Z 1002437d f i eelementweather.obj
 0001:0002337d       ??0?$_List_ptr@KV?$allocator@K@std@@@std@@IAE@V?$allocator@K@1@@Z 1002437d f i effectmanager.obj
 0001:0002337d       ??0?$_List_ptr@U?$pair@QAXPAVCEffectBody@@@std@@V?$allocator@U?$pair@QAXPAVCEffectBody@@@std@@@2@@std@@IAE@V?$allocator@U?$pair@QAXPAVCEffectBody@@@std@@@1@@Z 1002437d f i effectmanager.obj
 0001:000233ad       ??$_Allocate@U_Node@?$_List_nod@PAVCEElementSprite@@V?$allocator@PAVCEElementSprite@@@std@@@std@@@std@@YAPAU_Node@?$_List_nod@PAVCEElementSprite@@V?$allocator@PAVCEElementSprite@@@std@@@0@IPAU120@@Z 100243ad f i eelementweather.obj
 0001:000233ad       ??$_Allocate@U_Node@?$_List_nod@PAVCEElementBase@@V?$allocator@PAVCEElementBase@@@std@@@std@@@std@@YAPAU_Node@?$_List_nod@PAVCEElementBase@@V?$allocator@PAVCEElementBase@@@std@@@0@IPAU120@@Z 100243ad f i effectbody.obj
 0001:000233ad       ??$_Allocate@U_Node@?$_List_nod@KV?$allocator@K@std@@@std@@@std@@YAPAU_Node@?$_List_nod@KV?$allocator@K@std@@@0@IPAU120@@Z 100243ad f i effectmanager.obj
 0001:00023400       ??0CEffectBody@@QAE@XZ     10024400 f   effectbody.obj
 0001:00023486       ??1CEffectBody@@UAE@XZ     10024486 f   effectbody.obj
 0001:00023533       ?Clear@CEffectBody@@UAEXXZ 10024533 f   effectbody.obj
 0001:0002363d       ?SetElementInfo@CEffectBody@@UAEXPAUSt_ElementCreate@@@Z 1002463d f   effectbody.obj
 0001:0002366a       ?Create@CEffectBody@@UAE_N_N@Z 1002466a f   effectbody.obj
 0001:00023695       ?Destroy@CEffectBody@@UAEXXZ 10024695 f   effectbody.obj
 0001:000236ae       ?Free@CEffectBody@@UAEXXZ  100246ae f   effectbody.obj
 0001:000236f2       ?CreateElement@CEffectBody@@QAE_NPAUSt_ElementCreate@@H@Z 100246f2 f   effectbody.obj
 0001:00023ad6       ?DestroyAllElements@CEffectBody@@IAEXXZ 10024ad6 f   effectbody.obj
 0001:00023ba0       ?FreeElement@CEffectBody@@IAEXPAVCEElementBase@@@Z 10024ba0 f   effectbody.obj
 0001:00023bd4       ?Move@CEffectBody@@QAE?AW4_ENUM_RESULT_EFFECT_MOVE@@KAA_NH@Z 10024bd4 f   effectbody.obj
 0001:00023d08       ?MoveElement@CEffectBody@@IAEXKH@Z 10024d08 f   effectbody.obj
 0001:00023ede       ?GetTextureHandle@CEffectBody@@UAEXAAV?$vector@PAXV?$allocator@PAX@std@@@std@@@Z 10024ede f   effectbody.obj
 0001:00023f7f       ?ReloadTexture@CEffectBody@@UAEXXZ 10024f7f f   effectbody.obj
 0001:0002401b       ?Render@CEffectBody@@UAEXXZ 1002501b f   effectbody.obj
 0001:0002424d       ?SetResultMatrix@CEffectBody@@UAEXABUWzVector@@00@Z 1002524d f   effectbody.obj
 0001:00024323       ?SetResultMatrix@CEffectBody@@UAEXPBUWzMatrix@@00@Z 10025323 f   effectbody.obj
 0001:00024427       ?SetLifeInfo@CEffectBody@@QAEXKK@Z 10025427 f   effectbody.obj
 0001:00024464       ?SetAllElementTargetPos@CEffectBody@@QAEXABUWzVector@@@Z 10025464 f   effectbody.obj
 0001:00024505       ?AddSoundInfo@CEffectBody@@IAEXPBUSt_ElementCreate@@K@Z 10025505 f   effectbody.obj
 0001:000245b4       ?InitAllSoundInfos@CEffectBody@@IAEXXZ 100255b4 f   effectbody.obj
 0001:0002463b       ?FreeAllSoundInfos@CEffectBody@@IAEXXZ 1002563b f   effectbody.obj
 0001:000246da       ?ProcessSound@CEffectBody@@IAEXXZ 100256da f   effectbody.obj
 0001:000247e0       ?GetType@CEffectBody@@UBE?AW4ENUM_EELEMENT_TYPE@@XZ 100257e0 f i effectbody.obj
 0001:000247ec       ?UpdateBBox@CEffectBody@@IAEXXZ 100257ec f i effectbody.obj
 0001:00024847       ?Alloc@CSoundInfoManager@@QAEPAUSt_SoundInfo@@XZ 10025847 f i effectbody.obj
 0001:0002488c       ?Free@CSoundInfoManager@@QAEXPAUSt_SoundInfo@@@Z 1002588c f i effectbody.obj
 0001:000248d1       ?Put@CSoundInfoManager@@QAE_NPAUSt_SoundInfo@@@Z 100258d1 f i effectbody.obj
 0001:00024926       ?begin@?$list@PAVCEElementBase@@V?$allocator@PAVCEElementBase@@@std@@@std@@QAE?AV?$_Iterator@$00@12@XZ 10025926 f i effectbody.obj
 0001:00024926       ?begin@?$list@U?$pair@$$CBKV?$basic_string@DU?$char_traits@D@std@@V?$allocator@D@2@@std@@@std@@V?$allocator@U?$pair@$$CBKV?$basic_string@DU?$char_traits@D@std@@V?$allocator@D@2@@std@@@std@@@2@@std@@QBE?AV?$_Const_iterator@$00@12@XZ 10025926 f i effectmanager.obj
 0001:00024926       ?begin@?$list@U?$pair@QAXPAVCEffectBody@@@std@@V?$allocator@U?$pair@QAXPAVCEffectBody@@@std@@@2@@std@@QAE?AV?$_Iterator@$00@12@XZ 10025926 f i effectmanager.obj
 0001:00024926       ?begin@?$list@KV?$allocator@K@std@@@std@@QAE?AV?$_Iterator@$00@12@XZ 10025926 f i effectmanager_save.obj
 0001:00024926       ?begin@?$list@U?$pair@$$CBKPAUSt_BodyCreate@@@std@@V?$allocator@U?$pair@$$CBKPAUSt_BodyCreate@@@std@@@2@@std@@QAE?AV?$_Iterator@$00@12@XZ 10025926 f i effectmanager.obj
 0001:00024926       ?begin@?$list@PAVCEElementSprite@@V?$allocator@PAVCEElementSprite@@@std@@@std@@QAE?AV?$_Iterator@$00@12@XZ 10025926 f i eelementweather.obj
 0001:00024974       ?push_back@?$vector@PAXV?$allocator@PAX@std@@@std@@QAEXABQAX@Z 10025974 f i effectmanager.obj
 0001:00024974       ?push_back@?$vector@PAUsEffectTexture@CEffectManager@@V?$allocator@PAUsEffectTexture@CEffectManager@@@std@@@std@@QAEXABQAUsEffectTexture@CEffectManager@@@Z 10025974 f i effectmanager.obj
 0001:00024974       ?push_back@?$vector@PAUSt_SoundInfo@@V?$allocator@PAUSt_SoundInfo@@@std@@@std@@QAEXABQAUSt_SoundInfo@@@Z 10025974 f i effectbody.obj
 0001:00024a3e       ?Alloc@?$CWzMemoryPool@VCEElementMesh@@@@QAEPAVCEElementMesh@@XZ 10025a3e f i effectbody.obj
 0001:00024af6       ?Alloc@?$CWzMemoryPool@VCEElementChain@@@@QAEPAVCEElementChain@@XZ 10025af6 f i effectbody.obj
 0001:00024bae       ?Alloc@?$CWzMemoryPool@VCEElementFlatChain@@@@QAEPAVCEElementFlatChain@@XZ 10025bae f i effectbody.obj
 0001:00024c66       ?Alloc@?$CWzMemoryPool@VCEElementDecal@@@@QAEPAVCEElementDecal@@XZ 10025c66 f i effectbody.obj
 0001:00024d1e       ?Alloc@?$CWzMemoryPool@VCEElementWeather@@@@QAEPAVCEElementWeather@@XZ 10025d1e f i effectbody.obj
 0001:00024dd6       ?_Tidy@?$list@KV?$allocator@K@std@@@std@@IAEXXZ 10025dd6 f i effectmanager.obj
 0001:00024dd6       ?_Tidy@?$list@PAVCEElementBase@@V?$allocator@PAVCEElementBase@@@std@@@std@@IAEXXZ 10025dd6 f i effectbody.obj
 0001:00024dd6       ?_Tidy@?$list@U?$pair@$$CBKPAUSt_BodyCreate@@@std@@V?$allocator@U?$pair@$$CBKPAUSt_BodyCreate@@@std@@@2@@std@@IAEXXZ 10025dd6 f i effectmanager.obj
 0001:00024dd6       ?_Tidy@?$list@U?$pair@QAXPAVCEffectBody@@@std@@V?$allocator@U?$pair@QAXPAVCEffectBody@@@std@@@2@@std@@IAEXXZ 10025dd6 f i effectmanager.obj
 0001:00024dd6       ?_Tidy@?$list@PAVCEElementSprite@@V?$allocator@PAVCEElementSprite@@@std@@@std@@IAEXXZ 10025dd6 f i eelementweather.obj
 0001:00024e0b       ?insert@?$vector@PAXV?$allocator@PAX@std@@@std@@QAE?AV?$_Vector_iterator@PAXV?$allocator@PAX@std@@@2@V?$_Vector_const_iterator@PAXV?$allocator@PAX@std@@@2@ABQAX@Z 10025e0b f i effectmanager.obj
 0001:00024e0b       ?insert@?$vector@PAUsEffectTexture@CEffectManager@@V?$allocator@PAUsEffectTexture@CEffectManager@@@std@@@std@@QAE?AV?$_Vector_iterator@PAUsEffectTexture@CEffectManager@@V?$allocator@PAUsEffectTexture@CEffectManager@@@std@@@2@V?$_Vector_const_iterator@PAUsEffectTexture@CEffectManager@@V?$allocator@PAUsEffectTexture@CEffectManager@@@std@@@2@ABQAUsEffectTexture@CEffectManager@@@Z 10025e0b f i effectmanager.obj
 0001:00024e0b       ?insert@?$vector@PAUSt_SoundInfo@@V?$allocator@PAUSt_SoundInfo@@@std@@@std@@QAE?AV?$_Vector_iterator@PAUSt_SoundInfo@@V?$allocator@PAUSt_SoundInfo@@@std@@@2@V?$_Vector_const_iterator@PAUSt_SoundInfo@@V?$allocator@PAUSt_SoundInfo@@@std@@@2@ABQAUSt_SoundInfo@@@Z 10025e0b f i effectbody.obj
 0001:00024e9b       ?_Buy@?$vector@PAUsEffectTexture@CEffectManager@@V?$allocator@PAUsEffectTexture@CEffectManager@@@std@@@std@@IAE_NI@Z 10025e9b f i effectmanager.obj
 0001:00024e9b       ?_Buy@?$vector@PAXV?$allocator@PAX@std@@@std@@IAE_NI@Z 10025e9b f i effectmanager.obj
 0001:00024e9b       ?_Buy@?$vector@PAUSt_SoundInfo@@V?$allocator@PAUSt_SoundInfo@@@std@@@std@@IAE_NI@Z 10025e9b f i effectbody.obj
 0001:00024f4d       ?_Tidy@?$vector@PAXV?$allocator@PAX@std@@@std@@IAEXXZ 10025f4d f i effectmanager.obj
 0001:00024f4d       ?_Tidy@?$vector@PAUSt_SoundInfo@@V?$allocator@PAUSt_SoundInfo@@@std@@@std@@IAEXXZ 10025f4d f i effectbody.obj
 0001:00024f4d       ?_Tidy@?$vector@PAUsEffectTexture@CEffectManager@@V?$allocator@PAUsEffectTexture@CEffectManager@@@std@@@std@@IAEXXZ 10025f4d f i effectmanager.obj
 0001:00024fbe       ??E?$_Vector_const_iterator@PAUSt_SoundInfo@@V?$allocator@PAUSt_SoundInfo@@@std@@@std@@QAEAAV01@XZ 10025fbe f i effectbody.obj
 0001:00024fbe       ??E?$_Vector_const_iterator@PAXV?$allocator@PAX@std@@@std@@QAEAAV01@XZ 10025fbe f i effectmanager.obj
 0001:00025031       ?AllocObject@?$CWzMemoryBand@VCEffectBody@@@@QAEPAVCEffectBody@@XZ 10026031 f i effectmanager.obj
 0001:00025031       ?AllocObject@?$CWzMemoryBand@VCEElementWeather@@@@QAEPAVCEElementWeather@@XZ 10026031 f i effectbody.obj
 0001:00025031       ?AllocObject@?$CWzMemoryBand@VCEElementChain@@@@QAEPAVCEElementChain@@XZ 10026031 f i effectbody.obj
 0001:00025031       ?AllocObject@?$CWzMemoryBand@VCEElementFlatChain@@@@QAEPAVCEElementFlatChain@@XZ 10026031 f i effectbody.obj
 0001:00025031       ?AllocObject@?$CWzMemoryBand@VCEElementSprite@@@@QAEPAVCEElementSprite@@XZ 10026031 f i eelementweather.obj
 0001:00025031       ?AllocObject@?$CWzMemoryBand@VCEElementDecal@@@@QAEPAVCEElementDecal@@XZ 10026031 f i effectbody.obj
 0001:00025031       ?AllocObject@?$CWzMemoryBand@VCEElementMesh@@@@QAEPAVCEElementMesh@@XZ 10026031 f i effectbody.obj
 0001:00025063       ?_Insert_n@?$vector@PAXV?$allocator@PAX@std@@@std@@IAEXV?$_Vector_const_iterator@PAXV?$allocator@PAX@std@@@2@IABQAX@Z 10026063 f i effectmanager.obj
 0001:00025063       ?_Insert_n@?$vector@PAUSt_SoundInfo@@V?$allocator@PAUSt_SoundInfo@@@std@@@std@@IAEXV?$_Vector_const_iterator@PAUSt_SoundInfo@@V?$allocator@PAUSt_SoundInfo@@@std@@@2@IABQAUSt_SoundInfo@@@Z 10026063 f i effectbody.obj
 0001:00025063       ?_Insert_n@?$vector@PAUsEffectTexture@CEffectManager@@V?$allocator@PAUsEffectTexture@CEffectManager@@@std@@@std@@IAEXV?$_Vector_const_iterator@PAUsEffectTexture@CEffectManager@@V?$allocator@PAUsEffectTexture@CEffectManager@@@std@@@2@IABQAUsEffectTexture@CEffectManager@@@Z 10026063 f i effectmanager.obj
 0001:00025671       ?_Xlen@?$vector@U_List_position@?$_Hash@V?$_Hmap_traits@KV?$basic_string@DU?$char_traits@D@std@@V?$allocator@D@2@@std@@V?$hash_compare@KU?$less@K@std@@@stdext@@V?$allocator@U?$pair@$$CBKV?$basic_string@DU?$char_traits@D@std@@V?$allocator@D@2@@std@@@std@@@2@$0A@@stdext@@@stdext@@V?$allocator@U_List_position@?$_Hash@V?$_Hmap_traits@KV?$basic_string@DU?$char_traits@D@std@@V?$allocator@D@2@@std@@V?$hash_compare@KU?$less@K@std@@@stdext@@V?$allocator@U?$pair@$$CBKV?$basic_string@DU?$char_traits@D@std@@V?$allocator@D@2@@std@@@std@@@2@$0A@@stdext@@@stdext@@@std@@@std@@KAXXZ 10026671 f i effectmanager.obj
 0001:00025671       ?_Xlen@?$vector@USt_AutoCtlParam@@V?$allocator@USt_AutoCtlParam@@@std@@@std@@KAXXZ 10026671 f i effectmanager.obj
 0001:00025671       ?_Xlen@?$vector@U_List_position@?$_Hash@V?$_Hmap_traits@KPAUSt_BodyCreate@@V?$hash_compare@KU?$less@K@std@@@stdext@@V?$allocator@U?$pair@$$CBKPAUSt_BodyCreate@@@std@@@std@@$0A@@stdext@@@stdext@@V?$allocator@U_List_position@?$_Hash@V?$_Hmap_traits@KPAUSt_BodyCreate@@V?$hash_compare@KU?$less@K@std@@@stdext@@V?$allocator@U?$pair@$$CBKPAUSt_BodyCreate@@@std@@@std@@$0A@@stdext@@@stdext@@@std@@@std@@KAXXZ 10026671 f i effectmanager.obj
 0001:00025671       ?_Xlen@?$vector@USt_EffLODParam@@V?$allocator@USt_EffLODParam@@@std@@@std@@KAXXZ 10026671 f i effectmanager.obj
 0001:00025671       ?_Xlen@?$vector@PAXV?$allocator@PAX@std@@@std@@KAXXZ 10026671 f i effectmanager.obj
 0001:00025671       ?_Xlen@?$vector@U_WZNCSPT@WzNaturalCubicSplineDyn@@V?$allocator@U_WZNCSPT@WzNaturalCubicSplineDyn@@@std@@@std@@KAXXZ 10026671 f i Common_p:wznaturalcubicsplinedyn.obj
 0001:00025671       ?_Xlen@?$vector@PAUSt_SoundInfo@@V?$allocator@PAUSt_SoundInfo@@@std@@@std@@KAXXZ 10026671 f i effectbody.obj
 0001:00025671       ?_Xlen@?$vector@U_List_position@?$_Hash@V?$_Hmap_traits@PAXPAVCEffectBody@@V?$hash_compare@PAXU?$less@PAX@std@@@stdext@@V?$allocator@U?$pair@QAXPAVCEffectBody@@@std@@@std@@$0A@@stdext@@@stdext@@V?$allocator@U_List_position@?$_Hash@V?$_Hmap_traits@PAXPAVCEffectBody@@V?$hash_compare@PAXU?$less@PAX@std@@@stdext@@V?$allocator@U?$pair@QAXPAVCEffectBody@@@std@@@std@@$0A@@stdext@@@stdext@@@std@@@std@@KAXXZ 10026671 f i effectmanager.obj
 0001:00025671       ?_Xlen@?$vector@PAUsEffectTexture@CEffectManager@@V?$allocator@PAUsEffectTexture@CEffectManager@@@std@@@std@@KAXXZ 10026671 f i effectmanager.obj
 0001:000256e8       ??0?$_Const_iterator@$00@?$list@PAVCEElementBase@@V?$allocator@PAVCEElementBase@@@std@@@std@@QAE@PAU_Node@?$_List_nod@PAVCEElementBase@@V?$allocator@PAVCEElementBase@@@std@@@2@PBV12@@Z 100266e8 f i effectbody.obj
 0001:000256e8       ??0?$_Const_iterator@$00@?$list@U?$pair@$$CBKPAUSt_BodyCreate@@@std@@V?$allocator@U?$pair@$$CBKPAUSt_BodyCreate@@@std@@@2@@std@@QAE@PAU_Node@?$_List_nod@U?$pair@$$CBKPAUSt_BodyCreate@@@std@@V?$allocator@U?$pair@$$CBKPAUSt_BodyCreate@@@std@@@2@@2@PBV12@@Z 100266e8 f i effectmanager.obj
 0001:000256e8       ??0?$_Const_iterator@$00@?$list@U?$pair@QAXPAVCEffectBody@@@std@@V?$allocator@U?$pair@QAXPAVCEffectBody@@@std@@@2@@std@@QAE@PAU_Node@?$_List_nod@U?$pair@QAXPAVCEffectBody@@@std@@V?$allocator@U?$pair@QAXPAVCEffectBody@@@std@@@2@@2@PBV12@@Z 100266e8 f i effectmanager.obj
 0001:000256e8       ??0?$_Const_iterator@$00@?$list@U?$pair@$$CBKV?$basic_string@DU?$char_traits@D@std@@V?$allocator@D@2@@std@@@std@@V?$allocator@U?$pair@$$CBKV?$basic_string@DU?$char_traits@D@std@@V?$allocator@D@2@@std@@@std@@@2@@std@@QAE@PAU_Node@?$_List_nod@U?$pair@$$CBKV?$basic_string@DU?$char_traits@D@std@@V?$allocator@D@2@@std@@@std@@V?$allocator@U?$pair@$$CBKV?$basic_string@DU?$char_traits@D@std@@V?$allocator@D@2@@std@@@std@@@2@@2@PBV12@@Z 100266e8 f i loadmanager.obj
 0001:000256e8       ??0?$_Const_iterator@$00@?$list@KV?$allocator@K@std@@@std@@QAE@PAU_Node@?$_List_nod@KV?$allocator@K@std@@@2@PBV12@@Z 100266e8 f i effectbody.obj
 0001:000256e8       ??0?$_Const_iterator@$00@?$list@HV?$allocator@H@std@@@std@@QAE@PAU_Node@?$_List_nod@HV?$allocator@H@std@@@2@PBV12@@Z 100266e8 f i effectmanager.obj
 0001:00025723       ??$unchecked_copy@PAPAUSt_SoundInfo@@PAPAU1@@stdext@@YAPAPAUSt_SoundInfo@@PAPAU1@00@Z 10026723 f i effectbody.obj
 0001:00025723       ??$unchecked_copy@PAPAUsEffectTexture@CEffectManager@@PAPAU12@@stdext@@YAPAPAUsEffectTexture@CEffectManager@@PAPAU12@00@Z 10026723 f i effectmanager.obj
 0001:00025723       ??$unchecked_copy@PAPAXPAPAX@stdext@@YAPAPAXPAPAX00@Z 10026723 f i effectmanager.obj
 0001:00025794       ??$_Allocate@PAUSt_SoundInfo@@@std@@YAPAPAUSt_SoundInfo@@IPAPAU1@@Z 10026794 f i effectbody.obj
 0001:00025794       ??$_Allocate@PAX@std@@YAPAPAXIPAPAX@Z 10026794 f i effectmanager.obj
 0001:00025794       ??$_Allocate@V_Aux_cont@std@@@std@@YAPAV_Aux_cont@0@IPAV10@@Z 10026794 f i effectmanager.obj
 0001:00025794       ??$_Allocate@PAUsEffectTexture@CEffectManager@@@std@@YAPAPAUsEffectTexture@CEffectManager@@IPAPAU12@@Z 10026794 f i effectmanager.obj
 0001:000257e7       ??$unchecked_fill_n@PAPAXIPAX@stdext@@YAXPAPAXIABQAX@Z 100267e7 f i effectmanager.obj
 0001:000257e7       ??$unchecked_fill_n@PAPAUSt_SoundInfo@@IPAU1@@stdext@@YAXPAPAUSt_SoundInfo@@IABQAU1@@Z 100267e7 f i effectbody.obj
 0001:000257e7       ??$unchecked_fill_n@PAPAUsEffectTexture@CEffectManager@@IPAU12@@stdext@@YAXPAPAUsEffectTexture@CEffectManager@@IABQAU12@@Z 100267e7 f i effectmanager.obj
 0001:00025851       ??_U@YAPAXI@Z              10026851 f   libcpmt:newaop.obj
 0001:0002585c       ??0length_error@std@@QAE@ABV?$basic_string@DU?$char_traits@D@std@@V?$allocator@D@2@@1@@Z 1002685c f i libcpmt:string.obj
 0001:00025879       ??0out_of_range@std@@QAE@ABV?$basic_string@DU?$char_traits@D@std@@V?$allocator@D@2@@1@@Z 10026879 f i libcpmt:string.obj
 0001:00025896       ?_Xlen@_String_base@std@@SAXXZ 10026896 f   libcpmt:string.obj
 0001:000258ce       ?_Xran@_String_base@std@@SAXXZ 100268ce f   libcpmt:string.obj
 0001:00025906       ??3@YAXPAX@Z               10026906 f   LIBCMT:delete.obj
 0001:00025911       ??0bad_alloc@std@@QAE@XZ   10026911 f i LIBCMT:new.obj
 0001:0002592c       ??2@YAPAXI@Z               1002692c f   LIBCMT:new.obj
 0001:00025991       ?_JumpToContinuation@@YGXPAXPAUEHRegistrationNode@@@Z 10026991 f   LIBCMT:_trnsctrl_.obj
 0001:000259c3       ?_CallMemberFunction1@@YGXPAX00@Z 100269c3 f   LIBCMT:_trnsctrl_.obj
 0001:000259c3       ?_CallMemberFunction2@@YGXPAX00H@Z 100269c3 f   LIBCMT:_trnsctrl_.obj
 0001:000259c3       ?_CallMemberFunction0@@YGXPAX0@Z 100269c3 f   LIBCMT:_trnsctrl_.obj
 0001:000259ca       ?_UnwindNestedFrames@@YGXPAUEHRegistrationNode@@PAUEHExceptionRecord@@@Z 100269ca f   LIBCMT:_trnsctrl_.obj
 0001:00025a1e       ___CxxFrameHandler3        10026a1e f   LIBCMT:_trnsctrl_.obj
 0001:00025a87       ?_CallSETranslator@@YAHPAUEHExceptionRecord@@PAUEHRegistrationNode@@PAX2PBU_s_FuncInfo@@H1@Z 10026a87 f   LIBCMT:_trnsctrl_.obj
 0001:00025bfd       ?_GetRangeOfTrysToCheck@@YAPBU_s_TryBlockMapEntry@@PBU_s_FuncInfo@@HHPAI1@Z 10026bfd f   LIBCMT:_trnsctrl_.obj
 0001:00025c72       __CreateFrameInfo          10026c72 f   LIBCMT:_trnsctrl_.obj
 0001:00025c9e       __IsExceptionObjectToBeDestroyed 10026c9e f   LIBCMT:_trnsctrl_.obj
 0001:00025cc5       __FindAndUnlinkFrame       10026cc5 f   LIBCMT:_trnsctrl_.obj
 0001:00025d17       ?_CallCatchBlock2@@YAPAXPAUEHRegistrationNode@@PBU_s_FuncInfo@@PAXHK@Z 10026d17 f   LIBCMT:_trnsctrl_.obj
 0001:00025d77       @__security_check_cookie@4 10026d77 f   LIBCMT:secchk.obj
 0001:00025d86       __cfltcvt_init             10026d86 f   LIBCMT:_fpinit_.obj
 0001:00025de6       __fpmath                   10026de6 f   LIBCMT:_fpinit_.obj
 0001:00025e09       ??1type_info@@UAE@XZ       10026e09 f   LIBCMT:typinfo.obj
 0001:00025e19       ??_Etype_info@@UAEPAXI@Z   10026e19 f i LIBCMT:typinfo.obj
 0001:00025e19       ??_Gtype_info@@UAEPAXI@Z   10026e19 f i LIBCMT:typinfo.obj
 0001:00025e3a       ??8type_info@@QBE_NABV0@@Z 10026e3a f   LIBCMT:typinfo.obj
 0001:00025e60       _memset                    10026e60 f   LIBCMT:memset.obj
 0001:00025eda       ??_V@YAXPAX@Z              10026eda f   LIBCMT:delete2.obj
 0001:00025ee5       __initp_misc_invarg        10026ee5 f   LIBCMT:invarg.obj
 0001:00025ef4       __invoke_watson            10026ef4 f   LIBCMT:invarg.obj
 0001:0002601c       __invalid_parameter        1002701c f   LIBCMT:invarg.obj
 0001:00026042       __invalid_parameter_noinfo 10027042 f   LIBCMT:invarg.obj
 0001:00026052       _sprintf                   10027052 f   LIBCMT:sprintf.obj
 0001:000260d0       __ftol2_sse                100270d0 f   LIBCMT:ftol2.obj
 0001:000260d9       __ftol2_pentium4           100270d9 f   LIBCMT:ftol2.obj
 0001:000260ec       __ftol2_sse_excpt          100270ec f   LIBCMT:ftol2.obj
 0001:00026106       __ftol2                    10027106 f   LIBCMT:ftol2.obj
 0001:0002617b       __CxxThrowException@8      1002717b f   LIBCMT:throw.obj
 0001:000261c7       ??0exception@std@@QAE@XZ   100271c7 f   LIBCMT:stdexcpt.obj
 0001:000261d8       ??0exception@std@@QAE@ABQBD@Z 100271d8 f   LIBCMT:stdexcpt.obj
 0001:0002622b       ??0exception@std@@QAE@ABQBDH@Z 1002722b f   LIBCMT:stdexcpt.obj
 0001:00026248       ??0exception@std@@QAE@ABV01@@Z 10027248 f   LIBCMT:stdexcpt.obj
 0001:000262a5       ??1exception@std@@UAE@XZ   100272a5 f   LIBCMT:stdexcpt.obj
 0001:000262bb       ?what@exception@std@@UBEPBDXZ 100272bb f   LIBCMT:stdexcpt.obj
 0001:000262c8       ??_Eexception@std@@UAEPAXI@Z 100272c8 f i LIBCMT:stdexcpt.obj
 0001:000262c8       ??_Gexception@std@@UAEPAXI@Z 100272c8 f i LIBCMT:stdexcpt.obj
 0001:000262e9       _memcpy_s                  100272e9 f   LIBCMT:memcpy_s.obj
 0001:00026366       _memmove_s                 10027366 f   LIBCMT:memmove_s.obj
 0001:000263c3       _ldiv                      100273c3 f   LIBCMT:ldiv.obj
 0001:000263d1       ??_L@YGXPAXIHP6EX0@Z1@Z    100273d1 f   LIBCMT:ehvecctr.obj
 0001:00026436       ?__ArrayUnwind@@YGXPAXIHP6EX0@Z@Z 10027436 f   LIBCMT:ehvecdtr.obj
 0001:00026494       ??_M@YGXPAXIHP6EX0@Z@Z     10027494 f   LIBCMT:ehvecdtr.obj
 0001:00026500       _memcpy                    10027500 f   LIBCMT:memcpy.obj
 0001:00026870       __CIsqrt                   10027870 f   LIBCMT:_sqrt_.obj
 0001:00026884       _sqrt                      10027884     LIBCMT:_sqrt_.obj
 0001:0002692a       ??0_LocaleUpdate@@QAE@PAUlocaleinfo_struct@@@Z 1002792a f i LIBCMT:stricmp.obj
 0001:000269b1       ___ascii_stricmp           100279b1 f   LIBCMT:stricmp.obj
 0001:000269ea       __stricmp_l                100279ea f   LIBCMT:stricmp.obj
 0001:00026abf       __stricmp                  10027abf f   LIBCMT:stricmp.obj
 0001:00026abf       _stricmp                   10027abf f   LIBCMT:stricmp.obj
 0001:00026b11       _rand                      10027b11 f   LIBCMT:rand.obj
 0001:00026b40       _memmove                   10027b40 f   LIBCMT:memmove.obj
 0001:00026f5f       ___onexitinit              10027f5f f   LIBCMT:onexit.obj
 0001:00026f90       __onexit                   10027f90 f   LIBCMT:onexit.obj
 0001:00026fcc       _atexit                    10027fcc f   LIBCMT:onexit.obj
 0001:00026ff0       _cos                       10027ff0 f   LIBCMT:_cos_.obj
 0001:00027030       __CIcos                    10028030 f   LIBCMT:_cos_.obj
 0001:0002706b       __CIcos_default            1002806b f   LIBCMT:_cos_.obj
 0001:0002707f       __cos_default              1002807f     LIBCMT:_cos_.obj
 0001:00027120       _sin                       10028120 f   LIBCMT:_sin_.obj
 0001:00027160       __CIsin                    10028160 f   LIBCMT:_sin_.obj
 0001:0002719b       __CIsin_default            1002819b f   LIBCMT:_sin_.obj
 0001:000271af       __sin_default              100281af     LIBCMT:_sin_.obj
 0001:00027249       __CRT_INIT@12              10028249 f   LIBCMT:dllcrt0.obj
 0001:00027474       __DllMainCRTStartup@12     10028474 f   LIBCMT:dllcrt0.obj
 0001:000274a0       _strlen                    100284a0 f   LIBCMT:strlen.obj
 0001:0002752b       __EH_prolog3               1002852b f   LIBCMT:ehprolg3.obj
 0001:0002755e       __EH_prolog3_catch         1002855e f   LIBCMT:ehprolg3.obj
 0001:00027594       _free                      10028594 f   LIBCMT:free.obj
 0001:00027622       _V6_HeapAlloc              10028622 f   LIBCMT:malloc.obj
 0001:00027671       _malloc                    10028671 f   LIBCMT:malloc.obj
 0001:0002773b       __initp_heap_handler       1002873b f   LIBCMT:handler.obj
 0001:0002774a       __callnewh                 1002874a f   LIBCMT:handler.obj
 0001:00027772       ??0bad_exception@std@@QAE@PBD@Z 10028772 f i LIBCMT:frame.obj
 0001:00027790       ??1bad_exception@std@@UAE@XZ 10028790 f i LIBCMT:frame.obj
 0001:0002779b       ??_Ebad_exception@std@@UAEPAXI@Z 1002879b f i LIBCMT:frame.obj
 0001:0002779b       ??_Gbad_exception@std@@UAEPAXI@Z 1002879b f i LIBCMT:frame.obj
 0001:000277c2       ___TypeMatch               100287c2 f   LIBCMT:frame.obj
 0001:00027821       ___FrameUnwindFilter       10028821 f   LIBCMT:frame.obj
 0001:0002786a       ___FrameUnwindToState      1002886a f   LIBCMT:frame.obj
 0001:00027990       ___DestructExceptionObject 10028990 f   LIBCMT:frame.obj
 0001:000279e5       ___AdjustPointer           100289e5 f   LIBCMT:frame.obj
 0001:00027c6e       ___BuildCatchObjectHelper  10028c6e f   LIBCMT:frame.obj
 0001:00027ded       ___BuildCatchObject        10028ded f   LIBCMT:frame.obj
 0001:00028328       ??0bad_exception@std@@QAE@ABV01@@Z 10029328 f i LIBCMT:frame.obj
 0001:00028345       ___InternalCxxFrameHandler 10029345 f   LIBCMT:frame.obj
 0001:0002842b       __encode_pointer           1002942b f   LIBCMT:tidtable.obj
 0001:0002849d       __encoded_null             1002949d f   LIBCMT:tidtable.obj
 0001:000284a6       __decode_pointer           100294a6 f   LIBCMT:tidtable.obj
 0001:00028518       ___crtTlsAlloc@4           10029518 f   LIBCMT:tidtable.obj
 0001:00028521       ___set_flsgetvalue         10029521 f   LIBCMT:tidtable.obj
 0001:00028555       __mtterm                   10029555 f   LIBCMT:tidtable.obj
 0001:00028592       __initptd                  10029592 f   LIBCMT:tidtable.obj
 0001:00028679       __getptd_noexit            10029679 f   LIBCMT:tidtable.obj
 0001:000286f2       __getptd                   100296f2 f   LIBCMT:tidtable.obj
 0001:0002870c       __freefls@4                1002970c f   LIBCMT:tidtable.obj
 0001:0002883b       __freeptd                  1002983b f   LIBCMT:tidtable.obj
 0001:000288a9       __mtinit                   100298a9 f   LIBCMT:tidtable.obj
 0001:00028a36       ?terminate@@YAXXZ          10029a36 f   LIBCMT:hooks.obj
 0001:00028a6f       ?unexpected@@YAXXZ         10029a6f f   LIBCMT:hooks.obj
 0001:00028a82       ?_inconsistency@@YAXXZ     10029a82 f   LIBCMT:hooks.obj
 0001:00028aba       __initp_eh_hooks           10029aba f   LIBCMT:hooks.obj
 0001:00028ad0       __CallSettingFrame@12      10029ad0 f   LIBCMT:lowhelpr.obj
 0001:00028af7       __NLG_Return               10029af7     LIBCMT:lowhelpr.obj
 0001:00028b1c       ___report_gsfailure        10029b1c f   LIBCMT:gs_report.obj
 0001:00028c22       __forcdecpt_l              10029c22 f   LIBCMT:cvt.obj
 0001:00028c95       __cropzeros_l              10029c95 f   LIBCMT:cvt.obj
 0001:00028d17       __positive                 10029d17 f   LIBCMT:cvt.obj
 0001:00028d33       __fassign_l                10029d33 f   LIBCMT:cvt.obj
 0001:00028d75       __fassign                  10029d75 f   LIBCMT:cvt.obj
 0001:00028dae       __forcdecpt                10029dae f   LIBCMT:cvt.obj
 0001:00028dc1       __cropzeros                10029dc1 f   LIBCMT:cvt.obj
 0001:00028f43       __cftoe_l                  10029f43 f   LIBCMT:cvt.obj
 0001:00029013       __cftoe                    1002a013 f   LIBCMT:cvt.obj
 0001:00029033       __cftoa_l                  1002a033 f   LIBCMT:cvt.obj
 0001:0002949d       __cftof_l                  1002a49d f   LIBCMT:cvt.obj
 0001:00029558       __cftog_l                  1002a558 f   LIBCMT:cvt.obj
 0001:00029652       __cfltcvt_l                1002a652 f   LIBCMT:cvt.obj
 0001:000296da       __cfltcvt                  1002a6da f   LIBCMT:cvt.obj
 0001:000296fd       __initp_misc_cfltcvt_tab   1002a6fd f   LIBCMT:cmiscdat.obj
 0001:0002971e       __setdefaultprecision      1002a71e f   LIBCMT:fp8.obj
 0001:00029749       __ms_p5_test_fdiv          1002a749 f   LIBCMT:_testfdiv_.obj
 0001:00029787       __ms_p5_mp_test_fdiv       1002a787 f   LIBCMT:_testfdiv_.obj
 0001:000297b0       ?_Type_info_dtor@type_info@@CAXPAV1@@Z 1002a7b0 f   LIBCMT:typname.obj
 0001:00029820       _strcmp                    1002a820 f   LIBCMT:strcmp.obj
 0001:000298ff       __VEC_memzero              1002a8ff f   LIBCMT:p4_memset.obj
 0001:000299de       __get_sse2_info            1002a9de f   LIBCMT:cpu_disp.obj
 0001:00029a40       ___sse2_available_init     1002aa40 f   LIBCMT:cpu_disp.obj
 0001:00029a4d       __crt_debugger_hook        1002aa4d f   LIBCMT:dbghook.obj
 0001:00029a55       __flsbuf                   1002aa55 f   LIBCMT:_flsbuf.obj
 0001:00029c5f       __output_l                 1002ac5f f   LIBCMT:output.obj
 0001:0002a7f7       __get_errno_from_oserr     1002b7f7 f   LIBCMT:dosmap.obj
 0001:0002a839       __errno                    1002b839 f   LIBCMT:dosmap.obj
 0001:0002a84c       ___doserrno                1002b84c f   LIBCMT:dosmap.obj
 0001:0002a85f       __dosmaperr                1002b85f f   LIBCMT:dosmap.obj
 0001:0002a882       _strcpy_s                  1002b882 f   LIBCMT:strcpy_s.obj
 0001:0002a8ec       __SEH_prolog4              1002b8ec f   LIBCMT:sehprolg4.obj
 0001:0002a931       __SEH_epilog4              1002b931 f   LIBCMT:sehprolg4.obj
 0001:0002a950       __except_handler4          1002b950 f   LIBCMT:chandler4.obj
 0001:0002ab63       __VEC_memcpy               1002bb63 f   LIBCMT:p4_memcpy.obj
 0001:0002ac50       __trandisp1                1002bc50 f   LIBCMT:_87disp_.obj
 0001:0002acb7       __trandisp2                1002bcb7 f   LIBCMT:_87disp_.obj
 0001:0002ad43       __rttospopde               1002bd43     LIBCMT:_87disp_.obj
 0001:0002ad48       __rttospop                 1002bd48     LIBCMT:_87disp_.obj
 0001:0002ad4a       __rtnospop                 1002bd4a     LIBCMT:_87disp_.obj
 0001:0002ad4c       __rttosnpop                1002bd4c     LIBCMT:_87disp_.obj
 0001:0002ad4d       __rtnospopde               1002bd4d     LIBCMT:_87disp_.obj
 0001:0002ad54       __rtzeropop                1002bd54     LIBCMT:_87disp_.obj
 0001:0002ad56       __rtzeronpop               1002bd56     LIBCMT:_87disp_.obj
 0001:0002ad5b       __rtonepop                 1002bd5b     LIBCMT:_87disp_.obj
 0001:0002ad5d       __rtonenpop                1002bd5d     LIBCMT:_87disp_.obj
 0001:0002ad62       __tosnan1                  1002bd62     LIBCMT:_87disp_.obj
 0001:0002ad8d       __nosnan2                  1002bd8d     LIBCMT:_87disp_.obj
 0001:0002ad8f       __tosnan2                  1002bd8f     LIBCMT:_87disp_.obj
 0001:0002adb7       __nan2                     1002bdb7     LIBCMT:_87disp_.obj
 0001:0002adf6       __rtindfpop                1002bdf6     LIBCMT:_87disp_.obj
 0001:0002adf8       __rtindfnpop               1002bdf8     LIBCMT:_87disp_.obj
 0001:0002ae09       __rttosnpopde              1002be09     LIBCMT:_87disp_.obj
 0001:0002ae13       __rtchsifneg               1002be13     LIBCMT:_87disp_.obj
 0001:0002ae20       __startTwoArgErrorHandling 1002be20 f   LIBCMT:_genexcep_.obj
 0001:0002ae37       __startOneArgErrorHandling 1002be37 f   LIBCMT:_genexcep_.obj
 0001:0002ae80       __twoToTOS                 1002be80 f   LIBCMT:_common_.obj
 0001:0002ae95       __load_CW                  1002be95 f   LIBCMT:_common_.obj
 0001:0002aeac       __convertTOStoQNaN         1002beac f   LIBCMT:_common_.obj
 0001:0002aec5       __fload_withFB             1002bec5 f   LIBCMT:_common_.obj
 0001:0002af08       __checkTOS_withFB          1002bf08 f   LIBCMT:_common_.obj
 0001:0002af1e       __fast_exit                1002bf1e f   LIBCMT:_common_.obj
 0001:0002af2b       __math_exit                1002bf2b f   LIBCMT:_common_.obj
 0001:0002af55       __check_overflow_exit      1002bf55 f   LIBCMT:_common_.obj
 0001:0002af69       __check_range_exit         1002bf69 f   LIBCMT:_common_.obj
 0001:0002b232       ___updatetmbcinfo          1002c232 f   LIBCMT:mbctype.obj
 0001:0002b352       __setmbcp_nolock           1002c352 f   LIBCMT:mbctype.obj
 0001:0002b537       __setmbcp                  1002c537 f   LIBCMT:mbctype.obj
 0001:0002b6d1       ___initmbctable            1002c6d1 f   LIBCMT:mbctype.obj
 0001:0002b6ef       ___freetlocinfo            1002c6ef f   LIBCMT:setlocal.obj
 0001:0002b838       ___addlocaleref            1002c838 f   LIBCMT:setlocal.obj
 0001:0002b8c7       ___removelocaleref         1002c8c7 f   LIBCMT:setlocal.obj
 0001:0002b99e       ___updatetlocinfo          1002c99e f   LIBCMT:setlocal.obj
 0001:0002ba14       __tolower_l                1002ca14 f   LIBCMT:tolower.obj
 0001:0002bb29       _tolower                   1002cb29 f   LIBCMT:tolower.obj
 0001:0002bb55       __malloc_crt               1002cb55 f   LIBCMT:crtheap.obj
 0001:0002bb9a       __calloc_crt               1002cb9a f   LIBCMT:crtheap.obj
 0001:0002bbe6       __realloc_crt              1002cbe6 f   LIBCMT:crtheap.obj
 0001:0002bc34       __msize                    1002cc34 f   LIBCMT:msize.obj
 0001:0002bcd7       __crt_waiting_on_module_handle 1002ccd7 f   LIBCMT:crt0dat.obj
 0001:0002bd07       __amsg_exit                1002cd07 f   LIBCMT:crt0dat.obj
 0001:0002bd30       ___crtCorExitProcess       1002cd30 f   LIBCMT:crt0dat.obj
 0001:0002bd5b       ___crtExitProcess          1002cd5b f   LIBCMT:crt0dat.obj
 0001:0002bd73       __lockexit                 1002cd73 f   LIBCMT:crt0dat.obj
 0001:0002bd7c       __unlockexit               1002cd7c f   LIBCMT:crt0dat.obj
 0001:0002bda2       __initterm_e               1002cda2 f   LIBCMT:crt0dat.obj
 0001:0002bdc6       __cinit                    1002cdc6 f   LIBCMT:crt0dat.obj
 0001:0002bf77       __exit                     1002cf77 f   LIBCMT:crt0dat.obj
 0001:0002bf8d       __cexit                    1002cf8d f   LIBCMT:crt0dat.obj
 0001:0002bf9c       __init_pointers            1002cf9c f   LIBCMT:crt0dat.obj
 0001:0002bfea       __sse2_mathfcns_init       1002cfea f   LIBCMT:_mathfcns_.obj
 0001:0002c000       __CIcos_pentium4           1002d000 f   LIBCMT:_cos_pentium4_.obj
 0001:0002c018       __cos_pentium4             1002d018     LIBCMT:_cos_pentium4_.obj
 0001:0002c1b0       __CIsin_pentium4           1002d1b0 f   LIBCMT:_sin_pentium4_.obj
 0001:0002c1c8       __sin_pentium4             1002d1c8     LIBCMT:_sin_pentium4_.obj
 0001:0002c378       __ioinit                   1002d378 f   LIBCMT:ioinit.obj
 0001:0002c5cc       __ioterm                   1002d5cc f   LIBCMT:ioinit.obj
 0001:0002c61a       __setenvp                  1002d61a f   LIBCMT:stdenvp.obj
 0001:0002c892       __setargv                  1002d892 f   LIBCMT:stdargv.obj
 0001:0002c94d       ___crtGetEnvironmentStringsA 1002d94d f   LIBCMT:a_env.obj
 0001:0002ca84       __RTC_Initialize           1002da84 f   LIBCMT:_initsect_.obj
 0001:0002caaa       __RTC_Terminate            1002daaa f   LIBCMT:_initsect_.obj
 0001:0002cad0       __heap_init                1002dad0 f   LIBCMT:heapinit.obj
 0001:0002cb00       __heap_term                1002db00 f   LIBCMT:heapinit.obj
 0001:0002cb74       __initp_misc_winxfltr      1002db74 f   LIBCMT:winxfltr.obj
 0001:0002cb74       __fpclear                  1002db74 f   LIBCMT:_fpinit_.obj
 0001:0002cb75       __XcptFilter               1002db75 f   LIBCMT:winxfltr.obj
 0001:0002ccd5       ___CppXcptFilter           1002dcd5 f   LIBCMT:winxfltr.obj
 0001:0002ccf5       ___security_init_cookie    1002dcf5 f   LIBCMT:gs_support.obj
 0001:0002cd8b       __mtinitlocks              1002dd8b f   LIBCMT:mlock.obj
 0001:0002cdd6       __mtdeletelocks            1002ddd6 f   LIBCMT:mlock.obj
 0001:0002ce2d       __unlock                   1002de2d f   LIBCMT:mlock.obj
 0001:0002ce44       __mtinitlocknum            1002de44 f   LIBCMT:mlock.obj
 0001:0002cf07       __lock                     1002df07 f   LIBCMT:mlock.obj
 0001:0002cf3a       ___sbh_find_block          1002df3a f   LIBCMT:sbheap.obj
 0001:0002cf6a       ___sbh_free_block          1002df6a f   LIBCMT:sbheap.obj
 0001:0002d280       ___sbh_alloc_new_region    1002e280 f   LIBCMT:sbheap.obj
 0001:0002d330       ___sbh_alloc_new_group     1002e330 f   LIBCMT:sbheap.obj
 0001:0002d438       ___sbh_resize_block        1002e438 f   LIBCMT:sbheap.obj
 0001:0002d719       ___sbh_alloc_block         1002e719 f   LIBCMT:sbheap.obj
 0001:0002d9fe       __NMSG_WRITE               1002e9fe f   LIBCMT:crt0msg.obj
 0001:0002dba9       __FF_MSGBANNER             1002eba9 f   LIBCMT:crt0msg.obj
 0001:0002dbe2       ?_ValidateWrite@@YAHPAXI@Z 1002ebe2 f   LIBCMT:validate.obj
 0001:0002dbe2       ?_ValidateExecute@@YAHP6GHXZ@Z 1002ebe2 f   LIBCMT:validate.obj
 0001:0002dbe2       ?_ValidateRead@@YAHPBXI@Z  1002ebe2 f   LIBCMT:validate.obj
 0001:0002dbf4       _abort                     1002ebf4 f   LIBCMT:abort.obj
 0001:0002dd0c       __global_unwind2           1002ed0c f   LIBCMT:exsup.obj
 0001:0002dd71       __local_unwind2            1002ed71 f   LIBCMT:exsup.obj
 0001:0002ddf5       __abnormal_termination     1002edf5 f   LIBCMT:exsup.obj
 0001:0002de18       __NLG_Notify1              1002ee18 f   LIBCMT:exsup.obj
 0001:0002de21       __NLG_Notify               1002ee21 f   LIBCMT:exsup.obj
 0001:0002de38       __NLG_Dispatch             1002ee38     LIBCMT:exsup.obj
 0001:0002de38       __NLG_Dispatch2            1002ee38     LIBCMT:exsup.obj
 0001:0002de40       __NLG_Call                 1002ee40 f   LIBCMT:exsup.obj
 0001:0002de42       __NLG_Return2              1002ee42     LIBCMT:exsup.obj
 0001:0002de50       _strrchr                   1002ee50 f   LIBCMT:strrchr.obj
 0001:0002de7d       __isalpha_l                1002ee7d f i LIBCMT:_ctype.obj
 0001:0002ded3       _isalpha                   1002eed3 f i LIBCMT:_ctype.obj
 0001:0002df03       __isdigit_l                1002ef03 f i LIBCMT:_ctype.obj
 0001:0002df54       _isdigit                   1002ef54 f i LIBCMT:_ctype.obj
 0001:0002df82       __isspace_l                1002ef82 f i LIBCMT:_ctype.obj
 0001:0002dfd3       _isspace                   1002efd3 f i LIBCMT:_ctype.obj
 0001:0002e001       __isalnum_l                1002f001 f i LIBCMT:_ctype.obj
 0001:0002e057       _isalnum                   1002f057 f i LIBCMT:_ctype.obj
 0001:0002e087       __atodbl_l                 1002f087 f   LIBCMT:atodbl.obj
 0001:0002e12f       __atoflt_l                 1002f12f f   LIBCMT:atodbl.obj
 0001:0002e1d7       __fptostr                  1002f1d7 f   LIBCMT:_fptostr.obj
 0001:0002e296       ___dtold                   1002f296 f   LIBCMT:_cfout_.obj
 0001:0002e353       __fltout2                  1002f353 f   LIBCMT:_cfout_.obj
 0001:0002e3f0       __alldvrm                  1002f3f0 f   LIBCMT:lldvrm.obj
 0001:0002e4d0       __aullshr                  1002f4d0 f   LIBCMT:ullshr.obj
 0001:0002e4ef       __fptrap                   1002f4ef f   LIBCMT:crt0fp.obj
 0001:0002e4f8       __controlfp_s              1002f4f8 f   LIBCMT:_contrlfp_.obj
 0001:0002e564       __local_unwind4            1002f564 f   LIBCMT:exsup4.obj
 0001:0002e63a       __seh_longjmp_unwind4@4    1002f63a f   LIBCMT:exsup4.obj
 0001:0002e656       @_EH4_CallFilterFunc@8     1002f656 f   LIBCMT:exsup4.obj
 0001:0002e66d       @_EH4_TransferToHandler@8  1002f66d f   LIBCMT:exsup4.obj
 0001:0002e686       @_EH4_GlobalUnwind@4       1002f686 f   LIBCMT:exsup4.obj
 0001:0002e6a0       @_EH4_LocalUnwind@16       1002f6a0 f   LIBCMT:exsup4.obj
 0001:0002e6b7       __lseeki64_nolock          1002f6b7 f   LIBCMT:lseeki64.obj
 0001:0002e73c       __lseeki64                 1002f73c f   LIBCMT:lseeki64.obj
 0001:0002e855       __write_nolock             1002f855 f   LIBCMT:write.obj
 0001:0002ef88       __write                    1002ff88 f   LIBCMT:write.obj
 0001:0002f064       __getbuf                   10030064 f   LIBCMT:_getbuf.obj
 0001:0002f0ad       __isatty                   100300ad f   LIBCMT:isatty.obj
 0001:0002f111       ___iob_func                10030111 f   LIBCMT:_file.obj
 0001:0002f117       ___initstdio               10030117 f   LIBCMT:_file.obj
 0001:0002f1c8       ___endstdio                100301c8 f   LIBCMT:_file.obj
 0001:0002f1e8       __lock_file                100301e8 f   LIBCMT:_file.obj
 0001:0002f229       __lock_file2               10030229 f   LIBCMT:_file.obj
 0001:0002f25b       __unlock_file              1003025b f   LIBCMT:_file.obj
 0001:0002f297       __unlock_file2             10030297 f   LIBCMT:_file.obj
 0001:0002f2c6       __fileno                   100302c6 f   LIBCMT:fileno.obj
 0001:0002f2f8       __get_printf_count_output  100302f8 f   LIBCMT:printf.obj
 0001:0002f30e       __wctomb_s_l               1003030e f   LIBCMT:wctomb.obj
 0001:0002f47a       _wctomb_s                  1003047a f   LIBCMT:wctomb.obj
 0001:0002f497       __isleadbyte_l             10030497 f i LIBCMT:_wctype.obj
 0001:0002f4cf       _isleadbyte                100304cf f i LIBCMT:_wctype.obj
 0001:0002f4f0       __aulldvrm                 100304f0 f   LIBCMT:ulldvrm.obj
 0001:0002f590       __ValidateImageBase        10030590 f   LIBCMT:pesect.obj
 0001:0002f5d0       __FindPESection            100305d0 f   LIBCMT:pesect.obj
 0001:0002f620       __IsNonwritableInCurrentImage 10030620 f   LIBCMT:pesect.obj
 0001:0002f6dd       __87except                 100306dd f   LIBCMT:_87except_.obj
 0001:0002f81c       __freea                    1003081c f i LIBCMT:a_map.obj
 0001:0002fbe1       ___crtLCMapStringA         10030be1 f   LIBCMT:a_map.obj
 0001:0002fde0       ___crtGetStringTypeA       10030de0 f   LIBCMT:a_str.obj
 0001:0002fe22       ___free_lc_time            10030e22 f   LIBCMT:inittime.obj
 0001:0002ffb7       ___free_lconv_num          10030fb7 f   LIBCMT:initnum.obj
 0001:0002fffc       ___free_lconv_mon          10030ffc f   LIBCMT:initmon.obj
 0001:0003008a       _strcat_s                  1003108a f   LIBCMT:strcat_s.obj
 0001:00030100       _strcspn                   10031100 f   LIBCMT:strcspn.obj
 0001:00030146       _strncpy_s                 10031146 f   LIBCMT:strncpy_s.obj
 0001:00030200       _strpbrk                   10031200 f   LIBCMT:strpbrk.obj
 0001:00030240       __isctype_l                10031240 f   LIBCMT:isctype.obj
 0001:000302f8       __calloc_impl              100312f8 f   LIBCMT:calloc_impl.obj
 0001:00030416       _realloc                   10031416 f   LIBCMT:realloc.obj
 0001:00030631       __initp_misc_winsig        10031631 f   LIBCMT:winsig.obj
 0001:00030686       ___get_sigabrt             10031686 f   LIBCMT:winsig.obj
 0001:00030693       _raise                     10031693 f   LIBCMT:winsig.obj
 0001:00030843       __initp_misc_rand_s        10031843 f   LIBCMT:rand_s.obj
 0001:00030852       __initp_misc_purevirt      10031852 f   LIBCMT:inithelp.obj
 0001:00030861       __initp_misc_initcrit      10031861 f   LIBCMT:initcrit.obj
 0001:00030870       ___crtInitCritSecAndSpinCount 10031870 f   LIBCMT:initcrit.obj
 0001:00030923       __ismbblead_l              10031923 f   LIBCMT:ismbbyte.obj
 0001:0003093c       __ismbblead                1003193c f   LIBCMT:ismbbyte.obj
 0001:00030954       ___crtMessageBoxA          10031954 f   LIBCMT:crtmbox.obj
 0001:00030abd       __set_error_mode           10031abd f   LIBCMT:errmode.obj
 0001:00030b08       __ld12tod                  10031b08 f   LIBCMT:_intrncvt_.obj
 0001:0003104c       __ld12tof                  1003204c f   LIBCMT:_intrncvt_.obj
 0001:00031590       ___strgtold12_l            10032590 f   LIBCMT:_strgtold_.obj
 0001:00031c88       _$I10_OUTPUT               10032c88 f   LIBCMT:_x10fout_.obj
 0001:000326da       __control87                100336da f i LIBCMT:_ieee87_.obj
 0001:000329f0       __allmul                   100339f0 f   LIBCMT:llmul.obj
 0001:00032a24       _atol                      10033a24 f   LIBCMT:atox.obj
 0001:00032a3a       __free_osfhnd              10033a3a f   LIBCMT:osfinfo.obj
 0001:00032ac0       __get_osfhandle            10033ac0 f   LIBCMT:osfinfo.obj
 0001:00032b37       ___lock_fhandle            10033b37 f   LIBCMT:osfinfo.obj
 0001:00032bd7       __unlock_fhandle           10033bd7 f   LIBCMT:osfinfo.obj
 0001:00032bfe       __putwch_nolock            10033bfe f   LIBCMT:putwch.obj
 0001:00032cc3       __mbtowc_l                 10033cc3 f   LIBCMT:mbtowc.obj
 0001:00032dda       _mbtowc                    10033dda f   LIBCMT:mbtowc.obj
 0001:00032e00       __alloca_probe             10033e00     LIBCMT:chkstk.obj
 0001:00032e00       __chkstk                   10033e00 f   LIBCMT:chkstk.obj
 0001:00032e2b       __fcloseall                10033e2b f   LIBCMT:closeall.obj
 0001:00032eca       __flush                    10033eca f   LIBCMT:fflush.obj
 0001:00032f32       __fflush_nolock            10033f32 f   LIBCMT:fflush.obj
 0001:00033054       __flushall                 10034054 f   LIBCMT:fflush.obj
 0001:0003328c       _strtol                    1003428c f   LIBCMT:strtol.obj
 0001:000332b7       __raise_exc_ex             100342b7 f   LIBCMT:_fpexcept_.obj
 0001:00033593       __raise_exc                10034593 f   LIBCMT:_fpexcept_.obj
 0001:000335b6       __handle_exc               100345b6 f   LIBCMT:_fpexcept_.obj
 0001:00033798       __set_errno_from_matherr   10034798 f   LIBCMT:_fpexcept_.obj
 0001:000337c5       __matherr                  100347c5 f   LIBCMT:_matherr_.obj
 0001:000337c8       __statfp                   100347c8 f   LIBCMT:_fpctrl_.obj
 0001:000337d8       __clrfp                    100347d8 f   LIBCMT:_fpctrl_.obj
 0001:000337e9       __ctrlfp                   100347e9 f   LIBCMT:_fpctrl_.obj
 0001:00033812       __set_statfp               10034812 f   LIBCMT:_fpctrl_.obj
 0001:0003386a       ___set_fpsr_sse2           1003486a f   LIBCMT:_fpctrl_.obj
 0001:000338dc       ___ansicp                  100348dc f   LIBCMT:convrtcp.obj
 0001:00033925       ___convertcp               10034925 f   LIBCMT:convrtcp.obj
 0001:00033ae0       __alloca_probe_16          10034ae0 f   LIBCMT:alloca16.obj
 0001:00033af6       __alloca_probe_8           10034af6     LIBCMT:alloca16.obj
 0001:00033b0c       ___mtold12                 10034b0c f   LIBCMT:_mantold_.obj
 0001:00033cda       ___initconout              10034cda f   LIBCMT:initcon.obj
 0001:00033cf9       ___termcon                 10034cf9 f   LIBCMT:initcon.obj
 0001:00033d26       __fclose_nolock            10034d26 f   LIBCMT:fclose.obj
 0001:00033d9d       _fclose                    10034d9d f   LIBCMT:fclose.obj
 0001:00033e19       __commit                   10034e19 f   LIBCMT:commit.obj
 0001:00033efa       __set_exp                  10034efa f   LIBCMT:_util_.obj
 0001:00033f26       __decomp                   10034f26 f   LIBCMT:_util_.obj
 0001:00033fe0       ___ascii_strnicmp          10034fe0 f   LIBCMT:_strnicm.obj
 0001:00034041       __close_nolock             10035041 f   LIBCMT:close.obj
 0001:000340dd       __close                    100350dd f   LIBCMT:close.obj
 0001:000341aa       __freebuf                  100351aa f   LIBCMT:_freebuf.obj
 0001:000341f0       _strchr                    100351f0 f   LIBCMT:strchr.obj
 0001:000341f6       ___from_strstr_to_strchr   100351f6     LIBCMT:strchr.obj
 0001:000342ae       ?GetModuleTitle@?A0x5958724f@WzLog@@YAPBDXZ 100352ae f   ProgramCommonLibForEngine_p:wzlogsystem.obj
 0001:0003436d       ??0WzLogSystem@WzLog@@QAE@XZ 1003536d f   ProgramCommonLibForEngine_p:wzlogsystem.obj
 0001:000343bb       ??1WzLogSystem@WzLog@@UAE@XZ 100353bb f   ProgramCommonLibForEngine_p:wzlogsystem.obj
 0001:000343dd       ?AddLogHandler@WzLogSystem@WzLog@@QAEXPAVWzLogHandler@2@@Z 100353dd f   ProgramCommonLibForEngine_p:wzlogsystem.obj
 0001:00034422       ?Initialize@WzLogSystem@WzLog@@QAEXXZ 10035422 f   ProgramCommonLibForEngine_p:wzlogsystem.obj
 0001:00034592       ?Release@WzLogSystem@WzLog@@QAEXXZ 10035592 f   ProgramCommonLibForEngine_p:wzlogsystem.obj
 0001:0003460d       ?WriteLog@WzLogSystem@WzLog@@QAEXW4WZLOG_TYPE@WzLogType@@PBD@Z 1003560d f   ProgramCommonLibForEngine_p:wzlogsystem.obj
 0001:00034656       ?InitializeWzLogSystem@@YAXXZ 10035656 f   ProgramCommonLibForEngine_p:wzlogsystem.obj
 0001:000346d1       ?ReleaseWzLogSystem@@YAXXZ 100356d1 f   ProgramCommonLibForEngine_p:wzlogsystem.obj
 0001:00034716       ?AddWzLogHandler@@YAXPAVWzLogHandler@WzLog@@@Z 10035716 f   ProgramCommonLibForEngine_p:wzlogsystem.obj
 0001:00034735       ?OutputWzLog@@YAXW4WZLOG_TYPE@WzLogType@@PBDZZ 10035735 f   ProgramCommonLibForEngine_p:wzlogsystem.obj
 0001:00034784       ??_EWzLogSystem@WzLog@@UAEPAXI@Z 10035784 f i ProgramCommonLibForEngine_p:wzlogsystem.obj
 0001:00034784       ??_GWzLogSystem@WzLog@@UAEPAXI@Z 10035784 f i ProgramCommonLibForEngine_p:wzlogsystem.obj
 0001:000347ab       ??_E?$CWzSingleton@VWzLogSystem@WzLog@@@@UAEPAXI@Z 100357ab f i ProgramCommonLibForEngine_p:wzlogsystem.obj
 0001:000347ab       ??_G?$CWzSingleton@VWzLogSystem@WzLog@@@@UAEPAXI@Z 100357ab f i ProgramCommonLibForEngine_p:wzlogsystem.obj
 0001:000347da       ??0CDiscAccess@@QAE@XZ     100357da f   ProgramCommonLibForEngine_p:discaccess.obj
 0001:00034863       ??1CDiscAccess@@QAE@XZ     10035863 f   ProgramCommonLibForEngine_p:discaccess.obj
 0001:000348d9       ?Create@CDiscAccess@@QAEHXZ 100358d9 f   ProgramCommonLibForEngine_p:discaccess.obj
 0001:0003491c       ?Destroy@CDiscAccess@@QAEXXZ 1003591c f   ProgramCommonLibForEngine_p:discaccess.obj
 0001:00034953       ?OpenDisc_Hard@CDiscAccess@@QAEHKPBD@Z 10035953 f   ProgramCommonLibForEngine_p:discaccess.obj
 0001:00034ac6       ?OpenDisc_Packer@CDiscAccess@@QAEHKPBD0W4ENUM_OPEN_PACKER_TYPE@@@Z 10035ac6 f   ProgramCommonLibForEngine_p:discaccess.obj
 0001:00034d9a       ?CloseDisc@CDiscAccess@@QAEXK@Z 10035d9a f   ProgramCommonLibForEngine_p:discaccess.obj
 0001:00034ecd       ?SetActiveDisc@CDiscAccess@@QAEHK@Z 10035ecd f   ProgramCommonLibForEngine_p:discaccess.obj
 0001:00034fd9       ?GetActiveDisc@CDiscAccess@@QAEKXZ 10035fd9 f   ProgramCommonLibForEngine_p:discaccess.obj
 0001:00035024       ?FixFileName@CDiscAccess@@AAEXPADPBD@Z 10036024 f   ProgramCommonLibForEngine_p:discaccess.obj
 0001:000350d5       ?OpenFile@CDiscAccess@@QAEPAXKPBDKKW4ENUM_OPEN_DISPOSITION@@@Z 100360d5 f   ProgramCommonLibForEngine_p:discaccess.obj
 0001:00035528       ?CloseFile@CDiscAccess@@QAEHPAX@Z 10036528 f   ProgramCommonLibForEngine_p:discaccess.obj
 0001:000356d2       ?SeekFile@CDiscAccess@@QAEKPAXJW4ENUM_SEEK_ORIGIN@@@Z 100366d2 f   ProgramCommonLibForEngine_p:discaccess.obj
 0001:000358c8       ?ReadFile@CDiscAccess@@QAEKPAX0K@Z 100368c8 f   ProgramCommonLibForEngine_p:discaccess.obj
 0001:00035a9e       ?WriteFile@CDiscAccess@@QAEKPAXPBXK@Z 10036a9e f   ProgramCommonLibForEngine_p:discaccess.obj
 0001:00035c74       ?FileExists@CDiscAccess@@QAEHKPBD@Z 10036c74 f   ProgramCommonLibForEngine_p:discaccess.obj
 0001:00036016       ?GetFileSize@CDiscAccess@@QAEKPAX@Z 10037016 f   ProgramCommonLibForEngine_p:discaccess.obj
 0001:0003619e       ?GetFileInformationByHandle@CDiscAccess@@QAEHPAXPAUSt_FileInformation@@@Z 1003719e f   ProgramCommonLibForEngine_p:discaccess.obj
 0001:00036490       ?CopyFileA@CDiscAccess@@QAEHKPBD0@Z 10037490 f   ProgramCommonLibForEngine_p:discaccess.obj
 0001:0003675b       ?DeleteFileA@CDiscAccess@@QAEHKPBD@Z 1003775b f   ProgramCommonLibForEngine_p:discaccess.obj
 0001:00036a1e       ?CreateDirectoryA@CDiscAccess@@QAEHKPBD@Z 10037a1e f   ProgramCommonLibForEngine_p:discaccess.obj
 0001:00036ce3       ?RemoveDirectoryA@CDiscAccess@@QAEHKPBD@Z 10037ce3 f   ProgramCommonLibForEngine_p:discaccess.obj
 0001:00036fa6       ??1CWzCriticalSection@@QAE@XZ 10037fa6 f i ProgramCommonLibForEngine_p:discaccess.obj
 0001:00036fc1       ??0?$CWzHandleManager@USt_DAFileInfo@@@@QAE@XZ 10037fc1 f i ProgramCommonLibForEngine_p:discaccess.obj
 0001:0003704d       ??1?$CWzHandleManager@USt_DAFileInfo@@@@UAE@XZ 1003804d f i ProgramCommonLibForEngine_p:discaccess.obj
 0001:000370b9       ?Add@?$CWzHandleManager@USt_DAFileInfo@@@@QAEPAXABUSt_DAFileInfo@@@Z 100380b9 f i ProgramCommonLibForEngine_p:discaccess.obj
 0001:0003718d       ?Release@?$CWzHandleManager@USt_DAFileInfo@@@@QAEHPAX@Z 1003818d f i ProgramCommonLibForEngine_p:discaccess.obj
 0001:00037239       ?GetData@?$CWzHandleManager@USt_DAFileInfo@@@@QBEABUSt_DAFileInfo@@PAX@Z 10038239 f i ProgramCommonLibForEngine_p:discaccess.obj
 0001:00037271       ??_E?$CWzHandleManager@USt_DAFileInfo@@@@UAEPAXI@Z 10038271 f i ProgramCommonLibForEngine_p:discaccess.obj
 0001:00037271       ??_G?$CWzHandleManager@USt_DAFileInfo@@@@UAEPAXI@Z 10038271 f i ProgramCommonLibForEngine_p:discaccess.obj
 0001:00037298       ?Clear@?$CWzHandleManager@USt_DAFileInfo@@@@QAEXXZ 10038298 f i ProgramCommonLibForEngine_p:discaccess.obj
 0001:000372de       ??0?$CWzArray@USt_DAFileInfo@@@@QAE@XZ 100382de f i ProgramCommonLibForEngine_p:discaccess.obj
 0001:00037347       ?Set@?$CWzArray@USt_DAFileInfo@@@@QAEXHABUSt_DAFileInfo@@@Z 10038347 f i ProgramCommonLibForEngine_p:discaccess.obj
 0001:0003739c       ?Get@?$CWzArray@USt_DAFileInfo@@@@QBEAAUSt_DAFileInfo@@H@Z 1003839c f i ProgramCommonLibForEngine_p:discaccess.obj
 0001:000373e3       ?Clear@?$CWzArray@USt_DAFileInfo@@@@QAEXXZ 100383e3 f i ProgramCommonLibForEngine_p:discaccess.obj
 0001:0003740c       ?MakeSureDimensionSize@?$CWzArray@USt_DAFileInfo@@@@AAEXH@Z 1003840c f i ProgramCommonLibForEngine_p:discaccess.obj
 0001:000374da       ??0CScriptRead@@QAE@XZ     100384da f   ProgramCommonLibForEngine_p:scriptread.obj
 0001:000374fb       ??1CScriptRead@@QAE@XZ     100384fb f   ProgramCommonLibForEngine_p:scriptread.obj
 0001:00037514       ?CreateDiscAccess@CScriptRead@@AAEXXZ 10038514 f   ProgramCommonLibForEngine_p:scriptread.obj
 0001:00037596       ?ReleaseDiscAccess@CScriptRead@@AAEXXZ 10038596 f   ProgramCommonLibForEngine_p:scriptread.obj
 0001:000375f8       ?Clear@CScriptRead@@AAEXXZ 100385f8 f   ProgramCommonLibForEngine_p:scriptread.obj
 0001:0003763f       ?SetDiscAccess@CScriptRead@@QAEXPAVCDiscAccess@@@Z 1003863f f   ProgramCommonLibForEngine_p:scriptread.obj
 0001:00037661       ?Create@CScriptRead@@QAEHPBD@Z 10038661 f   ProgramCommonLibForEngine_p:scriptread.obj
 0001:00037747       ?CreateFromBuffer@CScriptRead@@QAEHPBDH@Z 10038747 f   ProgramCommonLibForEngine_p:scriptread.obj
 0001:000377b3       ?Destroy@CScriptRead@@QAEXXZ 100387b3 f   ProgramCommonLibForEngine_p:scriptread.obj
 0001:000377e7       ?GetToken@CScriptRead@@QAE?AW4ENUM_TOKEN_TYPE@@W42@@Z 100387e7 f   ProgramCommonLibForEngine_p:scriptread.obj
 0001:00037aa1       ?GetC@CScriptRead@@AAEEXZ  10038aa1 f i ProgramCommonLibForEngine_p:scriptread.obj
 0001:00037ae5       ??0WzFileLogHandler@WzLog@@QAE@XZ 10038ae5 f   ProgramCommonLibForEngine_p:WzFileLogHandler.obj
 0001:00037b25       ?SetLogFilePath@WzFileLogHandler@WzLog@@QAEXPBD@Z 10038b25 f   ProgramCommonLibForEngine_p:WzFileLogHandler.obj
 0001:00037b6b       ?OnInitialize@WzFileLogHandler@WzLog@@EAEHXZ 10038b6b f   ProgramCommonLibForEngine_p:WzFileLogHandler.obj
 0001:00037ba7       ?OnRelease@WzFileLogHandler@WzLog@@EAEXXZ 10038ba7 f   ProgramCommonLibForEngine_p:WzFileLogHandler.obj
 0001:00037bcc       ?SetFilterLevel@WzFileLogHandler@WzLog@@QAEXH@Z 10038bcc f   ProgramCommonLibForEngine_p:WzFileLogHandler.obj
 0001:00037c04       ?WriteLog@WzFileLogHandler@WzLog@@EAEXW4WZLOG_TYPE@WzLogType@@PBD@Z 10038c04 f   ProgramCommonLibForEngine_p:WzFileLogHandler.obj
 0001:00037cb4       ?WriteLog@WzLogHandler@WzLog@@UAEXW4WZLOG_TYPE@WzLogType@@PBD@Z 10038cb4 f i ProgramCommonLibForEngine_p:WzFileLogHandler.obj
 0001:00037cb4       ?SetFilter@WzLogHandler@WzLog@@UAEXW4WZLOG_TYPE@WzLogType@@H@Z 10038cb4 f i ProgramCommonLibForEngine_p:WzFileLogHandler.obj
 0001:00037cbf       ?GetFilter@WzLogHandler@WzLog@@UAEHW4WZLOG_TYPE@WzLogType@@@Z 10038cbf f i ProgramCommonLibForEngine_p:WzFileLogHandler.obj
 0001:00037ccc       ??_EWzLogHandler@WzLog@@UAEPAXI@Z 10038ccc f i ProgramCommonLibForEngine_p:WzFileLogHandler.obj
 0001:00037ccc       ??_GWzFileLogHandler@WzLog@@UAEPAXI@Z 10038ccc f i ProgramCommonLibForEngine_p:WzFileLogHandler.obj
 0001:00037ccc       ??_GWzLogHandler@WzLog@@UAEPAXI@Z 10038ccc f i ProgramCommonLibForEngine_p:WzFileLogHandler.obj
 0001:00037ccc       ??_EWzFileLogHandler@WzLog@@UAEPAXI@Z 10038ccc f i ProgramCommonLibForEngine_p:WzFileLogHandler.obj
 0001:00037cf4       ?SetFilter@WzFileLogHandler@WzLog@@UAEXW4WZLOG_TYPE@WzLogType@@H@Z 10038cf4 f i ProgramCommonLibForEngine_p:WzFileLogHandler.obj
 0001:00037d0f       ?IsCPUID@FastMath@@YA_NXZ  10038d0f f   Common_p:wzfastmath.obj
 0001:00037d83       ?IsCPUSupport@FastMath@@YA_NW4SlIntrinsic@1@@Z 10038d83 f   Common_p:wzfastmath.obj
 0001:00037e5d       ?IsOSSupport@FastMath@@YA_NW4SlIntrinsic@1@@Z 10038e5d f   Common_p:wzfastmath.obj
 0001:00037f18       ?GetCPUCaps@FastMath@@YAXPAUCPUCaps@1@@Z 10038f18 f   Common_p:wzfastmath.obj
 0001:0003803c       ?Startup@FastMath@@YAXXZ   1003903c f   Common_p:wzfastmath.obj
 0001:000380d5       ??0WzNaturalCubicSplineDyn@@QAE@XZ 100390d5 f   Common_p:wznaturalcubicsplinedyn.obj
 0001:00038110       ??1WzNaturalCubicSplineDyn@@QAE@XZ 10039110 f   Common_p:wznaturalcubicsplinedyn.obj
 0001:00038182       ?Create@WzNaturalCubicSplineDyn@@QAE_NH@Z 10039182 f   Common_p:wznaturalcubicsplinedyn.obj
 0001:00038cc0       ?Destroy@WzNaturalCubicSplineDyn@@QAEXXZ 10039cc0 f   Common_p:wznaturalcubicsplinedyn.obj
 0001:00038d64       ?Add@WzNaturalCubicSplineDyn@@QAEXMM@Z 10039d64 f   Common_p:wznaturalcubicsplinedyn.obj
 0001:00038ea2       ?Calculate@WzNaturalCubicSplineDyn@@QAEHPAMM@Z 10039ea2 f   Common_p:wznaturalcubicsplinedyn.obj
 0001:0003958f       ??0?$vector@USt_EffLODParam@@V?$allocator@USt_EffLODParam@@@std@@@std@@QAE@XZ 1003a58f f i effectmanager.obj
 0001:0003958f       ??0?$vector@U_WZNCSPT@WzNaturalCubicSplineDyn@@V?$allocator@U_WZNCSPT@WzNaturalCubicSplineDyn@@@std@@@std@@QAE@XZ 1003a58f f i Common_p:wznaturalcubicsplinedyn.obj
 0001:0003958f       ??0?$vector@USt_AutoCtlParam@@V?$allocator@USt_AutoCtlParam@@@std@@@std@@QAE@XZ 1003a58f f i effectmanager.obj
 0001:00039611       ??A?$vector@U_WZNCSPT@WzNaturalCubicSplineDyn@@V?$allocator@U_WZNCSPT@WzNaturalCubicSplineDyn@@@std@@@std@@QAEAAU_WZNCSPT@WzNaturalCubicSplineDyn@@I@Z 1003a611 f i Common_p:wznaturalcubicsplinedyn.obj
 0001:00039645       ??$_Unchecked_move_backward@PAUSt_AutoCtlParam@@PAU1@@stdext@@YAPAUSt_AutoCtlParam@@PAU1@00@Z 1003a645 f i effectmanager.obj
 0001:00039645       ??$_Unchecked_move_backward@PAU_List_position@?$_Hash@V?$_Hmap_traits@KV?$basic_string@DU?$char_traits@D@std@@V?$allocator@D@2@@std@@V?$hash_compare@KU?$less@K@std@@@stdext@@V?$allocator@U?$pair@$$CBKV?$basic_string@DU?$char_traits@D@std@@V?$allocator@D@2@@std@@@std@@@2@$0A@@stdext@@@stdext@@PAU123@@stdext@@YAPAU_List_position@?$_Hash@V?$_Hmap_traits@KV?$basic_string@DU?$char_traits@D@std@@V?$allocator@D@2@@std@@V?$hash_compare@KU?$less@K@std@@@stdext@@V?$allocator@U?$pair@$$CBKV?$basic_string@DU?$char_traits@D@std@@V?$allocator@D@2@@std@@@std@@@2@$0A@@stdext@@@0@PAU120@00@Z 1003a645 f i effectmanager.obj
 0001:00039645       ??$_Unchecked_move_backward@PAUSt_EffLODParam@@PAU1@@stdext@@YAPAUSt_EffLODParam@@PAU1@00@Z 1003a645 f i effectmanager.obj
 0001:00039645       ??$_Unchecked_move_backward@PAU_WZNCSPT@WzNaturalCubicSplineDyn@@PAU12@@stdext@@YAPAU_WZNCSPT@WzNaturalCubicSplineDyn@@PAU12@00@Z 1003a645 f i Common_p:wznaturalcubicsplinedyn.obj
 0001:00039645       ??$_Unchecked_move_backward@PAU_List_position@?$_Hash@V?$_Hmap_traits@KPAUSt_BodyCreate@@V?$hash_compare@KU?$less@K@std@@@stdext@@V?$allocator@U?$pair@$$CBKPAUSt_BodyCreate@@@std@@@std@@$0A@@stdext@@@stdext@@PAU123@@stdext@@YAPAU_List_position@?$_Hash@V?$_Hmap_traits@KPAUSt_BodyCreate@@V?$hash_compare@KU?$less@K@std@@@stdext@@V?$allocator@U?$pair@$$CBKPAUSt_BodyCreate@@@std@@@std@@$0A@@stdext@@@0@PAU120@00@Z 1003a645 f i effectmanager.obj
 0001:00039645       ??$_Unchecked_move_backward@PAU_List_position@?$_Hash@V?$_Hmap_traits@PAXPAVCEffectBody@@V?$hash_compare@PAXU?$less@PAX@std@@@stdext@@V?$allocator@U?$pair@QAXPAVCEffectBody@@@std@@@std@@$0A@@stdext@@@stdext@@PAU123@@stdext@@YAPAU_List_position@?$_Hash@V?$_Hmap_traits@PAXPAVCEffectBody@@V?$hash_compare@PAXU?$less@PAX@std@@@stdext@@V?$allocator@U?$pair@QAXPAVCEffectBody@@@std@@@std@@$0A@@stdext@@@0@PAU120@00@Z 1003a645 f i effectmanager.obj
 0001:00039681       ?MatrixRotationX_Scalar@@YAPAUWzMatrix@@PAU1@M@Z 1003a681 f i Common_p:wzmath.obj
 0001:00039795       ?MatrixRotationY_Scalar@@YAPAUWzMatrix@@PAU1@M@Z 1003a795 f i Common_p:wzmath.obj
 0001:000398a8       ?MatrixRotationZ_Scalar@@YAPAUWzMatrix@@PAU1@M@Z 1003a8a8 f i Common_p:wzmath.obj
 0001:000399bc       ?QuaternionMultiply_Scalar@@YAPAUWzQuaternion@@PAU1@PBU1@1@Z 1003a9bc f i Common_p:wzmath.obj
 0001:00039aab       ?MatrixInverse@@YAPAUWzMatrix@@PAU1@PBU1@@Z 1003aaab f   Common_p:wzmath.obj
 0001:0003a367       ?MatrixRotationZYX@@YAPAUWzMatrix@@PAU1@PBUWzVector@@@Z 1003b367 f   Common_p:wzmath.obj
 0001:0003a533       ?MatrixRotationZXY@@YAPAUWzMatrix@@PAU1@PBUWzVector@@@Z 1003b533 f   Common_p:wzmath.obj
 0001:0003a6fc       ?MatrixMultiply_Scalar@@YAPAUWzMatrix@@PAU1@PBU1@1@Z 1003b6fc f   Common_p:wzmath.obj
 0001:0003aabb       ?MatrixMultiply4x3_Scalar@@YAPAUWzMatrix@@PAU1@PBU1@1@Z 1003babb f   Common_p:wzmath.obj
 0001:0003ad35       ?MatrixRotationX_SSE@@YAPAUWzMatrix@@PAU1@M@Z 1003bd35 f   Common_p:wzmath.obj
 0001:0003ad6c       ?MatrixRotationY_SSE@@YAPAUWzMatrix@@PAU1@M@Z 1003bd6c f   Common_p:wzmath.obj
 0001:0003ada0       ?MatrixRotationZ_SSE@@YAPAUWzMatrix@@PAU1@M@Z 1003bda0 f   Common_p:wzmath.obj
 0001:0003add4       ?MatrixMultiply_SSE@@YAPAUWzMatrix@@PAU1@PBU1@1@Z 1003bdd4 f   Common_p:wzmath.obj
 0001:0003aeef       ?MatrixRotationX_3DNOW@@YAPAUWzMatrix@@PAU1@M@Z 1003beef f   Common_p:wzmath.obj
 0001:0003af3a       ?MatrixRotationY_3DNOW@@YAPAUWzMatrix@@PAU1@M@Z 1003bf3a f   Common_p:wzmath.obj
 0001:0003af82       ?MatrixRotationZ_3DNOW@@YAPAUWzMatrix@@PAU1@M@Z 1003bf82 f   Common_p:wzmath.obj
 0001:0003afca       ?MatrixMultiply_3DNOW@@YAPAUWzMatrix@@PAU1@PBU1@1@Z 1003bfca f   Common_p:wzmath.obj
 0001:0003b18e       ?RotationToQuaternion@@YAPAUWzQuaternion@@PAU1@PBUWzVector@@@Z 1003c18e f   Common_p:wzmath.obj
 0001:0003b292       ?GetQuaternionToConvertVector@@YAPAUWzQuaternion@@PAU1@PBUWzVector@@1@Z 1003c292 f   Common_p:wzmath.obj
 0001:0003b3db       ?MatrixToQuaternion@@YAPAUWzQuaternion@@PAU1@PBUWzMatrix@@@Z 1003c3db f   Common_p:wzmath.obj
 0001:0003b5bc       ?QuaternionToAxisAngle@@YAXPAUWzVector@@PAMPBUWzQuaternion@@@Z 1003c5bc f   Common_p:wzmath.obj
 0001:0003b6b2       ?QuaternionSlerp@@YAPAUWzQuaternion@@PAU1@PBU1@1M@Z 1003c6b2 f   Common_p:wzmath.obj
 0001:0003b828       ?QuaternionMultiply_SSE@@YAPAUWzQuaternion@@PAU1@PBU1@1@Z 1003c828 f   Common_p:wzmath.obj
 0001:0003b89a       ?QuaternionMultiply_3DNOWEXT@@YAPAUWzQuaternion@@PAU1@PBU1@1@Z 1003c89a f   Common_p:wzmath.obj
 0001:0003b943       ?MatrixSetZero@@YAPAUWzMatrix@@PAU1@@Z 1003c943 f i Common_p:wzmath.obj
 0001:0003ba4a       ??0WzNaturalCubicSpline@@QAE@XZ 1003ca4a f   Common_p:wznaturalcubicspline.obj
 0001:0003ba63       ??1WzNaturalCubicSpline@@QAE@XZ 1003ca63 f   Common_p:wznaturalcubicspline.obj
 0001:0003ba6c       ?Create@WzNaturalCubicSpline@@QAE_NH@Z 1003ca6c f   Common_p:wznaturalcubicspline.obj
 0001:0003be64       ?Destroy@WzNaturalCubicSpline@@QAEXXZ 1003ce64 f   Common_p:wznaturalcubicspline.obj
 0001:0003be7a       ?Add@WzNaturalCubicSpline@@QAEXMM@Z 1003ce7a f   Common_p:wznaturalcubicspline.obj
 0001:0003bf35       ?Calculate@WzNaturalCubicSpline@@QAEHPAMM@Z 1003cf35 f   Common_p:wznaturalcubicspline.obj
 0001:0003c194       ?Math_GetOrthogonalVectors@@YAXPAUWzVector@@0PBU1@@Z 1003d194 f   Common_p:mathassistant.obj
 0001:0003c206       ?Math_GetRandomDirection@@YAPAUWzVector@@PAU1@PBU1@M@Z 1003d206 f   Common_p:mathassistant.obj
 0001:0003c31a       ?Math_GetRandomPosInBoundingVolume@@YAXPAUWzVector@@PBUWzBoundingVolume@@@Z 1003d31a f   Common_p:mathassistant.obj
 0001:0003c45a       _RtlUnwind@16              1003d45a f   kernel32:KERNEL32.dll
 0001:0003c460       __vsnprintf_l              1003d460 f   LIBCMT:vsnprint.obj
 0001:0003c513       __vsnprintf                1003d513 f   LIBCMT:vsnprint.obj
 0001:0003c530       __atof_l                   1003d530 f   LIBCMT:atof.obj
 0001:0003c5db       _atof                      1003d5db f   LIBCMT:atof.obj
 0001:0003c5ee       __snprintf                 1003d5ee f   LIBCMT:snprintf.obj
 0001:0003c6a0       _acos                      1003d6a0 f   LIBCMT:_acos_.obj
 0001:0003c6e0       __CIacos                   1003d6e0 f   LIBCMT:_acos_.obj
 0001:0003c71b       __CIacos_default           1003d71b f   LIBCMT:_acos_.obj
 0001:0003c72f       __acos_default             1003d72f     LIBCMT:_acos_.obj
 0001:0003c7e6       __fltin2                   1003d7e6 f   LIBCMT:_cfin_.obj
 0001:0003c890       __CIacos_pentium4          1003d890 f   LIBCMT:_acos_pentium4_.obj
 0001:0003c8a8       __acos_pentium4            1003d8a8     LIBCMT:_acos_pentium4_.obj
 0001:0003cde4       ___libm_error_support      1003dde4 f   LIBCMT:_libm_error_.obj
 0001:0003d0a0       ??1CAutoFree@@QAE@XZ       1003e0a0 f   wzFilePacker_static:wzFilePacker.obj
 0001:0003d0b0       ?CONVERT_PATHCHAR@CPackFile@@CAXPAD@Z 1003e0b0 f i wzFilePacker_static:wzFilePacker.obj
 0001:0003d110       ??0CPackFile@@QAE@XZ       1003e110 f   wzFilePacker_static:wzFilePacker.obj
 0001:0003d140       ?Close@CPackFile@@QAEXXZ   1003e140 f   wzFilePacker_static:wzFilePacker.obj
 0001:0003d160       ?OpenFile@CPackFile@@QAEPAXPBDK@Z 1003e160 f   wzFilePacker_static:wzFilePacker.obj
 0001:0003d190       ?DeleteFileA@CPackFile@@QAEHPBD@Z 1003e190 f   wzFilePacker_static:wzFilePacker.obj
 0001:0003d190       ?RemoveDirectoryA@CPackFile@@QAEHPBD@Z 1003e190 f   wzFilePacker_static:wzFilePacker.obj
 0001:0003d1b0       ?FileExists@CPackFile@@QAEHPBD@Z 1003e1b0 f   wzFilePacker_static:wzFilePacker.obj
 0001:0003d1d0       ?CreateDirectoryA@CPackFile@@QAEHPBD@Z 1003e1d0 f   wzFilePacker_static:wzFilePacker.obj
 0001:0003d200       ?CloseFile@CPackFile@@QAEXPAX@Z 1003e200 f   wzFilePacker_static:wzFilePacker.obj
 0001:0003d210       ?GetFileProperties@CPackFile@@QAEHPAXPAUFileProperties@@@Z 1003e210 f   wzFilePacker_static:wzFilePacker.obj
 0001:0003d2c0       ?ReadFile@CPackFile@@QAEHPAX0K@Z 1003e2c0 f   wzFilePacker_static:wzFilePacker.obj
 0001:0003d2e0       ?WriteFile@CPackFile@@QAEHPAXPBXK@Z 1003e2e0 f   wzFilePacker_static:wzFilePacker.obj
 0001:0003d300       ?GetFileSize@CPackFile@@QAEHPAXPA_K@Z 1003e300 f   wzFilePacker_static:wzFilePacker.obj
 0001:0003d310       ?GetFilePointer@CPackFile@@QAEHPAXPA_K@Z 1003e310 f   wzFilePacker_static:wzFilePacker.obj
 0001:0003d320       ?SetFilePointer@CPackFile@@QAEHPAX_KK@Z 1003e320 f   wzFilePacker_static:wzFilePacker.obj
 0001:0003d340       ?AddFile@CPackFile@@QAEHPBD0@Z 1003e340 f   wzFilePacker_static:wzFilePacker.obj
 0001:0003d450       ??1CPackFile@@QAE@XZ       1003e450 f   wzFilePacker_static:wzFilePacker.obj
 0001:0003d460       ?Open@CPackFile@@QAEPAXPBD0K@Z 1003e460 f   wzFilePacker_static:wzFilePacker.obj
 0001:0003d580       @geVFile_CloseAPI@0        1003e580 f   wzFilePacker_static:vfile.obj
 0001:0003d640       @geVFile_Open_Detail@20    1003e640 f   wzFilePacker_static:vfile.obj
 0001:0003d730       @geVFile_Open@12           1003e730 f   wzFilePacker_static:vfile.obj
 0001:0003d820       @geVFile_DeleteFile@8      1003e820 f   wzFilePacker_static:vfile.obj
 0001:0003d830       @geVFile_FileExists@8      1003e830 f   wzFilePacker_static:vfile.obj
 0001:0003d840       @geVFile_Close@4           1003e840 f   wzFilePacker_static:vfile.obj
 0001:0003d890       @geVFile_GetS@12           1003e890 f   wzFilePacker_static:vfile.obj
 0001:0003d8b0       @geVFile_Read@12           1003e8b0 f   wzFilePacker_static:vfile.obj
 0001:0003d8e0       @geVFile_Write@12          1003e8e0 f   wzFilePacker_static:vfile.obj
 0001:0003d910       @geVFile_Seek@16           1003e910 f   wzFilePacker_static:vfile.obj
 0001:0003d930       @geVFile_Tell@8            1003e930 f   wzFilePacker_static:vfile.obj
 0001:0003d940       @geVFile_Size@8            1003e940 f   wzFilePacker_static:vfile.obj
 0001:0003d950       @geVFile_GetProperties@8   1003e950 f   wzFilePacker_static:vfile.obj
 0001:0003d960       @geVFile_EnlargeDirectorySize@8 1003e960 f   wzFilePacker_static:vfile.obj
 0001:0003d970       @geVFile_SetVersion@8      1003e970 f   wzFilePacker_static:vfile.obj
 0001:0003d980       @geVFile_IsPrevVersion@4   1003e980 f   wzFilePacker_static:vfile.obj
 0001:0003d990       @geVFile_OpenNewSystem@20  1003e990 f   wzFilePacker_static:vfile.obj
 0001:0003dad0       _CopyVFile                 1003ead0 f   wzFilePacker_static:vFile_util.obj
 0001:0003dc40       _CopyOneFile               1003ec40 f   wzFilePacker_static:vFile_util.obj
 0001:0003dcc0       _MakeDirectory             1003ecc0 f   wzFilePacker_static:vFile_util.obj
 0001:0003ddb0       _geRam_Allocate            1003edb0 f   wzFilePacker_static:Ram.obj
 0001:0003ddd0       _geRam_Free_               1003edd0 f   wzFilePacker_static:Ram.obj
 0001:0003dde0       _geRam_Realloc             1003ede0 f   wzFilePacker_static:Ram.obj
 0001:0003de40       _Encrypt                   1003ee40 f   wzFilePacker_static:fsvfs.obj
 0001:0003de80       _Decrypt                   1003ee80 f   wzFilePacker_static:fsvfs.obj
 0001:0003f850       @FSVFS_GetAPIs@0           10040850 f   wzFilePacker_static:fsvfs.obj
 0001:00040010       @FSMemory_GetAPIs@0        10041010 f   wzFilePacker_static:FSMEMORY.obj
 0001:00040ca0       @FSDos_GetAPIs@0           10041ca0 f   wzFilePacker_static:fsdos.obj
 0001:00040cb0       _DirTree_Create            10041cb0 f   wzFilePacker_static:dirtree.obj
 0001:00040d00       _DirTree_Destroy           10041d00 f   wzFilePacker_static:dirtree.obj
 0001:00040fa0       _DirTree_SetFileSize       10041fa0 f   wzFilePacker_static:dirtree.obj
 0001:00040fc0       _DirTree_GetFileSize       10041fc0 f   wzFilePacker_static:dirtree.obj
 0001:00040fe0       _DirTree_WriteToFile       10041fe0 f   wzFilePacker_static:dirtree.obj
 0001:00041010       _DirTree_GetSize           10042010 f   wzFilePacker_static:dirtree.obj
 0001:00041430       _DirTree_CreateFromFile    10042430 f   wzFilePacker_static:dirtree.obj
 0001:000417b0       _DirTree_FindExact         100427b0 f   wzFilePacker_static:dirtree.obj
 0001:00041810       _DirTree_FindPartial       10042810 f   wzFilePacker_static:dirtree.obj
 0001:00041890       _DirTree_AddFile           10042890 f   wzFilePacker_static:dirtree.obj
 0001:00041960       _DirTree_Remove            10042960 f   wzFilePacker_static:dirtree.obj
 0001:000419f0       _DirTree_SetFileAttributes 100429f0 f   wzFilePacker_static:dirtree.obj
 0001:00041a10       _DirTree_GetFileAttributes 10042a10 f   wzFilePacker_static:dirtree.obj
 0001:00041a20       _DirTree_SetFileOffset     10042a20 f   wzFilePacker_static:dirtree.obj
 0001:00041a40       _DirTree_GetFileOffset     10042a40 f   wzFilePacker_static:dirtree.obj
 0001:00041a60       _DirTree_SetFileTime       10042a60 f   wzFilePacker_static:dirtree.obj
 0001:00041a80       _DirTree_GetFileTime       10042a80 f   wzFilePacker_static:dirtree.obj
 0001:00041aa0       _DirTree_SetFileHints      10042aa0 f   wzFilePacker_static:dirtree.obj
 0001:00041b10       _DirTree_GetFileHints      10042b10 f   wzFilePacker_static:dirtree.obj
 0001:00041b30       _DirTree_GetName           10042b30 f   wzFilePacker_static:dirtree.obj
 0001:00041b70       _DirTree_FileExists        10042b70 f   wzFilePacker_static:dirtree.obj
 0001:00041b90       _DirTree_CreateFinder      10042b90 f   wzFilePacker_static:dirtree.obj
 0001:00041cc0       _DirTree_DestroyFinder     10042cc0 f   wzFilePacker_static:dirtree.obj
 0001:00041d00       _DirTree_FinderGetNextFile 10042d00 f   wzFilePacker_static:dirtree.obj
 0001:00041dc0       _DirTree_SetAllFileOffset  10042dc0 f   wzFilePacker_static:dirtree.obj
 0001:00041e70       _DuplicateString           10042e70 f   wzFilePacker_static:dirtree-common.obj
 0001:00041eb0       _GetNextDir                10042eb0 f   wzFilePacker_static:dirtree-common.obj
 0001:00041ee0       _MatchPattern              10042ee0 f   wzFilePacker_static:dirtree-common.obj
 0001:00041f40       _PathHasDir                10042f40 f   wzFilePacker_static:dirtree-common.obj
 0001:00041f56       __mbsstr_l                 10042f56 f   LIBCMT:mbsstr.obj
 0001:00042097       __mbsstr                   10043097 f   LIBCMT:mbsstr.obj
 0001:000420b0       _memchr                    100430b0 f   LIBCMT:memchr.obj
 0001:00042160       _strncpy                   10043160 f   LIBCMT:strncpy.obj
 0001:00042476       __splitpath                10043476 f   LIBCMT:splitpat.obj
 0001:000424d0       _strstr                    100434d0 f   LIBCMT:strstr.obj
 0001:00042556       __mbsnbcpy_s               10043556 f   LIBCMT:mbsnbcpy_s.obj
 0001:00042573       __mbsnbcpy_s_l             10043573 f   LIBCMT:mbsnbcpy_s_l.obj
 0002:00000000       __imp_?SetCurrentAnimation@CWzUnitDraw@@QAEXKHHH@Z 10045000     3dfileaccess_p:3DFileAccess_p.dll
 0002:00000004       __imp_?SetScale@CWzUnitDraw@@QAEXMMMH@Z 10045004     3dfileaccess_p:3DFileAccess_p.dll
 0002:00000008       __imp_?SetRotation@CWzUnitDraw@@QAEXABUWzVector@@H@Z 10045008     3dfileaccess_p:3DFileAccess_p.dll
 0002:0000000c       __imp_?SetPosition@CWzUnitDraw@@QAEXABUWzVector@@H@Z 1004500c     3dfileaccess_p:3DFileAccess_p.dll
 0002:00000010       __imp__Func_ContactWzd     10045010     3dfileaccess_p:3DFileAccess_p.dll
 0002:00000014       __imp_?EnableShadowReceive@CWzUnitDraw@@QAEXHH@Z 10045014     3dfileaccess_p:3DFileAccess_p.dll
 0002:00000018       __imp_?EnableShadowCast@CWzUnitDraw@@QAEXHH@Z 10045018     3dfileaccess_p:3DFileAccess_p.dll
 0002:0000001c       __imp_?SetWzUnit@CWzUnitDraw@@QAEXPAVCWzUnit@@H@Z 1004501c     3dfileaccess_p:3DFileAccess_p.dll
 0002:00000020       \1773DFileAccess_p_NULL_THUNK_DATA 10045020     3dfileaccess_p:3DFileAccess_p.dll
 0002:00000024       __imp__EnterCriticalSection@4 10045024     kernel32:KERNEL32.dll
 0002:00000028       __imp__LeaveCriticalSection@4 10045028     kernel32:KERNEL32.dll
 0002:0000002c       __imp__RtlUnwind@16        1004502c     kernel32:KERNEL32.dll
 0002:00000030       __imp__TerminateProcess@8  10045030     kernel32:KERNEL32.dll
 0002:00000034       __imp__GetCurrentProcess@0 10045034     kernel32:KERNEL32.dll
 0002:00000038       __imp__UnhandledExceptionFilter@4 10045038     kernel32:KERNEL32.dll
 0002:0000003c       __imp__SetUnhandledExceptionFilter@4 1004503c     kernel32:KERNEL32.dll
 0002:00000040       __imp__IsDebuggerPresent@0 10045040     kernel32:KERNEL32.dll
 0002:00000044       __imp__RaiseException@16   10045044     kernel32:KERNEL32.dll
 0002:00000048       __imp__GetCurrentThreadId@0 10045048     kernel32:KERNEL32.dll
 0002:0000004c       __imp__GetCommandLineA@0   1004504c     kernel32:KERNEL32.dll
 0002:00000050       __imp__GetLastError@0      10045050     kernel32:KERNEL32.dll
 0002:00000054       __imp__HeapFree@12         10045054     kernel32:KERNEL32.dll
 0002:00000058       __imp__HeapAlloc@12        10045058     kernel32:KERNEL32.dll
 0002:0000005c       __imp__GetModuleHandleW@4  1004505c     kernel32:KERNEL32.dll
 0002:00000060       __imp__GetProcAddress@8    10045060     kernel32:KERNEL32.dll
 0002:00000064       __imp__TlsGetValue@4       10045064     kernel32:KERNEL32.dll
 0002:00000068       __imp__TlsAlloc@0          10045068     kernel32:KERNEL32.dll
 0002:0000006c       __imp__TlsSetValue@8       1004506c     kernel32:KERNEL32.dll
 0002:00000070       __imp__TlsFree@4           10045070     kernel32:KERNEL32.dll
 0002:00000074       __imp__InterlockedIncrement@4 10045074     kernel32:KERNEL32.dll
 0002:00000078       __imp__SetLastError@4      10045078     kernel32:KERNEL32.dll
 0002:0000007c       __imp__InterlockedDecrement@4 1004507c     kernel32:KERNEL32.dll
 0002:00000080       __imp__GetModuleHandleA@4  10045080     kernel32:KERNEL32.dll
 0002:00000084       __imp__GetCPInfo@8         10045084     kernel32:KERNEL32.dll
 0002:00000088       __imp__GetACP@0            10045088     kernel32:KERNEL32.dll
 0002:0000008c       __imp__GetOEMCP@0          1004508c     kernel32:KERNEL32.dll
 0002:00000090       __imp__IsValidCodePage@4   10045090     kernel32:KERNEL32.dll
 0002:00000094       __imp__Sleep@4             10045094     kernel32:KERNEL32.dll
 0002:00000098       __imp__HeapSize@12         10045098     kernel32:KERNEL32.dll
 0002:0000009c       __imp__ExitProcess@4       1004509c     kernel32:KERNEL32.dll
 0002:000000a0       __imp__SetHandleCount@4    100450a0     kernel32:KERNEL32.dll
 0002:000000a4       __imp__GetStdHandle@4      100450a4     kernel32:KERNEL32.dll
 0002:000000a8       __imp__GetFileType@4       100450a8     kernel32:KERNEL32.dll
 0002:000000ac       __imp__GetStartupInfoA@4   100450ac     kernel32:KERNEL32.dll
 0002:000000b0       __imp__DeleteCriticalSection@4 100450b0     kernel32:KERNEL32.dll
 0002:000000b4       __imp__GetModuleFileNameA@12 100450b4     kernel32:KERNEL32.dll
 0002:000000b8       __imp__FreeEnvironmentStringsA@4 100450b8     kernel32:KERNEL32.dll
 0002:000000bc       __imp__GetEnvironmentStrings@0 100450bc     kernel32:KERNEL32.dll
 0002:000000c0       __imp__FreeEnvironmentStringsW@4 100450c0     kernel32:KERNEL32.dll
 0002:000000c4       __imp__WideCharToMultiByte@32 100450c4     kernel32:KERNEL32.dll
 0002:000000c8       __imp__GetEnvironmentStringsW@0 100450c8     kernel32:KERNEL32.dll
 0002:000000cc       __imp__HeapCreate@12       100450cc     kernel32:KERNEL32.dll
 0002:000000d0       __imp__HeapDestroy@4       100450d0     kernel32:KERNEL32.dll
 0002:000000d4       __imp__VirtualFree@12      100450d4     kernel32:KERNEL32.dll
 0002:000000d8       __imp__QueryPerformanceCounter@4 100450d8     kernel32:KERNEL32.dll
 0002:000000dc       __imp__GetTickCount@0      100450dc     kernel32:KERNEL32.dll
 0002:000000e0       __imp__GetCurrentProcessId@0 100450e0     kernel32:KERNEL32.dll
 0002:000000e4       __imp__GetSystemTimeAsFileTime@4 100450e4     kernel32:KERNEL32.dll
 0002:000000e8       __imp__VirtualAlloc@16     100450e8     kernel32:KERNEL32.dll
 0002:000000ec       __imp__HeapReAlloc@16      100450ec     kernel32:KERNEL32.dll
 0002:000000f0       __imp__WriteFile@20        100450f0     kernel32:KERNEL32.dll
 0002:000000f4       __imp__SetFilePointer@16   100450f4     kernel32:KERNEL32.dll
 0002:000000f8       __imp__GetConsoleCP@0      100450f8     kernel32:KERNEL32.dll
 0002:000000fc       __imp__GetConsoleMode@8    100450fc     kernel32:KERNEL32.dll
 0002:00000100       __imp__LCMapStringA@24     10045100     kernel32:KERNEL32.dll
 0002:00000104       __imp__MultiByteToWideChar@24 10045104     kernel32:KERNEL32.dll
 0002:00000108       __imp__LCMapStringW@24     10045108     kernel32:KERNEL32.dll
 0002:0000010c       __imp__GetStringTypeA@20   1004510c     kernel32:KERNEL32.dll
 0002:00000110       __imp__GetStringTypeW@16   10045110     kernel32:KERNEL32.dll
 0002:00000114       __imp__GetLocaleInfoA@16   10045114     kernel32:KERNEL32.dll
 0002:00000118       __imp__LoadLibraryA@4      10045118     kernel32:KERNEL32.dll
 0002:0000011c       __imp__InitializeCriticalSectionAndSpinCount@8 1004511c     kernel32:KERNEL32.dll
 0002:00000120       __imp__SetStdHandle@8      10045120     kernel32:KERNEL32.dll
 0002:00000124       __imp__WriteConsoleA@20    10045124     kernel32:KERNEL32.dll
 0002:00000128       __imp__GetConsoleOutputCP@0 10045128     kernel32:KERNEL32.dll
 0002:0000012c       __imp__WriteConsoleW@20    1004512c     kernel32:KERNEL32.dll
 0002:00000130       __imp__CreateFileA@28      10045130     kernel32:KERNEL32.dll
 0002:00000134       __imp__CloseHandle@4       10045134     kernel32:KERNEL32.dll
 0002:00000138       __imp__FlushFileBuffers@4  10045138     kernel32:KERNEL32.dll
 0002:0000013c       __imp__InitializeCriticalSection@4 1004513c     kernel32:KERNEL32.dll
 0002:00000140       __imp__ReadFile@20         10045140     kernel32:KERNEL32.dll
 0002:00000144       __imp__FindClose@4         10045144     kernel32:KERNEL32.dll
 0002:00000148       __imp__FindFirstFileA@8    10045148     kernel32:KERNEL32.dll
 0002:0000014c       __imp__GetFileSize@8       1004514c     kernel32:KERNEL32.dll
 0002:00000150       __imp__GetFileInformationByHandle@8 10045150     kernel32:KERNEL32.dll
 0002:00000154       __imp__CopyFileA@12        10045154     kernel32:KERNEL32.dll
 0002:00000158       __imp__DeleteFileA@4       10045158     kernel32:KERNEL32.dll
 0002:0000015c       __imp__CreateDirectoryA@8  1004515c     kernel32:KERNEL32.dll
 0002:00000160       __imp__RemoveDirectoryA@4  10045160     kernel32:KERNEL32.dll
 0002:00000164       __imp__GetLocalTime@4      10045164     kernel32:KERNEL32.dll
 0002:00000168       __imp__MoveFileA@8         10045168     kernel32:KERNEL32.dll
 0002:0000016c       __imp__GetFileAttributesA@4 1004516c     kernel32:KERNEL32.dll
 0002:00000170       __imp__lstrlenA@4          10045170     kernel32:KERNEL32.dll
 0002:00000174       __imp__lstrcpyA@8          10045174     kernel32:KERNEL32.dll
 0002:00000178       __imp__FindNextFileA@8     10045178     kernel32:KERNEL32.dll
 0002:0000017c       __imp__OutputDebugStringA@4 1004517c     kernel32:KERNEL32.dll
 0002:00000180       __imp__SetFilePointerEx@20 10045180     kernel32:KERNEL32.dll
 0002:00000184       __imp__GetFileSizeEx@8     10045184     kernel32:KERNEL32.dll
 0002:00000188       __imp__SetEndOfFile@4      10045188     kernel32:KERNEL32.dll
 0002:0000018c       __imp__SetFileAttributesA@8 1004518c     kernel32:KERNEL32.dll
 0002:00000190       __imp__SetFileTime@16      10045190     kernel32:KERNEL32.dll
 0002:00000194       \177KERNEL32_NULL_THUNK_DATA 10045194     kernel32:KERNEL32.dll
 0002:00000198       __imp__SendMessageA@16     10045198     user32:USER32.dll
 0002:0000019c       __imp__wsprintfA           1004519c     user32:USER32.dll
 0002:000001a0       \177USER32_NULL_THUNK_DATA 100451a0     user32:USER32.dll
 0002:000001a4       ___xc_a                    100451a4     LIBCMT:crt0init.obj
 0002:000001c8       ___xc_z                    100451c8     LIBCMT:crt0init.obj
 0002:000001cc       ___xi_a                    100451cc     LIBCMT:crt0init.obj
 0002:000001e4       ___xi_z                    100451e4     LIBCMT:crt0init.obj
 0002:000001e8       ___xp_a                    100451e8     LIBCMT:crt0init.obj
 0002:000001f4       ___xp_z                    100451f4     LIBCMT:crt0init.obj
 0002:000001f8       ___xt_a                    100451f8     LIBCMT:crt0init.obj
 0002:000001fc       ___xt_z                    100451fc     LIBCMT:crt0init.obj
 0002:00000220       ??_7CEffectManager@@6B@    10045220     effectmanager.obj
 0002:00000228       ??_7?$CWzSingleton@VCEffectManager@@@@6B@ 10045228     effectmanager.obj
 0002:0000022c       ??_C@_0DI@NBLCIHCF@CEffectManager?3?3Create?$CI?$CJ?5?9?5?$LL?g?$LP?n?$LF@ 1004522c     effectmanager.obj
 0002:00000264       ??_C@_0CP@GIIGGMB@CEffectManager?3?3Create?$CI?$CJ?5?9?5?$LI?$NO?$LI?p?$LI@ 10045264     effectmanager.obj
 0002:00000294       __real@bf800000            10045294     effectmanager.obj
 0002:00000298       ??_C@_0DL@PEALBKBL@CEffectManager?3?3LoadTextureFiles@ 10045298     effectmanager.obj
 0002:000002d4       ??_C@_04HDOCAJNK@?$CFs?$CFs?$AA@ 100452d4     effectmanager.obj
 0002:000002dc       ??_C@_0DI@HBMCNBMG@CEffectManager?3?3LoadMeshFiles?$CI?$CFs@ 100452dc     effectmanager.obj
 0002:00000314       ??_C@_0DI@JDEEJMMC@CEffectManager?3?3LoadMeshFiles?$CI?$CFs@ 10045314     effectmanager.obj
 0002:0000034c       __real@411ccccd            1004534c     effectmanager.obj
 0002:00000350       __real@3f800000            10045350     effectmanager.obj
 0002:00000354       __real@3f000000            10045354     effectmanager.obj
 0002:00000358       __real@bf000000            10045358     effectmanager.obj
 0002:0000035c       ??_C@_0CP@EMIKEIJK@St_BodyCreate?3?3CreateSpline?$CI?$CJ?5?9?5@ 1004535c     effectmanager.obj
 0002:0000038c       ??_C@_0DF@OGMGPPLI@CEffectManager?3?3AddEffectInfo?$CI?$CJ?5@ 1004538c     effectmanager.obj
 0002:000003c4       ??_C@_0DJ@KFPCOKKD@CEffectManager?3?3CreateEffect?$CI?$CJ?5?9@ 100453c4     effectmanager.obj
 0002:00000400       ??_C@_0DG@DOJIEKJB@CEffectManager?3?3CreateEffect?$CI?$CJ?5?9@ 10045400     effectmanager.obj
 0002:00000438       ??_C@_0DJ@DMNJCHCK@CEffectManager?3?3CreateEffect?$CI?$CJ?5?9@ 10045438     effectmanager.obj
 0002:00000474       ??_C@_0DH@GJIMFFIJ@CEffectManager?3?3CreateEffect?$CI?$CJ?5?9@ 10045474     effectmanager.obj
 0002:000004b0       __real@408f400000000000    100454b0     effectmanager.obj
 0002:000004b8       ??_C@_0DM@MHMOOJPO@CEffectManager?3?3CreateElement?$CI?$CJ?5@ 100454b8     effectmanager.obj
 0002:000004f4       ??_C@_0DK@NMJIKJJI@CEffectManager?3?3CreateElement?$CI?$CJ?5@ 100454f4     effectmanager.obj
 0002:00000530       ??_C@_0DA@MDDIDKFJ@CEffectManager?3?3CreateElement?$CI?$CJ?5@ 10045530     effectmanager.obj
 0002:00000560       ??_C@_0ED@HCCLOJOK@CEffectManager?3?3CreateSelectedEl@ 10045560     effectmanager.obj
 0002:000005a8       ??_C@_0EA@KPHBOPFA@CEffectManager?3?3CreateSelectedEl@ 100455a8     effectmanager.obj
 0002:000005e8       ??_C@_0EF@HLJEBDIK@CEffectManager?3?3CreateSelectedEl@ 100455e8     effectmanager.obj
 0002:00000630       ??_C@_0ED@KGBCMJLM@CEffectManager?3?3CreateSelectedEl@ 10045630     effectmanager.obj
 0002:00000674       ??_C@_0DC@GHPGADKB@CEffectManager?3?3Move?$CI?$CJ?5?9?5EffectB@ 10045674     effectmanager.obj
 0002:000006a8       __real@404c000000000000    100456a8     effectmanager.obj
 0002:000006b0       __real@0000000000000000    100456b0     effectmanager.obj
 0002:000006b8       __real@41200000            100456b8     effectmanager.obj
 0002:000006bc       __real@41700000            100456bc     effectmanager.obj
 0002:000006c0       __real@41a00000            100456c0     effectmanager.obj
 0002:000006c4       __real@41c80000            100456c4     effectmanager.obj
 0002:000006cc       ??_7out_of_range@std@@6B@  100456cc     effectmanager.obj
 0002:000006d4       ??_C@_0BM@PAPJHAGI@invalid?5map?1set?$DMT?$DO?5iterator?$AA@ 100456d4     effectmanager.obj
 0002:000006f0       ?npos@?$basic_string@DU?$char_traits@D@std@@V?$allocator@D@2@@std@@2IB 100456f0     effectmanager.obj
 0002:000006f8       ??_7logic_error@std@@6B@   100456f8     effectmanager.obj
 0002:00000704       ??_7bad_alloc@std@@6B@     10045704     effectmanager.obj
 0002:0000070c       __real@40800000            1004570c     effectmanager.obj
 0002:00000710       ??_C@_0DB@IFHBLKCI@CWzMemoryPool?3?3AllocBand?$CI?$CJ?5?9?5new@ 10045710     effectmanager.obj
 0002:00000744       ??_C@_0CP@FBCCNEPE@CWzMemoryPool?3?3AllocBand?$CI?$CJ?5?9?5new@ 10045744     effectmanager.obj
 0002:00000778       ??_7length_error@std@@6B@  10045778     effectmanager.obj
 0002:00000780       ??_C@_0BD@OLBABOEK@vector?$DMT?$DO?5too?5long?$AA@ 10045780     effectmanager.obj
 0002:00000794       ??_C@_0CN@MNHKBHCO@CWzMemoryBand?3?3Create?$CI?$CJ?5?9?5freeLi@ 10045794     effectmanager.obj
 0002:000007c4       ??_C@_0CM@IMMGHPGC@CWzMemoryBand?3?3Create?$CI?$CJ?5?9?5objPoo@ 100457c4     effectmanager.obj
 0002:000007f0       ??_C@_0CE@ICGMELHO@CWzMemoryBand?3?3Create?$CI?$CJ?5?9?5?$MA?L?$LJ?L?5?$MA@ 100457f0     effectmanager.obj
 0002:00000814       ??_C@_0BB@MOGOBHAF@list?$DMT?$DO?5too?5long?$AA@ 10045814     effectmanager.obj
 0002:0000082c       ??_7?$CWzHandleManager@PAVCEffectBody@@@@6B@ 1004582c     effectmanager.obj
 0002:00000830       ??_C@_0EF@POPAIGIK@CWzArray?3?3Get?$CI?$CJ?5?9?5?$LN?G?F?P?$CB?$CB?5?$LO?$LC?$LH?$LJ?$LB?b?5@ 10045830     effectmanager.obj
 0002:00000878       ??_C@_0DI@BCCEGDCJ@CEffectManager?3?3LoadEffectFromFi@ 10045878     effectmanager_load.obj
 0002:000008b0       ??_C@_0DI@IFIOFIHC@CEffectManager?3?3LoadEffectFromFi@ 100458b0     effectmanager_load.obj
 0002:000008e8       ??_C@_0DD@FPHLACKP@CEffectManager?3?3LoadEffectFromFi@ 100458e8     effectmanager_load.obj
 0002:00000920       ??_C@_0EB@KCNDGCEN@CEffectManager?3?3LoadEffectFromFi@ 10045920     effectmanager_load.obj
 0002:00000964       ??_C@_0DP@LCKEKKMI@CEffectManager?3?3LoadEffectFromFi@ 10045964     effectmanager_load.obj
 0002:000009a4       ??_C@_0CK@DDGHBEHH@CEffectManager?3?3LoadEffectFromFi@ 100459a4     effectmanager_load.obj
 0002:000009d0       ??_C@_0DF@NCJNGDDI@CEffectManager?3?3UnLoadEffectFrom@ 100459d0     effectmanager_load.obj
 0002:00000a08       ??_C@_0ED@OKGHMGEI@CEffectManager?3?3UnLoadEffectFrom@ 10045a08     effectmanager_load.obj
 0002:00000a50       ??_C@_0EB@JGFPBCIN@CEffectManager?3?3UnLoadEffectFrom@ 10045a50     effectmanager_load.obj
 0002:00000a94       ??_C@_0CJ@DLHNCEMJ@CEffectManager?3?3Load?$CI?$CJ?5?9?5?A?$NP?$LK?$LJ?5Bo@ 10045a94     effectmanager_load.obj
 0002:00000ac0       ??_C@_0CL@JPKCKMMF@CEffectManager?3?3Load?$CI?$CJ?5?9?5?$MA?$NP?$LI?x?$LF?H?5@ 10045ac0     effectmanager_load.obj
 0002:00000aec       ??_C@_0CI@MKOLGGOG@CEffectManager?3?3Load?$CI?$CJ?5?9?5?$LJ?v?$MA?$PM?5?$MA?P@ 10045aec     effectmanager_load.obj
 0002:00000b14       ??_C@_0CA@IBOAPGOJ@CEffectManager?3?3Load?$CI?$CFs?$CJ?5?9?5?$LN?G?F?P?$AA@ 10045b14     effectmanager_load.obj
 0002:00000b34       ??_C@_0CK@ILJIMHEL@CEffectManager?3?3Load?$CI?$CFs?$CJ?5?9?5?F?D?$MA?O?5@ 10045b34     effectmanager_load.obj
 0002:00000b60       ??_C@_0DD@EMDMKFHL@CEffectManager?3?3LoadBodyInfoOld?$CI@ 10045b60     effectmanager_load.obj
 0002:00000b94       ??_C@_08HFAOPDFF@ver?4e0?45?$AA@ 10045b94     effectmanager_load.obj
 0002:00000ba0       ??_C@_0CC@DDFLGMIG@CEffectManager?3?3LoadBodyInfoOld?$CI@ 10045ba0     effectmanager_load.obj
 0002:00000bc4       ??_C@_08MGBMAKJP@ver?4e2?44?$AA@ 10045bc4     effectmanager_load.obj
 0002:00000bd0       ??_C@_08JAEGKNBJ@ver?4e2?42?$AA@ 10045bd0     effectmanager_load.obj
 0002:00000bdc       ??_C@_08HIBMOKHN@ver?4e1?48?$AA@ 10045bdc     effectmanager_load.obj
 0002:00000be8       ??_C@_08MAKAINBI@ver?4e0?48?$AA@ 10045be8     effectmanager_load.obj
 0002:00000bf4       ??_C@_08KCHAMPJL@ver?4e2?40?$AA@ 10045bf4     effectmanager_load.obj
 0002:00000c00       ??_C@_08EHDIJBNH@ver?4e0?47?$AA@ 10045c00     effectmanager_load.obj
 0002:00000c0c       ??_C@_08OGJPMHPD@ver?4e1?46?$AA@ 10045c0c     effectmanager_load.obj
 0002:00000c18       ??_C@_08KJNOFBDE@ver?4e1?41?$AA@ 10045c18     effectmanager_load.obj
 0002:00000c24       ??_C@_08CDFEFEND@ver?4e0?43?$AA@ 10045c24     effectmanager_load.obj
 0002:00000c30       ??_C@_0DC@ICKDBMBF@CEffectManager?3?3LoadCreateInfo?$CI?$CJ@ 10045c30     effectmanager_load.obj
 0002:00000c64       ??_C@_08JLOIDDLG@ver?4e1?43?$AA@ 10045c64     effectmanager_load.obj
 0002:00000c70       ??_C@_08LLGLPONK@ver?4e2?41?$AA@ 10045c70     effectmanager_load.obj
 0002:00000c7c       ??_C@_08ICPDACPH@ver?4e1?42?$AA@ 10045c7c     effectmanager_load.obj
 0002:00000c88       ??_C@_08GMBFMCBE@ver?4e0?44?$AA@ 10045c88     effectmanager_load.obj
 0002:00000c94       ??_C@_08NJLLLMFJ@ver?4e0?49?$AA@ 10045c94     effectmanager_load.obj
 0002:00000ca0       ??_C@_08DKEPGFJC@ver?4e0?42?$AA@ 10045ca0     effectmanager_load.obj
 0002:00000cac       ??_C@_08MNLCJEDA@ver?4e1?45?$AA@ 10045cac     effectmanager_load.obj
 0002:00000cb8       ??_C@_08IJFNJMFI@ver?4e2?43?$AA@ 10045cb8     effectmanager_load.obj
 0002:00000cc4       ??_C@_08NEKJKFHB@ver?4e1?44?$AA@ 10045cc4     effectmanager_load.obj
 0002:00000cd0       ??_C@_08NPAHDLNO@ver?4e2?45?$AA@ 10045cd0     effectmanager_load.obj
 0002:00000cdc       ??_C@_0BE@JONHPENG@map?1set?$DMT?$DO?5too?5long?$AA@ 10045cdc     effectmanager_load.obj
 0002:00000cf0       ??_C@_0DM@NLOKNALK@CEffectManager?3?3Save?$CI?$CJ?5?9?5?G?X?$LE?g?5ID@ 10045cf0     effectmanager_save.obj
 0002:00000d2c       ??_C@_0CJ@IDKGINNJ@CEffectManager?3?3Save?$CI?$CJ?5?9?5INVALID@ 10045d2c     effectmanager_save.obj
 0002:00000d58       ??_C@_0CA@NKLHPIBB@CEffectManager?3?3Save?$CI?$CFs?$CJ?5?9?5?$LN?G?F?P?$AA@ 10045d58     effectmanager_save.obj
 0002:00000d78       ??_C@_0CK@MOHGMECL@CEffectManager?3?3Save?$CI?$CFs?$CJ?5?9?5?F?D?$MA?O?5@ 10045d78     effectmanager_save.obj
 0002:00000da4       ??_C@_0DC@NGBIEKJL@CEffectManager?3?3SaveCreateInfo?$CI?$CJ@ 10045da4     effectmanager_save.obj
 0002:00000dd8       ??_C@_03JBJLGPFL@end?$AA@  10045dd8     loadmanager.obj
 0002:00000ddc       ??_C@_0DB@KAIDKHJP@CLoadBaseManager?3?3OnCreate?$CI?$CFs?$CJ?5?9@ 10045ddc     loadmanager.obj
 0002:00000e10       ??_C@_05FAGFPHJG@start?$AA@ 10045e10     loadmanager.obj
 0002:00000e18       ??_C@_0CJ@KEEJBENC@CLoadBaseManager?3?3OnCreate?$CI?$CFs?$CJ?5?9@ 10045e18     loadmanager.obj
 0002:00000e44       ??_C@_0DH@IOHBPHLD@CLoadBaseManager?3?3OnCreate?$CI?$CFs?$CJ?5?9@ 10045e44     loadmanager.obj
 0002:00000e7c       ??_C@_0DJ@DLIIFNGA@CMemoryManager?3?3Create?$CI?$CJ?5?9?5Effec@ 10045e7c     memorymanager.obj
 0002:00000eb8       ??_C@_0DG@IAFILEFD@CMemoryManager?3?3Create?$CI?$CJ?5?9?5Weath@ 10045eb8     memorymanager.obj
 0002:00000ef0       ??_C@_0DE@OKLLDDGH@CMemoryManager?3?3Create?$CI?$CJ?5?9?5Decal@ 10045ef0     memorymanager.obj
 0002:00000f24       ??_C@_0DI@DGJFEGKD@CMemoryManager?3?3Create?$CI?$CJ?5?9?5FlatC@ 10045f24     memorymanager.obj
 0002:00000f5c       ??_C@_0DE@KONEPMJN@CMemoryManager?3?3Create?$CI?$CJ?5?9?5Chain@ 10045f5c     memorymanager.obj
 0002:00000f90       ??_C@_0DD@LCPIGEPE@CMemoryManager?3?3Create?$CI?$CJ?5?9?5Mesh?5@ 10045f90     memorymanager.obj
 0002:00000fc4       ??_C@_0DF@IFKHBHKL@CMemoryManager?3?3Create?$CI?$CJ?5?9?5Sprit@ 10045fc4     memorymanager.obj
 0002:00000ffc       ??_C@_0CM@DFMKCGE@CWzMemoryPool?3?3Create?$CI?$CJ?5?9?5?$LL?u?5?$LJ?j?$LF@ 10045ffc     memorymanager.obj
 0002:00001028       ??_C@_0CE@BMHBIKBE@CWzMemoryPool?3?3Create?$CI?$CJ?5?9?5?$MA?L?$LJ?L?5?$MA@ 10046028     memorymanager.obj
 0002:0000104c       ??_C@_0P@GHFPNOJB@bad?5allocation?$AA@ 1004604c     stdafx.obj
 0002:00001064       ??_7CEElementBase@@6B@     10046064     eelementbase.obj
 0002:000010b4       ??_7CEElementChain@@6B@    100460b4     eelementchain.obj
 0002:00001100       __real@3ff0000000000000    10046100     eelementchain.obj
 0002:00001108       ??_C@_0DC@MBFIOBML@CEElementChain?3?3Create?$CI?$CJ?5?9?5?$LN?G?F?P?$CB@ 10046108     eelementchain.obj
 0002:0000113c       ??_C@_0DF@IMEKFDIE@CEElementChain?3?3Create?$CI?$CJ?5?9?5GetEf@ 1004613c     eelementchain.obj
 0002:00001174       ??_C@_0DC@DBOEGJLC@CEElementChain?3?3Create?$CI?$CJ?5?9?5?$LN?G?F?P?$CB@ 10046174     eelementchain.obj
 0002:000011a8       __real@3f1a36e2e0000000    100461a8     eelementchain.obj
 0002:000011b0       __mask@@NegFloat@          100461b0     eelementchain.obj
 0002:000011c0       __real@3fd0000000000000    100461c0     eelementchain.obj
 0002:000011cc       ??_7CEElementDecal@@6B@    100461cc     eelementdecal.obj
 0002:00001214       ??_C@_0CM@EDEHOHGF@CEElementDecal?3?3Create?$CI?$CJ?5?9?5?E?X?$LN?$LK?C@ 10046214     eelementdecal.obj
 0002:00001240       __real@437f0000            10046240     eelementdecal.obj
 0002:00001248       __real@3eb0c6f7a0000000    10046248     eelementdecal.obj
 0002:00001254       ??_7CEElementFlatChain@@6B@ 10046254     eelementflatchain.obj
 0002:0000129c       ??_C@_0DJ@BJDHAOHM@CEElementFlatChain?3?3Create?$CI?$CJ?5?9?5G@ 1004629c     eelementflatchain.obj
 0002:000012d8       ??_C@_0DG@OOHHIMN@CEElementFlatChain?3?3Create?$CI?$CJ?5?9?5?$LN@ 100462d8     eelementflatchain.obj
 0002:00001310       ??_C@_0DE@ODBAEFNL@CEElementFlatChain?3?3SetTailNum?$CI?$CJ@ 10046310     eelementflatchain.obj
 0002:00001348       __real@3f847ae140000000    10046348     eelementflatchain.obj
 0002:00001354       ??_7CEElementMesh@@6B@     10046354     eelementmesh.obj
 0002:0000139c       ??_C@_0DA@NEGPBJBH@CEElementMesh?3?3Create?$CI?$CJ?5?9?5New?5Un@ 1004639c     eelementmesh.obj
 0002:000013cc       ??_C@_0CN@BGDOBPLA@CEElementMesh?3?3Create?$CI?$CJ?5?9?5GetWzU@ 100463cc     eelementmesh.obj
 0002:000013fc       ??_C@_0CO@JIDHOFNI@CEElementMesh?3?3Create?$CI?$CJ?5?9?5?$LN?G?F?P?$CB?$CB@ 100463fc     eelementmesh.obj
 0002:0000142c       ??_C@_0DD@JBMNGFGG@CWzUnitDraw?3?3SetRotationByMatrix@ 1004642c     eelementmesh.obj
 0002:00001464       ??_7CEElementParticle@@6B@ 10046464     eelementparticle.obj
 0002:000014b0       __real@3fe0000000000000    100464b0     eelementparticle.obj
 0002:000014b8       ??_C@_0DC@DOIKNIKJ@CEElementParticle?3?3Create?$CI?$CJ?5?9?5?$LM?v@ 100464b8     eelementparticle.obj
 0002:000014f0       __real@3f50624de0000000    100464f0     eelementparticle.obj
 0002:000014fc       ??_7CEElementSprite@@6B@   100464fc     eelementsprite.obj
 0002:00001544       ??_C@_0DE@LCMDEELH@CEElementSprite?3?3Create?$CI?$CJ?5?9?5GetT@ 10046544     eelementsprite.obj
 0002:00001578       ??_C@_0DG@GDFGNEIP@CEElementSprite?3?3Create?$CI?$CJ?5?9?5GetE@ 10046578     eelementsprite.obj
 0002:000015b0       ??_C@_0DD@FEODKKHC@CEElementSprite?3?3Create?$CI?$CJ?5?9?5?$LN?G?F?P@ 100465b0     eelementsprite.obj
 0002:000015e8       __real@4000000000000000    100465e8     eelementsprite.obj
 0002:000015f0       __real@4059000000000000    100465f0     eelementsprite.obj
 0002:000015fc       ??_7CEElementWeather@@6B@  100465fc     eelementweather.obj
 0002:0000164c       ??_7CEffectBody@@6B@       1004664c     effectbody.obj
 0002:00001694       ??_C@_0DC@GMMHEJN@CEffectBody?3?3CreateElement?$CI?$CJ?5?9?5?$LI@ 10046694     effectbody.obj
 0002:000016c8       ??_C@_0DA@NBDIKHCM@CEffectBody?3?3CreateElement?$CI?$CJ?5?9?5U@ 100466c8     effectbody.obj
 0002:000016f8       ??_C@_0BA@JFNIOLAK@string?5too?5long?$AA@ 100466f8     libcpmt:string.obj
 0002:00001708       ??_C@_0BI@CFPLBAOH@invalid?5string?5position?$AA@ 10046708     libcpmt:string.obj
 0002:00001720       __FPinit                   10046720     LIBCMT:_fpinit_.obj
 0002:00001724       __FPmtinit                 10046724     LIBCMT:_fpinit_.obj
 0002:00001728       __FPmtterm                 10046728     LIBCMT:_fpinit_.obj
 0002:00001730       ??_7type_info@@6B@         10046730     LIBCMT:typinfo.obj
 0002:00001758       ??_7exception@std@@6B@     10046758     LIBCMT:stdexcpt.obj
 0002:00001760       ??_C@_0BC@EOODALEL@Unknown?5exception?$AA@ 10046760     LIBCMT:stdexcpt.obj
 0002:00001774       __pDefaultRawDllMain       10046774     LIBCMT:dllcrt0.obj
 0002:00001774       __pRawDllMain              10046774     LIBCMT:dllcrt0.obj
 0002:00001778       __pDestructExceptionObject 10046778     LIBCMT:frame.obj
 0002:00001780       ??_7bad_exception@std@@6B@ 10046780     LIBCMT:frame.obj
 0002:00001788       ??_C@_0O@DPKOEFFH@bad?5exception?$AA@ 10046788     LIBCMT:frame.obj
 0002:00001798       ??_C@_0O@NLDKAIKN@EncodePointer?$AA@ 10046798     LIBCMT:tidtable.obj
 0002:000017a8       ??_C@_1BK@DBDEIDLH@?$AAK?$AAE?$AAR?$AAN?$AAE?$AAL?$AA3?$AA2?$AA?4?$AAD?$AAL?$AAL?$AA?$AA@ 100467a8     LIBCMT:tidtable.obj
 0002:000017c4       ??_C@_0O@KBPMFGHI@DecodePointer?$AA@ 100467c4     LIBCMT:tidtable.obj
 0002:000017d4       ??_C@_07PEJMOBNF@FlsFree?$AA@ 100467d4     LIBCMT:tidtable.obj
 0002:000017dc       ??_C@_0M@JCPCPOEF@FlsSetValue?$AA@ 100467dc     LIBCMT:tidtable.obj
 0002:000017e8       ??_C@_0M@GDNOONDI@FlsGetValue?$AA@ 100467e8     LIBCMT:tidtable.obj
 0002:000017f4       ??_C@_08KNHFBNJ@FlsAlloc?$AA@ 100467f4     LIBCMT:tidtable.obj
 0002:00001808       ??_C@_05KLBDPFGC@e?$CL000?$AA@ 10046808     LIBCMT:cvt.obj
 0002:00001810       __real@4150017ec0000000    10046810     LIBCMT:_testfdiv_.obj
 0002:00001818       __real@4147ffff80000000    10046818     LIBCMT:_testfdiv_.obj
 0002:00001820       ??_C@_0BK@NHEOCAHP@IsProcessorFeaturePresent?$AA@ 10046820     LIBCMT:_testfdiv_.obj
 0002:0000183c       ??_C@_08CPNIBGIE@KERNEL32?$AA@ 1004683c     LIBCMT:_testfdiv_.obj
 0002:00001848       ??_C@_1O@CEDCILHN@?$AA?$CI?$AAn?$AAu?$AAl?$AAl?$AA?$CJ?$AA?$AA@ 10046848     LIBCMT:output.obj
 0002:00001858       ??_C@_06OJHGLDPL@?$CInull?$CJ?$AA@ 10046858     LIBCMT:output.obj
 0002:00001860       ___lookuptable             10046860     LIBCMT:output.obj
 0002:000018c8       __DEFAULT_CW_in_mem        100468c8     LIBCMT:_common_.obj
 0002:000018ca       __pi_by_2_to_61            100468ca     LIBCMT:_common_.obj
 0002:00001988       ??_C@_01NEMOKFLO@?$DN?$AA@ 10046988     LIBCMT:setlocal.obj
 0002:0000198a       ??_C@_00CNPNBAHC@?$AA@     1004698a     LIBCMT:setlocal.obj
 0002:0000198c       ??_C@_0P@MIGLKIOC@CorExitProcess?$AA@ 1004698c     LIBCMT:crt0dat.obj
 0002:0000199c       ??_C@_1BI@BGOHAHKC@?$AAm?$AAs?$AAc?$AAo?$AAr?$AAe?$AAe?$AA?4?$AAd?$AAl?$AAl?$AA?$AA@ 1004699c     LIBCMT:crt0dat.obj
 0002:00002b10       __XcptActTab               10047b10     LIBCMT:winxfltr.obj
 0002:00002b88       ??_C@_0P@GGKDKEEG@runtime?5error?5?$AA@ 10047b88     LIBCMT:crt0msg.obj
 0002:00002b98       ??_C@_02PCIJFNDE@?$AN?6?$AA@ 10047b98     LIBCMT:crt0msg.obj
 0002:00002b9c       ??_C@_0O@MJNIPGOH@TLOSS?5error?$AN?6?$AA@ 10047b9c     LIBCMT:crt0msg.obj
 0002:00002bac       ??_C@_0N@BONNPDHF@SING?5error?$AN?6?$AA@ 10047bac     LIBCMT:crt0msg.obj
 0002:00002bbc       ??_C@_0P@MBDAJNE@DOMAIN?5error?$AN?6?$AA@ 10047bbc     LIBCMT:crt0msg.obj
 0002:00002bd0       ??_C@_0JL@DFDOOABL@R6034?$AN?6An?5application?5has?5made?5a@ 10047bd0     LIBCMT:crt0msg.obj
 0002:00002c70       ??_C@_0PH@EPAFIJ@R6033?$AN?6?9?5Attempt?5to?5use?5MSIL?5cod@ 10047c70     LIBCMT:crt0msg.obj
 0002:00002d68       ??_C@_0DD@BKEEABMM@R6032?$AN?6?9?5not?5enough?5space?5for?5lo@ 10047d68     LIBCMT:crt0msg.obj
 0002:00002da0       ??_C@_0GD@OFKILIED@R6031?$AN?6?9?5Attempt?5to?5initialize?5t@ 10047da0     LIBCMT:crt0msg.obj
 0002:00002e04       ??_C@_0BP@LPMHJOKI@R6030?$AN?6?9?5CRT?5not?5initialized?$AN?6?$AA@ 10047e04     LIBCMT:crt0msg.obj
 0002:00002e24       ??_C@_0CF@KJDAIALP@R6028?$AN?6?9?5unable?5to?5initialize?5he@ 10047e24     LIBCMT:crt0msg.obj
 0002:00002e4c       ??_C@_0DF@GAKBPDFP@R6027?$AN?6?9?5not?5enough?5space?5for?5lo@ 10047e4c     LIBCMT:crt0msg.obj
 0002:00002e84       ??_C@_0DF@IBLNNAIG@R6026?$AN?6?9?5not?5enough?5space?5for?5st@ 10047e84     LIBCMT:crt0msg.obj
 0002:00002ebc       ??_C@_0CG@IOHKGFNJ@R6025?$AN?6?9?5pure?5virtual?5function?5c@ 10047ebc     LIBCMT:crt0msg.obj
 0002:00002ee4       ??_C@_0DF@JIJJFJDC@R6024?$AN?6?9?5not?5enough?5space?5for?5_o@ 10047ee4     LIBCMT:crt0msg.obj
 0002:00002f1c       ??_C@_0CJ@EGEJHFME@R6019?$AN?6?9?5unable?5to?5open?5console?5@ 10047f1c     LIBCMT:crt0msg.obj
 0002:00002f48       ??_C@_0CB@GNHNIELH@R6018?$AN?6?9?5unexpected?5heap?5error?$AN?6@ 10047f48     LIBCMT:crt0msg.obj
 0002:00002f6c       ??_C@_0CN@FOLDKNG@R6017?$AN?6?9?5unexpected?5multithread?5@ 10047f6c     LIBCMT:crt0msg.obj
 0002:00002f9c       ??_C@_0CM@FAHFJNHO@R6016?$AN?6?9?5not?5enough?5space?5for?5th@ 10047f9c     LIBCMT:crt0msg.obj
 0002:00002fc8       ??_C@_0JG@LBKMGKLD@?$AN?6This?5application?5has?5requested@ 10047fc8     LIBCMT:crt0msg.obj
 0002:00003060       ??_C@_0CM@FLCNIPKK@R6009?$AN?6?9?5not?5enough?5space?5for?5en@ 10048060     LIBCMT:crt0msg.obj
 0002:0000308c       ??_C@_0CK@KMMJOAPP@R6008?$AN?6?9?5not?5enough?5space?5for?5ar@ 1004808c     LIBCMT:crt0msg.obj
 0002:000030b8       ??_C@_0CN@LEKKICBM@R6002?$AN?6?9?5floating?5point?5support?5@ 100480b8     LIBCMT:crt0msg.obj
 0002:000030e8       ??_C@_0CF@GOGNBNAK@Microsoft?5Visual?5C?$CL?$CL?5Runtime?5Lib@ 100480e8     LIBCMT:crt0msg.obj
 0002:00003110       ??_C@_02PHMGELLB@?6?6?$AA@ 10048110     LIBCMT:crt0msg.obj
 0002:00003114       ??_C@_03KHICJKCI@?4?4?4?$AA@ 10048114     LIBCMT:crt0msg.obj
 0002:00003118       ??_C@_0BH@DNAGHKFM@?$DMprogram?5name?5unknown?$DO?$AA@ 10048118     LIBCMT:crt0msg.obj
 0002:00003130       ??_C@_0BK@OFGJDLJJ@Runtime?5Error?$CB?6?6Program?3?5?$AA@ 10048130     LIBCMT:crt0msg.obj
 0002:0000314c       ??_C@_0BK@CFCOFLF@?5Complete?5Object?5Locator?8?$AA@ 1004814c     LIBCMT:undname.obj
 0002:00003168       ??_C@_0BN@MECKDCOJ@?5Class?5Hierarchy?5Descriptor?8?$AA@ 10048168     LIBCMT:undname.obj
 0002:00003188       ??_C@_0BD@LGICGFMM@?5Base?5Class?5Array?8?$AA@ 10048188     LIBCMT:undname.obj
 0002:0000319c       ??_C@_0BM@LDKODKLH@?5Base?5Class?5Descriptor?5at?5?$CI?$AA@ 1004819c     LIBCMT:undname.obj
 0002:000031b8       ??_C@_0BC@DAFEJGAK@?5Type?5Descriptor?8?$AA@ 100481b8     LIBCMT:undname.obj
 0002:000031cc       ??_C@_0BM@PMGGMLDN@?$GAlocal?5static?5thread?5guard?8?$AA@ 100481cc     LIBCMT:undname.obj
 0002:000031e8       ??_C@_0CL@FGIJHLCE@?$GAmanaged?5vector?5copy?5constructor@ 100481e8     LIBCMT:undname.obj
 0002:00003214       ??_C@_0CJ@GJELGAMM@?$GAvector?5vbase?5copy?5constructor?5i@ 10048214     LIBCMT:undname.obj
 0002:00003240       ??_C@_0CD@CGAJBKEJ@?$GAvector?5copy?5constructor?5iterato@ 10048240     LIBCMT:undname.obj
 0002:00003264       ??_C@_0CB@PDBIFEP@?$GAdynamic?5atexit?5destructor?5for?5?8@ 10048264     LIBCMT:undname.obj
 0002:00003288       ??_C@_0BL@CLIPGLGB@?$GAdynamic?5initializer?5for?5?8?$AA@ 10048288     LIBCMT:undname.obj
 0002:000032a4       ??_C@_0CM@FCBBDIGB@?$GAeh?5vector?5vbase?5copy?5constructo@ 100482a4     LIBCMT:undname.obj
 0002:000032d0       ??_C@_0CG@HLDDJMAG@?$GAeh?5vector?5copy?5constructor?5iter@ 100482d0     LIBCMT:undname.obj
 0002:000032f8       ??_C@_0CF@IMGKMJNO@?$GAmanaged?5vector?5destructor?5itera@ 100482f8     LIBCMT:undname.obj
 0002:00003320       ??_C@_0CG@CFDHKGGD@?$GAmanaged?5vector?5constructor?5iter@ 10048320     LIBCMT:undname.obj
 0002:00003348       ??_C@_0BN@CKNJLHMB@?$GAplacement?5delete?$FL?$FN?5closure?8?$AA@ 10048348     LIBCMT:undname.obj
 0002:00003368       ??_C@_0BL@CNOONJFP@?$GAplacement?5delete?5closure?8?$AA@ 10048368     LIBCMT:undname.obj
 0002:00003384       ??_C@_0P@HJKNJFNN@?$GAomni?5callsig?8?$AA@ 10048384     LIBCMT:undname.obj
 0002:00003394       ??_C@_09LBNFPBCA@?5delete?$FL?$FN?$AA@ 10048394     LIBCMT:undname.obj
 0002:000033a0       ??_C@_06FHBGPFGH@?5new?$FL?$FN?$AA@ 100483a0     LIBCMT:undname.obj
 0002:000033a8       ??_C@_0CE@IIHCMGGL@?$GAlocal?5vftable?5constructor?5closu@ 100483a8     LIBCMT:undname.obj
 0002:000033cc       ??_C@_0BA@KKLDJDLB@?$GAlocal?5vftable?8?$AA@ 100483cc     LIBCMT:undname.obj
 0002:000033dc       ??_C@_05KHLCHHI@?$GARTTI?$AA@ 100483dc     LIBCMT:undname.obj
 0002:000033e4       ??_C@_03KLGMFNMG@?$GAEH?$AA@ 100483e4     LIBCMT:undname.obj
 0002:000033e8       ??_C@_0BA@KBCDOMBN@?$GAudt?5returning?8?$AA@ 100483e8     LIBCMT:undname.obj
 0002:000033f8       ??_C@_0BL@LLKPOHJI@?$GAcopy?5constructor?5closure?8?$AA@ 100483f8     LIBCMT:undname.obj
 0002:00003414       ??_C@_0CH@OOJPLCPH@?$GAeh?5vector?5vbase?5constructor?5ite@ 10048414     LIBCMT:undname.obj
 0002:0000343c       ??_C@_0CA@GCEOPDGL@?$GAeh?5vector?5destructor?5iterator?8?$AA@ 1004843c     LIBCMT:undname.obj
 0002:0000345c       ??_C@_0CB@JONCMFFK@?$GAeh?5vector?5constructor?5iterator?8@ 1004845c     LIBCMT:undname.obj
 0002:00003480       ??_C@_0BL@NILFHHPC@?$GAvirtual?5displacement?5map?8?$AA@ 10048480     LIBCMT:undname.obj
 0002:0000349c       ??_C@_0CE@IKBNEHA@?$GAvector?5vbase?5constructor?5iterat@ 1004849c     LIBCMT:undname.obj
 0002:000034c0       ??_C@_0BN@LFPFMEDL@?$GAvector?5destructor?5iterator?8?$AA@ 100484c0     LIBCMT:undname.obj
 0002:000034e0       ??_C@_0BO@PFGOCPJJ@?$GAvector?5constructor?5iterator?8?$AA@ 100484e0     LIBCMT:undname.obj
 0002:00003500       ??_C@_0BN@IMDCHIKM@?$GAscalar?5deleting?5destructor?8?$AA@ 10048500     LIBCMT:undname.obj
 0002:00003520       ??_C@_0BO@OBMKPJIG@?$GAdefault?5constructor?5closure?8?$AA@ 10048520     LIBCMT:undname.obj
 0002:00003540       ??_C@_0BN@DEGPLNFK@?$GAvector?5deleting?5destructor?8?$AA@ 10048540     LIBCMT:undname.obj
 0002:00003560       ??_C@_0BD@JDLKDPAB@?$GAvbase?5destructor?8?$AA@ 10048560     LIBCMT:undname.obj
 0002:00003574       ??_C@_08OBABFOLI@?$GAstring?8?$AA@ 10048574     LIBCMT:undname.obj
 0002:00003580       ??_C@_0BF@KDPPACIK@?$GAlocal?5static?5guard?8?$AA@ 10048580     LIBCMT:undname.obj
 0002:00003598       ??_C@_08LLFFHHDJ@?$GAtypeof?8?$AA@ 10048598     LIBCMT:undname.obj
 0002:000035a4       ??_C@_07FEEIOKP@?$GAvcall?8?$AA@ 100485a4     LIBCMT:undname.obj
 0002:000035ac       ??_C@_09BLBHBJP@?$GAvbtable?8?$AA@ 100485ac     LIBCMT:undname.obj
 0002:000035b8       ??_C@_09IFPLHPGF@?$GAvftable?8?$AA@ 100485b8     LIBCMT:undname.obj
 0002:000035c4       ??_C@_02MHEGNOJ@?$FO?$DN?$AA@ 100485c4     LIBCMT:undname.obj
 0002:000035c8       ??_C@_02DHLNPPGH@?$HM?$DN?$AA@ 100485c8     LIBCMT:undname.obj
 0002:000035cc       ??_C@_02FGJGFEAB@?$CG?$DN?$AA@ 100485cc     LIBCMT:undname.obj
 0002:000035d0       ??_C@_03CDNPDDLA@?$DM?$DM?$DN?$AA@ 100485d0     LIBCMT:undname.obj
 0002:000035d4       ??_C@_03IKFCCPFF@?$DO?$DO?$DN?$AA@ 100485d4     LIBCMT:undname.obj
 0002:000035d8       ??_C@_02FENAOKFI@?$CF?$DN?$AA@ 100485d8     LIBCMT:undname.obj
 0002:000035dc       ??_C@_02FJEHGPIO@?1?$DN?$AA@ 100485dc     LIBCMT:undname.obj
 0002:000035e0       ??_C@_02FKMDLLOA@?9?$DN?$AA@ 100485e0     LIBCMT:undname.obj
 0002:000035e4       ??_C@_02FOEOMHFC@?$CL?$DN?$AA@ 100485e4     LIBCMT:undname.obj
 0002:000035e8       ??_C@_02FPIMKNGF@?$CK?$DN?$AA@ 100485e8     LIBCMT:undname.obj
 0002:000035ec       ??_C@_02NONPIBCD@?$HM?$HM?$AA@ 100485ec     LIBCMT:undname.obj
 0002:000035f0       ??_C@_02PPKAJPJL@?$CG?$CG?$AA@ 100485f0     LIBCMT:undname.obj
 0002:000035f4       ??_C@_01DNKMNLPK@?$HM?$AA@ 100485f4     LIBCMT:undname.obj
 0002:000035f8       ??_C@_01JKBOJNNK@?$FO?$AA@ 100485f8     LIBCMT:undname.obj
 0002:000035fc       ??_C@_01PJKLJHI@?$HO?$AA@  100485fc     LIBCMT:undname.obj
 0002:00003600       ??_C@_02HCKGKOFO@?$CI?$CJ?$AA@ 10048600     LIBCMT:undname.obj
 0002:00003604       ??_C@_01IHBHIGKO@?0?$AA@   10048604     LIBCMT:undname.obj
 0002:00003608       ??_C@_02EEKDKGMJ@?$DO?$DN?$AA@ 10048608     LIBCMT:undname.obj
 0002:0000360c       ??_C@_01PPODPGHN@?$DO?$AA@ 1004860c     LIBCMT:undname.obj
 0002:00003610       ??_C@_02EHCHHCKH@?$DM?$DN?$AA@ 10048610     LIBCMT:undname.obj
 0002:00003614       ??_C@_01MNNFJEPP@?$DM?$AA@ 10048614     LIBCMT:undname.obj
 0002:00003618       ??_C@_01FGNFDNOH@?$CF?$AA@ 10048618     LIBCMT:undname.obj
 0002:0000361c       ??_C@_01KMDKNFGN@?1?$AA@   1004861c     LIBCMT:undname.obj
 0002:00003620       ??_C@_03MNHNFDLC@?9?$DO?$CK?$AA@ 10048620     LIBCMT:undname.obj
 0002:00003624       ??_C@_01HNPIGOCE@?$CG?$AA@ 10048624     LIBCMT:undname.obj
 0002:00003628       ??_C@_01MIFGBAGJ@?$CL?$AA@ 10048628     LIBCMT:undname.obj
 0002:0000362c       ??_C@_01JOAMLHOP@?9?$AA@   1004862c     LIBCMT:undname.obj
 0002:00003630       ??_C@_02BAABKJLB@?9?9?$AA@ 10048630     LIBCMT:undname.obj
 0002:00003634       ??_C@_02ECNGHCIF@?$CL?$CL?$AA@ 10048634     LIBCMT:undname.obj
 0002:00003638       ??_C@_01NBENCBCI@?$CK?$AA@ 10048638     LIBCMT:undname.obj
 0002:0000363c       ??_C@_02HBOOOICD@?9?$DO?$AA@ 1004863c     LIBCMT:undname.obj
 0002:00003640       ??_C@_08LHJFAFGD@operator?$AA@ 10048640     LIBCMT:undname.obj
 0002:0000364c       ??_C@_02GPECMEKF@?$FL?$FN?$AA@ 1004864c     LIBCMT:undname.obj
 0002:00003650       ??_C@_02FDNJECIE@?$CB?$DN?$AA@ 10048650     LIBCMT:undname.obj
 0002:00003654       ??_C@_02EGOFBIJA@?$DN?$DN?$AA@ 10048654     LIBCMT:undname.obj
 0002:00003658       ??_C@_01DCLJPIOD@?$CB?$AA@ 10048658     LIBCMT:undname.obj
 0002:0000365c       ??_C@_02FODMEDOG@?$DM?$DM?$AA@ 1004865c     LIBCMT:undname.obj
 0002:00003660       ??_C@_02GPIOPFAK@?$DO?$DO?$AA@ 10048660     LIBCMT:undname.obj
 0002:00003664       ??_C@_07FPCDHGMM@?5delete?$AA@ 10048664     LIBCMT:undname.obj
 0002:0000366c       ??_C@_04NIHEBCM@?5new?$AA@ 1004866c     LIBCMT:undname.obj
 0002:00003674       ??_C@_0M@GFIIJFMG@__unaligned?$AA@ 10048674     LIBCMT:undname.obj
 0002:00003680       ??_C@_0L@PILCLIHE@__restrict?$AA@ 10048680     LIBCMT:undname.obj
 0002:0000368c       ??_C@_07JOMMBBKO@__ptr64?$AA@ 1004868c     LIBCMT:undname.obj
 0002:00003694       ??_C@_09HIJEGCPM@__clrcall?$AA@ 10048694     LIBCMT:undname.obj
 0002:000036a0       ??_C@_0L@JMKHOMEK@__fastcall?$AA@ 100486a0     LIBCMT:undname.obj
 0002:000036ac       ??_C@_0L@NPHFGOKO@__thiscall?$AA@ 100486ac     LIBCMT:undname.obj
 0002:000036b8       ??_C@_09IFJBGAPI@__stdcall?$AA@ 100486b8     LIBCMT:undname.obj
 0002:000036c4       ??_C@_08GHMPAG@__pascal?$AA@ 100486c4     LIBCMT:undname.obj
 0002:000036d0       ??_C@_07KOLFKCDI@__cdecl?$AA@ 100486d0     LIBCMT:undname.obj
 0002:000036d8       ??_C@_08EHJDFFNH@__based?$CI?$AA@ 100486d8     LIBCMT:undname.obj
 0002:00003868       ___lookuptable_s           10048868     LIBCMT:outputs.obj
 0002:000038c4       __real@00000000            100488c4     effectmanager.obj
 0002:000038c4       ??_C@_13NOLLCAOD@?$AA?$AA?$AA?$AA@ 100488c4     LIBCMT:a_map.obj
 0002:000038c8       ___newctype                100488c8     LIBCMT:ctype.obj
 0002:00003bc8       __wctype                   10048bc8     LIBCMT:ctype.obj
 0002:00003dd0       ___newclmap                10048dd0     LIBCMT:ctype.obj
 0002:00003f50       ___newcumap                10048f50     LIBCMT:ctype.obj
 0002:000040d0       ??_C@_08JCCMCCIL@HH?3mm?3ss?$AA@ 100490d0     LIBCMT:strftime.obj
 0002:000040dc       ??_C@_0BE@CKGJFCPC@dddd?0?5MMMM?5dd?0?5yyyy?$AA@ 100490dc     LIBCMT:strftime.obj
 0002:000040f0       ??_C@_08BPBNCDIB@MM?1dd?1yy?$AA@ 100490f0     LIBCMT:strftime.obj
 0002:000040fc       ??_C@_02CJNFDJBF@PM?$AA@   100490fc     LIBCMT:strftime.obj
 0002:00004100       ??_C@_02DEDBPAFC@AM?$AA@   10049100     LIBCMT:strftime.obj
 0002:00004104       ??_C@_08EDHMEBNP@December?$AA@ 10049104     LIBCMT:strftime.obj
 0002:00004110       ??_C@_08HCHEGEOA@November?$AA@ 10049110     LIBCMT:strftime.obj
 0002:0000411c       ??_C@_07JJNFCEND@October?$AA@ 1004911c     LIBCMT:strftime.obj
 0002:00004124       ??_C@_09BHHEALKD@September?$AA@ 10049124     LIBCMT:strftime.obj
 0002:00004130       ??_C@_06LBBHFDDG@August?$AA@ 10049130     LIBCMT:strftime.obj
 0002:00004138       ??_C@_04MIEPOIFP@July?$AA@ 10049138     LIBCMT:strftime.obj
 0002:00004140       ??_C@_04CNLMGBGM@June?$AA@ 10049140     LIBCMT:strftime.obj
 0002:00004148       ??_C@_05DMJDNLEJ@April?$AA@ 10049148     LIBCMT:strftime.obj
 0002:00004150       ??_C@_05HPCKOFNC@March?$AA@ 10049150     LIBCMT:strftime.obj
 0002:00004158       ??_C@_08GNJGEPFN@February?$AA@ 10049158     LIBCMT:strftime.obj
 0002:00004164       ??_C@_07CGJPFGJA@January?$AA@ 10049164     LIBCMT:strftime.obj
 0002:0000416c       ??_C@_03MKABNOCG@Dec?$AA@  1004916c     LIBCMT:strftime.obj
 0002:00004170       ??_C@_03JPJOFNIA@Nov?$AA@  10049170     LIBCMT:strftime.obj
 0002:00004174       ??_C@_03BMAOKBAD@Oct?$AA@  10049174     LIBCMT:strftime.obj
 0002:00004178       ??_C@_03GGCAPAJC@Sep?$AA@  10049178     LIBCMT:strftime.obj
 0002:0000417c       ??_C@_03IFJFEIGA@Aug?$AA@  1004917c     LIBCMT:strftime.obj
 0002:00004180       ??_C@_03LBGABGKK@Jul?$AA@  10049180     LIBCMT:strftime.obj
 0002:00004184       ??_C@_03IDFGHECI@Jun?$AA@  10049184     LIBCMT:strftime.obj
 0002:00004188       ??_C@_03CNMDKL@May?$AA@    10049188     LIBCMT:strftime.obj
 0002:0000418c       ??_C@_03LEOLGMJP@Apr?$AA@  1004918c     LIBCMT:strftime.obj
 0002:00004190       ??_C@_03ODNJBKGA@Mar?$AA@  10049190     LIBCMT:strftime.obj
 0002:00004194       ??_C@_03HJBDCHOM@Feb?$AA@  10049194     LIBCMT:strftime.obj
 0002:00004198       ??_C@_03JIHJHPIE@Jan?$AA@  10049198     LIBCMT:strftime.obj
 0002:0000419c       ??_C@_08INBOOONO@Saturday?$AA@ 1004919c     LIBCMT:strftime.obj
 0002:000041a8       ??_C@_06JECMNKMI@Friday?$AA@ 100491a8     LIBCMT:strftime.obj
 0002:000041b0       ??_C@_08HACCIKIA@Thursday?$AA@ 100491b0     LIBCMT:strftime.obj
 0002:000041bc       ??_C@_09DLIGFAKA@Wednesday?$AA@ 100491bc     LIBCMT:strftime.obj
 0002:000041c8       ??_C@_07BAAGCFCM@Tuesday?$AA@ 100491c8     LIBCMT:strftime.obj
 0002:000041d0       ??_C@_06JLEDEDGH@Monday?$AA@ 100491d0     LIBCMT:strftime.obj
 0002:000041d8       ??_C@_06OOPIFAJ@Sunday?$AA@ 100491d8     LIBCMT:strftime.obj
 0002:000041e0       ??_C@_03FEFJNEK@Sat?$AA@   100491e0     LIBCMT:strftime.obj
 0002:000041e4       ??_C@_03IDIOELNC@Fri?$AA@  100491e4     LIBCMT:strftime.obj
 0002:000041e8       ??_C@_03IOFIKPDN@Thu?$AA@  100491e8     LIBCMT:strftime.obj
 0002:000041ec       ??_C@_03MHOMLAJA@Wed?$AA@  100491ec     LIBCMT:strftime.obj
 0002:000041f0       ??_C@_03NAGEINEP@Tue?$AA@  100491f0     LIBCMT:strftime.obj
 0002:000041f4       ??_C@_03PDAGKDH@Mon?$AA@   100491f4     LIBCMT:strftime.obj
 0002:000041f8       ??_C@_03KOEHGMDN@Sun?$AA@  100491f8     LIBCMT:strftime.obj
 0002:000041fc       ??_C@_0BI@DFKBFLJE@GetProcessWindowStation?$AA@ 100491fc     LIBCMT:crtmbox.obj
 0002:00004214       ??_C@_0BK@CIDNPOGP@GetUserObjectInformationA?$AA@ 10049214     LIBCMT:crtmbox.obj
 0002:00004230       ??_C@_0BD@HHGDFDBJ@GetLastActivePopup?$AA@ 10049230     LIBCMT:crtmbox.obj
 0002:00004244       ??_C@_0BA@HNOPNCHB@GetActiveWindow?$AA@ 10049244     LIBCMT:crtmbox.obj
 0002:00004254       ??_C@_0M@CHKKJDAI@MessageBoxA?$AA@ 10049254     LIBCMT:crtmbox.obj
 0002:00004260       ??_C@_0L@NDEGIDAG@USER32?4DLL?$AA@ 10049260     LIBCMT:crtmbox.obj
 0002:0000426c       ??_C@_06IMKFLFPG@1?$CDQNAN?$AA@ 1004926c     LIBCMT:_x10fout_.obj
 0002:00004274       ??_C@_05DNEBIAHO@1?$CDINF?$AA@ 10049274     LIBCMT:_x10fout_.obj
 0002:0000427c       ??_C@_05PHHOCPM@1?$CDIND?$AA@ 1004927c     LIBCMT:_x10fout_.obj
 0002:00004284       ??_C@_06PGGFOGJG@1?$CDSNAN?$AA@ 10049284     LIBCMT:_x10fout_.obj
 0002:0000428c       ??_C@_0L@KDOEJCKC@_nextafter?$AA@ 1004928c     LIBCMT:_fpexcept_.obj
 0002:00004298       ??_C@_05JGDBENOH@_logb?$AA@ 10049298     LIBCMT:_fpexcept_.obj
 0002:000042a0       ??_C@_03ONILCKOB@_yn?$AA@  100492a0     LIBCMT:_fpexcept_.obj
 0002:000042a4       ??_C@_03NAKIGLHK@_y1?$AA@  100492a4     LIBCMT:_fpexcept_.obj
 0002:000042a8       ??_C@_03MJLDFKDL@_y0?$AA@  100492a8     LIBCMT:_fpexcept_.obj
 0002:000042ac       ??_C@_05GKKHEGJL@frexp?$AA@ 100492ac     LIBCMT:_fpexcept_.obj
 0002:000042b4       ??_C@_04KEPJIHGP@fmod?$AA@ 100492b4     LIBCMT:_fpexcept_.obj
 0002:000042bc       ??_C@_06MEIMCGCF@_hypot?$AA@ 100492bc     LIBCMT:_fpexcept_.obj
 0002:000042c4       ??_C@_05KBKMEMPO@_cabs?$AA@ 100492c4     LIBCMT:_fpexcept_.obj
 0002:000042cc       ??_C@_05CEJMAHNP@ldexp?$AA@ 100492cc     LIBCMT:_fpexcept_.obj
 0002:000042d4       ??_C@_04EHEDPDJG@modf?$AA@ 100492d4     LIBCMT:_fpexcept_.obj
 0002:000042dc       ??_C@_04ODHECPBC@fabs?$AA@ 100492dc     LIBCMT:_fpexcept_.obj
 0002:000042e4       ??_C@_05PBJFFIGL@floor?$AA@ 100492e4     LIBCMT:_fpexcept_.obj
 0002:000042ec       ??_C@_04GFPJNGEK@ceil?$AA@ 100492ec     LIBCMT:_fpexcept_.obj
 0002:000042f4       ??_C@_03IIINPABG@tan?$AA@  100492f4     LIBCMT:_fpexcept_.obj
 0002:000042f8       ??_C@_03LALBNOCG@cos?$AA@  100492f8     LIBCMT:_fpexcept_.obj
 0002:000042fc       ??_C@_03BLEJJJBH@sin?$AA@  100492fc     LIBCMT:_fpexcept_.obj
 0002:00004300       ??_C@_04EIAKFFMI@sqrt?$AA@ 10049300     LIBCMT:_fpexcept_.obj
 0002:00004308       ??_C@_05KNGEOGJB@atan2?$AA@ 10049308     LIBCMT:_fpexcept_.obj
 0002:00004310       ??_C@_04MLLJIGOK@atan?$AA@ 10049310     LIBCMT:_fpexcept_.obj
 0002:00004318       ??_C@_04PDIFKINK@acos?$AA@ 10049318     LIBCMT:_fpexcept_.obj
 0002:00004320       ??_C@_04FIHNOPOL@asin?$AA@ 10049320     LIBCMT:_fpexcept_.obj
 0002:00004328       ??_C@_04FJHINJAO@tanh?$AA@ 10049328     LIBCMT:_fpexcept_.obj
 0002:00004330       ??_C@_04HPJJNFIM@cosh?$AA@ 10049330     LIBCMT:_fpexcept_.obj
 0002:00004338       ??_C@_04COOMCNPB@sinh?$AA@ 10049338     LIBCMT:_fpexcept_.obj
 0002:00004340       ??_C@_05HGHHAHAP@log10?$AA@ 10049340     LIBCMT:_fpexcept_.obj
 0002:00004348       ??_C@_03MGHMBJCF@log?$AA@  10049348     LIBCMT:_fpexcept_.obj
 0002:0000434c       ??_C@_03JGHBODFD@pow?$AA@  1004934c     LIBCMT:_fpexcept_.obj
 0002:00004350       ??_C@_03KHJOGHMM@exp?$AA@  10049350     LIBCMT:_fpexcept_.obj
 0002:00004354       ___dnames                  10049354     LIBCMT:timeset.obj
 0002:0000436c       ___mnames                  1004936c     LIBCMT:timeset.obj
 0002:00004394       ??_C@_07GPDNMNG@CONOUT$?$AA@ 10049394     LIBCMT:initcon.obj
 0002:000043a0       ??_7WzLogSystem@WzLog@@6B@ 100493a0     ProgramCommonLibForEngine_p:wzlogsystem.obj
 0002:000043a8       ??_7?$CWzSingleton@VWzLogSystem@WzLog@@@@6B@ 100493a8     ProgramCommonLibForEngine_p:wzlogsystem.obj
 0002:000043ac       ??_C@_09ONPMENGE@se_?$CFs?4log?$AA@ 100493ac     ProgramCommonLibForEngine_p:wzlogsystem.obj
 0002:000043b8       ??_C@_0N@PKIBJLNA@WzFilePacker?$AA@ 100493b8     ProgramCommonLibForEngine_p:discaccess.obj
 0002:000043c8       ??_C@_09LGACLDHG@Hard?5disk?$AA@ 100493c8     ProgramCommonLibForEngine_p:discaccess.obj
 0002:000043d4       ??_C@_04OHJIHAFH@None?$AA@ 100493d4     ProgramCommonLibForEngine_p:discaccess.obj
 0002:000043dc       ??_C@_0DM@LMNABLME@CDiscAccess?3?3CreateDefaultDisc?$CI?$CJ@ 100493dc     ProgramCommonLibForEngine_p:discaccess.obj
 0002:00004418       ??_C@_0DI@ODBJGFIE@CDiscAccess?3?3OpenDisc_Hard?$CI?$CJ?5?9?5?$MA@ 10049418     ProgramCommonLibForEngine_p:discaccess.obj
 0002:00004450       ??_C@_0DG@PHHHENLO@CDiscAccess?3?3OpenDisc_Hard?$CI?$CJ?5?9?5?$MA@ 10049450     ProgramCommonLibForEngine_p:discaccess.obj
 0002:00004488       ??_C@_0EC@PMCOJJDG@CDiscAccess?3?3OpenDisc_Packer?$CI?$CJ?5?9@ 10049488     ProgramCommonLibForEngine_p:discaccess.obj
 0002:000044d0       ??_C@_0EA@OAHIDHBK@CDiscAccess?3?3OpenDisc_Packer?$CI?$CJ?5?9@ 100494d0     ProgramCommonLibForEngine_p:discaccess.obj
 0002:00004510       ??_C@_0DK@JHDNEDFK@CDiscAccess?3?3OpenDisc_Packer?$CI?$CJ?5?9@ 10049510     ProgramCommonLibForEngine_p:discaccess.obj
 0002:0000454c       ??_C@_0DI@LMHJEMHG@CDiscAccess?3?3OpenDisc_Packer?$CI?$CJ?5?9@ 1004954c     ProgramCommonLibForEngine_p:discaccess.obj
 0002:00004584       ??_C@_0DC@PKNMHJEJ@CDiscAccess?3?3CloseDisc?$CI?$CJ?5?9?5?$MA?$NP?$LI?x?$LF@ 10049584     ProgramCommonLibForEngine_p:discaccess.obj
 0002:000045b8       ??_C@_0DG@BKNAKAGB@CDiscAccess?3?3SetActiveDisc?$CI?$CJ?5?9?5?$LP@ 100495b8     ProgramCommonLibForEngine_p:discaccess.obj
 0002:000045f0       ??_C@_0DG@HELNFJLI@CDiscAccess?3?3SetActiveDisc?$CI?$CJ?5?9?5?$MA@ 100495f0     ProgramCommonLibForEngine_p:discaccess.obj
 0002:00004628       ??_C@_0DA@FFFJLJGB@CDiscAccess?3?3OpenFile?$CI?$CJ?5?9?5Unknow@ 10049628     ProgramCommonLibForEngine_p:discaccess.obj
 0002:00004658       ??_C@_0CN@DICIKECD@CDiscAccess?3?3OpenFile?$CI?$CJ?5?9?5?F?D?$MA?O?5?$LP@ 10049658     ProgramCommonLibForEngine_p:discaccess.obj
 0002:0000469c       ??_C@_0DB@MADLHAJA@CDiscAccess?3?3CloseFile?$CI?$CJ?5?9?5Unkno@ 1004969c     ProgramCommonLibForEngine_p:discaccess.obj
 0002:000046d0       ??_C@_0DO@HDCEPBCE@CDiscAccess?3?3CloseFile?$CI?$CJ?5?9?5?F?D?$MA?O?A@ 100496d0     ProgramCommonLibForEngine_p:discaccess.obj
 0002:00004710       ??_C@_0DA@NFEJOLPK@CDiscAccess?3?3CloseFile?$CI?$CJ?5?9?5?$LJ?$KL?H?$LP?G@ 10049710     ProgramCommonLibForEngine_p:discaccess.obj
 0002:00004740       ??_C@_0DA@ELBBBMEA@CDiscAccess?3?3SeekFile?$CI?$CJ?5?9?5Unknow@ 10049740     ProgramCommonLibForEngine_p:discaccess.obj
 0002:00004770       ??_C@_0DA@IKILOBGB@CDiscAccess?3?3SeekFile?$CI?$CJ?5?9?5GetFil@ 10049770     ProgramCommonLibForEngine_p:discaccess.obj
 0002:000047a0       ??_C@_0DA@HPNNDICA@CDiscAccess?3?3SeekFile?$CI?$CJ?5?9?5SetFil@ 100497a0     ProgramCommonLibForEngine_p:discaccess.obj
 0002:000047dc       ??_C@_0DA@EMEGOIF@CDiscAccess?3?3ReadFile?$CI?$CJ?5?9?5Unknow@ 100497dc     ProgramCommonLibForEngine_p:discaccess.obj
 0002:0000480c       ??_C@_0CB@JLNJPHFF@CDiscAccess?3?3ReadFile?$CI?$CJ?5?9?5?$LN?G?F?P?$CB?$CB@ 1004980c     ProgramCommonLibForEngine_p:discaccess.obj
 0002:00004830       ??_C@_0DB@LJCMBAL@CDiscAccess?3?3WriteFile?$CI?$CJ?5?9?5Unkno@ 10049830     ProgramCommonLibForEngine_p:discaccess.obj
 0002:00004864       ??_C@_0CC@LNNIJHEL@CDiscAccess?3?3WriteFile?$CI?$CJ?5?9?5?$LN?G?F?P?$CB@ 10049864     ProgramCommonLibForEngine_p:discaccess.obj
 0002:00004888       ??_C@_0DC@NPAJAIAP@CDiscAccess?3?3FileExists?$CI?$CJ?5?9?5Unkn@ 10049888     ProgramCommonLibForEngine_p:discaccess.obj
 0002:000048bc       ??_C@_0DD@CJICJBIC@CDiscAccess?3?3GetFileSize?$CI?$CJ?5?9?5Unk@ 100498bc     ProgramCommonLibForEngine_p:discaccess.obj
 0002:000048f0       ??_C@_0CE@JGOLOJIE@CDiscAccess?3?3GetFileSize?$CI?$CJ?5?9?5?$LN?G?F@ 100498f0     ProgramCommonLibForEngine_p:discaccess.obj
 0002:00004918       ??_C@_0EC@JKIAEHOK@CDiscAccess?3?3GetFileInformationB@ 10049918     ProgramCommonLibForEngine_p:discaccess.obj
 0002:0000495c       ??_C@_0DB@PPIDBHIP@CDiscAccess?3?3GetFileInformationB@ 1004995c     ProgramCommonLibForEngine_p:discaccess.obj
 0002:00004990       ??_C@_0CP@EOGGFMOM@CDiscAccess?3?3AddFile?$CI?$CJ?5?9?5Unknown@ 10049990     ProgramCommonLibForEngine_p:discaccess.obj
 0002:000049c0       ??_C@_0DC@OKADKNGE@CDiscAccess?3?3DeleteFile?$CI?$CJ?5?9?5Unkn@ 100499c0     ProgramCommonLibForEngine_p:discaccess.obj
 0002:000049f4       ??_C@_0DH@LJINKHCI@CDiscAccess?3?3CreateDirectory?$CI?$CJ?5?9@ 100499f4     ProgramCommonLibForEngine_p:discaccess.obj
 0002:00004a2c       ??_C@_0DH@HLAJJPFC@CDiscAccess?3?3RemoveDirectory?$CI?$CJ?5?9@ 10049a2c     ProgramCommonLibForEngine_p:discaccess.obj
 0002:00004a68       ??_7?$CWzHandleManager@USt_DAFileInfo@@@@6B@ 10049a68     ProgramCommonLibForEngine_p:discaccess.obj
 0002:00004a6c       ??_C@_0CN@GBNFHBOA@CScriptRead?3?3Create?$CI?$CJ?5?9?5?F?D?$MA?O?5?$LL?g?$MA@ 10049a6c     ProgramCommonLibForEngine_p:scriptread.obj
 0002:00004a9c       ??_C@_0CM@DDLIJOAA@CScriptRead?3?3Create?$CI?$CJ?5?9?5OpenFile@ 10049a9c     ProgramCommonLibForEngine_p:scriptread.obj
 0002:00004ac8       ??_C@_0DH@BADBPNMD@CScriptRead?3?3CreateFromBuffer?$CI?$CJ?5@ 10049ac8     ProgramCommonLibForEngine_p:scriptread.obj
 0002:00004b00       ??_C@_0CP@NCBLOAEK@CScriptRead?3?3GetToken?$CI?$CJ?5?9?5?$MA?$NP?$LI?x?$LF?H@ 10049b00     ProgramCommonLibForEngine_p:scriptread.obj
 0002:00004b34       ??_7WzFileLogHandler@WzLog@@6B@ 10049b34     ProgramCommonLibForEngine_p:WzFileLogHandler.obj
 0002:00004b50       ??_7WzLogHandler@WzLog@@6B@ 10049b50     ProgramCommonLibForEngine_p:WzFileLogHandler.obj
 0002:00004b68       ??_C@_0BK@OPFMAPDK@?$FL?$CF02d?3?$CF02d?3?$CF02d?$FN?$FL?$CFs?$FN?5?$CFs?$AN?6?$AA@ 10049b68     ProgramCommonLibForEngine_p:WzFileLogHandler.obj
 0002:00004bc8       __real@4018000000000000    10049bc8     Common_p:wznaturalcubicsplinedyn.obj
 0002:00004bd0       ??_C@_0CA@NFKJJDJK@MatrixInverse?$CI?$CJ?5?9?5det?5is?5zero?$CB?$CB?$AA@ 10049bd0     Common_p:wzmath.obj
 0002:00004bf0       __real@3a83126f            10049bf0     Common_p:wzmath.obj
 0002:00004bf8       __real@3ee4f8b580000000    10049bf8     Common_p:wzmath.obj
 0002:00004c00       ??_C@_0DK@BLIFBBOF@Math_GetRandomPosInBoundingVolum@ 10049c00     Common_p:mathassistant.obj
 0002:00004c3c       __real@40490fdb            10049c3c     Common_p:mathassistant.obj
 0002:000064c8       ??_C@_05EOHGHCHD@exp10?$AA@ 1004b4c8     LIBCMT:_libm_error_.obj
 0002:000066e8       __real@4f800000            1004b6e8     wzFilePacker_static:wzFilePacker.obj
 0002:00006f50       ??_C@_0BI@LCBABOGN@header?5is?5Final?5Version?$AA@ 1004bf50     wzFilePacker_static:fsvfs.obj
 0002:00006f68       ??_C@_0P@FOHJAHFG@header?5invalid?$AA@ 1004bf68     wzFilePacker_static:fsvfs.obj
 0002:00006f78       ??_C@_0DM@MLIJDPNB@Now?5Packing?5File?5Version?5?3?5?$CFd?0?5P@ 1004bf78     wzFilePacker_static:fsvfs.obj
 0002:00006fb4       ??_C@_0DA@JPDHOIDD@?$CK?$CK?$CK?$CK?$CK?$CK?$CK?$CK?$CK?$CK?$CK?$CK?$CK?$CK?$CK?$CK?5N2_UpdateFilePo@ 1004bfb4     wzFilePacker_static:fsvfs.obj
 0002:00006fe4       ??_C@_0CO@LGMGIONK@?$CK?$CK?$CK?$CK?$CK?$CK?$CK?$CK?$CK?$CK?$CK?$CK?$CK?$CK?$CK?$CK?5N2_SetFilePoint@ 1004bfe4     wzFilePacker_static:fsvfs.obj
 0002:00007014       ??_C@_0DF@IHAPMOPK@?$CL?$CL?$CL?$CL?$CL?$CL?$CL?$CL?$CL?$CL?5ReadFail_4_Error?5?3?5?G?O@ 1004c014     wzFilePacker_static:fsvfs.obj
 0002:0000704c       ??_C@_0DH@HABJGGNC@?$CL?$CL?$CL?$CL?$CL?$CL?$CL?$CL?$CL?$CL?5ReadFail_3_Error?5?3?5?$MA?P@ 1004c04c     wzFilePacker_static:fsvfs.obj
 0002:00007084       ??_C@_0DG@LCJJILDN@?$CL?$CL?$CL?$CL?$CL?$CL?$CL?$CL?$CL?$CL?5ReadFail_2_Error?5?3?5?$LP?$MA@ 1004c084     wzFilePacker_static:fsvfs.obj
 0002:000070bc       ??_C@_0CG@GENKINJN@?$CL?$CL?$CL?$CL?$CL?$CL?$CL?$CL?$CL?$CL?5ReadFail_1_ErrorCode?5@ 1004c0bc     wzFilePacker_static:fsvfs.obj
 0002:000070e4       ??_C@_0BH@MMBDGEON@Remove?5Fsvfs?5Tree?5Fail?$AA@ 1004c0e4     wzFilePacker_static:fsvfs.obj
 0002:000070fc       ??_C@_0BK@PKGCLKLI@Remove?5Fsvfs?5Tree?5SUCCESS?$AA@ 1004c0fc     wzFilePacker_static:fsvfs.obj
 0002:00007118       ??_C@_0BM@OPDJPMGP@Not?5File?5SameName?5Tree?9Node?$AA@ 1004c118     wzFilePacker_static:fsvfs.obj
 0002:00007568       ??_C@_02CEGDFPFP@?4?2?$AA@ 1004c568     wzFilePacker_static:fsdos.obj
 0002:0000756c       ??_C@_0BP@PFJFMKGH@Win32_SetFilePointer_Error?3?$CFd?6?$AA@ 1004c56c     wzFilePacker_static:fsdos.obj
 0002:000079e0       __load_config_used         1004c9e0     LIBCMT:loadcfg.obj
 0002:00007a94       ??_R4?$CWzSingleton@VCEffectManager@@@@6B@ 1004ca94     effectmanager.obj
 0002:00007aa8       ??_R3?$CWzSingleton@VCEffectManager@@@@8 1004caa8     effectmanager.obj
 0002:00007ab8       ??_R2?$CWzSingleton@VCEffectManager@@@@8 1004cab8     effectmanager.obj
 0002:00007ac0       ??_R1A@?0A@EA@?$CWzSingleton@VCEffectManager@@@@8 1004cac0     effectmanager.obj
 0002:00007adc       ??_R4CEffectManager@@6B@   1004cadc     effectmanager.obj
 0002:00007af0       ??_R3CEffectManager@@8     1004caf0     effectmanager.obj
 0002:00007b00       ??_R2CEffectManager@@8     1004cb00     effectmanager.obj
 0002:00007b0c       ??_R1A@?0A@EA@CEffectManager@@8 1004cb0c     effectmanager.obj
 0002:00007b28       ??_R4out_of_range@std@@6B@ 1004cb28     effectmanager.obj
 0002:00007b3c       ??_R3out_of_range@std@@8   1004cb3c     effectmanager.obj
 0002:00007b4c       ??_R2out_of_range@std@@8   1004cb4c     effectmanager.obj
 0002:00007b5c       ??_R1A@?0A@EA@out_of_range@std@@8 1004cb5c     effectmanager.obj
 0002:00007b78       ??_R1A@?0A@EA@logic_error@std@@8 1004cb78     effectmanager.obj
 0002:00007b94       ??_R3logic_error@std@@8    1004cb94     effectmanager.obj
 0002:00007ba4       ??_R2logic_error@std@@8    1004cba4     effectmanager.obj
 0002:00007bb0       ??_R1A@?0A@EA@exception@std@@8 1004cbb0     effectmanager.obj
 0002:00007bcc       ??_R3exception@std@@8      1004cbcc     effectmanager.obj
 0002:00007bdc       ??_R2exception@std@@8      1004cbdc     effectmanager.obj
 0002:00007be4       ??_R4logic_error@std@@6B@  1004cbe4     effectmanager.obj
 0002:00007bf8       ??_R4bad_alloc@std@@6B@    1004cbf8     effectmanager.obj
 0002:00007c0c       ??_R3bad_alloc@std@@8      1004cc0c     effectmanager.obj
 0002:00007c1c       ??_R2bad_alloc@std@@8      1004cc1c     effectmanager.obj
 0002:00007c28       ??_R1A@?0A@EA@bad_alloc@std@@8 1004cc28     effectmanager.obj
 0002:00007c44       ??_R4length_error@std@@6B@ 1004cc44     effectmanager.obj
 0002:00007c58       ??_R3length_error@std@@8   1004cc58     effectmanager.obj
 0002:00007c68       ??_R2length_error@std@@8   1004cc68     effectmanager.obj
 0002:00007c78       ??_R1A@?0A@EA@length_error@std@@8 1004cc78     effectmanager.obj
 0002:00007c94       ??_R4?$CWzHandleManager@PAVCEffectBody@@@@6B@ 1004cc94     effectmanager.obj
 0002:00007ca8       ??_R3?$CWzHandleManager@PAVCEffectBody@@@@8 1004cca8     effectmanager.obj
 0002:00007cb8       ??_R2?$CWzHandleManager@PAVCEffectBody@@@@8 1004ccb8     effectmanager.obj
 0002:00007cc0       ??_R1A@?0A@EA@?$CWzHandleManager@PAVCEffectBody@@@@8 1004ccc0     effectmanager.obj
 0002:00007cdc       ??_R4CEElementBase@@6B@    1004ccdc     eelementbase.obj
 0002:00007cf0       ??_R3CEElementBase@@8      1004ccf0     eelementbase.obj
 0002:00007d00       ??_R2CEElementBase@@8      1004cd00     eelementbase.obj
 0002:00007d08       ??_R1A@?0A@EA@CEElementBase@@8 1004cd08     eelementbase.obj
 0002:00007d24       ??_R4CEElementChain@@6B@   1004cd24     eelementchain.obj
 0002:00007d38       ??_R3CEElementChain@@8     1004cd38     eelementchain.obj
 0002:00007d48       ??_R2CEElementChain@@8     1004cd48     eelementchain.obj
 0002:00007d58       ??_R1A@?0A@EA@CEElementChain@@8 1004cd58     eelementchain.obj
 0002:00007d74       ??_R1A@?0A@EA@CEElementParticle@@8 1004cd74     eelementchain.obj
 0002:00007d90       ??_R3CEElementParticle@@8  1004cd90     eelementchain.obj
 0002:00007da0       ??_R2CEElementParticle@@8  1004cda0     eelementchain.obj
 0002:00007dac       ??_R4CEElementDecal@@6B@   1004cdac     eelementdecal.obj
 0002:00007dc0       ??_R3CEElementDecal@@8     1004cdc0     eelementdecal.obj
 0002:00007dd0       ??_R2CEElementDecal@@8     1004cdd0     eelementdecal.obj
 0002:00007ddc       ??_R1A@?0A@EA@CEElementDecal@@8 1004cddc     eelementdecal.obj
 0002:00007df8       ??_R4CEElementFlatChain@@6B@ 1004cdf8     eelementflatchain.obj
 0002:00007e0c       ??_R3CEElementFlatChain@@8 1004ce0c     eelementflatchain.obj
 0002:00007e1c       ??_R2CEElementFlatChain@@8 1004ce1c     eelementflatchain.obj
 0002:00007e28       ??_R1A@?0A@EA@CEElementFlatChain@@8 1004ce28     eelementflatchain.obj
 0002:00007e44       ??_R4CEElementMesh@@6B@    1004ce44     eelementmesh.obj
 0002:00007e58       ??_R3CEElementMesh@@8      1004ce58     eelementmesh.obj
 0002:00007e68       ??_R2CEElementMesh@@8      1004ce68     eelementmesh.obj
 0002:00007e78       ??_R1A@?0A@EA@CEElementMesh@@8 1004ce78     eelementmesh.obj
 0002:00007e94       ??_R4CEElementParticle@@6B@ 1004ce94     eelementparticle.obj
 0002:00007ea8       ??_R4CEElementSprite@@6B@  1004cea8     eelementsprite.obj
 0002:00007ebc       ??_R3CEElementSprite@@8    1004cebc     eelementsprite.obj
 0002:00007ecc       ??_R2CEElementSprite@@8    1004cecc     eelementsprite.obj
 0002:00007edc       ??_R1A@?0A@EA@CEElementSprite@@8 1004cedc     eelementsprite.obj
 0002:00007ef8       ??_R4CEElementWeather@@6B@ 1004cef8     eelementweather.obj
 0002:00007f0c       ??_R3CEElementWeather@@8   1004cf0c     eelementweather.obj
 0002:00007f1c       ??_R2CEElementWeather@@8   1004cf1c     eelementweather.obj
 0002:00007f28       ??_R1A@?0A@EA@CEElementWeather@@8 1004cf28     eelementweather.obj
 0002:00007f44       ??_R4CEffectBody@@6B@      1004cf44     effectbody.obj
 0002:00007f58       ??_R3CEffectBody@@8        1004cf58     effectbody.obj
 0002:00007f68       ??_R2CEffectBody@@8        1004cf68     effectbody.obj
 0002:00007f78       ??_R1A@?0A@EA@CEffectBody@@8 1004cf78     effectbody.obj
 0002:00007f94       ??_R4type_info@@6B@        1004cf94     LIBCMT:typinfo.obj
 0002:00007fa8       ??_R3type_info@@8          1004cfa8     LIBCMT:typinfo.obj
 0002:00007fb8       ??_R2type_info@@8          1004cfb8     LIBCMT:typinfo.obj
 0002:00007fc0       ??_R1A@?0A@EA@type_info@@8 1004cfc0     LIBCMT:typinfo.obj
 0002:00007fdc       ??_R4exception@std@@6B@    1004cfdc     LIBCMT:stdexcpt.obj
 0002:00007ff0       ??_R4bad_exception@std@@6B@ 1004cff0     LIBCMT:frame.obj
 0002:00008004       ??_R3bad_exception@std@@8  1004d004     LIBCMT:frame.obj
 0002:00008014       ??_R2bad_exception@std@@8  1004d014     LIBCMT:frame.obj
 0002:00008020       ??_R1A@?0A@EA@bad_exception@std@@8 1004d020     LIBCMT:frame.obj
 0002:0000803c       ??_R4?$CWzSingleton@VWzLogSystem@WzLog@@@@6B@ 1004d03c     ProgramCommonLibForEngine_p:wzlogsystem.obj
 0002:00008050       ??_R3?$CWzSingleton@VWzLogSystem@WzLog@@@@8 1004d050     ProgramCommonLibForEngine_p:wzlogsystem.obj
 0002:00008060       ??_R2?$CWzSingleton@VWzLogSystem@WzLog@@@@8 1004d060     ProgramCommonLibForEngine_p:wzlogsystem.obj
 0002:00008068       ??_R1A@?0A@EA@?$CWzSingleton@VWzLogSystem@WzLog@@@@8 1004d068     ProgramCommonLibForEngine_p:wzlogsystem.obj
 0002:00008084       ??_R4WzLogSystem@WzLog@@6B@ 1004d084     ProgramCommonLibForEngine_p:wzlogsystem.obj
 0002:00008098       ??_R3WzLogSystem@WzLog@@8  1004d098     ProgramCommonLibForEngine_p:wzlogsystem.obj
 0002:000080a8       ??_R2WzLogSystem@WzLog@@8  1004d0a8     ProgramCommonLibForEngine_p:wzlogsystem.obj
 0002:000080b4       ??_R1A@?0A@EA@WzLogSystem@WzLog@@8 1004d0b4     ProgramCommonLibForEngine_p:wzlogsystem.obj
 0002:000080d0       ??_R4?$CWzHandleManager@USt_DAFileInfo@@@@6B@ 1004d0d0     ProgramCommonLibForEngine_p:discaccess.obj
 0002:000080e4       ??_R3?$CWzHandleManager@USt_DAFileInfo@@@@8 1004d0e4     ProgramCommonLibForEngine_p:discaccess.obj
 0002:000080f4       ??_R2?$CWzHandleManager@USt_DAFileInfo@@@@8 1004d0f4     ProgramCommonLibForEngine_p:discaccess.obj
 0002:000080fc       ??_R1A@?0A@EA@?$CWzHandleManager@USt_DAFileInfo@@@@8 1004d0fc     ProgramCommonLibForEngine_p:discaccess.obj
 0002:00008118       ??_R4WzLogHandler@WzLog@@6B@ 1004d118     ProgramCommonLibForEngine_p:WzFileLogHandler.obj
 0002:0000812c       ??_R3WzLogHandler@WzLog@@8 1004d12c     ProgramCommonLibForEngine_p:WzFileLogHandler.obj
 0002:0000813c       ??_R2WzLogHandler@WzLog@@8 1004d13c     ProgramCommonLibForEngine_p:WzFileLogHandler.obj
 0002:00008144       ??_R1A@?0A@EA@WzLogHandler@WzLog@@8 1004d144     ProgramCommonLibForEngine_p:WzFileLogHandler.obj
 0002:00008160       ??_R4WzFileLogHandler@WzLog@@6B@ 1004d160     ProgramCommonLibForEngine_p:WzFileLogHandler.obj
 0002:00008174       ??_R3WzFileLogHandler@WzLog@@8 1004d174     ProgramCommonLibForEngine_p:WzFileLogHandler.obj
 0002:00008184       ??_R2WzFileLogHandler@WzLog@@8 1004d184     ProgramCommonLibForEngine_p:WzFileLogHandler.obj
 0002:00008190       ??_R1A@?0A@EA@WzFileLogHandler@WzLog@@8 1004d190     ProgramCommonLibForEngine_p:WzFileLogHandler.obj
 0002:000081b0       ___safe_se_handler_table   1004d1b0     <linker-defined>
 0002:00008348       ___rtc_iaa                 1004d348     LIBCMT:_initsect_.obj
 0002:0000834c       ___rtc_izz                 1004d34c     LIBCMT:_initsect_.obj
 0002:00008350       ___rtc_taa                 1004d350     LIBCMT:_initsect_.obj
 0002:00008354       ___rtc_tzz                 1004d354     LIBCMT:_initsect_.obj
 0002:000089f8       __TI3?AVout_of_range@std@@ 1004d9f8     effectmanager.obj
 0002:00008a34       __CTA3?AVout_of_range@std@@ 1004da34     effectmanager.obj
 0002:00008a44       __CT??_R0?AVout_of_range@std@@@8??0out_of_range@std@@QAE@ABV01@@Z40 1004da44     effectmanager.obj
 0002:00008a60       __CT??_R0?AVlogic_error@std@@@8??0logic_error@std@@QAE@ABV01@@Z40 1004da60     effectmanager.obj
 0002:00008a7c       __CT??_R0?AVexception@std@@@8??0exception@std@@QAE@ABV01@@Z12 1004da7c     effectmanager.obj
 0002:00008b50       __TI2?AVbad_alloc@std@@    1004db50     effectmanager.obj
 0002:00008b60       __CTA2?AVbad_alloc@std@@   1004db60     effectmanager.obj
 0002:00008b6c       __CT??_R0?AVbad_alloc@std@@@8??0bad_alloc@std@@QAE@ABV01@@Z12 1004db6c     effectmanager.obj
 0002:00008d24       __TI3?AVlength_error@std@@ 1004dd24     effectmanager.obj
 0002:00008d34       __CTA3?AVlength_error@std@@ 1004dd34     effectmanager.obj
 0002:00008d44       __CT??_R0?AVlength_error@std@@@8??0length_error@std@@QAE@ABV01@@Z40 1004dd44     effectmanager.obj
 0002:00009acc       __TI2?AVbad_exception@std@@ 1004eacc     LIBCMT:frame.obj
 0002:00009adc       __CTA2?AVbad_exception@std@@ 1004eadc     LIBCMT:frame.obj
 0002:00009ae8       __CT??_R0?AVbad_exception@std@@@8??0bad_exception@std@@QAE@ABV01@@Z12 1004eae8     LIBCMT:frame.obj
 0002:0000a2e0       __IMPORT_DESCRIPTOR_KERNEL32 1004f2e0     kernel32:KERNEL32.dll
 0002:0000a2f4       __IMPORT_DESCRIPTOR_USER32 1004f2f4     user32:USER32.dll
 0002:0000a308       __IMPORT_DESCRIPTOR_3DFileAccess_p 1004f308     3dfileaccess_p:3DFileAccess_p.dll
 0002:0000a31c       __NULL_IMPORT_DESCRIPTOR   1004f31c     kernel32:KERNEL32.dll
 0003:00000000       ?wvScale@?1??CreateEffect@CEffectManager@@QAEPAXKABUWzVector@@H@Z@4U3@A 10051000     dllaccess.obj
 0003:0000000c       ??_R0?AV?$CWzSingleton@VCEffectManager@@@@@8 1005100c     effectmanager.obj
 0003:0000003c       ??_R0?AVCEffectManager@@@8 1005103c     effectmanager.obj
 0003:00000068       ??_R0?AVout_of_range@std@@@8 10051068     effectmanager.obj
 0003:00000088       ??_R0?AVlogic_error@std@@@8 10051088     effectmanager.obj
 0003:000000a8       ??_R0?AVexception@std@@@8  100510a8     effectmanager.obj
 0003:000000c4       ??_R0?AVbad_alloc@std@@@8  100510c4     effectmanager.obj
 0003:000000e0       ??_R0?AVlength_error@std@@@8 100510e0     effectmanager.obj
 0003:00000100       ??_R0?AV?$CWzHandleManager@PAVCEffectBody@@@@@8 10051100     effectmanager.obj
 0003:00000138       ??_R0?AVCEElementBase@@@8  10051138     eelementbase.obj
 0003:00000154       ??_R0?AVCEElementChain@@@8 10051154     eelementchain.obj
 0003:00000174       ??_R0?AVCEElementParticle@@@8 10051174     eelementchain.obj
 0003:00000194       ??_R0?AVCEElementDecal@@@8 10051194     eelementdecal.obj
 0003:000001b4       ??_R0?AVCEElementFlatChain@@@8 100511b4     eelementflatchain.obj
 0003:000001d8       ??_R0?AVCEElementMesh@@@8  100511d8     eelementmesh.obj
 0003:000001f4       ??_R0?AVCEElementSprite@@@8 100511f4     eelementsprite.obj
 0003:00000214       ??_R0?AVCEElementWeather@@@8 10051214     eelementweather.obj
 0003:00000234       ??_R0?AVCEffectBody@@@8    10051234     effectbody.obj
 0003:0000025c       ___security_cookie         1005125c     LIBCMT:gs_cookie.obj
 0003:00000260       ___security_cookie_complement 10051260     LIBCMT:gs_cookie.obj
 0003:00000264       __fltused                  10051264     LIBCMT:_fpinit_.obj
 0003:00000268       __ldused                   10051268     LIBCMT:_fpinit_.obj
 0003:00000270       ??_R0?AVtype_info@@@8      10051270     LIBCMT:typinfo.obj
 0003:000002d4       ??_R0?AVbad_exception@std@@@8 100512d4     LIBCMT:frame.obj
 0003:000002f4       ___flsindex                100512f4     LIBCMT:tidtable.obj
 0003:000002f8       ___getvalueindex           100512f8     LIBCMT:tidtable.obj
 0003:00000300       __cfltcvt_tab              10051300     LIBCMT:cmiscdat.obj
 0003:00000330       ___nullstring              10051330     LIBCMT:output.obj
 0003:00000334       ___wnullstring             10051334     LIBCMT:output.obj
 0003:000004b0       __indefinite               100514b0     LIBCMT:_87disp_.obj
 0003:000004ba       __piby2                    100514ba     LIBCMT:_87disp_.obj
 0003:000004e0       ___initialmbcinfo          100514e0     LIBCMT:mbctype.obj
 0003:00000700       __mbctype                  10051700     LIBCMT:mbctype.obj
 0003:00000808       __mbcasemap                10051808     LIBCMT:mbctype.obj
 0003:00000908       ___ptmbcinfo               10051908     LIBCMT:mbctype.obj
 0003:00000a04       ___globallocalestatus      10051a04     LIBCMT:glstatus.obj
 0003:00000a08       ___clocalestr              10051a08     LIBCMT:nlsdata2.obj
 0003:00000a10       ___initiallocinfo          10051a10     LIBCMT:nlsdata2.obj
 0003:00000ae8       ___ptlocinfo               10051ae8     LIBCMT:nlsdata2.obj
 0003:00000aec       ___lc_clike                10051aec     LIBCMT:nlsdata2.obj
 0003:00000af0       ___initiallocalestructinfo 10051af0     LIBCMT:nlsdata2.obj
 0003:00000af8       __aexit_rtn                10051af8     LIBCMT:crt0dat.obj
 0003:00000b00       ___badioinfo               10051b00     LIBCMT:ioinit.obj
 0003:00000b40       __amblksiz                 10051b40     LIBCMT:heapinit.obj
 0003:00000b44       __First_FPE_Indx           10051b44     LIBCMT:winxfltr.obj
 0003:00000b48       __Num_FPE                  10051b48     LIBCMT:winxfltr.obj
 0003:00000b4c       __XcptActTabSize           10051b4c     LIBCMT:winxfltr.obj
 0003:00000b50       __XcptActTabCount          10051b50     LIBCMT:winxfltr.obj
 0003:00000d30       ___abort_behavior          10051d30     LIBCMT:abort.obj
 0003:00000d34       __NLG_Destination          10051d34     LIBCMT:exsup.obj
 0003:00000d50       __iob                      10051d50     LIBCMT:_file.obj
 0003:00000fd0       __pctype                   10051fd0     LIBCMT:ctype.obj
 0003:00000fd4       __pwctype                  10051fd4     LIBCMT:ctype.obj
 0003:00000fd8       ___lc_time_c               10051fd8     LIBCMT:strftime.obj
 0003:00001090       ___lc_time_curr            10052090     LIBCMT:strftime.obj
 0003:00001094       ___lconv_static_decimal    10052094     LIBCMT:lconv.obj
 0003:00001098       ___lconv_c                 10052098     LIBCMT:lconv.obj
 0003:000010c8       ___lconv                   100520c8     LIBCMT:lconv.obj
 0003:000010cc       ___mb_cur_max              100520cc     LIBCMT:nlsdata1.obj
 0003:000010d0       ___decimal_point           100520d0     LIBCMT:nlsdata1.obj
 0003:000010d4       ___decimal_point_length    100520d4     LIBCMT:nlsdata1.obj
 0003:00001208       __matherr_flag             10052208     LIBCMT:_matherr_.obj
 0003:00001230       __timezone                 10052230     LIBCMT:timeset.obj
 0003:00001234       __daylight                 10052234     LIBCMT:timeset.obj
 0003:00001238       __dstbias                  10052238     LIBCMT:timeset.obj
 0003:000012c0       __tzname                   100522c0     LIBCMT:timeset.obj
 0003:000012e0       __pow10pos                 100522e0     LIBCMT:_constpow_.obj
 0003:00001440       __pow10neg                 10052440     LIBCMT:_constpow_.obj
 0003:0000159c       __coninpfh                 1005259c     LIBCMT:initcon.obj
 0003:000015a0       __confh                    100525a0     LIBCMT:initcon.obj
 0003:000015a8       __d_inf                    100525a8     LIBCMT:_util_.obj
 0003:000015b0       __d_ind                    100525b0     LIBCMT:_util_.obj
 0003:000015b8       __d_max                    100525b8     LIBCMT:_util_.obj
 0003:000015c0       __d_min                    100525c0     LIBCMT:_util_.obj
 0003:000015c8       __d_mzero                  100525c8     LIBCMT:_util_.obj
 0003:000015d0       __lpdays                   100525d0     LIBCMT:days.obj
 0003:00001604       __days                     10052604     LIBCMT:days.obj
 0003:00001640       ??_R0?AV?$CWzSingleton@VWzLogSystem@WzLog@@@@@8 10052640     ProgramCommonLibForEngine_p:wzlogsystem.obj
 0003:00001674       ??_R0?AVWzLogSystem@WzLog@@@8 10052674     ProgramCommonLibForEngine_p:wzlogsystem.obj
 0003:00001698       ?g_lpszDiscType@@3PAPBDA   10052698     ProgramCommonLibForEngine_p:discaccess.obj
 0003:000016a4       ??_R0?AV?$CWzHandleManager@USt_DAFileInfo@@@@@8 100526a4     ProgramCommonLibForEngine_p:discaccess.obj
 0003:000016d8       ??_R0?AVWzLogHandler@WzLog@@@8 100526d8     ProgramCommonLibForEngine_p:WzFileLogHandler.obj
 0003:000016fc       ??_R0?AVWzFileLogHandler@WzLog@@@8 100526fc     ProgramCommonLibForEngine_p:WzFileLogHandler.obj
 0003:00001730       ?g_MatMulFunc@@3P6APAUWzMatrix@@PAU1@PBU1@1@ZA 10052730     Common_p:wzmath.obj
 0003:00001734       ?g_MatMul4x3Func@@3P6APAUWzMatrix@@PAU1@PBU1@1@ZA 10052734     Common_p:wzmath.obj
 0003:00001738       ?g_MatRotXFunc@@3P6APAUWzMatrix@@PAU1@M@ZA 10052738     Common_p:wzmath.obj
 0003:0000173c       ?g_MatRotYFunc@@3P6APAUWzMatrix@@PAU1@M@ZA 1005273c     Common_p:wzmath.obj
 0003:00001740       ?g_MatRotZFunc@@3P6APAUWzMatrix@@PAU1@M@ZA 10052740     Common_p:wzmath.obj
 0003:00001744       ?g_QuatMulFunc@@3P6APAUWzQuaternion@@PAU1@PBU1@1@ZA 10052744     Common_p:wzmath.obj
 0003:00001750       ?_PMPM@@3PAIA              10052750     Common_p:wzmath.obj
 0003:00001760       ?_PPMM@@3PAIA              10052760     Common_p:wzmath.obj
 0003:00001770       ?_MPPM@@3PAIA              10052770     Common_p:wzmath.obj
 0003:00001780       ?_PM@@3PAIA                10052780     Common_p:wzmath.obj
 0003:00001790       ?_MP@@3PAIA                10052790     Common_p:wzmath.obj
 0003:000017c4       _cchCurDir                 100527c4     wzFilePacker_static:vFile_util.obj
 0003:00001910       __lookuptrailbytes         10052910     LIBCMT:read.obj
 0003:00001a20       ?wvRot@?1??CreateEffect@CEffectManager@@QAEPAXKABUWzVector@@H@Z@4U3@A 10052a20     dllaccess.obj
 0003:00001a2c       ?wvRot@?1??CreateEffect@CEffectManager@@QAEPAXKABUWzVector@@0H@Z@4U3@A 10052a2c     dllaccess.obj
 0003:00001a38       ?s_instance@?$CWzSingleton@VWzLogSystem@WzLog@@@@0PAVWzLogSystem@WzLog@@A 10052a38     dllaccess.obj
 0003:00001a3c       ?s_instance@?$CWzSingleton@VCEffectManager@@@@0PAVCEffectManager@@A 10052a3c     effectmanager.obj
 0003:00001a4c       ?wvTest@?3??Outside_Frustum_AABB@@YAGPBUWzFrustum@@PBUBvAABB@@@Z@4UWzVector@@A 10052a4c     effectmanager.obj
 0003:00001a58       ?m_dummyData@?$CWzHandleManager@PAVCEffectBody@@@@1PAVCEffectBody@@A 10052a58     effectmanager.obj
 0003:00001a5c       ?m_nullData@?$CWzHandleManager@PAVCEffectBody@@@@1PAVCEffectBody@@A 10052a5c     effectmanager.obj
 0003:00001a60       ?m_dummyData@?$CWzArray@G@@0GA 10052a60     effectmanager.obj
 0003:00001a64       ?m_dummyData@?$CWzArray@PAVCEffectBody@@@@0PAVCEffectBody@@A 10052a64     effectmanager.obj
 0003:00001a68       ?g_effDbgInfo@@3USt_EffDbgInfo@@A 10052a68     effectmanager.obj
 0003:00001aa8       ?g_cSplineX@@3VWzNaturalCubicSpline@@A 10052aa8     eelementflatchain.obj
 0003:00001ca0       ?g_cSplineY@@3VWzNaturalCubicSpline@@A 10052ca0     eelementflatchain.obj
 0003:00001e98       ?g_cSplineZ@@3VWzNaturalCubicSpline@@A 10052e98     eelementflatchain.obj
 0003:00002090       ?g_cSpline2X@@3VWzNaturalCubicSpline@@A 10053090     eelementflatchain.obj
 0003:00002288       ?g_cSpline2Y@@3VWzNaturalCubicSpline@@A 10053288     eelementflatchain.obj
 0003:00002480       ?g_cSpline2Z@@3VWzNaturalCubicSpline@@A 10053480     eelementflatchain.obj
 0003:00002674       ?m_dummyData@?$CWzArray@PAUWzRenderInfo@@@@0PAUWzRenderInfo@@A 10053674     eelementmesh.obj
 0003:00002678       ?m_dummyData@?$CWzArray@PAVWzAnimationInfo@@@@0PAVWzAnimationInfo@@A 10053678     eelementmesh.obj
 0003:0000267c       ?m_dummyData@?$CWzArray@PAVCWzUnitSubType@@@@0PAVCWzUnitSubType@@A 1005367c     eelementmesh.obj
 0003:00002680       ?m_dummyData@?$CWzHashTable@PAUSt_WzUnitContainer@@K@@1PAUSt_WzUnitContainer@@A 10053680     eelementmesh.obj
 0003:00002720       ?fInWX@?1??QuaternionToMatrix@@YAPAUWzMatrix@@PAU2@PBUWzQuaternion@@@Z@4MA 10053720     eelementsprite.obj
 0003:00002724       ?fInWY@?1??QuaternionToMatrix@@YAPAUWzMatrix@@PAU2@PBUWzQuaternion@@@Z@4MA 10053724     eelementsprite.obj
 0003:00002728       ?fInWZ@?1??QuaternionToMatrix@@YAPAUWzMatrix@@PAU2@PBUWzQuaternion@@@Z@4MA 10053728     eelementsprite.obj
 0003:0000272c       ?fInYZ@?1??QuaternionToMatrix@@YAPAUWzMatrix@@PAU2@PBUWzQuaternion@@@Z@4MA 1005372c     eelementsprite.obj
 0003:00002730       ?fInXZ@?1??QuaternionToMatrix@@YAPAUWzMatrix@@PAU2@PBUWzQuaternion@@@Z@4MA 10053730     eelementsprite.obj
 0003:00002734       ?fInXY@?1??QuaternionToMatrix@@YAPAUWzMatrix@@PAU2@PBUWzQuaternion@@@Z@4MA 10053734     eelementsprite.obj
 0003:00002738       ?fInZZ@?1??QuaternionToMatrix@@YAPAUWzMatrix@@PAU2@PBUWzQuaternion@@@Z@4MA 10053738     eelementsprite.obj
 0003:0000273c       ?fInYY@?1??QuaternionToMatrix@@YAPAUWzMatrix@@PAU2@PBUWzQuaternion@@@Z@4MA 1005373c     eelementsprite.obj
 0003:00002740       ?fInXX@?1??QuaternionToMatrix@@YAPAUWzMatrix@@PAU2@PBUWzQuaternion@@@Z@4MA 10053740     eelementsprite.obj
 0003:00002744       ?m_dummyData@?$CWzHandleManager@PAUSt_TextureContainer@@@@1PAUSt_TextureContainer@@A 10053744     eelementsprite.obj
 0003:00002748       ?m_dummyData@?$CWzArray@PAUSt_TextureContainer@@@@0PAUSt_TextureContainer@@A 10053748     eelementsprite.obj
 0003:00002788       ?cb@?1??GetCube@CDivideCube@@QAEXKPAUSt_Cube@@@Z@4U3@A 10053788     eelementweather.obj
 0003:00002824       ___fastflag                10053824     LIBCMT:_fpinit_.obj
 0003:00002828       __adjust_fdiv              10053828     LIBCMT:_fpinit_.obj
 0003:0000282c       ___pInvalidArgHandler      1005382c     LIBCMT:invarg.obj
 0003:00002834       __aenvptr                  10053834     LIBCMT:dllcrt0.obj
 0003:00002838       __wenvptr                  10053838     LIBCMT:dllcrt0.obj
 0003:0000283c       ___error_mode              1005383c     LIBCMT:dllcrt0.obj
 0003:00002840       ___app_type                10053840     LIBCMT:dllcrt0.obj
 0003:00002844       ?_pnhHeap@@3P6AHI@ZA       10053844     LIBCMT:handler.obj
 0003:00002848       _gpFlsAlloc                10053848     LIBCMT:tidtable.obj
 0003:0000284c       _gpFlsGetValue             1005384c     LIBCMT:tidtable.obj
 0003:00002850       _gpFlsSetValue             10053850     LIBCMT:tidtable.obj
 0003:00002854       _gpFlsFree                 10053854     LIBCMT:tidtable.obj
 0003:00002858       ?__pInconsistency@@3P6AXXZA 10053858     LIBCMT:hooks.obj
 0003:00002b90       ___mbulinfo                10053b90     LIBCMT:mbctype.obj
 0003:00002b9c       ___mbcodepage              10053b9c     LIBCMT:mbctype.obj
 0003:00002ba0       ___ismbcodepage            10053ba0     LIBCMT:mbctype.obj
 0003:00002ba4       ___mblcid                  10053ba4     LIBCMT:mbctype.obj
 0003:00002ba8       ___locale_changed          10053ba8     LIBCMT:setlocal.obj
 0003:00002bac       ___lc_handle               10053bac     LIBCMT:nlsdata2.obj
 0003:00002bc4       ___lc_codepage             10053bc4     LIBCMT:nlsdata2.obj
 0003:00002bc8       ___lc_collate_cp           10053bc8     LIBCMT:nlsdata2.obj
 0003:00002bcc       __maxwait                  10053bcc     LIBCMT:crtheap.obj
 0003:00002bd0       __umaskval                 10053bd0     LIBCMT:crt0dat.obj
 0003:00002bd4       ___argc                    10053bd4     LIBCMT:crt0dat.obj
 0003:00002bd8       ___argv                    10053bd8     LIBCMT:crt0dat.obj
 0003:00002bdc       ___wargv                   10053bdc     LIBCMT:crt0dat.obj
 0003:00002be0       __environ                  10053be0     LIBCMT:crt0dat.obj
 0003:00002be4       ___initenv                 10053be4     LIBCMT:crt0dat.obj
 0003:00002be8       __wenviron                 10053be8     LIBCMT:crt0dat.obj
 0003:00002bec       ___winitenv                10053bec     LIBCMT:crt0dat.obj
 0003:00002bf0       __pgmptr                   10053bf0     LIBCMT:crt0dat.obj
 0003:00002bf4       __wpgmptr                  10053bf4     LIBCMT:crt0dat.obj
 0003:00002bf8       __exitflag                 10053bf8     LIBCMT:crt0dat.obj
 0003:00002bfc       __C_Termination_Done       10053bfc     LIBCMT:crt0dat.obj
 0003:00002c00       __C_Exit_Done              10053c00     LIBCMT:crt0dat.obj
 0003:00002d14       __crtheap                  10053d14     LIBCMT:heapinit.obj
 0003:00002e68       ___sbh_pHeaderDefer        10053e68     LIBCMT:sbheap.obj
 0003:00003184       __newmode                  10054184     LIBCMT:_newmode.obj
 0003:00003188       __outputformat             10054188     LIBCMT:outputformat.obj
 0003:000031a0       ?pArgList@UnDecorator@@0PAVReplicator@@A 100541a0     LIBCMT:undname.obj
 0003:000031a4       ?pZNameList@UnDecorator@@0PAVReplicator@@A 100541a4     LIBCMT:undname.obj
 0003:000031a8       ?pTemplateArgList@UnDecorator@@0PAVReplicator@@A 100541a8     LIBCMT:undname.obj
 0003:000031ac       ?gName@UnDecorator@@0PBDB  100541ac     LIBCMT:undname.obj
 0003:000031b0       ?name@UnDecorator@@0PBDB   100541b0     LIBCMT:undname.obj
 0003:000031b4       ?outputString@UnDecorator@@0PADA 100541b4     LIBCMT:undname.obj
 0003:000031b8       ?maxStringLength@UnDecorator@@0HA 100541b8     LIBCMT:undname.obj
 0003:000031bc       ?disableFlags@UnDecorator@@0KA 100541bc     LIBCMT:undname.obj
 0003:000031c0       ?m_pGetParameter@UnDecorator@@0P6APADJ@ZA 100541c0     LIBCMT:undname.obj
 0003:000031c4       ?fExplicitTemplateParams@UnDecorator@@0_NA 100541c4     LIBCMT:undname.obj
 0003:000031c5       ?fGetTemplateArgumentList@UnDecorator@@0_NA 100541c5     LIBCMT:undname.obj
 0003:000031c8       __cflush                   100541c8     LIBCMT:_file.obj
 0003:000031d8       ___lconv_static_null       100541d8     LIBCMT:lconv.obj
 0003:000031fc       ___pPurecall               100541fc     LIBCMT:inithelp.obj
 0003:00003218       __stdbuf                   10054218     LIBCMT:_sftbuf.obj
 0003:000038ec       ?m_dummyData@?$CWzHandleManager@USt_DAFileInfo@@@@1USt_DAFileInfo@@A 100548ec     ProgramCommonLibForEngine_p:discaccess.obj
 0003:000038f4       ?m_nullData@?$CWzHandleManager@USt_DAFileInfo@@@@1USt_DAFileInfo@@A 100548f4     ProgramCommonLibForEngine_p:discaccess.obj
 0003:000038fc       ?m_dummyData@?$CWzArray@USt_DAFileInfo@@@@0USt_DAFileInfo@@A 100548fc     ProgramCommonLibForEngine_p:discaccess.obj
 0003:00003d50       ?autofree@@3VCAutoFree@@A  10054d50     wzFilePacker_static:wzFilePacker.obj
 0003:00003d60       _dwTreeCount               10054d60     wzFilePacker_static:vfile.obj
 0003:00003d64       _g_nTreeArrayCount         10054d64     wzFilePacker_static:vfile.obj
 0003:00003d68       _g_ulStartBinaryOffset     10054d68     wzFilePacker_static:vfile.obj
 0003:00003d70       _g_ulTatalBinarySize       10054d70     wzFilePacker_static:vfile.obj
 0003:00003d7c       _bCurDirCreated            10054d7c     wzFilePacker_static:vFile_util.obj
 0003:0000468c       __commode                  1005568c     LIBCMT:ncommode.obj
 0003:00004690       __fmode                    10055690     LIBCMT:txtmode.obj
 0003:00004694       __pmatherr                 10055694     <common>
 0003:00004698       ___piob                    10055698     <common>
 0003:000046a0       __bufin                    100556a0     <common>
 0003:000056a0       __nstream                  100566a0     <common>
 0003:000056a4       ___sbh_cntHeaderList       100566a4     <common>
 0003:000056a8       ___sbh_pHeaderList         100566a8     <common>
 0003:000056ac       ___sbh_threshold           100566ac     <common>
 0003:000056b0       ___sbh_pHeaderScan         100566b0     <common>
 0003:000056b4       ___sbh_sizeHeaderList      100566b4     <common>
 0003:000056b8       ___sbh_indGroupDefer       100566b8     <common>
 0003:000056bc       ___active_heap             100566bc     <common>
 0003:000056c0       __nhandle                  100566c0     <common>
 0003:000056e0       ___pioinfo                 100566e0     <common>
 0003:000057e0       ___use_sse2_mathfcns       100567e0     <common>
 0003:000057e4       ___env_initialized         100567e4     <common>
 0003:000057e8       ___onexitend               100567e8     <common>
 0003:000057ec       ___onexitbegin             100567ec     <common>
 0003:000057f0       ___mbctype_initialized     100567f0     <common>
 0003:000057f4       ___dyn_tls_init_callback   100567f4     <common>
 0003:000057f8       __debugger_hook_dummy      100567f8     <common>
 0003:000057fc       ___sse2_available          100567fc     <common>
 0003:00005800       __acmdln                   10056800     <common>
 0003:00005804       _StupidUnusedPointer       10056804     <common>
 0003:00005820       _g_TreeList                10056820     <common>

 entry point at        0001:00027474

 Static symbols

 0001:00002e16       ??$AllocNew@UsEffectTexture@CEffectManager@@@CMemoryPool@@YAPAUsEffectTexture@CEffectManager@@XZ 10003e16 f   effectmanager.obj
 0001:00002e91       ??$AllocDelete@UsEffectTexture@CEffectManager@@@CMemoryPool@@YAXPAUsEffectTexture@CEffectManager@@@Z 10003e91 f   effectmanager.obj
 0001:00002ed7       ??$AllocNew@USt_BodyCreate@@@CMemoryPool@@YAPAUSt_BodyCreate@@XZ 10003ed7 f   effectmanager.obj
 0001:00002f3f       ??$AllocDelete@USt_BodyCreate@@@CMemoryPool@@YAXPAUSt_BodyCreate@@@Z 10003f3f f   effectmanager.obj
 0001:0000971f       __catch$?_Copy@?$basic_string@DU?$char_traits@D@std@@V?$allocator@D@2@@std@@IAEXII@Z$0 1000a71f f i effectmanager.obj
 0001:0000974b       __catch$?_Copy@?$basic_string@DU?$char_traits@D@std@@V?$allocator@D@2@@std@@IAEXII@Z$1 1000a74b f i effectmanager.obj
 0001:00009de0       __catch$?_Buynode@?$list@KV?$allocator@K@std@@@std@@IAEPAU_Node@?$_List_nod@KV?$allocator@K@std@@@2@XZ$0 1000ade0 f i effectmanager.obj
 0001:00009de0       __catch$?_Buynode@?$list@PAVCEElementSprite@@V?$allocator@PAVCEElementSprite@@@std@@@std@@IAEPAU_Node@?$_List_nod@PAVCEElementSprite@@V?$allocator@PAVCEElementSprite@@@std@@@2@XZ$0 1000ade0 f i effectmanager.obj
 0001:00009de0       __catch$?_Buynode@?$list@PAVCEElementBase@@V?$allocator@PAVCEElementBase@@@std@@@std@@IAEPAU_Node@?$_List_nod@PAVCEElementBase@@V?$allocator@PAVCEElementBase@@@std@@@2@XZ$0 1000ade0 f i effectmanager.obj
 0001:0000b8eb       __catch$?_Copy@?$_Tree@V?$_Tmap_traits@JUWzVector@@U?$less@J@std@@V?$allocator@U?$pair@$$CBJUWzVector@@@std@@@3@$0A@@std@@@std@@IAEPAU_Node@?$_Tree_nod@V?$_Tmap_traits@JUWzVector@@U?$less@J@std@@V?$allocator@U?$pair@$$CBJUWzVector@@@std@@@3@$0A@@std@@@2@PAU342@0@Z$0 1000c8eb f i effectmanager.obj
 0001:0000bb02       __catch$?_Copy@?$_Tree@V?$_Tmap_traits@JMU?$less@J@std@@V?$allocator@U?$pair@$$CBJM@std@@@2@$0A@@std@@@std@@IAEPAU_Node@?$_Tree_nod@V?$_Tmap_traits@JMU?$less@J@std@@V?$allocator@U?$pair@$$CBJM@std@@@2@$0A@@std@@@2@PAU342@0@Z$0 1000cb02 f i effectmanager.obj
 0001:0000c7bd       __catch$?_Buynode@?$_Tree@V?$_Tmap_traits@JUWzVector@@U?$less@J@std@@V?$allocator@U?$pair@$$CBJUWzVector@@@std@@@3@$0A@@std@@@std@@IAEPAU_Node@?$_Tree_nod@V?$_Tmap_traits@JUWzVector@@U?$less@J@std@@V?$allocator@U?$pair@$$CBJUWzVector@@@std@@@3@$0A@@std@@@2@XZ$0 1000d7bd f i effectmanager.obj
 0001:0000c896       __catch$?_Buynode@?$_Tree@V?$_Tmap_traits@JUWzVector@@U?$less@J@std@@V?$allocator@U?$pair@$$CBJUWzVector@@@std@@@3@$0A@@std@@@std@@IAEPAU_Node@?$_Tree_nod@V?$_Tmap_traits@JUWzVector@@U?$less@J@std@@V?$allocator@U?$pair@$$CBJUWzVector@@@std@@@3@$0A@@std@@@2@PAU342@00ABU?$pair@$$CBJUWzVector@@@2@D@Z$0 1000d896 f i effectmanager.obj
 0001:0000c9a4       __catch$?_Buynode@?$_Tree@V?$_Tmap_traits@JMU?$less@J@std@@V?$allocator@U?$pair@$$CBJM@std@@@2@$0A@@std@@@std@@IAEPAU_Node@?$_Tree_nod@V?$_Tmap_traits@JMU?$less@J@std@@V?$allocator@U?$pair@$$CBJM@std@@@2@$0A@@std@@@2@XZ$0 1000d9a4 f i effectmanager.obj
 0001:0000ca81       __catch$?_Buynode@?$_Tree@V?$_Tmap_traits@JMU?$less@J@std@@V?$allocator@U?$pair@$$CBJM@std@@@2@$0A@@std@@@std@@IAEPAU_Node@?$_Tree_nod@V?$_Tmap_traits@JMU?$less@J@std@@V?$allocator@U?$pair@$$CBJM@std@@@2@$0A@@std@@@2@PAU342@00ABU?$pair@$$CBJM@2@D@Z$0 1000da81 f i effectmanager.obj
 0001:0000ce2c       __catch$?_Buynode@?$list@U?$pair@$$CBKPAUSt_BodyCreate@@@std@@V?$allocator@U?$pair@$$CBKPAUSt_BodyCreate@@@std@@@2@@std@@IAEPAU_Node@?$_List_nod@U?$pair@$$CBKPAUSt_BodyCreate@@@std@@V?$allocator@U?$pair@$$CBKPAUSt_BodyCreate@@@std@@@2@@2@XZ$0 1000de2c f i effectmanager.obj
 0001:0000ce2c       __catch$?_Buynode@?$list@U?$pair@QAXPAVCEffectBody@@@std@@V?$allocator@U?$pair@QAXPAVCEffectBody@@@std@@@2@@std@@IAEPAU_Node@?$_List_nod@U?$pair@QAXPAVCEffectBody@@@std@@V?$allocator@U?$pair@QAXPAVCEffectBody@@@std@@@2@@2@XZ$0 1000de2c f i effectmanager.obj
 0001:0000d308       __catch$?_Buynode@?$list@U?$pair@$$CBKPAUSt_BodyCreate@@@std@@V?$allocator@U?$pair@$$CBKPAUSt_BodyCreate@@@std@@@2@@std@@IAEPAU_Node@?$_List_nod@U?$pair@$$CBKPAUSt_BodyCreate@@@std@@V?$allocator@U?$pair@$$CBKPAUSt_BodyCreate@@@std@@@2@@2@PAU342@0ABU?$pair@$$CBKPAUSt_BodyCreate@@@2@@Z$0 1000e308 f i effectmanager.obj
 0001:0000d308       __catch$?_Buynode@?$list@U?$pair@QAXPAVCEffectBody@@@std@@V?$allocator@U?$pair@QAXPAVCEffectBody@@@std@@@2@@std@@IAEPAU_Node@?$_List_nod@U?$pair@QAXPAVCEffectBody@@@std@@V?$allocator@U?$pair@QAXPAVCEffectBody@@@std@@@2@@2@PAU342@0ABU?$pair@QAXPAVCEffectBody@@@2@@Z$0 1000e308 f i effectmanager.obj
 0001:0000d6a5       __catch$?_Insert_n@?$vector@U_List_position@?$_Hash@V?$_Hmap_traits@KV?$basic_string@DU?$char_traits@D@std@@V?$allocator@D@2@@std@@V?$hash_compare@KU?$less@K@std@@@stdext@@V?$allocator@U?$pair@$$CBKV?$basic_string@DU?$char_traits@D@std@@V?$allocator@D@2@@std@@@std@@@2@$0A@@stdext@@@stdext@@V?$allocator@U_List_position@?$_Hash@V?$_Hmap_traits@KV?$basic_string@DU?$char_traits@D@std@@V?$allocator@D@2@@std@@V?$hash_compare@KU?$less@K@std@@@stdext@@V?$allocator@U?$pair@$$CBKV?$basic_string@DU?$char_traits@D@std@@V?$allocator@D@2@@std@@@std@@@2@$0A@@stdext@@@stdext@@@std@@@std@@IAEXV?$_Vector_const_iterator@U_List_position@?$_Hash@V?$_Hmap_traits@KV?$basic_string@DU?$char_traits@D@std@@V?$allocator@D@2@@std@@V?$hash_compare@KU?$less@K@std@@@stdext@@V?$allocator@U?$pair@$$CBKV?$basic_string@DU?$char_traits@D@std@@V?$allocator@D@2@@std@@@std@@@2@$0A@@stdext@@@stdext@@V?$allocator@U_List_position@?$_Hash@V?$_Hmap_traits@KV?$basic_string@DU?$char_traits@D@std@@V?$allocator@D@2@@std@@V?$hash_compare@KU?$less@K@std@@@stdext@@V?$allocator@U?$pair@$$CBKV?$basic_string@DU?$char_traits@D@std@@V?$allocator@D@2@@std@@@std@@@2@$0A@@stdext@@@stdext@@@std@@@2@IABU_List_position@?$_Hash@V?$_Hmap_traits@KV?$basic_string@DU?$char_traits@D@std@@V?$allocator@D@2@@std@@V?$hash_compare@KU?$less@K@std@@@stdext@@V?$allocator@U?$pair@$$CBKV?$basic_string@DU?$char_traits@D@std@@V?$allocator@D@2@@std@@@std@@@2@$0A@@stdext@@@stdext@@@Z$0 1000e6a5 f i effectmanager.obj
 0001:0000d6a5       __catch$?_Insert_n@?$vector@U_List_position@?$_Hash@V?$_Hmap_traits@PAXPAVCEffectBody@@V?$hash_compare@PAXU?$less@PAX@std@@@stdext@@V?$allocator@U?$pair@QAXPAVCEffectBody@@@std@@@std@@$0A@@stdext@@@stdext@@V?$allocator@U_List_position@?$_Hash@V?$_Hmap_traits@PAXPAVCEffectBody@@V?$hash_compare@PAXU?$less@PAX@std@@@stdext@@V?$allocator@U?$pair@QAXPAVCEffectBody@@@std@@@std@@$0A@@stdext@@@stdext@@@std@@@std@@IAEXV?$_Vector_const_iterator@U_List_position@?$_Hash@V?$_Hmap_traits@PAXPAVCEffectBody@@V?$hash_compare@PAXU?$less@PAX@std@@@stdext@@V?$allocator@U?$pair@QAXPAVCEffectBody@@@std@@@std@@$0A@@stdext@@@stdext@@V?$allocator@U_List_position@?$_Hash@V?$_Hmap_traits@PAXPAVCEffectBody@@V?$hash_compare@PAXU?$less@PAX@std@@@stdext@@V?$allocator@U?$pair@QAXPAVCEffectBody@@@std@@@std@@$0A@@stdext@@@stdext@@@std@@@2@IABU_List_position@?$_Hash@V?$_Hmap_traits@PAXPAVCEffectBody@@V?$hash_compare@PAXU?$less@PAX@std@@@stdext@@V?$allocator@U?$pair@QAXPAVCEffectBody@@@std@@@std@@$0A@@stdext@@@stdext@@@Z$0 1000e6a5 f i effectmanager.obj
 0001:0000d6a5       __catch$?_Insert_n@?$vector@USt_AutoCtlParam@@V?$allocator@USt_AutoCtlParam@@@std@@@std@@IAEXV?$_Vector_const_iterator@USt_AutoCtlParam@@V?$allocator@USt_AutoCtlParam@@@std@@@2@IABUSt_AutoCtlParam@@@Z$0 1000e6a5 f i effectmanager.obj
 0001:0000d6a5       __catch$?_Insert_n@?$vector@USt_EffLODParam@@V?$allocator@USt_EffLODParam@@@std@@@std@@IAEXV?$_Vector_const_iterator@USt_EffLODParam@@V?$allocator@USt_EffLODParam@@@std@@@2@IABUSt_EffLODParam@@@Z$0 1000e6a5 f i effectmanager.obj
 0001:0000d6a5       __catch$?_Insert_n@?$vector@U_WZNCSPT@WzNaturalCubicSplineDyn@@V?$allocator@U_WZNCSPT@WzNaturalCubicSplineDyn@@@std@@@std@@IAEXV?$_Vector_const_iterator@U_WZNCSPT@WzNaturalCubicSplineDyn@@V?$allocator@U_WZNCSPT@WzNaturalCubicSplineDyn@@@std@@@2@IABU_WZNCSPT@WzNaturalCubicSplineDyn@@@Z$0 1000e6a5 f i effectmanager.obj
 0001:0000d6a5       __catch$?_Insert_n@?$vector@U_List_position@?$_Hash@V?$_Hmap_traits@KPAUSt_BodyCreate@@V?$hash_compare@KU?$less@K@std@@@stdext@@V?$allocator@U?$pair@$$CBKPAUSt_BodyCreate@@@std@@@std@@$0A@@stdext@@@stdext@@V?$allocator@U_List_position@?$_Hash@V?$_Hmap_traits@KPAUSt_BodyCreate@@V?$hash_compare@KU?$less@K@std@@@stdext@@V?$allocator@U?$pair@$$CBKPAUSt_BodyCreate@@@std@@@std@@$0A@@stdext@@@stdext@@@std@@@std@@IAEXV?$_Vector_const_iterator@U_List_position@?$_Hash@V?$_Hmap_traits@KPAUSt_BodyCreate@@V?$hash_compare@KU?$less@K@std@@@stdext@@V?$allocator@U?$pair@$$CBKPAUSt_BodyCreate@@@std@@@std@@$0A@@stdext@@@stdext@@V?$allocator@U_List_position@?$_Hash@V?$_Hmap_traits@KPAUSt_BodyCreate@@V?$hash_compare@KU?$less@K@std@@@stdext@@V?$allocator@U?$pair@$$CBKPAUSt_BodyCreate@@@std@@@std@@$0A@@stdext@@@stdext@@@std@@@2@IABU_List_position@?$_Hash@V?$_Hmap_traits@KPAUSt_BodyCreate@@V?$hash_compare@KU?$less@K@std@@@stdext@@V?$allocator@U?$pair@$$CBKPAUSt_BodyCreate@@@std@@@std@@$0A@@stdext@@@stdext@@@Z$0 1000e6a5 f i effectmanager.obj
 0001:0000d95f       __catch$?_Insert_n@?$vector@U_List_position@?$_Hash@V?$_Hmap_traits@KV?$basic_string@DU?$char_traits@D@std@@V?$allocator@D@2@@std@@V?$hash_compare@KU?$less@K@std@@@stdext@@V?$allocator@U?$pair@$$CBKV?$basic_string@DU?$char_traits@D@std@@V?$allocator@D@2@@std@@@std@@@2@$0A@@stdext@@@stdext@@V?$allocator@U_List_position@?$_Hash@V?$_Hmap_traits@KV?$basic_string@DU?$char_traits@D@std@@V?$allocator@D@2@@std@@V?$hash_compare@KU?$less@K@std@@@stdext@@V?$allocator@U?$pair@$$CBKV?$basic_string@DU?$char_traits@D@std@@V?$allocator@D@2@@std@@@std@@@2@$0A@@stdext@@@stdext@@@std@@@std@@IAEXV?$_Vector_const_iterator@U_List_position@?$_Hash@V?$_Hmap_traits@KV?$basic_string@DU?$char_traits@D@std@@V?$allocator@D@2@@std@@V?$hash_compare@KU?$less@K@std@@@stdext@@V?$allocator@U?$pair@$$CBKV?$basic_string@DU?$char_traits@D@std@@V?$allocator@D@2@@std@@@std@@@2@$0A@@stdext@@@stdext@@V?$allocator@U_List_position@?$_Hash@V?$_Hmap_traits@KV?$basic_string@DU?$char_traits@D@std@@V?$allocator@D@2@@std@@V?$hash_compare@KU?$less@K@std@@@stdext@@V?$allocator@U?$pair@$$CBKV?$basic_string@DU?$char_traits@D@std@@V?$allocator@D@2@@std@@@std@@@2@$0A@@stdext@@@stdext@@@std@@@2@IABU_List_position@?$_Hash@V?$_Hmap_traits@KV?$basic_string@DU?$char_traits@D@std@@V?$allocator@D@2@@std@@V?$hash_compare@KU?$less@K@std@@@stdext@@V?$allocator@U?$pair@$$CBKV?$basic_string@DU?$char_traits@D@std@@V?$allocator@D@2@@std@@@std@@@2@$0A@@stdext@@@stdext@@@Z$2 1000e95f f i effectmanager.obj
 0001:0000d95f       __catch$?_Insert_n@?$vector@USt_AutoCtlParam@@V?$allocator@USt_AutoCtlParam@@@std@@@std@@IAEXV?$_Vector_const_iterator@USt_AutoCtlParam@@V?$allocator@USt_AutoCtlParam@@@std@@@2@IABUSt_AutoCtlParam@@@Z$2 1000e95f f i effectmanager.obj
 0001:0000d95f       __catch$?_Insert_n@?$vector@U_List_position@?$_Hash@V?$_Hmap_traits@PAXPAVCEffectBody@@V?$hash_compare@PAXU?$less@PAX@std@@@stdext@@V?$allocator@U?$pair@QAXPAVCEffectBody@@@std@@@std@@$0A@@stdext@@@stdext@@V?$allocator@U_List_position@?$_Hash@V?$_Hmap_traits@PAXPAVCEffectBody@@V?$hash_compare@PAXU?$less@PAX@std@@@stdext@@V?$allocator@U?$pair@QAXPAVCEffectBody@@@std@@@std@@$0A@@stdext@@@stdext@@@std@@@std@@IAEXV?$_Vector_const_iterator@U_List_position@?$_Hash@V?$_Hmap_traits@PAXPAVCEffectBody@@V?$hash_compare@PAXU?$less@PAX@std@@@stdext@@V?$allocator@U?$pair@QAXPAVCEffectBody@@@std@@@std@@$0A@@stdext@@@stdext@@V?$allocator@U_List_position@?$_Hash@V?$_Hmap_traits@PAXPAVCEffectBody@@V?$hash_compare@PAXU?$less@PAX@std@@@stdext@@V?$allocator@U?$pair@QAXPAVCEffectBody@@@std@@@std@@$0A@@stdext@@@stdext@@@std@@@2@IABU_List_position@?$_Hash@V?$_Hmap_traits@PAXPAVCEffectBody@@V?$hash_compare@PAXU?$less@PAX@std@@@stdext@@V?$allocator@U?$pair@QAXPAVCEffectBody@@@std@@@std@@$0A@@stdext@@@stdext@@@Z$2 1000e95f f i effectmanager.obj
 0001:0000d95f       __catch$?_Insert_n@?$vector@USt_EffLODParam@@V?$allocator@USt_EffLODParam@@@std@@@std@@IAEXV?$_Vector_const_iterator@USt_EffLODParam@@V?$allocator@USt_EffLODParam@@@std@@@2@IABUSt_EffLODParam@@@Z$2 1000e95f f i effectmanager.obj
 0001:0000d95f       __catch$?_Insert_n@?$vector@U_WZNCSPT@WzNaturalCubicSplineDyn@@V?$allocator@U_WZNCSPT@WzNaturalCubicSplineDyn@@@std@@@std@@IAEXV?$_Vector_const_iterator@U_WZNCSPT@WzNaturalCubicSplineDyn@@V?$allocator@U_WZNCSPT@WzNaturalCubicSplineDyn@@@std@@@2@IABU_WZNCSPT@WzNaturalCubicSplineDyn@@@Z$2 1000e95f f i effectmanager.obj
 0001:0000d95f       __catch$?_Insert_n@?$vector@U_List_position@?$_Hash@V?$_Hmap_traits@KPAUSt_BodyCreate@@V?$hash_compare@KU?$less@K@std@@@stdext@@V?$allocator@U?$pair@$$CBKPAUSt_BodyCreate@@@std@@@std@@$0A@@stdext@@@stdext@@V?$allocator@U_List_position@?$_Hash@V?$_Hmap_traits@KPAUSt_BodyCreate@@V?$hash_compare@KU?$less@K@std@@@stdext@@V?$allocator@U?$pair@$$CBKPAUSt_BodyCreate@@@std@@@std@@$0A@@stdext@@@stdext@@@std@@@std@@IAEXV?$_Vector_const_iterator@U_List_position@?$_Hash@V?$_Hmap_traits@KPAUSt_BodyCreate@@V?$hash_compare@KU?$less@K@std@@@stdext@@V?$allocator@U?$pair@$$CBKPAUSt_BodyCreate@@@std@@@std@@$0A@@stdext@@@stdext@@V?$allocator@U_List_position@?$_Hash@V?$_Hmap_traits@KPAUSt_BodyCreate@@V?$hash_compare@KU?$less@K@std@@@stdext@@V?$allocator@U?$pair@$$CBKPAUSt_BodyCreate@@@std@@@std@@$0A@@stdext@@@stdext@@@std@@@2@IABU_List_position@?$_Hash@V?$_Hmap_traits@KPAUSt_BodyCreate@@V?$hash_compare@KU?$less@K@std@@@stdext@@V?$allocator@U?$pair@$$CBKPAUSt_BodyCreate@@@std@@@std@@$0A@@stdext@@@stdext@@@Z$2 1000e95f f i effectmanager.obj
 0001:0000e820       __catch$??$_Uninit_fill_n@PAU_WZNCSPT@WzNaturalCubicSplineDyn@@IU12@V?$allocator@U_WZNCSPT@WzNaturalCubicSplineDyn@@@std@@@std@@YAXPAU_WZNCSPT@WzNaturalCubicSplineDyn@@IABU12@AAV?$allocator@U_WZNCSPT@WzNaturalCubicSplineDyn@@@0@U_Nonscalar_ptr_iterator_tag@0@U_Range_checked_iterator_tag@0@@Z$0 1000f820 f i effectmanager.obj
 0001:0000e820       __catch$??$_Uninit_fill_n@PAU_List_position@?$_Hash@V?$_Hmap_traits@KV?$basic_string@DU?$char_traits@D@std@@V?$allocator@D@2@@std@@V?$hash_compare@KU?$less@K@std@@@stdext@@V?$allocator@U?$pair@$$CBKV?$basic_string@DU?$char_traits@D@std@@V?$allocator@D@2@@std@@@std@@@2@$0A@@stdext@@@stdext@@IU123@V?$allocator@U_List_position@?$_Hash@V?$_Hmap_traits@KV?$basic_string@DU?$char_traits@D@std@@V?$allocator@D@2@@std@@V?$hash_compare@KU?$less@K@std@@@stdext@@V?$allocator@U?$pair@$$CBKV?$basic_string@DU?$char_traits@D@std@@V?$allocator@D@2@@std@@@std@@@2@$0A@@stdext@@@stdext@@@std@@@std@@YAXPAU_List_position@?$_Hash@V?$_Hmap_traits@KV?$basic_string@DU?$char_traits@D@std@@V?$allocator@D@2@@std@@V?$hash_compare@KU?$less@K@std@@@stdext@@V?$allocator@U?$pair@$$CBKV?$basic_string@DU?$char_traits@D@std@@V?$allocator@D@2@@std@@@std@@@2@$0A@@stdext@@@stdext@@IABU123@AAV?$allocator@U_List_position@?$_Hash@V?$_Hmap_traits@KV?$basic_string@DU?$char_traits@D@std@@V?$allocator@D@2@@std@@V?$hash_compare@KU?$less@K@std@@@stdext@@V?$allocator@U?$pair@$$CBKV?$basic_string@DU?$char_traits@D@std@@V?$allocator@D@2@@std@@@std@@@2@$0A@@stdext@@@stdext@@@0@U_Nonscalar_ptr_iterator_tag@0@U_Range_checked_iterator_tag@0@@Z$0 1000f820 f i effectmanager.obj
 0001:0000e820       __catch$??$_Uninit_fill_n@PAU_List_position@?$_Hash@V?$_Hmap_traits@KPAUSt_BodyCreate@@V?$hash_compare@KU?$less@K@std@@@stdext@@V?$allocator@U?$pair@$$CBKPAUSt_BodyCreate@@@std@@@std@@$0A@@stdext@@@stdext@@IU123@V?$allocator@U_List_position@?$_Hash@V?$_Hmap_traits@KPAUSt_BodyCreate@@V?$hash_compare@KU?$less@K@std@@@stdext@@V?$allocator@U?$pair@$$CBKPAUSt_BodyCreate@@@std@@@std@@$0A@@stdext@@@stdext@@@std@@@std@@YAXPAU_List_position@?$_Hash@V?$_Hmap_traits@KPAUSt_BodyCreate@@V?$hash_compare@KU?$less@K@std@@@stdext@@V?$allocator@U?$pair@$$CBKPAUSt_BodyCreate@@@std@@@std@@$0A@@stdext@@@stdext@@IABU123@AAV?$allocator@U_List_position@?$_Hash@V?$_Hmap_traits@KPAUSt_BodyCreate@@V?$hash_compare@KU?$less@K@std@@@stdext@@V?$allocator@U?$pair@$$CBKPAUSt_BodyCreate@@@std@@@std@@$0A@@stdext@@@stdext@@@0@U_Nonscalar_ptr_iterator_tag@0@U_Range_checked_iterator_tag@0@@Z$0 1000f820 f i effectmanager.obj
 0001:0000e820       __catch$??$_Uninit_fill_n@PAUSt_AutoCtlParam@@IU1@V?$allocator@USt_AutoCtlParam@@@std@@@std@@YAXPAUSt_AutoCtlParam@@IABU1@AAV?$allocator@USt_AutoCtlParam@@@0@U_Nonscalar_ptr_iterator_tag@0@U_Range_checked_iterator_tag@0@@Z$0 1000f820 f i effectmanager.obj
 0001:0000e820       __catch$??$_Uninit_fill_n@PAU_List_position@?$_Hash@V?$_Hmap_traits@PAXPAVCEffectBody@@V?$hash_compare@PAXU?$less@PAX@std@@@stdext@@V?$allocator@U?$pair@QAXPAVCEffectBody@@@std@@@std@@$0A@@stdext@@@stdext@@IU123@V?$allocator@U_List_position@?$_Hash@V?$_Hmap_traits@PAXPAVCEffectBody@@V?$hash_compare@PAXU?$less@PAX@std@@@stdext@@V?$allocator@U?$pair@QAXPAVCEffectBody@@@std@@@std@@$0A@@stdext@@@stdext@@@std@@@std@@YAXPAU_List_position@?$_Hash@V?$_Hmap_traits@PAXPAVCEffectBody@@V?$hash_compare@PAXU?$less@PAX@std@@@stdext@@V?$allocator@U?$pair@QAXPAVCEffectBody@@@std@@@std@@$0A@@stdext@@@stdext@@IABU123@AAV?$allocator@U_List_position@?$_Hash@V?$_Hmap_traits@PAXPAVCEffectBody@@V?$hash_compare@PAXU?$less@PAX@std@@@stdext@@V?$allocator@U?$pair@QAXPAVCEffectBody@@@std@@@std@@$0A@@stdext@@@stdext@@@0@U_Nonscalar_ptr_iterator_tag@0@U_Range_checked_iterator_tag@0@@Z$0 1000f820 f i effectmanager.obj
 0001:0000e820       __catch$??$_Uninit_fill_n@PAUSt_EffLODParam@@IU1@V?$allocator@USt_EffLODParam@@@std@@@std@@YAXPAUSt_EffLODParam@@IABU1@AAV?$allocator@USt_EffLODParam@@@0@U_Nonscalar_ptr_iterator_tag@0@U_Range_checked_iterator_tag@0@@Z$0 1000f820 f i effectmanager.obj
 0001:0000e93b       __catch$??$_Insert@V?$_Const_iterator@$00@?$list@U?$pair@QAXPAVCEffectBody@@@std@@V?$allocator@U?$pair@QAXPAVCEffectBody@@@std@@@2@@std@@@?$list@U?$pair@QAXPAVCEffectBody@@@std@@V?$allocator@U?$pair@QAXPAVCEffectBody@@@std@@@2@@std@@QAEXV?$_Const_iterator@$00@01@00Uforward_iterator_tag@1@@Z$0 1000f93b f i effectmanager.obj
 0001:0000e93b       __catch$??$_Insert@V?$_Const_iterator@$00@?$list@U?$pair@$$CBKPAUSt_BodyCreate@@@std@@V?$allocator@U?$pair@$$CBKPAUSt_BodyCreate@@@std@@@2@@std@@@?$list@U?$pair@$$CBKPAUSt_BodyCreate@@@std@@V?$allocator@U?$pair@$$CBKPAUSt_BodyCreate@@@std@@@2@@std@@QAEXV?$_Const_iterator@$00@01@00Uforward_iterator_tag@1@@Z$0 1000f93b f i effectmanager.obj
 0001:0000ec23       __catch$??$_Insert@V?$_Const_iterator@$00@?$list@KV?$allocator@K@std@@@std@@@?$list@KV?$allocator@K@std@@@std@@QAEXV?$_Const_iterator@$00@01@00Uforward_iterator_tag@1@@Z$0 1000fc23 f i effectmanager.obj
 0001:0000ed8a       __catch$??$_Uninit_copy@PAU_List_position@?$_Hash@V?$_Hmap_traits@KV?$basic_string@DU?$char_traits@D@std@@V?$allocator@D@2@@std@@V?$hash_compare@KU?$less@K@std@@@stdext@@V?$allocator@U?$pair@$$CBKV?$basic_string@DU?$char_traits@D@std@@V?$allocator@D@2@@std@@@std@@@2@$0A@@stdext@@@stdext@@PAU123@V?$allocator@U_List_position@?$_Hash@V?$_Hmap_traits@KV?$basic_string@DU?$char_traits@D@std@@V?$allocator@D@2@@std@@V?$hash_compare@KU?$less@K@std@@@stdext@@V?$allocator@U?$pair@$$CBKV?$basic_string@DU?$char_traits@D@std@@V?$allocator@D@2@@std@@@std@@@2@$0A@@stdext@@@stdext@@@std@@@std@@YAPAU_List_position@?$_Hash@V?$_Hmap_traits@KV?$basic_string@DU?$char_traits@D@std@@V?$allocator@D@2@@std@@V?$hash_compare@KU?$less@K@std@@@stdext@@V?$allocator@U?$pair@$$CBKV?$basic_string@DU?$char_traits@D@std@@V?$allocator@D@2@@std@@@std@@@2@$0A@@stdext@@@stdext@@PAU123@00AAV?$allocator@U_List_position@?$_Hash@V?$_Hmap_traits@KV?$basic_string@DU?$char_traits@D@std@@V?$allocator@D@2@@std@@V?$hash_compare@KU?$less@K@std@@@stdext@@V?$allocator@U?$pair@$$CBKV?$basic_string@DU?$char_traits@D@std@@V?$allocator@D@2@@std@@@std@@@2@$0A@@stdext@@@stdext@@@0@U_Nonscalar_ptr_iterator_tag@0@U_Range_checked_iterator_tag@0@@Z$0 1000fd8a f i effectmanager.obj
 0001:0000ed8a       __catch$??$_Uninit_copy@PAU_List_position@?$_Hash@V?$_Hmap_traits@KPAUSt_BodyCreate@@V?$hash_compare@KU?$less@K@std@@@stdext@@V?$allocator@U?$pair@$$CBKPAUSt_BodyCreate@@@std@@@std@@$0A@@stdext@@@stdext@@PAU123@V?$allocator@U_List_position@?$_Hash@V?$_Hmap_traits@KPAUSt_BodyCreate@@V?$hash_compare@KU?$less@K@std@@@stdext@@V?$allocator@U?$pair@$$CBKPAUSt_BodyCreate@@@std@@@std@@$0A@@stdext@@@stdext@@@std@@@std@@YAPAU_List_position@?$_Hash@V?$_Hmap_traits@KPAUSt_BodyCreate@@V?$hash_compare@KU?$less@K@std@@@stdext@@V?$allocator@U?$pair@$$CBKPAUSt_BodyCreate@@@std@@@std@@$0A@@stdext@@@stdext@@PAU123@00AAV?$allocator@U_List_position@?$_Hash@V?$_Hmap_traits@KPAUSt_BodyCreate@@V?$hash_compare@KU?$less@K@std@@@stdext@@V?$allocator@U?$pair@$$CBKPAUSt_BodyCreate@@@std@@@std@@$0A@@stdext@@@stdext@@@0@U_Nonscalar_ptr_iterator_tag@0@U_Range_checked_iterator_tag@0@@Z$0 1000fd8a f i effectmanager.obj
 0001:0000ed8a       __catch$??$_Uninit_copy@PAUSt_AutoCtlParam@@PAU1@V?$allocator@USt_AutoCtlParam@@@std@@@std@@YAPAUSt_AutoCtlParam@@PAU1@00AAV?$allocator@USt_AutoCtlParam@@@0@U_Nonscalar_ptr_iterator_tag@0@U_Range_checked_iterator_tag@0@@Z$0 1000fd8a f i effectmanager.obj
 0001:0000ed8a       __catch$??$_Uninit_copy@PAU_List_position@?$_Hash@V?$_Hmap_traits@PAXPAVCEffectBody@@V?$hash_compare@PAXU?$less@PAX@std@@@stdext@@V?$allocator@U?$pair@QAXPAVCEffectBody@@@std@@@std@@$0A@@stdext@@@stdext@@PAU123@V?$allocator@U_List_position@?$_Hash@V?$_Hmap_traits@PAXPAVCEffectBody@@V?$hash_compare@PAXU?$less@PAX@std@@@stdext@@V?$allocator@U?$pair@QAXPAVCEffectBody@@@std@@@std@@$0A@@stdext@@@stdext@@@std@@@std@@YAPAU_List_position@?$_Hash@V?$_Hmap_traits@PAXPAVCEffectBody@@V?$hash_compare@PAXU?$less@PAX@std@@@stdext@@V?$allocator@U?$pair@QAXPAVCEffectBody@@@std@@@std@@$0A@@stdext@@@stdext@@PAU123@00AAV?$allocator@U_List_position@?$_Hash@V?$_Hmap_traits@PAXPAVCEffectBody@@V?$hash_compare@PAXU?$less@PAX@std@@@stdext@@V?$allocator@U?$pair@QAXPAVCEffectBody@@@std@@@std@@$0A@@stdext@@@stdext@@@0@U_Nonscalar_ptr_iterator_tag@0@U_Range_checked_iterator_tag@0@@Z$0 1000fd8a f i effectmanager.obj
 0001:0000ed8a       __catch$??$_Uninit_copy@PAU_WZNCSPT@WzNaturalCubicSplineDyn@@PAU12@V?$allocator@U_WZNCSPT@WzNaturalCubicSplineDyn@@@std@@@std@@YAPAU_WZNCSPT@WzNaturalCubicSplineDyn@@PAU12@00AAV?$allocator@U_WZNCSPT@WzNaturalCubicSplineDyn@@@0@U_Nonscalar_ptr_iterator_tag@0@U_Range_checked_iterator_tag@0@@Z$0 1000fd8a f i effectmanager.obj
 0001:0000ed8a       __catch$??$_Uninit_copy@PAUSt_EffLODParam@@PAU1@V?$allocator@USt_EffLODParam@@@std@@@std@@YAPAUSt_EffLODParam@@PAU1@00AAV?$allocator@USt_EffLODParam@@@0@U_Nonscalar_ptr_iterator_tag@0@U_Range_checked_iterator_tag@0@@Z$0 1000fd8a f i effectmanager.obj
 0001:00012604       ??$AllocNew@USt_BodyCreate@@@CMemoryPool@@YAPAUSt_BodyCreate@@XZ 10013604 f   effectmanager_load.obj
 0001:0001266c       ??$AllocNew@USt_ElementCreate@@@CMemoryPool@@YAPAUSt_ElementCreate@@XZ 1001366c f   effectmanager_load.obj
 0001:000126c7       ??$AllocNew@USt_Create_Info@@@CMemoryPool@@YAPAUSt_Create_Info@@XZ 100136c7 f   effectmanager_load.obj
 0001:0001272f       ??$AllocNew@USt_Move_Info@@@CMemoryPool@@YAPAUSt_Move_Info@@XZ 1001372f f   effectmanager_load.obj
 0001:00012797       ??$AllocNew@USt_Change_Info@@@CMemoryPool@@YAPAUSt_Change_Info@@XZ 10013797 f   effectmanager_load.obj
 0001:000127ff       ??$AllocNew@USt_Visual_Info@@@CMemoryPool@@YAPAUSt_Visual_Info@@XZ 100137ff f   effectmanager_load.obj
 0001:00017f40       __catch$?_Buynode@?$list@U?$pair@$$CBKV?$basic_string@DU?$char_traits@D@std@@V?$allocator@D@2@@std@@@std@@V?$allocator@U?$pair@$$CBKV?$basic_string@DU?$char_traits@D@std@@V?$allocator@D@2@@std@@@std@@@2@@std@@IAEPAU_Node@?$_List_nod@U?$pair@$$CBKV?$basic_string@DU?$char_traits@D@std@@V?$allocator@D@2@@std@@@std@@V?$allocator@U?$pair@$$CBKV?$basic_string@DU?$char_traits@D@std@@V?$allocator@D@2@@std@@@std@@@2@@2@XZ$0 10018f40 f i loadmanager.obj
 0001:000181cb       __catch$?_Buynode@?$list@U?$pair@$$CBKV?$basic_string@DU?$char_traits@D@std@@V?$allocator@D@2@@std@@@std@@V?$allocator@U?$pair@$$CBKV?$basic_string@DU?$char_traits@D@std@@V?$allocator@D@2@@std@@@std@@@2@@std@@IAEPAU_Node@?$_List_nod@U?$pair@$$CBKV?$basic_string@DU?$char_traits@D@std@@V?$allocator@D@2@@std@@@std@@V?$allocator@U?$pair@$$CBKV?$basic_string@DU?$char_traits@D@std@@V?$allocator@D@2@@std@@@std@@@2@@2@PAU342@0ABU?$pair@$$CBKV?$basic_string@DU?$char_traits@D@std@@V?$allocator@D@2@@std@@@2@@Z$0 100191cb f i loadmanager.obj
 0001:000184a5       __catch$??$_Insert@V?$_Const_iterator@$00@?$list@U?$pair@$$CBKV?$basic_string@DU?$char_traits@D@std@@V?$allocator@D@2@@std@@@std@@V?$allocator@U?$pair@$$CBKV?$basic_string@DU?$char_traits@D@std@@V?$allocator@D@2@@std@@@std@@@2@@std@@@?$list@U?$pair@$$CBKV?$basic_string@DU?$char_traits@D@std@@V?$allocator@D@2@@std@@@std@@V?$allocator@U?$pair@$$CBKV?$basic_string@DU?$char_traits@D@std@@V?$allocator@D@2@@std@@@std@@@2@@std@@QAEXV?$_Const_iterator@$00@01@00Uforward_iterator_tag@1@@Z$0 100194a5 f i loadmanager.obj
 0001:0002327e       __catch$?_Buynode@?$list@KV?$allocator@K@std@@@std@@IAEPAU_Node@?$_List_nod@KV?$allocator@K@std@@@2@PAU342@0ABK@Z$0 1002427e f i eelementweather.obj
 0001:0002327e       __catch$?_Buynode@?$list@PAVCEElementSprite@@V?$allocator@PAVCEElementSprite@@@std@@@std@@IAEPAU_Node@?$_List_nod@PAVCEElementSprite@@V?$allocator@PAVCEElementSprite@@@std@@@2@PAU342@0ABQAVCEElementSprite@@@Z$0 1002427e f i eelementweather.obj
 0001:0002327e       __catch$?_Buynode@?$list@PAVCEElementBase@@V?$allocator@PAVCEElementBase@@@std@@@std@@IAEPAU_Node@?$_List_nod@PAVCEElementBase@@V?$allocator@PAVCEElementBase@@@std@@@2@PAU342@0ABQAVCEElementBase@@@Z$0 1002427e f i eelementweather.obj
 0001:000252aa       __catch$?_Insert_n@?$vector@PAUSt_SoundInfo@@V?$allocator@PAUSt_SoundInfo@@@std@@@std@@IAEXV?$_Vector_const_iterator@PAUSt_SoundInfo@@V?$allocator@PAUSt_SoundInfo@@@std@@@2@IABQAUSt_SoundInfo@@@Z$0 100262aa f i effectbody.obj
 0001:000252aa       __catch$?_Insert_n@?$vector@PAXV?$allocator@PAX@std@@@std@@IAEXV?$_Vector_const_iterator@PAXV?$allocator@PAX@std@@@2@IABQAX@Z$0 100262aa f i effectbody.obj
 0001:000252aa       __catch$?_Insert_n@?$vector@PAUsEffectTexture@CEffectManager@@V?$allocator@PAUsEffectTexture@CEffectManager@@@std@@@std@@IAEXV?$_Vector_const_iterator@PAUsEffectTexture@CEffectManager@@V?$allocator@PAUsEffectTexture@CEffectManager@@@std@@@2@IABQAUsEffectTexture@CEffectManager@@@Z$0 100262aa f i effectbody.obj
 0001:000254d5       __catch$?_Insert_n@?$vector@PAUsEffectTexture@CEffectManager@@V?$allocator@PAUsEffectTexture@CEffectManager@@@std@@@std@@IAEXV?$_Vector_const_iterator@PAUsEffectTexture@CEffectManager@@V?$allocator@PAUsEffectTexture@CEffectManager@@@std@@@2@IABQAUsEffectTexture@CEffectManager@@@Z$2 100264d5 f i effectbody.obj
 0001:000254d5       __catch$?_Insert_n@?$vector@PAUSt_SoundInfo@@V?$allocator@PAUSt_SoundInfo@@@std@@@std@@IAEXV?$_Vector_const_iterator@PAUSt_SoundInfo@@V?$allocator@PAUSt_SoundInfo@@@std@@@2@IABQAUSt_SoundInfo@@@Z$2 100264d5 f i effectbody.obj
 0001:000254d5       __catch$?_Insert_n@?$vector@PAXV?$allocator@PAX@std@@@std@@IAEXV?$_Vector_const_iterator@PAXV?$allocator@PAX@std@@@2@IABQAX@Z$2 100264d5 f i effectbody.obj
 0001:00025a54       ?CatchGuardHandler@@YA?AW4_EXCEPTION_DISPOSITION@@PAUEHExceptionRecord@@PAUCatchGuardRN@@PAX2@Z 10026a54 f   LIBCMT:_trnsctrl_.obj
 0001:00025b5e       ?TranslatorGuardHandler@@YA?AW4_EXCEPTION_DISPOSITION@@PAUEHExceptionRecord@@PAUTranslatorGuardRN@@PAX2@Z 10026b5e f   LIBCMT:_trnsctrl_.obj
 0001:00026ea5       __onexit_nolock            10027ea5 f   LIBCMT:onexit.obj
 0001:0002737e       ___DllMainCRTStartup       1002837e f   LIBCMT:dllcrt0.obj
 0001:0002794b       ?ExFilterRethrow@@YAHPAU_EXCEPTION_POINTERS@@@Z 1002894b f   LIBCMT:frame.obj
 0001:00027a0e       ?IsInExceptionSpec@@YAEPAUEHExceptionRecord@@PBU_s_ESTypeList@@@Z 10028a0e f   LIBCMT:frame.obj
 0001:00027a89       ?CallUnexpected@@YAXPBU_s_ESTypeList@@@Z 10028a89 f   LIBCMT:frame.obj
 0001:00027aba       __catch$?CallUnexpected@@YAXPBU_s_ESTypeList@@@Z$0 10028aba f   LIBCMT:frame.obj
 0001:00027ad2       ?CallCatchBlock@@YAPAXPAUEHExceptionRecord@@PAUEHRegistrationNode@@PAU_CONTEXT@@PBU_s_FuncInfo@@PAXHK@Z 10028ad2 f   LIBCMT:frame.obj
 0001:00027e7f       ?CatchIt@@YAXPAUEHExceptionRecord@@PAUEHRegistrationNode@@PAU_CONTEXT@@PAXPBU_s_FuncInfo@@PBU_s_HandlerType@@PBU_s_CatchableType@@PBU_s_TryBlockMapEntry@@H1E@Z 10028e7f f   LIBCMT:frame.obj
 0001:00027eed       ?FindHandlerForForeignException@@YAXPAUEHExceptionRecord@@PAUEHRegistrationNode@@PAU_CONTEXT@@PAXPBU_s_FuncInfo@@HH1@Z 10028eed f   LIBCMT:frame.obj
 0001:00027fe1       ?FindHandler@@YAXPAUEHExceptionRecord@@PAUEHRegistrationNode@@PAU_CONTEXT@@PAXPBU_s_FuncInfo@@EH1@Z 10028fe1 f   LIBCMT:frame.obj
 0001:00028d8f       __shift                    10029d8f f   LIBCMT:cvt.obj
 0001:00028dd4       __cftoe2_l                 10029dd4 f   LIBCMT:cvt.obj
 0001:000293a6       __cftof2_l                 1002a3a6 f   LIBCMT:cvt.obj
 0001:000298a8       _fastzero_I                1002a8a8 f   LIBCMT:p4_memset.obj
 0001:0002998e       _has_osfxsr_set            1002a98e f   LIBCMT:cpu_disp.obj
 0001:00029bb9       _write_char                1002abb9 f   LIBCMT:output.obj
 0001:00029bec       _write_multi_char          1002abec f   LIBCMT:output.obj
 0001:00029c12       _write_string              1002ac12 f   LIBCMT:output.obj
 0001:0002aadc       _fastcopy_I                1002badc f   LIBCMT:p4_memcpy.obj
 0001:0002b00c       ?CPtoLCID@@YAHH@Z          1002c00c f   LIBCMT:mbctype.obj
 0001:0002b03b       ?setSBCS@@YAXPAUthreadmbcinfostruct@@@Z 1002c03b f   LIBCMT:mbctype.obj
 0001:0002b09f       ?setSBUpLow@@YAXPAUthreadmbcinfostruct@@@Z 1002c09f f   LIBCMT:mbctype.obj
 0001:0002b2d6       ?getSystemCP@@YAHH@Z       1002c2d6 f   LIBCMT:mbctype.obj
 0001:0002b960       __updatetlocinfoEx_nolock  1002c960 f   LIBCMT:setlocal.obj
 0001:0002bd85       __initterm                 1002cd85 f   LIBCMT:crt0dat.obj
 0001:0002be4b       _doexit                    1002ce4b f   LIBCMT:crt0dat.obj
 0001:0002c6f8       _parse_cmdline             1002d6f8 f   LIBCMT:stdargv.obj
 0001:0002dd2c       __unwind_handler           1002ed2c f   LIBCMT:exsup.obj
 0001:0002e5f4       __unwind_handler4          1002f5f4 f   LIBCMT:exsup4.obj
 0001:0002f83c       ?__crtLCMapStringA_stat@@YAHPAUlocaleinfo_struct@@KKPBDHPADHHH@Z 1003083c f   LIBCMT:a_map.obj
 0001:0002fc26       ?__crtGetStringTypeA_stat@@YAHPAUlocaleinfo_struct@@KPBDHPAGHHH@Z 10030c26 f   LIBCMT:a_str.obj
 0001:0003064f       _siglookup                 1003164f f   LIBCMT:winsig.obj
 0001:000308d0       ?x_ismbbtype_l@@YAHPAUlocaleinfo_struct@@IHH@Z 100318d0 f   LIBCMT:ismbbyte.obj
 0001:000325ac       __hw_cw                    100335ac f   LIBCMT:_ieee87_.obj
 0001:0003263a       ___hw_cw_sse2              1003363a f   LIBCMT:_ieee87_.obj
 0001:00032f7a       _flsall                    10033f7a f   LIBCMT:fflush.obj
 0001:0003305d       ?strtoxl@@YAKPAUlocaleinfo_struct@@PBDPAPBDHH@Z 1003405d f   LIBCMT:strtol.obj
 0001:0003d530       @geVFile_RegisterFileSystemInternal@8 1003e530 f   wzFilePacker_static:vfile.obj
 0001:0003d5a0       _RegisterBuiltInAPIs       1003e5a0 f   wzFilePacker_static:vfile.obj
 0001:0003d610       @CheckOpenFlags@4          1003e610 f   wzFilePacker_static:vfile.obj
 0001:0003dd90       _geRam_DoCriticalCallback  1003ed90 f   wzFilePacker_static:Ram.obj
 0001:0003dec0       @FSVFS_FinderCreate@12     1003eec0 f   wzFilePacker_static:fsvfs.obj
 0001:0003df30       @FSVFS_FinderGetNextFile@4 1003ef30 f   wzFilePacker_static:fsvfs.obj
 0001:0003df50       @FSVFS_FinderGetProperties@8 1003ef50 f   wzFilePacker_static:fsvfs.obj
 0001:0003dfb0       @FSVFS_FinderDestroy@4     1003efb0 f   wzFilePacker_static:fsvfs.obj
 0001:0003dfe0       @FSVFS_OpenNewSystem@16    1003efe0 f   wzFilePacker_static:fsvfs.obj
 0001:0003e6c0       @FSVFS_MakeSpace@24        1003f6c0 f   wzFilePacker_static:fsvfs.obj
 0001:0003e960       @FSVFS_EnlargeDirectorySize@8 1003f960 f   wzFilePacker_static:fsvfs.obj
 0001:0003ea40       @FSVFS_Close@4             1003fa40 f   wzFilePacker_static:fsvfs.obj
 0001:0003ebb0       @ForceFilePos@4            1003fbb0 f   wzFilePacker_static:fsvfs.obj
 0001:0003ebd0       _ClampOperationSize        1003fbd0 f   wzFilePacker_static:fsvfs.obj
 0001:0003ec10       @UpdateFilePos@4           1003fc10 f   wzFilePacker_static:fsvfs.obj
 0001:0003ecf0       @FSVFS_GetS@12             1003fcf0 f   wzFilePacker_static:fsvfs.obj
 0001:0003ed40       @FSVFS_Read@12             1003fd40 f   wzFilePacker_static:fsvfs.obj
 0001:0003eeb0       @FSVFS_Write@12            1003feb0 f   wzFilePacker_static:fsvfs.obj
 0001:0003ef10       @FSVFS_Seek@16             1003ff10 f   wzFilePacker_static:fsvfs.obj
 0001:0003efa0       @FSVFS_EOF@4               1003ffa0 f   wzFilePacker_static:fsvfs.obj
 0001:0003efc0       @FSVFS_Tell@8              1003ffc0 f   wzFilePacker_static:fsvfs.obj
 0001:0003efe0       @FSVFS_Size@8              1003ffe0 f   wzFilePacker_static:fsvfs.obj
 0001:0003f000       @FSVFS_GetProperties@8     10040000 f   wzFilePacker_static:fsvfs.obj
 0001:0003f050       @FSVFS_SetAttributes@8     10040050 f   wzFilePacker_static:fsvfs.obj
 0001:0003f070       @FSVFS_SetTime@8           10040070 f   wzFilePacker_static:fsvfs.obj
 0001:0003f080       @FSVFS_SetHints@8          10040080 f   wzFilePacker_static:fsvfs.obj
 0001:0003f090       @FSVFS_FileExists@12       10040090 f   wzFilePacker_static:fsvfs.obj
 0001:0003f0b0       _FSVFS_GetVoidSpace        100400b0 f   wzFilePacker_static:fsvfs.obj
 0001:0003f540       _FSVFS_SetVoidSpace        10040540 f   wzFilePacker_static:fsvfs.obj
 0001:0003f860       @FSVFS_Open@20             10040860 f   wzFilePacker_static:fsvfs.obj
 0001:0003fa20       @FSVFS_DeleteFile@12       10040a20 f   wzFilePacker_static:fsvfs.obj
 0001:0003fb60       @FSMemory_FinderCreate@12  10040b60 f   wzFilePacker_static:FSMEMORY.obj
 0001:0003fb60       @FSMemory_FileExists@12    10040b60 f   wzFilePacker_static:FSMEMORY.obj
 0001:0003fb60       @FSMemory_DeleteFile@12    10040b60 f   wzFilePacker_static:FSMEMORY.obj
 0001:0003fb70       @FSMemory_FinderDestroy@4  10040b70 f   wzFilePacker_static:FSMEMORY.obj
 0001:0003fb80       @FSMemory_Open@20          10040b80 f   wzFilePacker_static:FSMEMORY.obj
 0001:0003fb90       @FSMemory_OpenNewSystem@16 10040b90 f   wzFilePacker_static:FSMEMORY.obj
 0001:0003fc50       @FSMemory_UpdateContext@16 10040c50 f   wzFilePacker_static:FSMEMORY.obj
 0001:0003fc80       @FSMemory_Close@4          10040c80 f   wzFilePacker_static:FSMEMORY.obj
 0001:0003fcc0       @ClampOperationSize@12     10040cc0 f   wzFilePacker_static:FSMEMORY.obj
 0001:0003fd00       @DataPtr@4                 10040d00 f   wzFilePacker_static:FSMEMORY.obj
 0001:0003fd10       @FSMemory_GetS@12          10040d10 f   wzFilePacker_static:FSMEMORY.obj
 0001:0003fd70       @FSMemory_Read@12          10040d70 f   wzFilePacker_static:FSMEMORY.obj
 0001:0003fdd0       @TestForExpansion@12       10040dd0 f   wzFilePacker_static:FSMEMORY.obj
 0001:0003fe50       @FSMemory_Write@12         10040e50 f   wzFilePacker_static:FSMEMORY.obj
 0001:0003fed0       @FSMemory_Seek@16          10040ed0 f   wzFilePacker_static:FSMEMORY.obj
 0001:0003ffa0       @FSMemory_EOF@4            10040fa0 f   wzFilePacker_static:FSMEMORY.obj
 0001:0003ffc0       @FSMemory_Tell@8           10040fc0 f   wzFilePacker_static:FSMEMORY.obj
 0001:0003ffe0       @FSMemory_Size@8           10040fe0 f   wzFilePacker_static:FSMEMORY.obj
 0001:00040000       @FSMemory_Disperse@16      10041000 f   wzFilePacker_static:FSMEMORY.obj
 0001:00040000       @FSVFS_RenameFile@16       10041000 f   wzFilePacker_static:FSMEMORY.obj
 0001:00040000       @FSMemory_SetSize@12       10041000 f   wzFilePacker_static:FSMEMORY.obj
 0001:00040000       @FSMemory_RenameFile@16    10041000 f   wzFilePacker_static:FSMEMORY.obj
 0001:00040000       @FSVFS_SetSize@12          10041000 f   wzFilePacker_static:FSMEMORY.obj
 0001:00040000       @FSVFS_UpdateContext@16    10041000 f   wzFilePacker_static:FSMEMORY.obj
 0001:00040000       @FSDos_Disperse@16         10041000 f   wzFilePacker_static:FSMEMORY.obj
 0001:00040000       @FSDos_UpdateContext@16    10041000 f   wzFilePacker_static:FSMEMORY.obj
 0001:00040000       @FSVFS_Disperse@16         10041000 f   wzFilePacker_static:FSMEMORY.obj
 0001:00040020       _BuildFileName             10041020 f   wzFilePacker_static:fsdos.obj
 0001:000400f0       @FSDos_FinderCreate@12     100410f0 f   wzFilePacker_static:fsdos.obj
 0001:000401c0       @FSDos_FinderGetNextFile@4 100411c0 f   wzFilePacker_static:fsdos.obj
 0001:00040230       @FSDos_FinderGetProperties@8 10041230 f   wzFilePacker_static:fsdos.obj
 0001:000402b0       @FSDos_FinderDestroy@4     100412b0 f   wzFilePacker_static:fsdos.obj
 0001:000402e0       _IsRootDirectory           100412e0 f   wzFilePacker_static:fsdos.obj
 0001:00040330       @FSDos_Open@20             10041330 f   wzFilePacker_static:fsdos.obj
 0001:00040530       @FSDos_OpenNewSystem@16    10041530 f   wzFilePacker_static:fsdos.obj
 0001:00040550       @FSDos_Close@4             10041550 f   wzFilePacker_static:fsdos.obj
 0001:000405a0       @FSDos_GetS@12             100415a0 f   wzFilePacker_static:fsdos.obj
 0001:00040680       @FSDos_Read@12             10041680 f   wzFilePacker_static:fsdos.obj
 0001:000406e0       @FSDos_Write@12            100416e0 f   wzFilePacker_static:fsdos.obj
 0001:00040720       @FSDos_Seek@16             10041720 f   wzFilePacker_static:fsdos.obj
 0001:000407e0       @FSDos_EOF@4               100417e0 f   wzFilePacker_static:fsdos.obj
 0001:00040870       @FSDos_Tell@8              10041870 f   wzFilePacker_static:fsdos.obj
 0001:000408e0       @FSDos_Size@8              100418e0 f   wzFilePacker_static:fsdos.obj
 0001:00040950       @FSDos_GetProperties@8     10041950 f   wzFilePacker_static:fsdos.obj
 0001:00040a10       @FSDos_SetSize@12          10041a10 f   wzFilePacker_static:fsdos.obj
 0001:00040a60       @FSDos_SetAttributes@8     10041a60 f   wzFilePacker_static:fsdos.obj
 0001:00040a90       @FSDos_SetTime@8           10041a90 f   wzFilePacker_static:fsdos.obj
 0001:00040ac0       @FSMemory_EnlargeDirectorySize@8 10041ac0 f   wzFilePacker_static:fsdos.obj
 0001:00040ac0       @FSMemory_SetHints@8       10041ac0 f   wzFilePacker_static:fsdos.obj
 0001:00040ac0       @FSMemory_SetTime@8        10041ac0 f   wzFilePacker_static:fsdos.obj
 0001:00040ac0       @FSMemory_SetAttributes@8  10041ac0 f   wzFilePacker_static:fsdos.obj
 0001:00040ac0       @FSMemory_GetProperties@8  10041ac0 f   wzFilePacker_static:fsdos.obj
 0001:00040ac0       @FSDos_EnlargeDirectorySize@8 10041ac0 f   wzFilePacker_static:fsdos.obj
 0001:00040ac0       @FSMemory_FinderGetProperties@8 10041ac0 f   wzFilePacker_static:fsdos.obj
 0001:00040ac0       @FSMemory_FinderGetNextFile@4 10041ac0 f   wzFilePacker_static:fsdos.obj
 0001:00040ac0       @FSDos_SetHints@8          10041ac0 f   wzFilePacker_static:fsdos.obj
 0001:00040ad0       @FSDos_FileExists@12       10041ad0 f   wzFilePacker_static:fsdos.obj
 0001:00040b60       @FSDos_DeleteFile@12       10041b60 f   wzFilePacker_static:fsdos.obj
 0001:00040bf0       @FSDos_RenameFile@16       10041bf0 f   wzFilePacker_static:fsdos.obj
 0001:00040d60       _WriteTree                 10041d60 f   wzFilePacker_static:dirtree.obj
 0001:00040ee0       _DirTree_WriteToFile1      10041ee0 f   wzFilePacker_static:dirtree.obj
 0001:00041080       _ReadTree                  10042080 f   wzFilePacker_static:dirtree.obj
 0001:000412d0       _ReadTreeCount             100422d0 f   wzFilePacker_static:dirtree.obj
 0001:00042284       __splitpath_helper         10043284 f   LIBCMT:splitpat.obj
 0001:00042790       __unwindfunclet$??0CEffectManager@@QAE@XZ$0 10043790 f   effectmanager.obj
 0001:00042798       __unwindfunclet$??0CEffectManager@@QAE@XZ$1 10043798 f   effectmanager.obj
 0001:000427a3       __unwindfunclet$??0CEffectManager@@QAE@XZ$2 100437a3 f   effectmanager.obj
 0001:000427ae       __unwindfunclet$??0CEffectManager@@QAE@XZ$3 100437ae f   effectmanager.obj
 0001:000427b9       __unwindfunclet$??0CEffectManager@@QAE@XZ$4 100437b9 f   effectmanager.obj
 0001:000427c7       __unwindfunclet$??0CEffectManager@@QAE@XZ$5 100437c7 f   effectmanager.obj
 0001:000427d5       __unwindfunclet$??0CEffectManager@@QAE@XZ$6 100437d5 f   effectmanager.obj
 0001:000427e3       __unwindfunclet$??0CEffectManager@@QAE@XZ$7 100437e3 f   effectmanager.obj
 0001:000427f1       __unwindfunclet$??0CEffectManager@@QAE@XZ$8 100437f1 f   effectmanager.obj
 0001:000427ff       __unwindfunclet$??0CEffectManager@@QAE@XZ$9 100437ff f   effectmanager.obj
 0001:0004280d       __unwindfunclet$??0CEffectManager@@QAE@XZ$10 1004380d f   effectmanager.obj
 0001:0004281b       __ehhandler$??0CEffectManager@@QAE@XZ 1004381b f   effectmanager.obj
 0001:00042836       __unwindfunclet$??1CEffectManager@@UAE@XZ$0 10043836 f   effectmanager.obj
 0001:00042841       __unwindfunclet$??1CEffectManager@@UAE@XZ$1 10043841 f   effectmanager.obj
 0001:0004284f       __unwindfunclet$??1CEffectManager@@UAE@XZ$2 1004384f f   effectmanager.obj
 0001:0004285d       __unwindfunclet$??1CEffectManager@@UAE@XZ$3 1004385d f   effectmanager.obj
 0001:0004286b       __unwindfunclet$??1CEffectManager@@UAE@XZ$4 1004386b f   effectmanager.obj
 0001:0004287c       __unwindfunclet$??1CEffectManager@@UAE@XZ$5 1004387c f   effectmanager.obj
 0001:0004288d       __unwindfunclet$??1CEffectManager@@UAE@XZ$6 1004388d f   effectmanager.obj
 0001:0004289e       __unwindfunclet$??1CEffectManager@@UAE@XZ$7 1004389e f   effectmanager.obj
 0001:000428af       __unwindfunclet$??1CEffectManager@@UAE@XZ$8 100438af f   effectmanager.obj
 0001:000428c0       __unwindfunclet$??1CEffectManager@@UAE@XZ$9 100438c0 f   effectmanager.obj
 0001:000428d1       __unwindfunclet$??1CEffectManager@@UAE@XZ$10 100438d1 f   effectmanager.obj
 0001:000428e2       __unwindfunclet$??1CEffectManager@@UAE@XZ$11 100438e2 f   effectmanager.obj
 0001:000428ea       __unwindfunclet$??1CEffectManager@@UAE@XZ$13 100438ea f   effectmanager.obj
 0001:000428f2       __unwindfunclet$??1CEffectManager@@UAE@XZ$15 100438f2 f   effectmanager.obj
 0001:000428fa       __unwindfunclet$??1CEffectManager@@UAE@XZ$41 100438fa f   effectmanager.obj
 0001:00042905       __ehhandler$??1CEffectManager@@UAE@XZ 10043905 f   effectmanager.obj
 0001:00042923       __unwindfunclet$?Create@CEffectManager@@QAE_NPAVCDrawBase@@PAVCWorldBase@@@Z$2 10043923 f   effectmanager.obj
 0001:0004292d       __ehhandler$?Create@CEffectManager@@QAE_NPAVCDrawBase@@PAVCWorldBase@@@Z 1004392d f   effectmanager.obj
 0001:00042948       __unwindfunclet$?ReleaseEffectTexture@CEffectManager@@QAEXXZ$0 10043948 f   effectmanager.obj
 0001:00042950       __ehhandler$?ReleaseEffectTexture@CEffectManager@@QAEXXZ 10043950 f   effectmanager.obj
 0001:0004296e       __unwindfunclet$?LoadTextureFiles@CEffectManager@@QAE_NPBD0W4EENUM_LOAD_TYPE@@@Z$0 1004396e f   effectmanager.obj
 0001:00042979       __ehhandler$?LoadTextureFiles@CEffectManager@@QAE_NPBD0W4EENUM_LOAD_TYPE@@@Z 10043979 f   effectmanager.obj
 0001:000429a1       __unwindfunclet$?LoadMeshFiles@CEffectManager@@QAE_NPBD0W4EENUM_LOAD_TYPE@@@Z$0 100439a1 f   effectmanager.obj
 0001:000429ac       __ehhandler$?LoadMeshFiles@CEffectManager@@QAE_NPBD0W4EENUM_LOAD_TYPE@@@Z 100439ac f   effectmanager.obj
 0001:000429d4       __unwindfunclet$??$AllocNew@UsEffectTexture@CEffectManager@@@CMemoryPool@@YAPAUsEffectTexture@CEffectManager@@XZ$0 100439d4 f   effectmanager.obj
 0001:000429de       __ehhandler$??$AllocNew@UsEffectTexture@CEffectManager@@@CMemoryPool@@YAPAUsEffectTexture@CEffectManager@@XZ 100439de f   effectmanager.obj
 0001:000429f9       __unwindfunclet$??$AllocNew@USt_BodyCreate@@@CMemoryPool@@YAPAUSt_BodyCreate@@XZ$0 100439f9 f   effectmanager.obj
 0001:00042a03       __ehhandler$??$AllocNew@USt_BodyCreate@@@CMemoryPool@@YAPAUSt_BodyCreate@@XZ 10043a03 f   effectmanager.obj
 0001:00042a1e       __unwindfunclet$??4St_BodyCreate@@QAEAAU0@ABU0@@Z$1 10043a1e f   effectmanager.obj
 0001:00042a28       __unwindfunclet$??4St_BodyCreate@@QAEAAU0@ABU0@@Z$2 10043a28 f   effectmanager.obj
 0001:00042a35       __unwindfunclet$??4St_BodyCreate@@QAEAAU0@ABU0@@Z$3 10043a35 f   effectmanager.obj
 0001:00042a42       __unwindfunclet$??4St_BodyCreate@@QAEAAU0@ABU0@@Z$4 10043a42 f   effectmanager.obj
 0001:00042a4f       __ehhandler$??4St_BodyCreate@@QAEAAU0@ABU0@@Z 10043a4f f   effectmanager.obj
 0001:00042a6d       __unwindfunclet$??0St_Create_Info@@QAE@XZ$0 10043a6d f   effectmanager.obj
 0001:00042a78       __unwindfunclet$??0St_Create_Info@@QAE@XZ$1 10043a78 f   effectmanager.obj
 0001:00042a83       __ehhandler$??0St_Create_Info@@QAE@XZ 10043a83 f   effectmanager.obj
 0001:00042a9e       __unwindfunclet$??1?$map@JUWzVector@@U?$less@J@std@@V?$allocator@U?$pair@$$CBJUWzVector@@@std@@@3@@std@@QAE@XZ$1 10043a9e f   effectmanager.obj
 0001:00042a9e       __unwindfunclet$??1?$map@JMU?$less@J@std@@V?$allocator@U?$pair@$$CBJM@std@@@2@@std@@QAE@XZ$1 10043a9e f   effectmanager.obj
 0001:00042aa6       __ehhandler$??1?$map@JUWzVector@@U?$less@J@std@@V?$allocator@U?$pair@$$CBJUWzVector@@@std@@@3@@std@@QAE@XZ 10043aa6 f   effectmanager.obj
 0001:00042aa6       __ehhandler$??1?$map@JMU?$less@J@std@@V?$allocator@U?$pair@$$CBJM@std@@@2@@std@@QAE@XZ 10043aa6 f   effectmanager.obj
 0001:00042ac1       __unwindfunclet$??0St_Move_Info@@QAE@XZ$0 10043ac1 f   effectmanager.obj
 0001:00042acc       __unwindfunclet$??0St_Move_Info@@QAE@XZ$1 10043acc f   effectmanager.obj
 0001:00042ad7       __ehhandler$??0St_Move_Info@@QAE@XZ 10043ad7 f   effectmanager.obj
 0001:00042af2       __unwindfunclet$??0St_Change_Info@@QAE@XZ$0 10043af2 f   effectmanager.obj
 0001:00042afd       __unwindfunclet$??0St_Change_Info@@QAE@XZ$1 10043afd f   effectmanager.obj
 0001:00042b0b       __unwindfunclet$??0St_Change_Info@@QAE@XZ$2 10043b0b f   effectmanager.obj
 0001:00042b19       __unwindfunclet$??0St_Change_Info@@QAE@XZ$3 10043b19 f   effectmanager.obj
 0001:00042b27       __unwindfunclet$??0St_Change_Info@@QAE@XZ$4 10043b27 f   effectmanager.obj
 0001:00042b38       __unwindfunclet$??0St_Change_Info@@QAE@XZ$5 10043b38 f   effectmanager.obj
 0001:00042b49       __unwindfunclet$??0St_Change_Info@@QAE@XZ$6 10043b49 f   effectmanager.obj
 0001:00042b5a       __unwindfunclet$??0St_Change_Info@@QAE@XZ$7 10043b5a f   effectmanager.obj
 0001:00042b6b       __unwindfunclet$??0St_Change_Info@@QAE@XZ$8 10043b6b f   effectmanager.obj
 0001:00042b7c       __unwindfunclet$??0St_Change_Info@@QAE@XZ$9 10043b7c f   effectmanager.obj
 0001:00042b8d       __unwindfunclet$??0St_Change_Info@@QAE@XZ$10 10043b8d f   effectmanager.obj
 0001:00042b9e       __unwindfunclet$??0St_Change_Info@@QAE@XZ$11 10043b9e f   effectmanager.obj
 0001:00042baf       __unwindfunclet$??0St_Change_Info@@QAE@XZ$12 10043baf f   effectmanager.obj
 0001:00042bc0       __unwindfunclet$??0St_Change_Info@@QAE@XZ$13 10043bc0 f   effectmanager.obj
 0001:00042bd1       __unwindfunclet$??0St_Change_Info@@QAE@XZ$14 10043bd1 f   effectmanager.obj
 0001:00042be2       __unwindfunclet$??0St_Change_Info@@QAE@XZ$15 10043be2 f   effectmanager.obj
 0001:00042bf3       __ehhandler$??0St_Change_Info@@QAE@XZ 10043bf3 f   effectmanager.obj
 0001:00042c0e       __unwindfunclet$?CreateSpline@St_BodyCreate@@QAEXPAUSt_ElementCreate@@@Z$0 10043c0e f   effectmanager.obj
 0001:00042c18       __unwindfunclet$?CreateSpline@St_BodyCreate@@QAEXPAUSt_ElementCreate@@@Z$1 10043c18 f   effectmanager.obj
 0001:00042c22       __unwindfunclet$?CreateSpline@St_BodyCreate@@QAEXPAUSt_ElementCreate@@@Z$2 10043c22 f   effectmanager.obj
 0001:00042c2c       __unwindfunclet$?CreateSpline@St_BodyCreate@@QAEXPAUSt_ElementCreate@@@Z$3 10043c2c f   effectmanager.obj
 0001:00042c36       __unwindfunclet$?CreateSpline@St_BodyCreate@@QAEXPAUSt_ElementCreate@@@Z$4 10043c36 f   effectmanager.obj
 0001:00042c40       __unwindfunclet$?CreateSpline@St_BodyCreate@@QAEXPAUSt_ElementCreate@@@Z$5 10043c40 f   effectmanager.obj
 0001:00042c4a       __unwindfunclet$?CreateSpline@St_BodyCreate@@QAEXPAUSt_ElementCreate@@@Z$6 10043c4a f   effectmanager.obj
 0001:00042c54       __unwindfunclet$?CreateSpline@St_BodyCreate@@QAEXPAUSt_ElementCreate@@@Z$7 10043c54 f   effectmanager.obj
 0001:00042c5e       __unwindfunclet$?CreateSpline@St_BodyCreate@@QAEXPAUSt_ElementCreate@@@Z$8 10043c5e f   effectmanager.obj
 0001:00042c68       __unwindfunclet$?CreateSpline@St_BodyCreate@@QAEXPAUSt_ElementCreate@@@Z$9 10043c68 f   effectmanager.obj
 0001:00042c75       __unwindfunclet$?CreateSpline@St_BodyCreate@@QAEXPAUSt_ElementCreate@@@Z$10 10043c75 f   effectmanager.obj
 0001:00042c82       __unwindfunclet$?CreateSpline@St_BodyCreate@@QAEXPAUSt_ElementCreate@@@Z$11 10043c82 f   effectmanager.obj
 0001:00042c8f       __unwindfunclet$?CreateSpline@St_BodyCreate@@QAEXPAUSt_ElementCreate@@@Z$12 10043c8f f   effectmanager.obj
 0001:00042c9c       __unwindfunclet$?CreateSpline@St_BodyCreate@@QAEXPAUSt_ElementCreate@@@Z$13 10043c9c f   effectmanager.obj
 0001:00042ca9       __unwindfunclet$?CreateSpline@St_BodyCreate@@QAEXPAUSt_ElementCreate@@@Z$14 10043ca9 f   effectmanager.obj
 0001:00042cb6       __unwindfunclet$?CreateSpline@St_BodyCreate@@QAEXPAUSt_ElementCreate@@@Z$15 10043cb6 f   effectmanager.obj
 0001:00042cc3       __unwindfunclet$?CreateSpline@St_BodyCreate@@QAEXPAUSt_ElementCreate@@@Z$16 10043cc3 f   effectmanager.obj
 0001:00042cd0       __unwindfunclet$?CreateSpline@St_BodyCreate@@QAEXPAUSt_ElementCreate@@@Z$17 10043cd0 f   effectmanager.obj
 0001:00042cdd       __unwindfunclet$?CreateSpline@St_BodyCreate@@QAEXPAUSt_ElementCreate@@@Z$18 10043cdd f   effectmanager.obj
 0001:00042cea       __unwindfunclet$?CreateSpline@St_BodyCreate@@QAEXPAUSt_ElementCreate@@@Z$19 10043cea f   effectmanager.obj
 0001:00042cf7       __unwindfunclet$?CreateSpline@St_BodyCreate@@QAEXPAUSt_ElementCreate@@@Z$20 10043cf7 f   effectmanager.obj
 0001:00042d04       __unwindfunclet$?CreateSpline@St_BodyCreate@@QAEXPAUSt_ElementCreate@@@Z$21 10043d04 f   effectmanager.obj
 0001:00042d11       __ehhandler$?CreateSpline@St_BodyCreate@@QAEXPAUSt_ElementCreate@@@Z 10043d11 f   effectmanager.obj
 0001:00042d2f       __unwindfunclet$??1St_Change_Info@@QAE@XZ$0 10043d2f f   effectmanager.obj
 0001:00042d3a       __unwindfunclet$??1St_Change_Info@@QAE@XZ$1 10043d3a f   effectmanager.obj
 0001:00042d48       __unwindfunclet$??1St_Change_Info@@QAE@XZ$2 10043d48 f   effectmanager.obj
 0001:00042d56       __unwindfunclet$??1St_Change_Info@@QAE@XZ$3 10043d56 f   effectmanager.obj
 0001:00042d64       __unwindfunclet$??1St_Change_Info@@QAE@XZ$4 10043d64 f   effectmanager.obj
 0001:00042d75       __unwindfunclet$??1St_Change_Info@@QAE@XZ$5 10043d75 f   effectmanager.obj
 0001:00042d86       __unwindfunclet$??1St_Change_Info@@QAE@XZ$6 10043d86 f   effectmanager.obj
 0001:00042d97       __unwindfunclet$??1St_Change_Info@@QAE@XZ$7 10043d97 f   effectmanager.obj
 0001:00042da8       __unwindfunclet$??1St_Change_Info@@QAE@XZ$8 10043da8 f   effectmanager.obj
 0001:00042db9       __unwindfunclet$??1St_Change_Info@@QAE@XZ$9 10043db9 f   effectmanager.obj
 0001:00042dca       __unwindfunclet$??1St_Change_Info@@QAE@XZ$10 10043dca f   effectmanager.obj
 0001:00042ddb       __unwindfunclet$??1St_Change_Info@@QAE@XZ$11 10043ddb f   effectmanager.obj
 0001:00042dec       __unwindfunclet$??1St_Change_Info@@QAE@XZ$12 10043dec f   effectmanager.obj
 0001:00042dfd       __unwindfunclet$??1St_Change_Info@@QAE@XZ$13 10043dfd f   effectmanager.obj
 0001:00042e0e       __unwindfunclet$??1St_Change_Info@@QAE@XZ$14 10043e0e f   effectmanager.obj
 0001:00042e1f       __unwindfunclet$??1St_Change_Info@@QAE@XZ$17 10043e1f f   effectmanager.obj
 0001:00042e27       __unwindfunclet$??1St_Change_Info@@QAE@XZ$24 10043e27 f   effectmanager.obj
 0001:00042e2f       __unwindfunclet$??1St_Change_Info@@QAE@XZ$31 10043e2f f   effectmanager.obj
 0001:00042e37       __unwindfunclet$??1St_Change_Info@@QAE@XZ$38 10043e37 f   effectmanager.obj
 0001:00042e3f       __unwindfunclet$??1St_Change_Info@@QAE@XZ$45 10043e3f f   effectmanager.obj
 0001:00042e47       __unwindfunclet$??1St_Change_Info@@QAE@XZ$52 10043e47 f   effectmanager.obj
 0001:00042e4f       __unwindfunclet$??1St_Change_Info@@QAE@XZ$59 10043e4f f   effectmanager.obj
 0001:00042e57       __unwindfunclet$??1St_Change_Info@@QAE@XZ$66 10043e57 f   effectmanager.obj
 0001:00042e5f       __unwindfunclet$??1St_Change_Info@@QAE@XZ$73 10043e5f f   effectmanager.obj
 0001:00042e67       __unwindfunclet$??1St_Change_Info@@QAE@XZ$80 10043e67 f   effectmanager.obj
 0001:00042e6f       __unwindfunclet$??1St_Change_Info@@QAE@XZ$87 10043e6f f   effectmanager.obj
 0001:00042e77       __unwindfunclet$??1St_Change_Info@@QAE@XZ$94 10043e77 f   effectmanager.obj
 0001:00042e7f       __unwindfunclet$??1St_Change_Info@@QAE@XZ$101 10043e7f f   effectmanager.obj
 0001:00042e87       __unwindfunclet$??1St_Change_Info@@QAE@XZ$108 10043e87 f   effectmanager.obj
 0001:00042e8f       __unwindfunclet$??1St_Change_Info@@QAE@XZ$115 10043e8f f   effectmanager.obj
 0001:00042e9a       __unwindfunclet$??1St_Change_Info@@QAE@XZ$122 10043e9a f   effectmanager.obj
 0001:00042ea5       __ehhandler$??1St_Change_Info@@QAE@XZ 10043ea5 f   effectmanager.obj
 0001:00042ec3       __unwindfunclet$??1St_Move_Info@@QAE@XZ$0 10043ec3 f   effectmanager.obj
 0001:00042ece       __unwindfunclet$??1St_Move_Info@@QAE@XZ$3 10043ece f   effectmanager.obj
 0001:00042ed6       __unwindfunclet$??1St_Move_Info@@QAE@XZ$10 10043ed6 f   effectmanager.obj
 0001:00042ede       __ehhandler$??1St_Move_Info@@QAE@XZ 10043ede f   effectmanager.obj
 0001:00042ef9       __unwindfunclet$??1St_Create_Info@@QAE@XZ$0 10043ef9 f   effectmanager.obj
 0001:00042f04       __unwindfunclet$??1St_Create_Info@@QAE@XZ$2 10043f04 f   effectmanager.obj
 0001:00042f0c       __unwindfunclet$??1St_Create_Info@@QAE@XZ$8 10043f0c f   effectmanager.obj
 0001:00042f14       __ehhandler$??1St_Create_Info@@QAE@XZ 10043f14 f   effectmanager.obj
 0001:00042f2f       __unwindfunclet$??0?$list@U?$pair@$$CBKPAUSt_BodyCreate@@@std@@V?$allocator@U?$pair@$$CBKPAUSt_BodyCreate@@@std@@@2@@std@@QAE@ABV?$allocator@U?$pair@$$CBKPAUSt_BodyCreate@@@std@@@1@@Z$0 10043f2f f   effectmanager.obj
 0001:00042f2f       __unwindfunclet$??0?$list@PAVCEElementBase@@V?$allocator@PAVCEElementBase@@@std@@@std@@QAE@XZ$0 10043f2f f   effectmanager.obj
 0001:00042f2f       __unwindfunclet$??0?$list@U?$pair@QAXPAVCEffectBody@@@std@@V?$allocator@U?$pair@QAXPAVCEffectBody@@@std@@@2@@std@@QAE@ABV?$allocator@U?$pair@QAXPAVCEffectBody@@@std@@@1@@Z$0 10043f2f f   effectmanager.obj
 0001:00042f2f       __unwindfunclet$??0?$list@PAVCEElementSprite@@V?$allocator@PAVCEElementSprite@@@std@@@std@@QAE@XZ$0 10043f2f f   effectmanager.obj
 0001:00042f2f       __unwindfunclet$??0?$list@KV?$allocator@K@std@@@std@@QAE@XZ$0 10043f2f f   effectmanager.obj
 0001:00042f2f       __unwindfunclet$??0?$list@U?$pair@$$CBKV?$basic_string@DU?$char_traits@D@std@@V?$allocator@D@2@@std@@@std@@V?$allocator@U?$pair@$$CBKV?$basic_string@DU?$char_traits@D@std@@V?$allocator@D@2@@std@@@std@@@2@@std@@QAE@ABV?$allocator@U?$pair@$$CBKV?$basic_string@DU?$char_traits@D@std@@V?$allocator@D@2@@std@@@std@@@1@@Z$0 10043f2f f   effectmanager.obj
 0001:00042f37       __ehhandler$??0?$list@KV?$allocator@K@std@@@std@@QAE@XZ 10043f37 f   effectmanager.obj
 0001:00042f37       __ehhandler$??0?$list@U?$pair@QAXPAVCEffectBody@@@std@@V?$allocator@U?$pair@QAXPAVCEffectBody@@@std@@@2@@std@@QAE@ABV?$allocator@U?$pair@QAXPAVCEffectBody@@@std@@@1@@Z 10043f37 f   effectmanager.obj
 0001:00042f37       __ehhandler$??0?$list@U?$pair@$$CBKPAUSt_BodyCreate@@@std@@V?$allocator@U?$pair@$$CBKPAUSt_BodyCreate@@@std@@@2@@std@@QAE@ABV?$allocator@U?$pair@$$CBKPAUSt_BodyCreate@@@std@@@1@@Z 10043f37 f   effectmanager.obj
 0001:00042f37       __ehhandler$??0?$list@PAVCEElementBase@@V?$allocator@PAVCEElementBase@@@std@@@std@@QAE@XZ 10043f37 f   effectmanager.obj
 0001:00042f37       __ehhandler$??0?$list@PAVCEElementSprite@@V?$allocator@PAVCEElementSprite@@@std@@@std@@QAE@XZ 10043f37 f   effectmanager.obj
 0001:00042f37       __ehhandler$??0?$list@U?$pair@$$CBKV?$basic_string@DU?$char_traits@D@std@@V?$allocator@D@2@@std@@@std@@V?$allocator@U?$pair@$$CBKV?$basic_string@DU?$char_traits@D@std@@V?$allocator@D@2@@std@@@std@@@2@@std@@QAE@ABV?$allocator@U?$pair@$$CBKV?$basic_string@DU?$char_traits@D@std@@V?$allocator@D@2@@std@@@std@@@1@@Z 10043f37 f   effectmanager.obj
 0001:00042f52       __unwindfunclet$??1?$_Hash@V?$_Hmap_traits@KPAUSt_BodyCreate@@V?$hash_compare@KU?$less@K@std@@@stdext@@V?$allocator@U?$pair@$$CBKPAUSt_BodyCreate@@@std@@@std@@$0A@@stdext@@@stdext@@QAE@XZ$0 10043f52 f   effectmanager.obj
 0001:00042f52       __unwindfunclet$??1?$_Hash@V?$_Hmap_traits@PAXPAVCEffectBody@@V?$hash_compare@PAXU?$less@PAX@std@@@stdext@@V?$allocator@U?$pair@QAXPAVCEffectBody@@@std@@@std@@$0A@@stdext@@@stdext@@QAE@XZ$0 10043f52 f   effectmanager.obj
 0001:00042f5a       __unwindfunclet$??1?$_Hash@V?$_Hmap_traits@KPAUSt_BodyCreate@@V?$hash_compare@KU?$less@K@std@@@stdext@@V?$allocator@U?$pair@$$CBKPAUSt_BodyCreate@@@std@@@std@@$0A@@stdext@@@stdext@@QAE@XZ$1 10043f5a f   effectmanager.obj
 0001:00042f5a       __unwindfunclet$??1?$_Hash@V?$_Hmap_traits@PAXPAVCEffectBody@@V?$hash_compare@PAXU?$less@PAX@std@@@stdext@@V?$allocator@U?$pair@QAXPAVCEffectBody@@@std@@@std@@$0A@@stdext@@@stdext@@QAE@XZ$1 10043f5a f   effectmanager.obj
 0001:00042f65       __unwindfunclet$??1?$_Hash@V?$_Hmap_traits@KPAUSt_BodyCreate@@V?$hash_compare@KU?$less@K@std@@@stdext@@V?$allocator@U?$pair@$$CBKPAUSt_BodyCreate@@@std@@@std@@$0A@@stdext@@@stdext@@QAE@XZ$3 10043f65 f   effectmanager.obj
 0001:00042f65       __unwindfunclet$??1?$_Hash@V?$_Hmap_traits@PAXPAVCEffectBody@@V?$hash_compare@PAXU?$less@PAX@std@@@stdext@@V?$allocator@U?$pair@QAXPAVCEffectBody@@@std@@@std@@$0A@@stdext@@@stdext@@QAE@XZ$3 10043f65 f   effectmanager.obj
 0001:00042f6d       __unwindfunclet$??1?$_Hash@V?$_Hmap_traits@KPAUSt_BodyCreate@@V?$hash_compare@KU?$less@K@std@@@stdext@@V?$allocator@U?$pair@$$CBKPAUSt_BodyCreate@@@std@@@std@@$0A@@stdext@@@stdext@@QAE@XZ$6 10043f6d f   effectmanager.obj
 0001:00042f6d       __unwindfunclet$??1?$_Hash@V?$_Hmap_traits@PAXPAVCEffectBody@@V?$hash_compare@PAXU?$less@PAX@std@@@stdext@@V?$allocator@U?$pair@QAXPAVCEffectBody@@@std@@@std@@$0A@@stdext@@@stdext@@QAE@XZ$6 10043f6d f   effectmanager.obj
 0001:00042f75       __ehhandler$??1?$_Hash@V?$_Hmap_traits@KPAUSt_BodyCreate@@V?$hash_compare@KU?$less@K@std@@@stdext@@V?$allocator@U?$pair@$$CBKPAUSt_BodyCreate@@@std@@@std@@$0A@@stdext@@@stdext@@QAE@XZ 10043f75 f   effectmanager.obj
 0001:00042f75       __ehhandler$??1?$_Hash@V?$_Hmap_traits@PAXPAVCEffectBody@@V?$hash_compare@PAXU?$less@PAX@std@@@stdext@@V?$allocator@U?$pair@QAXPAVCEffectBody@@@std@@@std@@$0A@@stdext@@@stdext@@QAE@XZ 10043f75 f   effectmanager.obj
 0001:00042f90       __unwindfunclet$??1?$vector@U_List_position@?$_Hash@V?$_Hmap_traits@KPAUSt_BodyCreate@@V?$hash_compare@KU?$less@K@std@@@stdext@@V?$allocator@U?$pair@$$CBKPAUSt_BodyCreate@@@std@@@std@@$0A@@stdext@@@stdext@@V?$allocator@U_List_position@?$_Hash@V?$_Hmap_traits@KPAUSt_BodyCreate@@V?$hash_compare@KU?$less@K@std@@@stdext@@V?$allocator@U?$pair@$$CBKPAUSt_BodyCreate@@@std@@@std@@$0A@@stdext@@@stdext@@@std@@@std@@QAE@XZ$0 10043f90 f   effectmanager.obj
 0001:00042f90       __unwindfunclet$??1?$vector@U_List_position@?$_Hash@V?$_Hmap_traits@PAXPAVCEffectBody@@V?$hash_compare@PAXU?$less@PAX@std@@@stdext@@V?$allocator@U?$pair@QAXPAVCEffectBody@@@std@@@std@@$0A@@stdext@@@stdext@@V?$allocator@U_List_position@?$_Hash@V?$_Hmap_traits@PAXPAVCEffectBody@@V?$hash_compare@PAXU?$less@PAX@std@@@stdext@@V?$allocator@U?$pair@QAXPAVCEffectBody@@@std@@@std@@$0A@@stdext@@@stdext@@@std@@@std@@QAE@XZ$0 10043f90 f   effectmanager.obj
 0001:00042f90       __unwindfunclet$??1?$vector@USt_AutoCtlParam@@V?$allocator@USt_AutoCtlParam@@@std@@@std@@QAE@XZ$0 10043f90 f   effectmanager.obj
 0001:00042f90       __unwindfunclet$??1?$vector@U_List_position@?$_Hash@V?$_Hmap_traits@KV?$basic_string@DU?$char_traits@D@std@@V?$allocator@D@2@@std@@V?$hash_compare@KU?$less@K@std@@@stdext@@V?$allocator@U?$pair@$$CBKV?$basic_string@DU?$char_traits@D@std@@V?$allocator@D@2@@std@@@std@@@2@$0A@@stdext@@@stdext@@V?$allocator@U_List_position@?$_Hash@V?$_Hmap_traits@KV?$basic_string@DU?$char_traits@D@std@@V?$allocator@D@2@@std@@V?$hash_compare@KU?$less@K@std@@@stdext@@V?$allocator@U?$pair@$$CBKV?$basic_string@DU?$char_traits@D@std@@V?$allocator@D@2@@std@@@std@@@2@$0A@@stdext@@@stdext@@@std@@@std@@QAE@XZ$0 10043f90 f   effectmanager.obj
 0001:00042f90       __unwindfunclet$??1?$vector@U_WZNCSPT@WzNaturalCubicSplineDyn@@V?$allocator@U_WZNCSPT@WzNaturalCubicSplineDyn@@@std@@@std@@QAE@XZ$0 10043f90 f   effectmanager.obj
 0001:00042f90       __unwindfunclet$??1?$vector@USt_EffLODParam@@V?$allocator@USt_EffLODParam@@@std@@@std@@QAE@XZ$0 10043f90 f   effectmanager.obj
 0001:00042f98       __ehhandler$??1?$vector@USt_AutoCtlParam@@V?$allocator@USt_AutoCtlParam@@@std@@@std@@QAE@XZ 10043f98 f   effectmanager.obj
 0001:00042f98       __ehhandler$??1?$vector@U_List_position@?$_Hash@V?$_Hmap_traits@PAXPAVCEffectBody@@V?$hash_compare@PAXU?$less@PAX@std@@@stdext@@V?$allocator@U?$pair@QAXPAVCEffectBody@@@std@@@std@@$0A@@stdext@@@stdext@@V?$allocator@U_List_position@?$_Hash@V?$_Hmap_traits@PAXPAVCEffectBody@@V?$hash_compare@PAXU?$less@PAX@std@@@stdext@@V?$allocator@U?$pair@QAXPAVCEffectBody@@@std@@@std@@$0A@@stdext@@@stdext@@@std@@@std@@QAE@XZ 10043f98 f   effectmanager.obj
 0001:00042f98       __ehhandler$??1?$vector@USt_EffLODParam@@V?$allocator@USt_EffLODParam@@@std@@@std@@QAE@XZ 10043f98 f   effectmanager.obj
 0001:00042f98       __ehhandler$??1?$vector@U_List_position@?$_Hash@V?$_Hmap_traits@KPAUSt_BodyCreate@@V?$hash_compare@KU?$less@K@std@@@stdext@@V?$allocator@U?$pair@$$CBKPAUSt_BodyCreate@@@std@@@std@@$0A@@stdext@@@stdext@@V?$allocator@U_List_position@?$_Hash@V?$_Hmap_traits@KPAUSt_BodyCreate@@V?$hash_compare@KU?$less@K@std@@@stdext@@V?$allocator@U?$pair@$$CBKPAUSt_BodyCreate@@@std@@@std@@$0A@@stdext@@@stdext@@@std@@@std@@QAE@XZ 10043f98 f   effectmanager.obj
 0001:00042f98       __ehhandler$??1?$vector@U_List_position@?$_Hash@V?$_Hmap_traits@KV?$basic_string@DU?$char_traits@D@std@@V?$allocator@D@2@@std@@V?$hash_compare@KU?$less@K@std@@@stdext@@V?$allocator@U?$pair@$$CBKV?$basic_string@DU?$char_traits@D@std@@V?$allocator@D@2@@std@@@std@@@2@$0A@@stdext@@@stdext@@V?$allocator@U_List_position@?$_Hash@V?$_Hmap_traits@KV?$basic_string@DU?$char_traits@D@std@@V?$allocator@D@2@@std@@V?$hash_compare@KU?$less@K@std@@@stdext@@V?$allocator@U?$pair@$$CBKV?$basic_string@DU?$char_traits@D@std@@V?$allocator@D@2@@std@@@std@@@2@$0A@@stdext@@@stdext@@@std@@@std@@QAE@XZ 10043f98 f   effectmanager.obj
 0001:00042f98       __ehhandler$??1?$vector@U_WZNCSPT@WzNaturalCubicSplineDyn@@V?$allocator@U_WZNCSPT@WzNaturalCubicSplineDyn@@@std@@@std@@QAE@XZ 10043f98 f   effectmanager.obj
 0001:00042fb3       __unwindfunclet$?erase@?$_Tree@V?$_Tmap_traits@JMU?$less@J@std@@V?$allocator@U?$pair@$$CBJM@std@@@2@$0A@@std@@@std@@QAE?AViterator@12@Vconst_iterator@12@@Z$0 10043fb3 f   effectmanager.obj
 0001:00042fb3       __unwindfunclet$?erase@?$_Tree@V?$_Tmap_traits@JUWzVector@@U?$less@J@std@@V?$allocator@U?$pair@$$CBJUWzVector@@@std@@@3@$0A@@std@@@std@@QAE?AViterator@12@Vconst_iterator@12@@Z$0 10043fb3 f   effectmanager.obj
 0001:00042fbb       __ehhandler$?erase@?$_Tree@V?$_Tmap_traits@JUWzVector@@U?$less@J@std@@V?$allocator@U?$pair@$$CBJUWzVector@@@std@@@3@$0A@@std@@@std@@QAE?AViterator@12@Vconst_iterator@12@@Z 10043fbb f   effectmanager.obj
 0001:00042fbb       __ehhandler$?erase@?$_Tree@V?$_Tmap_traits@JMU?$less@J@std@@V?$allocator@U?$pair@$$CBJM@std@@@2@$0A@@std@@@std@@QAE?AViterator@12@Vconst_iterator@12@@Z 10043fbb f   effectmanager.obj
 0001:00042fd9       __unwindfunclet$??0logic_error@std@@QAE@ABV?$basic_string@DU?$char_traits@D@std@@V?$allocator@D@2@@1@@Z$0 10043fd9 f   effectmanager.obj
 0001:00042fd9       __unwindfunclet$??0logic_error@std@@QAE@ABV01@@Z$0 10043fd9 f   effectmanager.obj
 0001:00042fe1       __ehhandler$??0logic_error@std@@QAE@ABV?$basic_string@DU?$char_traits@D@std@@V?$allocator@D@2@@1@@Z 10043fe1 f   effectmanager.obj
 0001:00042fe1       __ehhandler$??0logic_error@std@@QAE@ABV01@@Z 10043fe1 f   effectmanager.obj
 0001:00042ffc       __ehhandler$?_Copy@?$basic_string@DU?$char_traits@D@std@@V?$allocator@D@2@@std@@IAEXII@Z 10043ffc f   effectmanager.obj
 0001:0004301a       __ehhandler$?_Buynode@?$list@PAVCEElementSprite@@V?$allocator@PAVCEElementSprite@@@std@@@std@@IAEPAU_Node@?$_List_nod@PAVCEElementSprite@@V?$allocator@PAVCEElementSprite@@@std@@@2@XZ 1004401a f   effectmanager.obj
 0001:0004301a       __ehhandler$?_Buynode@?$list@PAVCEElementBase@@V?$allocator@PAVCEElementBase@@@std@@@std@@IAEPAU_Node@?$_List_nod@PAVCEElementBase@@V?$allocator@PAVCEElementBase@@@std@@@2@XZ 1004401a f   effectmanager.obj
 0001:0004301a       __ehhandler$?_Buynode@?$list@KV?$allocator@K@std@@@std@@IAEPAU_Node@?$_List_nod@KV?$allocator@K@std@@@2@XZ 1004401a f   effectmanager.obj
 0001:00043035       __unwindfunclet$??0?$_Tree@V?$_Tmap_traits@JUWzVector@@U?$less@J@std@@V?$allocator@U?$pair@$$CBJUWzVector@@@std@@@3@$0A@@std@@@std@@QAE@ABU?$less@J@1@ABV?$allocator@U?$pair@$$CBJUWzVector@@@std@@@1@@Z$0 10044035 f   effectmanager.obj
 0001:00043035       __unwindfunclet$??0?$_Tree@V?$_Tmap_traits@JMU?$less@J@std@@V?$allocator@U?$pair@$$CBJM@std@@@2@$0A@@std@@@std@@QAE@ABU?$less@J@1@ABV?$allocator@U?$pair@$$CBJM@std@@@1@@Z$0 10044035 f   effectmanager.obj
 0001:0004303d       __ehhandler$??0?$_Tree@V?$_Tmap_traits@JMU?$less@J@std@@V?$allocator@U?$pair@$$CBJM@std@@@2@$0A@@std@@@std@@QAE@ABU?$less@J@1@ABV?$allocator@U?$pair@$$CBJM@std@@@1@@Z 1004403d f   effectmanager.obj
 0001:0004303d       __ehhandler$??0?$_Tree@V?$_Tmap_traits@JUWzVector@@U?$less@J@std@@V?$allocator@U?$pair@$$CBJUWzVector@@@std@@@3@$0A@@std@@@std@@QAE@ABU?$less@J@1@ABV?$allocator@U?$pair@$$CBJUWzVector@@@std@@@1@@Z 1004403d f   effectmanager.obj
 0001:00043058       __unwindfunclet$??0?$_Hash@V?$_Hmap_traits@KPAUSt_BodyCreate@@V?$hash_compare@KU?$less@K@std@@@stdext@@V?$allocator@U?$pair@$$CBKPAUSt_BodyCreate@@@std@@@std@@$0A@@stdext@@@stdext@@QAE@ABV?$hash_compare@KU?$less@K@std@@@1@ABV?$allocator@U?$pair@$$CBKPAUSt_BodyCreate@@@std@@@std@@@Z$0 10044058 f   effectmanager.obj
 0001:00043058       __unwindfunclet$??0?$_Hash@V?$_Hmap_traits@PAXPAVCEffectBody@@V?$hash_compare@PAXU?$less@PAX@std@@@stdext@@V?$allocator@U?$pair@QAXPAVCEffectBody@@@std@@@std@@$0A@@stdext@@@stdext@@QAE@ABV?$hash_compare@PAXU?$less@PAX@std@@@1@ABV?$allocator@U?$pair@QAXPAVCEffectBody@@@std@@@std@@@Z$0 10044058 f   effectmanager.obj
 0001:00043063       __unwindfunclet$??0?$_Hash@V?$_Hmap_traits@PAXPAVCEffectBody@@V?$hash_compare@PAXU?$less@PAX@std@@@stdext@@V?$allocator@U?$pair@QAXPAVCEffectBody@@@std@@@std@@$0A@@stdext@@@stdext@@QAE@ABV?$hash_compare@PAXU?$less@PAX@std@@@1@ABV?$allocator@U?$pair@QAXPAVCEffectBody@@@std@@@std@@@Z$1 10044063 f   effectmanager.obj
 0001:00043063       __unwindfunclet$??0?$_Hash@V?$_Hmap_traits@KPAUSt_BodyCreate@@V?$hash_compare@KU?$less@K@std@@@stdext@@V?$allocator@U?$pair@$$CBKPAUSt_BodyCreate@@@std@@@std@@$0A@@stdext@@@stdext@@QAE@ABV?$hash_compare@KU?$less@K@std@@@1@ABV?$allocator@U?$pair@$$CBKPAUSt_BodyCreate@@@std@@@std@@@Z$1 10044063 f   effectmanager.obj
 0001:00043071       __unwindfunclet$??0?$_Hash@V?$_Hmap_traits@KPAUSt_BodyCreate@@V?$hash_compare@KU?$less@K@std@@@stdext@@V?$allocator@U?$pair@$$CBKPAUSt_BodyCreate@@@std@@@std@@$0A@@stdext@@@stdext@@QAE@ABV?$hash_compare@KU?$less@K@std@@@1@ABV?$allocator@U?$pair@$$CBKPAUSt_BodyCreate@@@std@@@std@@@Z$2 10044071 f   effectmanager.obj
 0001:00043071       __unwindfunclet$??0?$_Hash@V?$_Hmap_traits@PAXPAVCEffectBody@@V?$hash_compare@PAXU?$less@PAX@std@@@stdext@@V?$allocator@U?$pair@QAXPAVCEffectBody@@@std@@@std@@$0A@@stdext@@@stdext@@QAE@ABV?$hash_compare@PAXU?$less@PAX@std@@@1@ABV?$allocator@U?$pair@QAXPAVCEffectBody@@@std@@@std@@@Z$2 10044071 f   effectmanager.obj
 0001:0004307f       __ehhandler$??0?$_Hash@V?$_Hmap_traits@KPAUSt_BodyCreate@@V?$hash_compare@KU?$less@K@std@@@stdext@@V?$allocator@U?$pair@$$CBKPAUSt_BodyCreate@@@std@@@std@@$0A@@stdext@@@stdext@@QAE@ABV?$hash_compare@KU?$less@K@std@@@1@ABV?$allocator@U?$pair@$$CBKPAUSt_BodyCreate@@@std@@@std@@@Z 1004407f f   effectmanager.obj
 0001:0004307f       __ehhandler$??0?$_Hash@V?$_Hmap_traits@PAXPAVCEffectBody@@V?$hash_compare@PAXU?$less@PAX@std@@@stdext@@V?$allocator@U?$pair@QAXPAVCEffectBody@@@std@@@std@@$0A@@stdext@@@stdext@@QAE@ABV?$hash_compare@PAXU?$less@PAX@std@@@1@ABV?$allocator@U?$pair@QAXPAVCEffectBody@@@std@@@std@@@Z 1004407f f   effectmanager.obj
 0001:0004309d       __unwindfunclet$??1?$list@KV?$allocator@K@std@@@std@@QAE@XZ$0 1004409d f   effectmanager.obj
 0001:0004309d       __unwindfunclet$??1?$list@PAVCEElementBase@@V?$allocator@PAVCEElementBase@@@std@@@std@@QAE@XZ$0 1004409d f   effectmanager.obj
 0001:0004309d       __unwindfunclet$??1?$list@U?$pair@$$CBKPAUSt_BodyCreate@@@std@@V?$allocator@U?$pair@$$CBKPAUSt_BodyCreate@@@std@@@2@@std@@QAE@XZ$0 1004409d f   effectmanager.obj
 0001:0004309d       __unwindfunclet$??1?$list@U?$pair@QAXPAVCEffectBody@@@std@@V?$allocator@U?$pair@QAXPAVCEffectBody@@@std@@@2@@std@@QAE@XZ$0 1004409d f   effectmanager.obj
 0001:000430a5       __ehhandler$??1?$list@U?$pair@QAXPAVCEffectBody@@@std@@V?$allocator@U?$pair@QAXPAVCEffectBody@@@std@@@2@@std@@QAE@XZ 100440a5 f   effectmanager.obj
 0001:000430a5       __ehhandler$??1?$list@KV?$allocator@K@std@@@std@@QAE@XZ 100440a5 f   effectmanager.obj
 0001:000430a5       __ehhandler$??1?$list@PAVCEElementBase@@V?$allocator@PAVCEElementBase@@@std@@@std@@QAE@XZ 100440a5 f   effectmanager.obj
 0001:000430a5       __ehhandler$??1?$list@U?$pair@$$CBKPAUSt_BodyCreate@@@std@@V?$allocator@U?$pair@$$CBKPAUSt_BodyCreate@@@std@@@2@@std@@QAE@XZ 100440a5 f   effectmanager.obj
 0001:000430c0       __ehhandler$?_Copy@?$_Tree@V?$_Tmap_traits@JUWzVector@@U?$less@J@std@@V?$allocator@U?$pair@$$CBJUWzVector@@@std@@@3@$0A@@std@@@std@@IAEPAU_Node@?$_Tree_nod@V?$_Tmap_traits@JUWzVector@@U?$less@J@std@@V?$allocator@U?$pair@$$CBJUWzVector@@@std@@@3@$0A@@std@@@2@PAU342@0@Z 100440c0 f   effectmanager.obj
 0001:000430db       __ehhandler$?_Copy@?$_Tree@V?$_Tmap_traits@JMU?$less@J@std@@V?$allocator@U?$pair@$$CBJM@std@@@2@$0A@@std@@@std@@IAEPAU_Node@?$_Tree_nod@V?$_Tmap_traits@JMU?$less@J@std@@V?$allocator@U?$pair@$$CBJM@std@@@2@$0A@@std@@@2@PAU342@0@Z 100440db f   effectmanager.obj
 0001:000430f6       __unwindfunclet$??0?$_Container_base_aux_alloc_real@V?$allocator@U_List_position@?$_Hash@V?$_Hmap_traits@PAXPAVCEffectBody@@V?$hash_compare@PAXU?$less@PAX@std@@@stdext@@V?$allocator@U?$pair@QAXPAVCEffectBody@@@std@@@std@@$0A@@stdext@@@stdext@@@std@@@std@@IAE@V?$allocator@U_List_position@?$_Hash@V?$_Hmap_traits@PAXPAVCEffectBody@@V?$hash_compare@PAXU?$less@PAX@std@@@stdext@@V?$allocator@U?$pair@QAXPAVCEffectBody@@@std@@@std@@$0A@@stdext@@@stdext@@@1@@Z$0 100440f6 f   effectmanager.obj
 0001:000430f6       __unwindfunclet$??0?$_Container_base_aux_alloc_real@V?$allocator@PAUsEffectTexture@CEffectManager@@@std@@@std@@IAE@V?$allocator@PAUsEffectTexture@CEffectManager@@@1@@Z$0 100440f6 f   effectmanager.obj
 0001:000430f6       __unwindfunclet$??0?$_Container_base_aux_alloc_real@V?$allocator@K@std@@@std@@IAE@V?$allocator@K@1@@Z$0 100440f6 f   effectmanager.obj
 0001:000430f6       __unwindfunclet$??0?$_Container_base_aux_alloc_real@V?$allocator@U_List_position@?$_Hash@V?$_Hmap_traits@KPAUSt_BodyCreate@@V?$hash_compare@KU?$less@K@std@@@stdext@@V?$allocator@U?$pair@$$CBKPAUSt_BodyCreate@@@std@@@std@@$0A@@stdext@@@stdext@@@std@@@std@@IAE@V?$allocator@U_List_position@?$_Hash@V?$_Hmap_traits@KPAUSt_BodyCreate@@V?$hash_compare@KU?$less@K@std@@@stdext@@V?$allocator@U?$pair@$$CBKPAUSt_BodyCreate@@@std@@@std@@$0A@@stdext@@@stdext@@@1@@Z$0 100440f6 f   effectmanager.obj
 0001:000430f6       __unwindfunclet$??0?$_Container_base_aux_alloc_real@V?$allocator@PAVCEElementSprite@@@std@@@std@@IAE@V?$allocator@PAVCEElementSprite@@@1@@Z$0 100440f6 f   effectmanager.obj
 0001:000430f6       __unwindfunclet$??0?$_Container_base_aux_alloc_real@V?$allocator@PAVCEElementBase@@@std@@@std@@IAE@V?$allocator@PAVCEElementBase@@@1@@Z$0 100440f6 f   effectmanager.obj
 0001:000430f6       __unwindfunclet$??0?$_Container_base_aux_alloc_real@V?$allocator@USt_AutoCtlParam@@@std@@@std@@IAE@V?$allocator@USt_AutoCtlParam@@@1@@Z$0 100440f6 f   effectmanager.obj
 0001:000430f6       __unwindfunclet$??0?$_Container_base_aux_alloc_real@V?$allocator@U?$pair@$$CBJUWzVector@@@std@@@std@@@std@@IAE@V?$allocator@U?$pair@$$CBJUWzVector@@@std@@@1@@Z$0 100440f6 f   effectmanager.obj
 0001:000430f6       __unwindfunclet$??0?$_Container_base_aux_alloc_real@V?$allocator@PAUSt_SoundInfo@@@std@@@std@@IAE@V?$allocator@PAUSt_SoundInfo@@@1@@Z$0 100440f6 f   effectmanager.obj
 0001:000430f6       __unwindfunclet$??0?$_Container_base_aux_alloc_real@V?$allocator@U?$pair@$$CBJM@std@@@std@@@std@@IAE@V?$allocator@U?$pair@$$CBJM@std@@@1@@Z$0 100440f6 f   effectmanager.obj
 0001:000430f6       __unwindfunclet$??0?$_Container_base_aux_alloc_real@V?$allocator@PAX@std@@@std@@IAE@V?$allocator@PAX@1@@Z$0 100440f6 f   effectmanager.obj
 0001:000430f6       __unwindfunclet$??0?$_Container_base_aux_alloc_real@V?$allocator@U_WZNCSPT@WzNaturalCubicSplineDyn@@@std@@@std@@IAE@V?$allocator@U_WZNCSPT@WzNaturalCubicSplineDyn@@@1@@Z$0 100440f6 f   effectmanager.obj
 0001:000430f6       __unwindfunclet$??0?$_Container_base_aux_alloc_real@V?$allocator@USt_EffLODParam@@@std@@@std@@IAE@V?$allocator@USt_EffLODParam@@@1@@Z$0 100440f6 f   effectmanager.obj
 0001:000430f6       __unwindfunclet$??0?$_Container_base_aux_alloc_real@V?$allocator@U?$pair@$$CBKPAUSt_BodyCreate@@@std@@@std@@@std@@IAE@V?$allocator@U?$pair@$$CBKPAUSt_BodyCreate@@@std@@@1@@Z$0 100440f6 f   effectmanager.obj
 0001:000430f6       __unwindfunclet$??0?$_Container_base_aux_alloc_real@V?$allocator@U?$pair@$$CBKV?$basic_string@DU?$char_traits@D@std@@V?$allocator@D@2@@std@@@std@@@std@@@std@@IAE@V?$allocator@U?$pair@$$CBKV?$basic_string@DU?$char_traits@D@std@@V?$allocator@D@2@@std@@@std@@@1@@Z$0 100440f6 f   effectmanager.obj
 0001:000430f6       __unwindfunclet$??0?$_Container_base_aux_alloc_real@V?$allocator@U?$pair@QAXPAVCEffectBody@@@std@@@std@@@std@@IAE@V?$allocator@U?$pair@QAXPAVCEffectBody@@@std@@@1@@Z$0 100440f6 f   effectmanager.obj
 0001:000430f6       __unwindfunclet$??0?$_Container_base_aux_alloc_real@V?$allocator@U_List_position@?$_Hash@V?$_Hmap_traits@KV?$basic_string@DU?$char_traits@D@std@@V?$allocator@D@2@@std@@V?$hash_compare@KU?$less@K@std@@@stdext@@V?$allocator@U?$pair@$$CBKV?$basic_string@DU?$char_traits@D@std@@V?$allocator@D@2@@std@@@std@@@2@$0A@@stdext@@@stdext@@@std@@@std@@IAE@V?$allocator@U_List_position@?$_Hash@V?$_Hmap_traits@KV?$basic_string@DU?$char_traits@D@std@@V?$allocator@D@2@@std@@V?$hash_compare@KU?$less@K@std@@@stdext@@V?$allocator@U?$pair@$$CBKV?$basic_string@DU?$char_traits@D@std@@V?$allocator@D@2@@std@@@std@@@2@$0A@@stdext@@@stdext@@@1@@Z$0 100440f6 f   effectmanager.obj
 0001:000430fe       __ehhandler$??0?$_Container_base_aux_alloc_real@V?$allocator@U_List_position@?$_Hash@V?$_Hmap_traits@KV?$basic_string@DU?$char_traits@D@std@@V?$allocator@D@2@@std@@V?$hash_compare@KU?$less@K@std@@@stdext@@V?$allocator@U?$pair@$$CBKV?$basic_string@DU?$char_traits@D@std@@V?$allocator@D@2@@std@@@std@@@2@$0A@@stdext@@@stdext@@@std@@@std@@IAE@V?$allocator@U_List_position@?$_Hash@V?$_Hmap_traits@KV?$basic_string@DU?$char_traits@D@std@@V?$allocator@D@2@@std@@V?$hash_compare@KU?$less@K@std@@@stdext@@V?$allocator@U?$pair@$$CBKV?$basic_string@DU?$char_traits@D@std@@V?$allocator@D@2@@std@@@std@@@2@$0A@@stdext@@@stdext@@@1@@Z 100440fe f   effectmanager.obj
 0001:000430fe       __ehhandler$??0?$_Container_base_aux_alloc_real@V?$allocator@USt_EffLODParam@@@std@@@std@@IAE@V?$allocator@USt_EffLODParam@@@1@@Z 100440fe f   effectmanager.obj
 0001:000430fe       __ehhandler$??0?$_Container_base_aux_alloc_real@V?$allocator@U?$pair@QAXPAVCEffectBody@@@std@@@std@@@std@@IAE@V?$allocator@U?$pair@QAXPAVCEffectBody@@@std@@@1@@Z 100440fe f   effectmanager.obj
 0001:000430fe       __ehhandler$??0?$_Container_base_aux_alloc_real@V?$allocator@U?$pair@$$CBKPAUSt_BodyCreate@@@std@@@std@@@std@@IAE@V?$allocator@U?$pair@$$CBKPAUSt_BodyCreate@@@std@@@1@@Z 100440fe f   effectmanager.obj
 0001:000430fe       __ehhandler$??0?$_Container_base_aux_alloc_real@V?$allocator@U?$pair@$$CBJM@std@@@std@@@std@@IAE@V?$allocator@U?$pair@$$CBJM@std@@@1@@Z 100440fe f   effectmanager.obj
 0001:000430fe       __ehhandler$??0?$_Container_base_aux_alloc_real@V?$allocator@PAX@std@@@std@@IAE@V?$allocator@PAX@1@@Z 100440fe f   effectmanager.obj
 0001:000430fe       __ehhandler$??0?$_Container_base_aux_alloc_real@V?$allocator@U?$pair@$$CBJUWzVector@@@std@@@std@@@std@@IAE@V?$allocator@U?$pair@$$CBJUWzVector@@@std@@@1@@Z 100440fe f   effectmanager.obj
 0001:000430fe       __ehhandler$??0?$_Container_base_aux_alloc_real@V?$allocator@PAUSt_SoundInfo@@@std@@@std@@IAE@V?$allocator@PAUSt_SoundInfo@@@1@@Z 100440fe f   effectmanager.obj
 0001:000430fe       __ehhandler$??0?$_Container_base_aux_alloc_real@V?$allocator@U?$pair@$$CBKV?$basic_string@DU?$char_traits@D@std@@V?$allocator@D@2@@std@@@std@@@std@@@std@@IAE@V?$allocator@U?$pair@$$CBKV?$basic_string@DU?$char_traits@D@std@@V?$allocator@D@2@@std@@@std@@@1@@Z 100440fe f   effectmanager.obj
 0001:000430fe       __ehhandler$??0?$_Container_base_aux_alloc_real@V?$allocator@USt_AutoCtlParam@@@std@@@std@@IAE@V?$allocator@USt_AutoCtlParam@@@1@@Z 100440fe f   effectmanager.obj
 0001:000430fe       __ehhandler$??0?$_Container_base_aux_alloc_real@V?$allocator@K@std@@@std@@IAE@V?$allocator@K@1@@Z 100440fe f   effectmanager.obj
 0001:000430fe       __ehhandler$??0?$_Container_base_aux_alloc_real@V?$allocator@U_List_position@?$_Hash@V?$_Hmap_traits@PAXPAVCEffectBody@@V?$hash_compare@PAXU?$less@PAX@std@@@stdext@@V?$allocator@U?$pair@QAXPAVCEffectBody@@@std@@@std@@$0A@@stdext@@@stdext@@@std@@@std@@IAE@V?$allocator@U_List_position@?$_Hash@V?$_Hmap_traits@PAXPAVCEffectBody@@V?$hash_compare@PAXU?$less@PAX@std@@@stdext@@V?$allocator@U?$pair@QAXPAVCEffectBody@@@std@@@std@@$0A@@stdext@@@stdext@@@1@@Z 100440fe f   effectmanager.obj
 0001:000430fe       __ehhandler$??0?$_Container_base_aux_alloc_real@V?$allocator@PAVCEElementSprite@@@std@@@std@@IAE@V?$allocator@PAVCEElementSprite@@@1@@Z 100440fe f   effectmanager.obj
 0001:000430fe       __ehhandler$??0?$_Container_base_aux_alloc_real@V?$allocator@PAUsEffectTexture@CEffectManager@@@std@@@std@@IAE@V?$allocator@PAUsEffectTexture@CEffectManager@@@1@@Z 100440fe f   effectmanager.obj
 0001:000430fe       __ehhandler$??0?$_Container_base_aux_alloc_real@V?$allocator@U_List_position@?$_Hash@V?$_Hmap_traits@KPAUSt_BodyCreate@@V?$hash_compare@KU?$less@K@std@@@stdext@@V?$allocator@U?$pair@$$CBKPAUSt_BodyCreate@@@std@@@std@@$0A@@stdext@@@stdext@@@std@@@std@@IAE@V?$allocator@U_List_position@?$_Hash@V?$_Hmap_traits@KPAUSt_BodyCreate@@V?$hash_compare@KU?$less@K@std@@@stdext@@V?$allocator@U?$pair@$$CBKPAUSt_BodyCreate@@@std@@@std@@$0A@@stdext@@@stdext@@@1@@Z 100440fe f   effectmanager.obj
 0001:000430fe       __ehhandler$??0?$_Container_base_aux_alloc_real@V?$allocator@U_WZNCSPT@WzNaturalCubicSplineDyn@@@std@@@std@@IAE@V?$allocator@U_WZNCSPT@WzNaturalCubicSplineDyn@@@1@@Z 100440fe f   effectmanager.obj
 0001:000430fe       __ehhandler$??0?$_Container_base_aux_alloc_real@V?$allocator@PAVCEElementBase@@@std@@@std@@IAE@V?$allocator@PAVCEElementBase@@@1@@Z 100440fe f   effectmanager.obj
 0001:00043119       __unwindfunclet$??0?$vector@U_List_position@?$_Hash@V?$_Hmap_traits@PAXPAVCEffectBody@@V?$hash_compare@PAXU?$less@PAX@std@@@stdext@@V?$allocator@U?$pair@QAXPAVCEffectBody@@@std@@@std@@$0A@@stdext@@@stdext@@V?$allocator@U_List_position@?$_Hash@V?$_Hmap_traits@PAXPAVCEffectBody@@V?$hash_compare@PAXU?$less@PAX@std@@@stdext@@V?$allocator@U?$pair@QAXPAVCEffectBody@@@std@@@std@@$0A@@stdext@@@stdext@@@std@@@std@@QAE@ABV?$allocator@U_List_position@?$_Hash@V?$_Hmap_traits@PAXPAVCEffectBody@@V?$hash_compare@PAXU?$less@PAX@std@@@stdext@@V?$allocator@U?$pair@QAXPAVCEffectBody@@@std@@@std@@$0A@@stdext@@@stdext@@@1@@Z$0 10044119 f   effectmanager.obj
 0001:00043119       __unwindfunclet$??0?$vector@USt_AutoCtlParam@@V?$allocator@USt_AutoCtlParam@@@std@@@std@@QAE@XZ$0 10044119 f   effectmanager.obj
 0001:00043119       __unwindfunclet$??0?$vector@U_List_position@?$_Hash@V?$_Hmap_traits@KV?$basic_string@DU?$char_traits@D@std@@V?$allocator@D@2@@std@@V?$hash_compare@KU?$less@K@std@@@stdext@@V?$allocator@U?$pair@$$CBKV?$basic_string@DU?$char_traits@D@std@@V?$allocator@D@2@@std@@@std@@@2@$0A@@stdext@@@stdext@@V?$allocator@U_List_position@?$_Hash@V?$_Hmap_traits@KV?$basic_string@DU?$char_traits@D@std@@V?$allocator@D@2@@std@@V?$hash_compare@KU?$less@K@std@@@stdext@@V?$allocator@U?$pair@$$CBKV?$basic_string@DU?$char_traits@D@std@@V?$allocator@D@2@@std@@@std@@@2@$0A@@stdext@@@stdext@@@std@@@std@@QAE@ABV?$allocator@U_List_position@?$_Hash@V?$_Hmap_traits@KV?$basic_string@DU?$char_traits@D@std@@V?$allocator@D@2@@std@@V?$hash_compare@KU?$less@K@std@@@stdext@@V?$allocator@U?$pair@$$CBKV?$basic_string@DU?$char_traits@D@std@@V?$allocator@D@2@@std@@@std@@@2@$0A@@stdext@@@stdext@@@1@@Z$0 10044119 f   effectmanager.obj
 0001:00043119       __unwindfunclet$??0?$vector@PAUsEffectTexture@CEffectManager@@V?$allocator@PAUsEffectTexture@CEffectManager@@@std@@@std@@QAE@XZ$0 10044119 f   effectmanager.obj
 0001:00043119       __unwindfunclet$??0?$vector@PAXV?$allocator@PAX@std@@@std@@QAE@XZ$0 10044119 f   effectmanager.obj
 0001:00043119       __unwindfunclet$??0?$vector@PAUSt_SoundInfo@@V?$allocator@PAUSt_SoundInfo@@@std@@@std@@QAE@XZ$0 10044119 f   effectmanager.obj
 0001:00043119       __unwindfunclet$??0?$vector@USt_EffLODParam@@V?$allocator@USt_EffLODParam@@@std@@@std@@QAE@XZ$0 10044119 f   effectmanager.obj
 0001:00043119       __unwindfunclet$??0?$vector@U_WZNCSPT@WzNaturalCubicSplineDyn@@V?$allocator@U_WZNCSPT@WzNaturalCubicSplineDyn@@@std@@@std@@QAE@XZ$0 10044119 f   effectmanager.obj
 0001:00043119       __unwindfunclet$??0?$vector@U_List_position@?$_Hash@V?$_Hmap_traits@KPAUSt_BodyCreate@@V?$hash_compare@KU?$less@K@std@@@stdext@@V?$allocator@U?$pair@$$CBKPAUSt_BodyCreate@@@std@@@std@@$0A@@stdext@@@stdext@@V?$allocator@U_List_position@?$_Hash@V?$_Hmap_traits@KPAUSt_BodyCreate@@V?$hash_compare@KU?$less@K@std@@@stdext@@V?$allocator@U?$pair@$$CBKPAUSt_BodyCreate@@@std@@@std@@$0A@@stdext@@@stdext@@@std@@@std@@QAE@ABV?$allocator@U_List_position@?$_Hash@V?$_Hmap_traits@KPAUSt_BodyCreate@@V?$hash_compare@KU?$less@K@std@@@stdext@@V?$allocator@U?$pair@$$CBKPAUSt_BodyCreate@@@std@@@std@@$0A@@stdext@@@stdext@@@1@@Z$0 10044119 f   effectmanager.obj
 0001:00043124       __ehhandler$??0?$vector@U_List_position@?$_Hash@V?$_Hmap_traits@KPAUSt_BodyCreate@@V?$hash_compare@KU?$less@K@std@@@stdext@@V?$allocator@U?$pair@$$CBKPAUSt_BodyCreate@@@std@@@std@@$0A@@stdext@@@stdext@@V?$allocator@U_List_position@?$_Hash@V?$_Hmap_traits@KPAUSt_BodyCreate@@V?$hash_compare@KU?$less@K@std@@@stdext@@V?$allocator@U?$pair@$$CBKPAUSt_BodyCreate@@@std@@@std@@$0A@@stdext@@@stdext@@@std@@@std@@QAE@ABV?$allocator@U_List_position@?$_Hash@V?$_Hmap_traits@KPAUSt_BodyCreate@@V?$hash_compare@KU?$less@K@std@@@stdext@@V?$allocator@U?$pair@$$CBKPAUSt_BodyCreate@@@std@@@std@@$0A@@stdext@@@stdext@@@1@@Z 10044124 f   effectmanager.obj
 0001:00043124       __ehhandler$??0?$vector@USt_AutoCtlParam@@V?$allocator@USt_AutoCtlParam@@@std@@@std@@QAE@XZ 10044124 f   effectmanager.obj
 0001:00043124       __ehhandler$??0?$vector@PAXV?$allocator@PAX@std@@@std@@QAE@XZ 10044124 f   effectmanager.obj
 0001:00043124       __ehhandler$??0?$vector@U_WZNCSPT@WzNaturalCubicSplineDyn@@V?$allocator@U_WZNCSPT@WzNaturalCubicSplineDyn@@@std@@@std@@QAE@XZ 10044124 f   effectmanager.obj
 0001:00043124       __ehhandler$??0?$vector@USt_EffLODParam@@V?$allocator@USt_EffLODParam@@@std@@@std@@QAE@XZ 10044124 f   effectmanager.obj
 0001:00043124       __ehhandler$??0?$vector@PAUSt_SoundInfo@@V?$allocator@PAUSt_SoundInfo@@@std@@@std@@QAE@XZ 10044124 f   effectmanager.obj
 0001:00043124       __ehhandler$??0?$vector@PAUsEffectTexture@CEffectManager@@V?$allocator@PAUsEffectTexture@CEffectManager@@@std@@@std@@QAE@XZ 10044124 f   effectmanager.obj
 0001:00043124       __ehhandler$??0?$vector@U_List_position@?$_Hash@V?$_Hmap_traits@PAXPAVCEffectBody@@V?$hash_compare@PAXU?$less@PAX@std@@@stdext@@V?$allocator@U?$pair@QAXPAVCEffectBody@@@std@@@std@@$0A@@stdext@@@stdext@@V?$allocator@U_List_position@?$_Hash@V?$_Hmap_traits@PAXPAVCEffectBody@@V?$hash_compare@PAXU?$less@PAX@std@@@stdext@@V?$allocator@U?$pair@QAXPAVCEffectBody@@@std@@@std@@$0A@@stdext@@@stdext@@@std@@@std@@QAE@ABV?$allocator@U_List_position@?$_Hash@V?$_Hmap_traits@PAXPAVCEffectBody@@V?$hash_compare@PAXU?$less@PAX@std@@@stdext@@V?$allocator@U?$pair@QAXPAVCEffectBody@@@std@@@std@@$0A@@stdext@@@stdext@@@1@@Z 10044124 f   effectmanager.obj
 0001:00043124       __ehhandler$??0?$vector@U_List_position@?$_Hash@V?$_Hmap_traits@KV?$basic_string@DU?$char_traits@D@std@@V?$allocator@D@2@@std@@V?$hash_compare@KU?$less@K@std@@@stdext@@V?$allocator@U?$pair@$$CBKV?$basic_string@DU?$char_traits@D@std@@V?$allocator@D@2@@std@@@std@@@2@$0A@@stdext@@@stdext@@V?$allocator@U_List_position@?$_Hash@V?$_Hmap_traits@KV?$basic_string@DU?$char_traits@D@std@@V?$allocator@D@2@@std@@V?$hash_compare@KU?$less@K@std@@@stdext@@V?$allocator@U?$pair@$$CBKV?$basic_string@DU?$char_traits@D@std@@V?$allocator@D@2@@std@@@std@@@2@$0A@@stdext@@@stdext@@@std@@@std@@QAE@ABV?$allocator@U_List_position@?$_Hash@V?$_Hmap_traits@KV?$basic_string@DU?$char_traits@D@std@@V?$allocator@D@2@@std@@V?$hash_compare@KU?$less@K@std@@@stdext@@V?$allocator@U?$pair@$$CBKV?$basic_string@DU?$char_traits@D@std@@V?$allocator@D@2@@std@@@std@@@2@$0A@@stdext@@@stdext@@@1@@Z 10044124 f   effectmanager.obj
 0001:00043142       __ehhandler$?_Buynode@?$_Tree@V?$_Tmap_traits@JUWzVector@@U?$less@J@std@@V?$allocator@U?$pair@$$CBJUWzVector@@@std@@@3@$0A@@std@@@std@@IAEPAU_Node@?$_Tree_nod@V?$_Tmap_traits@JUWzVector@@U?$less@J@std@@V?$allocator@U?$pair@$$CBJUWzVector@@@std@@@3@$0A@@std@@@2@XZ 10044142 f   effectmanager.obj
 0001:0004315d       __ehhandler$?_Buynode@?$_Tree@V?$_Tmap_traits@JUWzVector@@U?$less@J@std@@V?$allocator@U?$pair@$$CBJUWzVector@@@std@@@3@$0A@@std@@@std@@IAEPAU_Node@?$_Tree_nod@V?$_Tmap_traits@JUWzVector@@U?$less@J@std@@V?$allocator@U?$pair@$$CBJUWzVector@@@std@@@3@$0A@@std@@@2@PAU342@00ABU?$pair@$$CBJUWzVector@@@2@D@Z 1004415d f   effectmanager.obj
 0001:00043178       __ehhandler$?_Buynode@?$_Tree@V?$_Tmap_traits@JMU?$less@J@std@@V?$allocator@U?$pair@$$CBJM@std@@@2@$0A@@std@@@std@@IAEPAU_Node@?$_Tree_nod@V?$_Tmap_traits@JMU?$less@J@std@@V?$allocator@U?$pair@$$CBJM@std@@@2@$0A@@std@@@2@XZ 10044178 f   effectmanager.obj
 0001:00043193       __ehhandler$?_Buynode@?$_Tree@V?$_Tmap_traits@JMU?$less@J@std@@V?$allocator@U?$pair@$$CBJM@std@@@2@$0A@@std@@@std@@IAEPAU_Node@?$_Tree_nod@V?$_Tmap_traits@JMU?$less@J@std@@V?$allocator@U?$pair@$$CBJM@std@@@2@$0A@@std@@@2@PAU342@00ABU?$pair@$$CBJM@2@D@Z 10044193 f   effectmanager.obj
 0001:000431ae       __ehhandler$?_Buynode@?$list@U?$pair@$$CBKPAUSt_BodyCreate@@@std@@V?$allocator@U?$pair@$$CBKPAUSt_BodyCreate@@@std@@@2@@std@@IAEPAU_Node@?$_List_nod@U?$pair@$$CBKPAUSt_BodyCreate@@@std@@V?$allocator@U?$pair@$$CBKPAUSt_BodyCreate@@@std@@@2@@2@XZ 100441ae f   effectmanager.obj
 0001:000431ae       __ehhandler$?_Buynode@?$list@U?$pair@QAXPAVCEffectBody@@@std@@V?$allocator@U?$pair@QAXPAVCEffectBody@@@std@@@2@@std@@IAEPAU_Node@?$_List_nod@U?$pair@QAXPAVCEffectBody@@@std@@V?$allocator@U?$pair@QAXPAVCEffectBody@@@std@@@2@@2@XZ 100441ae f   effectmanager.obj
 0001:000431c9       __ehhandler$?_Buynode@?$list@U?$pair@$$CBKPAUSt_BodyCreate@@@std@@V?$allocator@U?$pair@$$CBKPAUSt_BodyCreate@@@std@@@2@@std@@IAEPAU_Node@?$_List_nod@U?$pair@$$CBKPAUSt_BodyCreate@@@std@@V?$allocator@U?$pair@$$CBKPAUSt_BodyCreate@@@std@@@2@@2@PAU342@0ABU?$pair@$$CBKPAUSt_BodyCreate@@@2@@Z 100441c9 f   effectmanager.obj
 0001:000431c9       __ehhandler$?_Buynode@?$list@U?$pair@QAXPAVCEffectBody@@@std@@V?$allocator@U?$pair@QAXPAVCEffectBody@@@std@@@2@@std@@IAEPAU_Node@?$_List_nod@U?$pair@QAXPAVCEffectBody@@@std@@V?$allocator@U?$pair@QAXPAVCEffectBody@@@std@@@2@@2@PAU342@0ABU?$pair@QAXPAVCEffectBody@@@2@@Z 100441c9 f   effectmanager.obj
 0001:000431e4       __unwindfunclet$?_Incsize@?$list@PAVCEElementBase@@V?$allocator@PAVCEElementBase@@@std@@@std@@IAEXI@Z$0 100441e4 f   effectmanager.obj
 0001:000431e4       __unwindfunclet$?_Incsize@?$list@U?$pair@$$CBKV?$basic_string@DU?$char_traits@D@std@@V?$allocator@D@2@@std@@@std@@V?$allocator@U?$pair@$$CBKV?$basic_string@DU?$char_traits@D@std@@V?$allocator@D@2@@std@@@std@@@2@@std@@IAEXI@Z$0 100441e4 f   effectmanager.obj
 0001:000431e4       __unwindfunclet$?_Incsize@?$list@U?$pair@$$CBKPAUSt_BodyCreate@@@std@@V?$allocator@U?$pair@$$CBKPAUSt_BodyCreate@@@std@@@2@@std@@IAEXI@Z$0 100441e4 f   effectmanager.obj
 0001:000431e4       __unwindfunclet$?_Incsize@?$list@U?$pair@QAXPAVCEffectBody@@@std@@V?$allocator@U?$pair@QAXPAVCEffectBody@@@std@@@2@@std@@IAEXI@Z$0 100441e4 f   effectmanager.obj
 0001:000431e4       __unwindfunclet$?_Incsize@?$list@PAVCEElementSprite@@V?$allocator@PAVCEElementSprite@@@std@@@std@@IAEXI@Z$0 100441e4 f   effectmanager.obj
 0001:000431e4       __unwindfunclet$?_Incsize@?$list@KV?$allocator@K@std@@@std@@IAEXI@Z$0 100441e4 f   effectmanager.obj
 0001:000431ec       __ehhandler$?_Incsize@?$list@U?$pair@QAXPAVCEffectBody@@@std@@V?$allocator@U?$pair@QAXPAVCEffectBody@@@std@@@2@@std@@IAEXI@Z 100441ec f   effectmanager.obj
 0001:000431ec       __ehhandler$?_Incsize@?$list@U?$pair@$$CBKPAUSt_BodyCreate@@@std@@V?$allocator@U?$pair@$$CBKPAUSt_BodyCreate@@@std@@@2@@std@@IAEXI@Z 100441ec f   effectmanager.obj
 0001:000431ec       __ehhandler$?_Incsize@?$list@PAVCEElementBase@@V?$allocator@PAVCEElementBase@@@std@@@std@@IAEXI@Z 100441ec f   effectmanager.obj
 0001:000431ec       __ehhandler$?_Incsize@?$list@U?$pair@$$CBKV?$basic_string@DU?$char_traits@D@std@@V?$allocator@D@2@@std@@@std@@V?$allocator@U?$pair@$$CBKV?$basic_string@DU?$char_traits@D@std@@V?$allocator@D@2@@std@@@std@@@2@@std@@IAEXI@Z 100441ec f   effectmanager.obj
 0001:000431ec       __ehhandler$?_Incsize@?$list@KV?$allocator@K@std@@@std@@IAEXI@Z 100441ec f   effectmanager.obj
 0001:000431ec       __ehhandler$?_Incsize@?$list@PAVCEElementSprite@@V?$allocator@PAVCEElementSprite@@@std@@@std@@IAEXI@Z 100441ec f   effectmanager.obj
 0001:0004320a       __ehhandler$?_Insert_n@?$vector@U_List_position@?$_Hash@V?$_Hmap_traits@PAXPAVCEffectBody@@V?$hash_compare@PAXU?$less@PAX@std@@@stdext@@V?$allocator@U?$pair@QAXPAVCEffectBody@@@std@@@std@@$0A@@stdext@@@stdext@@V?$allocator@U_List_position@?$_Hash@V?$_Hmap_traits@PAXPAVCEffectBody@@V?$hash_compare@PAXU?$less@PAX@std@@@stdext@@V?$allocator@U?$pair@QAXPAVCEffectBody@@@std@@@std@@$0A@@stdext@@@stdext@@@std@@@std@@IAEXV?$_Vector_const_iterator@U_List_position@?$_Hash@V?$_Hmap_traits@PAXPAVCEffectBody@@V?$hash_compare@PAXU?$less@PAX@std@@@stdext@@V?$allocator@U?$pair@QAXPAVCEffectBody@@@std@@@std@@$0A@@stdext@@@stdext@@V?$allocator@U_List_position@?$_Hash@V?$_Hmap_traits@PAXPAVCEffectBody@@V?$hash_compare@PAXU?$less@PAX@std@@@stdext@@V?$allocator@U?$pair@QAXPAVCEffectBody@@@std@@@std@@$0A@@stdext@@@stdext@@@std@@@2@IABU_List_position@?$_Hash@V?$_Hmap_traits@PAXPAVCEffectBody@@V?$hash_compare@PAXU?$less@PAX@std@@@stdext@@V?$allocator@U?$pair@QAXPAVCEffectBody@@@std@@@std@@$0A@@stdext@@@stdext@@@Z 1004420a f   effectmanager.obj
 0001:0004320a       __ehhandler$?_Insert_n@?$vector@USt_EffLODParam@@V?$allocator@USt_EffLODParam@@@std@@@std@@IAEXV?$_Vector_const_iterator@USt_EffLODParam@@V?$allocator@USt_EffLODParam@@@std@@@2@IABUSt_EffLODParam@@@Z 1004420a f   effectmanager.obj
 0001:0004320a       __ehhandler$?_Insert_n@?$vector@USt_AutoCtlParam@@V?$allocator@USt_AutoCtlParam@@@std@@@std@@IAEXV?$_Vector_const_iterator@USt_AutoCtlParam@@V?$allocator@USt_AutoCtlParam@@@std@@@2@IABUSt_AutoCtlParam@@@Z 1004420a f   effectmanager.obj
 0001:0004320a       __ehhandler$?_Insert_n@?$vector@U_List_position@?$_Hash@V?$_Hmap_traits@KPAUSt_BodyCreate@@V?$hash_compare@KU?$less@K@std@@@stdext@@V?$allocator@U?$pair@$$CBKPAUSt_BodyCreate@@@std@@@std@@$0A@@stdext@@@stdext@@V?$allocator@U_List_position@?$_Hash@V?$_Hmap_traits@KPAUSt_BodyCreate@@V?$hash_compare@KU?$less@K@std@@@stdext@@V?$allocator@U?$pair@$$CBKPAUSt_BodyCreate@@@std@@@std@@$0A@@stdext@@@stdext@@@std@@@std@@IAEXV?$_Vector_const_iterator@U_List_position@?$_Hash@V?$_Hmap_traits@KPAUSt_BodyCreate@@V?$hash_compare@KU?$less@K@std@@@stdext@@V?$allocator@U?$pair@$$CBKPAUSt_BodyCreate@@@std@@@std@@$0A@@stdext@@@stdext@@V?$allocator@U_List_position@?$_Hash@V?$_Hmap_traits@KPAUSt_BodyCreate@@V?$hash_compare@KU?$less@K@std@@@stdext@@V?$allocator@U?$pair@$$CBKPAUSt_BodyCreate@@@std@@@std@@$0A@@stdext@@@stdext@@@std@@@2@IABU_List_position@?$_Hash@V?$_Hmap_traits@KPAUSt_BodyCreate@@V?$hash_compare@KU?$less@K@std@@@stdext@@V?$allocator@U?$pair@$$CBKPAUSt_BodyCreate@@@std@@@std@@$0A@@stdext@@@stdext@@@Z 1004420a f   effectmanager.obj
 0001:0004320a       __ehhandler$?_Insert_n@?$vector@U_List_position@?$_Hash@V?$_Hmap_traits@KV?$basic_string@DU?$char_traits@D@std@@V?$allocator@D@2@@std@@V?$hash_compare@KU?$less@K@std@@@stdext@@V?$allocator@U?$pair@$$CBKV?$basic_string@DU?$char_traits@D@std@@V?$allocator@D@2@@std@@@std@@@2@$0A@@stdext@@@stdext@@V?$allocator@U_List_position@?$_Hash@V?$_Hmap_traits@KV?$basic_string@DU?$char_traits@D@std@@V?$allocator@D@2@@std@@V?$hash_compare@KU?$less@K@std@@@stdext@@V?$allocator@U?$pair@$$CBKV?$basic_string@DU?$char_traits@D@std@@V?$allocator@D@2@@std@@@std@@@2@$0A@@stdext@@@stdext@@@std@@@std@@IAEXV?$_Vector_const_iterator@U_List_position@?$_Hash@V?$_Hmap_traits@KV?$basic_string@DU?$char_traits@D@std@@V?$allocator@D@2@@std@@V?$hash_compare@KU?$less@K@std@@@stdext@@V?$allocator@U?$pair@$$CBKV?$basic_string@DU?$char_traits@D@std@@V?$allocator@D@2@@std@@@std@@@2@$0A@@stdext@@@stdext@@V?$allocator@U_List_position@?$_Hash@V?$_Hmap_traits@KV?$basic_string@DU?$char_traits@D@std@@V?$allocator@D@2@@std@@V?$hash_compare@KU?$less@K@std@@@stdext@@V?$allocator@U?$pair@$$CBKV?$basic_string@DU?$char_traits@D@std@@V?$allocator@D@2@@std@@@std@@@2@$0A@@stdext@@@stdext@@@std@@@2@IABU_List_position@?$_Hash@V?$_Hmap_traits@KV?$basic_string@DU?$char_traits@D@std@@V?$allocator@D@2@@std@@V?$hash_compare@KU?$less@K@std@@@stdext@@V?$allocator@U?$pair@$$CBKV?$basic_string@DU?$char_traits@D@std@@V?$allocator@D@2@@std@@@std@@@2@$0A@@stdext@@@stdext@@@Z 1004420a f   effectmanager.obj
 0001:0004320a       __ehhandler$?_Insert_n@?$vector@U_WZNCSPT@WzNaturalCubicSplineDyn@@V?$allocator@U_WZNCSPT@WzNaturalCubicSplineDyn@@@std@@@std@@IAEXV?$_Vector_const_iterator@U_WZNCSPT@WzNaturalCubicSplineDyn@@V?$allocator@U_WZNCSPT@WzNaturalCubicSplineDyn@@@std@@@2@IABU_WZNCSPT@WzNaturalCubicSplineDyn@@@Z 1004420a f   effectmanager.obj
 0001:00043228       __unwindfunclet$??1?$CWzHandleManager@USt_DAFileInfo@@@@UAE@XZ$0 10044228 f   effectmanager.obj
 0001:00043228       __unwindfunclet$??1?$CWzHandleManager@PAVCEffectBody@@@@UAE@XZ$0 10044228 f   effectmanager.obj
 0001:00043233       __unwindfunclet$??1?$CWzHandleManager@PAVCEffectBody@@@@UAE@XZ$1 10044233 f   effectmanager.obj
 0001:00043233       __unwindfunclet$??1?$CWzHandleManager@USt_DAFileInfo@@@@UAE@XZ$1 10044233 f   effectmanager.obj
 0001:0004323e       __ehhandler$??1?$CWzHandleManager@USt_DAFileInfo@@@@UAE@XZ 1004423e f   effectmanager.obj
 0001:0004323e       __ehhandler$??1?$CWzHandleManager@PAVCEffectBody@@@@UAE@XZ 1004423e f   effectmanager.obj
 0001:00043259       __unwindfunclet$??0St_BodyCreate@@QAE@XZ$0 10044259 f   effectmanager.obj
 0001:00043264       __unwindfunclet$??0St_BodyCreate@@QAE@XZ$1 10044264 f   effectmanager.obj
 0001:0004326f       __unwindfunclet$??0St_BodyCreate@@QAE@XZ$2 1004426f f   effectmanager.obj
 0001:0004327a       __unwindfunclet$??0St_BodyCreate@@QAE@XZ$3 1004427a f   effectmanager.obj
 0001:00043285       __ehhandler$??0St_BodyCreate@@QAE@XZ 10044285 f   effectmanager.obj
 0001:000432a0       __unwindfunclet$??1St_BodyCreate@@QAE@XZ$0 100442a0 f   effectmanager.obj
 0001:000432ae       __unwindfunclet$??1St_BodyCreate@@QAE@XZ$1 100442ae f   effectmanager.obj
 0001:000432bc       __unwindfunclet$??1St_BodyCreate@@QAE@XZ$2 100442bc f   effectmanager.obj
 0001:000432ca       __unwindfunclet$??1St_BodyCreate@@QAE@XZ$3 100442ca f   effectmanager.obj
 0001:000432d8       __unwindfunclet$??1St_BodyCreate@@QAE@XZ$5 100442d8 f   effectmanager.obj
 0001:000432e0       __unwindfunclet$??1St_BodyCreate@@QAE@XZ$8 100442e0 f   effectmanager.obj
 0001:000432e8       __unwindfunclet$??1St_BodyCreate@@QAE@XZ$11 100442e8 f   effectmanager.obj
 0001:000432f0       __unwindfunclet$??1St_BodyCreate@@QAE@XZ$14 100442f0 f   effectmanager.obj
 0001:000432fb       __unwindfunclet$??1St_BodyCreate@@QAE@XZ$17 100442fb f   effectmanager.obj
 0001:00043306       __ehhandler$??1St_BodyCreate@@QAE@XZ 10044306 f   effectmanager.obj
 0001:00043324       __ehhandler$??$_Uninit_fill_n@PAUSt_EffLODParam@@IU1@V?$allocator@USt_EffLODParam@@@std@@@std@@YAXPAUSt_EffLODParam@@IABU1@AAV?$allocator@USt_EffLODParam@@@0@U_Nonscalar_ptr_iterator_tag@0@U_Range_checked_iterator_tag@0@@Z 10044324 f   effectmanager.obj
 0001:00043324       __ehhandler$??$_Uninit_fill_n@PAU_List_position@?$_Hash@V?$_Hmap_traits@PAXPAVCEffectBody@@V?$hash_compare@PAXU?$less@PAX@std@@@stdext@@V?$allocator@U?$pair@QAXPAVCEffectBody@@@std@@@std@@$0A@@stdext@@@stdext@@IU123@V?$allocator@U_List_position@?$_Hash@V?$_Hmap_traits@PAXPAVCEffectBody@@V?$hash_compare@PAXU?$less@PAX@std@@@stdext@@V?$allocator@U?$pair@QAXPAVCEffectBody@@@std@@@std@@$0A@@stdext@@@stdext@@@std@@@std@@YAXPAU_List_position@?$_Hash@V?$_Hmap_traits@PAXPAVCEffectBody@@V?$hash_compare@PAXU?$less@PAX@std@@@stdext@@V?$allocator@U?$pair@QAXPAVCEffectBody@@@std@@@std@@$0A@@stdext@@@stdext@@IABU123@AAV?$allocator@U_List_position@?$_Hash@V?$_Hmap_traits@PAXPAVCEffectBody@@V?$hash_compare@PAXU?$less@PAX@std@@@stdext@@V?$allocator@U?$pair@QAXPAVCEffectBody@@@std@@@std@@$0A@@stdext@@@stdext@@@0@U_Nonscalar_ptr_iterator_tag@0@U_Range_checked_iterator_tag@0@@Z 10044324 f   effectmanager.obj
 0001:00043324       __ehhandler$??$_Uninit_fill_n@PAUSt_AutoCtlParam@@IU1@V?$allocator@USt_AutoCtlParam@@@std@@@std@@YAXPAUSt_AutoCtlParam@@IABU1@AAV?$allocator@USt_AutoCtlParam@@@0@U_Nonscalar_ptr_iterator_tag@0@U_Range_checked_iterator_tag@0@@Z 10044324 f   effectmanager.obj
 0001:00043324       __ehhandler$??$_Uninit_fill_n@PAU_List_position@?$_Hash@V?$_Hmap_traits@KPAUSt_BodyCreate@@V?$hash_compare@KU?$less@K@std@@@stdext@@V?$allocator@U?$pair@$$CBKPAUSt_BodyCreate@@@std@@@std@@$0A@@stdext@@@stdext@@IU123@V?$allocator@U_List_position@?$_Hash@V?$_Hmap_traits@KPAUSt_BodyCreate@@V?$hash_compare@KU?$less@K@std@@@stdext@@V?$allocator@U?$pair@$$CBKPAUSt_BodyCreate@@@std@@@std@@$0A@@stdext@@@stdext@@@std@@@std@@YAXPAU_List_position@?$_Hash@V?$_Hmap_traits@KPAUSt_BodyCreate@@V?$hash_compare@KU?$less@K@std@@@stdext@@V?$allocator@U?$pair@$$CBKPAUSt_BodyCreate@@@std@@@std@@$0A@@stdext@@@stdext@@IABU123@AAV?$allocator@U_List_position@?$_Hash@V?$_Hmap_traits@KPAUSt_BodyCreate@@V?$hash_compare@KU?$less@K@std@@@stdext@@V?$allocator@U?$pair@$$CBKPAUSt_BodyCreate@@@std@@@std@@$0A@@stdext@@@stdext@@@0@U_Nonscalar_ptr_iterator_tag@0@U_Range_checked_iterator_tag@0@@Z 10044324 f   effectmanager.obj
 0001:00043324       __ehhandler$??$_Uninit_fill_n@PAU_WZNCSPT@WzNaturalCubicSplineDyn@@IU12@V?$allocator@U_WZNCSPT@WzNaturalCubicSplineDyn@@@std@@@std@@YAXPAU_WZNCSPT@WzNaturalCubicSplineDyn@@IABU12@AAV?$allocator@U_WZNCSPT@WzNaturalCubicSplineDyn@@@0@U_Nonscalar_ptr_iterator_tag@0@U_Range_checked_iterator_tag@0@@Z 10044324 f   effectmanager.obj
 0001:00043324       __ehhandler$??$_Uninit_fill_n@PAU_List_position@?$_Hash@V?$_Hmap_traits@KV?$basic_string@DU?$char_traits@D@std@@V?$allocator@D@2@@std@@V?$hash_compare@KU?$less@K@std@@@stdext@@V?$allocator@U?$pair@$$CBKV?$basic_string@DU?$char_traits@D@std@@V?$allocator@D@2@@std@@@std@@@2@$0A@@stdext@@@stdext@@IU123@V?$allocator@U_List_position@?$_Hash@V?$_Hmap_traits@KV?$basic_string@DU?$char_traits@D@std@@V?$allocator@D@2@@std@@V?$hash_compare@KU?$less@K@std@@@stdext@@V?$allocator@U?$pair@$$CBKV?$basic_string@DU?$char_traits@D@std@@V?$allocator@D@2@@std@@@std@@@2@$0A@@stdext@@@stdext@@@std@@@std@@YAXPAU_List_position@?$_Hash@V?$_Hmap_traits@KV?$basic_string@DU?$char_traits@D@std@@V?$allocator@D@2@@std@@V?$hash_compare@KU?$less@K@std@@@stdext@@V?$allocator@U?$pair@$$CBKV?$basic_string@DU?$char_traits@D@std@@V?$allocator@D@2@@std@@@std@@@2@$0A@@stdext@@@stdext@@IABU123@AAV?$allocator@U_List_position@?$_Hash@V?$_Hmap_traits@KV?$basic_string@DU?$char_traits@D@std@@V?$allocator@D@2@@std@@V?$hash_compare@KU?$less@K@std@@@stdext@@V?$allocator@U?$pair@$$CBKV?$basic_string@DU?$char_traits@D@std@@V?$allocator@D@2@@std@@@std@@@2@$0A@@stdext@@@stdext@@@0@U_Nonscalar_ptr_iterator_tag@0@U_Range_checked_iterator_tag@0@@Z 10044324 f   effectmanager.obj
 0001:0004333f       __ehhandler$??$_Insert@V?$_Const_iterator@$00@?$list@U?$pair@QAXPAVCEffectBody@@@std@@V?$allocator@U?$pair@QAXPAVCEffectBody@@@std@@@2@@std@@@?$list@U?$pair@QAXPAVCEffectBody@@@std@@V?$allocator@U?$pair@QAXPAVCEffectBody@@@std@@@2@@std@@QAEXV?$_Const_iterator@$00@01@00Uforward_iterator_tag@1@@Z 1004433f f   effectmanager.obj
 0001:0004333f       __ehhandler$??$_Insert@V?$_Const_iterator@$00@?$list@U?$pair@$$CBKPAUSt_BodyCreate@@@std@@V?$allocator@U?$pair@$$CBKPAUSt_BodyCreate@@@std@@@2@@std@@@?$list@U?$pair@$$CBKPAUSt_BodyCreate@@@std@@V?$allocator@U?$pair@$$CBKPAUSt_BodyCreate@@@std@@@2@@std@@QAEXV?$_Const_iterator@$00@01@00Uforward_iterator_tag@1@@Z 1004433f f   effectmanager.obj
 0001:0004335d       __ehhandler$??$_Insert@V?$_Const_iterator@$00@?$list@KV?$allocator@K@std@@@std@@@?$list@KV?$allocator@K@std@@@std@@QAEXV?$_Const_iterator@$00@01@00Uforward_iterator_tag@1@@Z 1004435d f   effectmanager.obj
 0001:0004337b       __ehhandler$??$_Uninit_copy@PAUSt_AutoCtlParam@@PAU1@V?$allocator@USt_AutoCtlParam@@@std@@@std@@YAPAUSt_AutoCtlParam@@PAU1@00AAV?$allocator@USt_AutoCtlParam@@@0@U_Nonscalar_ptr_iterator_tag@0@U_Range_checked_iterator_tag@0@@Z 1004437b f   effectmanager.obj
 0001:0004337b       __ehhandler$??$_Uninit_copy@PAUSt_EffLODParam@@PAU1@V?$allocator@USt_EffLODParam@@@std@@@std@@YAPAUSt_EffLODParam@@PAU1@00AAV?$allocator@USt_EffLODParam@@@0@U_Nonscalar_ptr_iterator_tag@0@U_Range_checked_iterator_tag@0@@Z 1004437b f   effectmanager.obj
 0001:0004337b       __ehhandler$??$_Uninit_copy@PAU_List_position@?$_Hash@V?$_Hmap_traits@KV?$basic_string@DU?$char_traits@D@std@@V?$allocator@D@2@@std@@V?$hash_compare@KU?$less@K@std@@@stdext@@V?$allocator@U?$pair@$$CBKV?$basic_string@DU?$char_traits@D@std@@V?$allocator@D@2@@std@@@std@@@2@$0A@@stdext@@@stdext@@PAU123@V?$allocator@U_List_position@?$_Hash@V?$_Hmap_traits@KV?$basic_string@DU?$char_traits@D@std@@V?$allocator@D@2@@std@@V?$hash_compare@KU?$less@K@std@@@stdext@@V?$allocator@U?$pair@$$CBKV?$basic_string@DU?$char_traits@D@std@@V?$allocator@D@2@@std@@@std@@@2@$0A@@stdext@@@stdext@@@std@@@std@@YAPAU_List_position@?$_Hash@V?$_Hmap_traits@KV?$basic_string@DU?$char_traits@D@std@@V?$allocator@D@2@@std@@V?$hash_compare@KU?$less@K@std@@@stdext@@V?$allocator@U?$pair@$$CBKV?$basic_string@DU?$char_traits@D@std@@V?$allocator@D@2@@std@@@std@@@2@$0A@@stdext@@@stdext@@PAU123@00AAV?$allocator@U_List_position@?$_Hash@V?$_Hmap_traits@KV?$basic_string@DU?$char_traits@D@std@@V?$allocator@D@2@@std@@V?$hash_compare@KU?$less@K@std@@@stdext@@V?$allocator@U?$pair@$$CBKV?$basic_string@DU?$char_traits@D@std@@V?$allocator@D@2@@std@@@std@@@2@$0A@@stdext@@@stdext@@@0@U_Nonscalar_ptr_iterator_tag@0@U_Range_checked_iterator_tag@0@@Z 1004437b f   effectmanager.obj
 0001:0004337b       __ehhandler$??$_Uninit_copy@PAU_List_position@?$_Hash@V?$_Hmap_traits@KPAUSt_BodyCreate@@V?$hash_compare@KU?$less@K@std@@@stdext@@V?$allocator@U?$pair@$$CBKPAUSt_BodyCreate@@@std@@@std@@$0A@@stdext@@@stdext@@PAU123@V?$allocator@U_List_position@?$_Hash@V?$_Hmap_traits@KPAUSt_BodyCreate@@V?$hash_compare@KU?$less@K@std@@@stdext@@V?$allocator@U?$pair@$$CBKPAUSt_BodyCreate@@@std@@@std@@$0A@@stdext@@@stdext@@@std@@@std@@YAPAU_List_position@?$_Hash@V?$_Hmap_traits@KPAUSt_BodyCreate@@V?$hash_compare@KU?$less@K@std@@@stdext@@V?$allocator@U?$pair@$$CBKPAUSt_BodyCreate@@@std@@@std@@$0A@@stdext@@@stdext@@PAU123@00AAV?$allocator@U_List_position@?$_Hash@V?$_Hmap_traits@KPAUSt_BodyCreate@@V?$hash_compare@KU?$less@K@std@@@stdext@@V?$allocator@U?$pair@$$CBKPAUSt_BodyCreate@@@std@@@std@@$0A@@stdext@@@stdext@@@0@U_Nonscalar_ptr_iterator_tag@0@U_Range_checked_iterator_tag@0@@Z 1004437b f   effectmanager.obj
 0001:0004337b       __ehhandler$??$_Uninit_copy@PAU_List_position@?$_Hash@V?$_Hmap_traits@PAXPAVCEffectBody@@V?$hash_compare@PAXU?$less@PAX@std@@@stdext@@V?$allocator@U?$pair@QAXPAVCEffectBody@@@std@@@std@@$0A@@stdext@@@stdext@@PAU123@V?$allocator@U_List_position@?$_Hash@V?$_Hmap_traits@PAXPAVCEffectBody@@V?$hash_compare@PAXU?$less@PAX@std@@@stdext@@V?$allocator@U?$pair@QAXPAVCEffectBody@@@std@@@std@@$0A@@stdext@@@stdext@@@std@@@std@@YAPAU_List_position@?$_Hash@V?$_Hmap_traits@PAXPAVCEffectBody@@V?$hash_compare@PAXU?$less@PAX@std@@@stdext@@V?$allocator@U?$pair@QAXPAVCEffectBody@@@std@@@std@@$0A@@stdext@@@stdext@@PAU123@00AAV?$allocator@U_List_position@?$_Hash@V?$_Hmap_traits@PAXPAVCEffectBody@@V?$hash_compare@PAXU?$less@PAX@std@@@stdext@@V?$allocator@U?$pair@QAXPAVCEffectBody@@@std@@@std@@$0A@@stdext@@@stdext@@@0@U_Nonscalar_ptr_iterator_tag@0@U_Range_checked_iterator_tag@0@@Z 1004437b f   effectmanager.obj
 0001:0004337b       __ehhandler$??$_Uninit_copy@PAU_WZNCSPT@WzNaturalCubicSplineDyn@@PAU12@V?$allocator@U_WZNCSPT@WzNaturalCubicSplineDyn@@@std@@@std@@YAPAU_WZNCSPT@WzNaturalCubicSplineDyn@@PAU12@00AAV?$allocator@U_WZNCSPT@WzNaturalCubicSplineDyn@@@0@U_Nonscalar_ptr_iterator_tag@0@U_Range_checked_iterator_tag@0@@Z 1004437b f   effectmanager.obj
 0001:00043396       __unwindfunclet$?LoadEffectFromFile@CEffectManager@@QAE_NPBD0W4EENUM_LOAD_TYPE@@H@Z$0 10044396 f   effectmanager_load.obj
 0001:000433a1       __ehhandler$?LoadEffectFromFile@CEffectManager@@QAE_NPBD0W4EENUM_LOAD_TYPE@@H@Z 100443a1 f   effectmanager_load.obj
 0001:000433c9       __unwindfunclet$?UnLoadEffectFromFile@CEffectManager@@QAEXPBD@Z$0 100443c9 f   effectmanager_load.obj
 0001:000433d1       __ehhandler$?UnLoadEffectFromFile@CEffectManager@@QAEXPBD@Z 100443d1 f   effectmanager_load.obj
 0001:000433ef       __unwindfunclet$??$AllocNew@USt_BodyCreate@@@CMemoryPool@@YAPAUSt_BodyCreate@@XZ$0 100443ef f   effectmanager_load.obj
 0001:000433f9       __ehhandler$??$AllocNew@USt_BodyCreate@@@CMemoryPool@@YAPAUSt_BodyCreate@@XZ 100443f9 f   effectmanager_load.obj
 0001:00043414       __unwindfunclet$??$AllocNew@USt_Create_Info@@@CMemoryPool@@YAPAUSt_Create_Info@@XZ$0 10044414 f   effectmanager_load.obj
 0001:0004341e       __ehhandler$??$AllocNew@USt_Create_Info@@@CMemoryPool@@YAPAUSt_Create_Info@@XZ 1004441e f   effectmanager_load.obj
 0001:00043439       __unwindfunclet$??$AllocNew@USt_Move_Info@@@CMemoryPool@@YAPAUSt_Move_Info@@XZ$0 10044439 f   effectmanager_load.obj
 0001:00043443       __ehhandler$??$AllocNew@USt_Move_Info@@@CMemoryPool@@YAPAUSt_Move_Info@@XZ 10044443 f   effectmanager_load.obj
 0001:0004345e       __unwindfunclet$??$AllocNew@USt_Change_Info@@@CMemoryPool@@YAPAUSt_Change_Info@@XZ$0 1004445e f   effectmanager_load.obj
 0001:00043468       __ehhandler$??$AllocNew@USt_Change_Info@@@CMemoryPool@@YAPAUSt_Change_Info@@XZ 10044468 f   effectmanager_load.obj
 0001:00043483       __unwindfunclet$??$AllocNew@USt_Visual_Info@@@CMemoryPool@@YAPAUSt_Visual_Info@@XZ$0 10044483 f   effectmanager_load.obj
 0001:0004348d       __ehhandler$??$AllocNew@USt_Visual_Info@@@CMemoryPool@@YAPAUSt_Visual_Info@@XZ 1004448d f   effectmanager_load.obj
 0001:000434a8       __unwindfunclet$?_Insert@?$_Tree@V?$_Tmap_traits@JMU?$less@J@std@@V?$allocator@U?$pair@$$CBJM@std@@@2@$0A@@std@@@std@@IAE?AViterator@12@_NPAU_Node@?$_Tree_nod@V?$_Tmap_traits@JMU?$less@J@std@@V?$allocator@U?$pair@$$CBJM@std@@@2@$0A@@std@@@2@ABU?$pair@$$CBJM@2@@Z$0 100444a8 f   effectmanager_load.obj
 0001:000434a8       __unwindfunclet$?_Insert@?$_Tree@V?$_Tmap_traits@JUWzVector@@U?$less@J@std@@V?$allocator@U?$pair@$$CBJUWzVector@@@std@@@3@$0A@@std@@@std@@IAE?AViterator@12@_NPAU_Node@?$_Tree_nod@V?$_Tmap_traits@JUWzVector@@U?$less@J@std@@V?$allocator@U?$pair@$$CBJUWzVector@@@std@@@3@$0A@@std@@@2@ABU?$pair@$$CBJUWzVector@@@2@@Z$0 100444a8 f   effectmanager_load.obj
 0001:000434b0       __ehhandler$?_Insert@?$_Tree@V?$_Tmap_traits@JUWzVector@@U?$less@J@std@@V?$allocator@U?$pair@$$CBJUWzVector@@@std@@@3@$0A@@std@@@std@@IAE?AViterator@12@_NPAU_Node@?$_Tree_nod@V?$_Tmap_traits@JUWzVector@@U?$less@J@std@@V?$allocator@U?$pair@$$CBJUWzVector@@@std@@@3@$0A@@std@@@2@ABU?$pair@$$CBJUWzVector@@@2@@Z 100444b0 f   effectmanager_load.obj
 0001:000434b0       __ehhandler$?_Insert@?$_Tree@V?$_Tmap_traits@JMU?$less@J@std@@V?$allocator@U?$pair@$$CBJM@std@@@2@$0A@@std@@@std@@IAE?AViterator@12@_NPAU_Node@?$_Tree_nod@V?$_Tmap_traits@JMU?$less@J@std@@V?$allocator@U?$pair@$$CBJM@std@@@2@$0A@@std@@@2@ABU?$pair@$$CBJM@2@@Z 100444b0 f   effectmanager_load.obj
 0001:000434ce       __unwindfunclet$?CreateFromFile@CLoadBaseManager@@QAEHPBDPAVCDiscAccess@@W4EENUM_LOAD_TYPE@@@Z$0 100444ce f   loadmanager.obj
 0001:000434d9       __unwindfunclet$?CreateFromFile@CLoadBaseManager@@QAEHPBDPAVCDiscAccess@@W4EENUM_LOAD_TYPE@@@Z$1 100444d9 f   loadmanager.obj
 0001:000434e4       __unwindfunclet$?CreateFromFile@CLoadBaseManager@@QAEHPBDPAVCDiscAccess@@W4EENUM_LOAD_TYPE@@@Z$2 100444e4 f   loadmanager.obj
 0001:000434ef       __ehhandler$?CreateFromFile@CLoadBaseManager@@QAEHPBDPAVCDiscAccess@@W4EENUM_LOAD_TYPE@@@Z 100444ef f   loadmanager.obj
 0001:00043517       __unwindfunclet$?Merge@CLoadBaseManager@@QAEXABV1@@Z$0 10044517 f   loadmanager.obj
 0001:0004351f       __ehhandler$?Merge@CLoadBaseManager@@QAEXABV1@@Z 1004451f f   loadmanager.obj
 0001:0004353d       __unwindfunclet$??1?$_Hash@V?$_Hmap_traits@KV?$basic_string@DU?$char_traits@D@std@@V?$allocator@D@2@@std@@V?$hash_compare@KU?$less@K@std@@@stdext@@V?$allocator@U?$pair@$$CBKV?$basic_string@DU?$char_traits@D@std@@V?$allocator@D@2@@std@@@std@@@2@$0A@@stdext@@@stdext@@QAE@XZ$0 1004453d f   loadmanager.obj
 0001:00043545       __unwindfunclet$??1?$_Hash@V?$_Hmap_traits@KV?$basic_string@DU?$char_traits@D@std@@V?$allocator@D@2@@std@@V?$hash_compare@KU?$less@K@std@@@stdext@@V?$allocator@U?$pair@$$CBKV?$basic_string@DU?$char_traits@D@std@@V?$allocator@D@2@@std@@@std@@@2@$0A@@stdext@@@stdext@@QAE@XZ$1 10044545 f   loadmanager.obj
 0001:00043550       __unwindfunclet$??1?$_Hash@V?$_Hmap_traits@KV?$basic_string@DU?$char_traits@D@std@@V?$allocator@D@2@@std@@V?$hash_compare@KU?$less@K@std@@@stdext@@V?$allocator@U?$pair@$$CBKV?$basic_string@DU?$char_traits@D@std@@V?$allocator@D@2@@std@@@std@@@2@$0A@@stdext@@@stdext@@QAE@XZ$3 10044550 f   loadmanager.obj
 0001:00043558       __unwindfunclet$??1?$_Hash@V?$_Hmap_traits@KV?$basic_string@DU?$char_traits@D@std@@V?$allocator@D@2@@std@@V?$hash_compare@KU?$less@K@std@@@stdext@@V?$allocator@U?$pair@$$CBKV?$basic_string@DU?$char_traits@D@std@@V?$allocator@D@2@@std@@@std@@@2@$0A@@stdext@@@stdext@@QAE@XZ$6 10044558 f   loadmanager.obj
 0001:00043560       __ehhandler$??1?$_Hash@V?$_Hmap_traits@KV?$basic_string@DU?$char_traits@D@std@@V?$allocator@D@2@@std@@V?$hash_compare@KU?$less@K@std@@@stdext@@V?$allocator@U?$pair@$$CBKV?$basic_string@DU?$char_traits@D@std@@V?$allocator@D@2@@std@@@std@@@2@$0A@@stdext@@@stdext@@QAE@XZ 10044560 f   loadmanager.obj
 0001:0004357b       __unwindfunclet$??0?$_Hash@V?$_Hmap_traits@KV?$basic_string@DU?$char_traits@D@std@@V?$allocator@D@2@@std@@V?$hash_compare@KU?$less@K@std@@@stdext@@V?$allocator@U?$pair@$$CBKV?$basic_string@DU?$char_traits@D@std@@V?$allocator@D@2@@std@@@std@@@2@$0A@@stdext@@@stdext@@QAE@ABV?$hash_compare@KU?$less@K@std@@@1@ABV?$allocator@U?$pair@$$CBKV?$basic_string@DU?$char_traits@D@std@@V?$allocator@D@2@@std@@@std@@@std@@@Z$0 1004457b f   loadmanager.obj
 0001:00043586       __unwindfunclet$??0?$_Hash@V?$_Hmap_traits@KV?$basic_string@DU?$char_traits@D@std@@V?$allocator@D@2@@std@@V?$hash_compare@KU?$less@K@std@@@stdext@@V?$allocator@U?$pair@$$CBKV?$basic_string@DU?$char_traits@D@std@@V?$allocator@D@2@@std@@@std@@@2@$0A@@stdext@@@stdext@@QAE@ABV?$hash_compare@KU?$less@K@std@@@1@ABV?$allocator@U?$pair@$$CBKV?$basic_string@DU?$char_traits@D@std@@V?$allocator@D@2@@std@@@std@@@std@@@Z$1 10044586 f   loadmanager.obj
 0001:00043594       __unwindfunclet$??0?$_Hash@V?$_Hmap_traits@KV?$basic_string@DU?$char_traits@D@std@@V?$allocator@D@2@@std@@V?$hash_compare@KU?$less@K@std@@@stdext@@V?$allocator@U?$pair@$$CBKV?$basic_string@DU?$char_traits@D@std@@V?$allocator@D@2@@std@@@std@@@2@$0A@@stdext@@@stdext@@QAE@ABV?$hash_compare@KU?$less@K@std@@@1@ABV?$allocator@U?$pair@$$CBKV?$basic_string@DU?$char_traits@D@std@@V?$allocator@D@2@@std@@@std@@@std@@@Z$2 10044594 f   loadmanager.obj
 0001:000435a2       __ehhandler$??0?$_Hash@V?$_Hmap_traits@KV?$basic_string@DU?$char_traits@D@std@@V?$allocator@D@2@@std@@V?$hash_compare@KU?$less@K@std@@@stdext@@V?$allocator@U?$pair@$$CBKV?$basic_string@DU?$char_traits@D@std@@V?$allocator@D@2@@std@@@std@@@2@$0A@@stdext@@@stdext@@QAE@ABV?$hash_compare@KU?$less@K@std@@@1@ABV?$allocator@U?$pair@$$CBKV?$basic_string@DU?$char_traits@D@std@@V?$allocator@D@2@@std@@@std@@@std@@@Z 100445a2 f   loadmanager.obj
 0001:000435c0       __unwindfunclet$??1?$vector@PAUsEffectTexture@CEffectManager@@V?$allocator@PAUsEffectTexture@CEffectManager@@@std@@@std@@QAE@XZ$0 100445c0 f   loadmanager.obj
 0001:000435c0       __unwindfunclet$??1?$list@U?$pair@$$CBKV?$basic_string@DU?$char_traits@D@std@@V?$allocator@D@2@@std@@@std@@V?$allocator@U?$pair@$$CBKV?$basic_string@DU?$char_traits@D@std@@V?$allocator@D@2@@std@@@std@@@2@@std@@QAE@XZ$0 100445c0 f   loadmanager.obj
 0001:000435c0       __unwindfunclet$??1?$vector@PAXV?$allocator@PAX@std@@@std@@QAE@XZ$0 100445c0 f   loadmanager.obj
 0001:000435c8       __ehhandler$??1?$list@U?$pair@$$CBKV?$basic_string@DU?$char_traits@D@std@@V?$allocator@D@2@@std@@@std@@V?$allocator@U?$pair@$$CBKV?$basic_string@DU?$char_traits@D@std@@V?$allocator@D@2@@std@@@std@@@2@@std@@QAE@XZ 100445c8 f   loadmanager.obj
 0001:000435c8       __ehhandler$??1?$vector@PAXV?$allocator@PAX@std@@@std@@QAE@XZ 100445c8 f   loadmanager.obj
 0001:000435c8       __ehhandler$??1?$vector@PAUsEffectTexture@CEffectManager@@V?$allocator@PAUsEffectTexture@CEffectManager@@@std@@@std@@QAE@XZ 100445c8 f   loadmanager.obj
 0001:000435e3       __ehhandler$?_Buynode@?$list@U?$pair@$$CBKV?$basic_string@DU?$char_traits@D@std@@V?$allocator@D@2@@std@@@std@@V?$allocator@U?$pair@$$CBKV?$basic_string@DU?$char_traits@D@std@@V?$allocator@D@2@@std@@@std@@@2@@std@@IAEPAU_Node@?$_List_nod@U?$pair@$$CBKV?$basic_string@DU?$char_traits@D@std@@V?$allocator@D@2@@std@@@std@@V?$allocator@U?$pair@$$CBKV?$basic_string@DU?$char_traits@D@std@@V?$allocator@D@2@@std@@@std@@@2@@2@XZ 100445e3 f   loadmanager.obj
 0001:000435fe       __ehhandler$?_Buynode@?$list@U?$pair@$$CBKV?$basic_string@DU?$char_traits@D@std@@V?$allocator@D@2@@std@@@std@@V?$allocator@U?$pair@$$CBKV?$basic_string@DU?$char_traits@D@std@@V?$allocator@D@2@@std@@@std@@@2@@std@@IAEPAU_Node@?$_List_nod@U?$pair@$$CBKV?$basic_string@DU?$char_traits@D@std@@V?$allocator@D@2@@std@@@std@@V?$allocator@U?$pair@$$CBKV?$basic_string@DU?$char_traits@D@std@@V?$allocator@D@2@@std@@@std@@@2@@2@PAU342@0ABU?$pair@$$CBKV?$basic_string@DU?$char_traits@D@std@@V?$allocator@D@2@@std@@@2@@Z 100445fe f   loadmanager.obj
 0001:00043619       __unwindfunclet$??$_Construct@U?$pair@$$CBKV?$basic_string@DU?$char_traits@D@std@@V?$allocator@D@2@@std@@@std@@U12@@std@@YAXPAU?$pair@$$CBKV?$basic_string@DU?$char_traits@D@std@@V?$allocator@D@2@@std@@@0@ABU10@@Z$0 10044619 f   loadmanager.obj
 0001:00043627       __ehhandler$??$_Construct@U?$pair@$$CBKV?$basic_string@DU?$char_traits@D@std@@V?$allocator@D@2@@std@@@std@@U12@@std@@YAXPAU?$pair@$$CBKV?$basic_string@DU?$char_traits@D@std@@V?$allocator@D@2@@std@@@0@ABU10@@Z 10044627 f   loadmanager.obj
 0001:00043642       __ehhandler$??$_Insert@V?$_Const_iterator@$00@?$list@U?$pair@$$CBKV?$basic_string@DU?$char_traits@D@std@@V?$allocator@D@2@@std@@@std@@V?$allocator@U?$pair@$$CBKV?$basic_string@DU?$char_traits@D@std@@V?$allocator@D@2@@std@@@std@@@2@@std@@@?$list@U?$pair@$$CBKV?$basic_string@DU?$char_traits@D@std@@V?$allocator@D@2@@std@@@std@@V?$allocator@U?$pair@$$CBKV?$basic_string@DU?$char_traits@D@std@@V?$allocator@D@2@@std@@@std@@@2@@std@@QAEXV?$_Const_iterator@$00@01@00Uforward_iterator_tag@1@@Z 10044642 f   loadmanager.obj
 0001:00043660       __unwindfunclet$?Create@?$CWzMemoryBand@VCEElementChain@@@@QAE_NH@Z$2 10044660 f   memorymanager.obj
 0001:00043660       __unwindfunclet$?Create@?$CWzMemoryBand@VCEElementMesh@@@@QAE_NH@Z$2 10044660 f   memorymanager.obj
 0001:00043660       __unwindfunclet$?Create@?$CWzMemoryBand@VCEElementFlatChain@@@@QAE_NH@Z$2 10044660 f   memorymanager.obj
 0001:00043660       __unwindfunclet$?Create@?$CWzMemoryBand@VCEElementDecal@@@@QAE_NH@Z$2 10044660 f   memorymanager.obj
 0001:00043660       __unwindfunclet$?Create@?$CWzMemoryBand@VCEffectBody@@@@QAE_NH@Z$2 10044660 f   memorymanager.obj
 0001:00043660       __unwindfunclet$?Create@?$CWzMemoryBand@VCEElementSprite@@@@QAE_NH@Z$2 10044660 f   memorymanager.obj
 0001:00043660       __unwindfunclet$?Create@?$CWzMemoryBand@VCEElementWeather@@@@QAE_NH@Z$2 10044660 f   memorymanager.obj
 0001:0004366a       __ehhandler$?Create@?$CWzMemoryBand@VCEElementDecal@@@@QAE_NH@Z 1004466a f   memorymanager.obj
 0001:0004366a       __ehhandler$?Create@?$CWzMemoryBand@VCEElementFlatChain@@@@QAE_NH@Z 1004466a f   memorymanager.obj
 0001:0004366a       __ehhandler$?Create@?$CWzMemoryBand@VCEffectBody@@@@QAE_NH@Z 1004466a f   memorymanager.obj
 0001:0004366a       __ehhandler$?Create@?$CWzMemoryBand@VCEElementChain@@@@QAE_NH@Z 1004466a f   memorymanager.obj
 0001:0004366a       __ehhandler$?Create@?$CWzMemoryBand@VCEElementMesh@@@@QAE_NH@Z 1004466a f   memorymanager.obj
 0001:0004366a       __ehhandler$?Create@?$CWzMemoryBand@VCEElementSprite@@@@QAE_NH@Z 1004466a f   memorymanager.obj
 0001:0004366a       __ehhandler$?Create@?$CWzMemoryBand@VCEElementWeather@@@@QAE_NH@Z 1004466a f   memorymanager.obj
 0001:00043685       __unwindfunclet$?GetTextureInfo@CManagerTexture@@QAEPAUSt_TextureContainer@@PAX@Z$0 10044685 f   eelementsprite.obj
 0001:0004368d       __ehhandler$?GetTextureInfo@CManagerTexture@@QAEPAUSt_TextureContainer@@PAX@Z 1004468d f   eelementsprite.obj
 0001:000436a8       __unwindfunclet$??0CEElementWeather@@QAE@XZ$0 100446a8 f   eelementweather.obj
 0001:000436b0       __unwindfunclet$??0CEElementWeather@@QAE@XZ$1 100446b0 f   eelementweather.obj
 0001:000436be       __ehhandler$??0CEElementWeather@@QAE@XZ 100446be f   eelementweather.obj
 0001:000436d9       __unwindfunclet$??1CEElementWeather@@UAE@XZ$0 100446d9 f   eelementweather.obj
 0001:000436e1       __unwindfunclet$??1CEElementWeather@@UAE@XZ$1 100446e1 f   eelementweather.obj
 0001:000436ef       __unwindfunclet$??1CEElementWeather@@UAE@XZ$3 100446ef f   eelementweather.obj
 0001:000436f7       __ehhandler$??1CEElementWeather@@UAE@XZ 100446f7 f   eelementweather.obj
 0001:00043712       __ehhandler$?_Buynode@?$list@PAVCEElementSprite@@V?$allocator@PAVCEElementSprite@@@std@@@std@@IAEPAU_Node@?$_List_nod@PAVCEElementSprite@@V?$allocator@PAVCEElementSprite@@@std@@@2@PAU342@0ABQAVCEElementSprite@@@Z 10044712 f   eelementweather.obj
 0001:00043712       __ehhandler$?_Buynode@?$list@PAVCEElementBase@@V?$allocator@PAVCEElementBase@@@std@@@std@@IAEPAU_Node@?$_List_nod@PAVCEElementBase@@V?$allocator@PAVCEElementBase@@@std@@@2@PAU342@0ABQAVCEElementBase@@@Z 10044712 f   eelementweather.obj
 0001:00043712       __ehhandler$?_Buynode@?$list@KV?$allocator@K@std@@@std@@IAEPAU_Node@?$_List_nod@KV?$allocator@K@std@@@2@PAU342@0ABK@Z 10044712 f   eelementweather.obj
 0001:0004372d       __unwindfunclet$??0CEffectBody@@QAE@XZ$0 1004472d f   effectbody.obj
 0001:00043738       __unwindfunclet$??0CEffectBody@@QAE@XZ$1 10044738 f   effectbody.obj
 0001:00043749       __ehhandler$??0CEffectBody@@QAE@XZ 10044749 f   effectbody.obj
 0001:00043767       __unwindfunclet$??1CEffectBody@@UAE@XZ$0 10044767 f   effectbody.obj
 0001:0004376f       __unwindfunclet$??1CEffectBody@@UAE@XZ$1 1004476f f   effectbody.obj
 0001:0004377d       __unwindfunclet$??1CEffectBody@@UAE@XZ$3 1004477d f   effectbody.obj
 0001:00043785       __unwindfunclet$??1CEffectBody@@UAE@XZ$6 10044785 f   effectbody.obj
 0001:0004378d       __ehhandler$??1CEffectBody@@UAE@XZ 1004478d f   effectbody.obj
 0001:000437a8       __ehhandler$?_Insert_n@?$vector@PAUsEffectTexture@CEffectManager@@V?$allocator@PAUsEffectTexture@CEffectManager@@@std@@@std@@IAEXV?$_Vector_const_iterator@PAUsEffectTexture@CEffectManager@@V?$allocator@PAUsEffectTexture@CEffectManager@@@std@@@2@IABQAUsEffectTexture@CEffectManager@@@Z 100447a8 f   effectbody.obj
 0001:000437a8       __ehhandler$?_Insert_n@?$vector@PAUSt_SoundInfo@@V?$allocator@PAUSt_SoundInfo@@@std@@@std@@IAEXV?$_Vector_const_iterator@PAUSt_SoundInfo@@V?$allocator@PAUSt_SoundInfo@@@std@@@2@IABQAUSt_SoundInfo@@@Z 100447a8 f   effectbody.obj
 0001:000437a8       __ehhandler$?_Insert_n@?$vector@PAXV?$allocator@PAX@std@@@std@@IAEXV?$_Vector_const_iterator@PAXV?$allocator@PAX@std@@@2@IABQAX@Z 100447a8 f   effectbody.obj
 0001:000437c6       __unwindfunclet$?_Xlen@?$vector@U_WZNCSPT@WzNaturalCubicSplineDyn@@V?$allocator@U_WZNCSPT@WzNaturalCubicSplineDyn@@@std@@@std@@KAXXZ$0 100447c6 f   effectbody.obj
 0001:000437c6       __unwindfunclet$?_Xlen@?$vector@U_List_position@?$_Hash@V?$_Hmap_traits@KPAUSt_BodyCreate@@V?$hash_compare@KU?$less@K@std@@@stdext@@V?$allocator@U?$pair@$$CBKPAUSt_BodyCreate@@@std@@@std@@$0A@@stdext@@@stdext@@V?$allocator@U_List_position@?$_Hash@V?$_Hmap_traits@KPAUSt_BodyCreate@@V?$hash_compare@KU?$less@K@std@@@stdext@@V?$allocator@U?$pair@$$CBKPAUSt_BodyCreate@@@std@@@std@@$0A@@stdext@@@stdext@@@std@@@std@@KAXXZ$0 100447c6 f   effectbody.obj
 0001:000437c6       __unwindfunclet$?_Xlen@?$vector@USt_EffLODParam@@V?$allocator@USt_EffLODParam@@@std@@@std@@KAXXZ$0 100447c6 f   effectbody.obj
 0001:000437c6       __unwindfunclet$?_Xlen@?$vector@U_List_position@?$_Hash@V?$_Hmap_traits@PAXPAVCEffectBody@@V?$hash_compare@PAXU?$less@PAX@std@@@stdext@@V?$allocator@U?$pair@QAXPAVCEffectBody@@@std@@@std@@$0A@@stdext@@@stdext@@V?$allocator@U_List_position@?$_Hash@V?$_Hmap_traits@PAXPAVCEffectBody@@V?$hash_compare@PAXU?$less@PAX@std@@@stdext@@V?$allocator@U?$pair@QAXPAVCEffectBody@@@std@@@std@@$0A@@stdext@@@stdext@@@std@@@std@@KAXXZ$0 100447c6 f   effectbody.obj
 0001:000437c6       __unwindfunclet$?_Xlen@?$vector@USt_AutoCtlParam@@V?$allocator@USt_AutoCtlParam@@@std@@@std@@KAXXZ$0 100447c6 f   effectbody.obj
 0001:000437c6       __unwindfunclet$?_Xlen@?$vector@U_List_position@?$_Hash@V?$_Hmap_traits@KV?$basic_string@DU?$char_traits@D@std@@V?$allocator@D@2@@std@@V?$hash_compare@KU?$less@K@std@@@stdext@@V?$allocator@U?$pair@$$CBKV?$basic_string@DU?$char_traits@D@std@@V?$allocator@D@2@@std@@@std@@@2@$0A@@stdext@@@stdext@@V?$allocator@U_List_position@?$_Hash@V?$_Hmap_traits@KV?$basic_string@DU?$char_traits@D@std@@V?$allocator@D@2@@std@@V?$hash_compare@KU?$less@K@std@@@stdext@@V?$allocator@U?$pair@$$CBKV?$basic_string@DU?$char_traits@D@std@@V?$allocator@D@2@@std@@@std@@@2@$0A@@stdext@@@stdext@@@std@@@std@@KAXXZ$0 100447c6 f   effectbody.obj
 0001:000437c6       __unwindfunclet$?_Xlen@?$vector@PAUsEffectTexture@CEffectManager@@V?$allocator@PAUsEffectTexture@CEffectManager@@@std@@@std@@KAXXZ$0 100447c6 f   effectbody.obj
 0001:000437c6       __unwindfunclet$?_Xlen@?$vector@PAXV?$allocator@PAX@std@@@std@@KAXXZ$0 100447c6 f   effectbody.obj
 0001:000437c6       __unwindfunclet$?_Xlen@?$vector@PAUSt_SoundInfo@@V?$allocator@PAUSt_SoundInfo@@@std@@@std@@KAXXZ$0 100447c6 f   effectbody.obj
 0001:000437ce       __ehhandler$?_Xlen@?$vector@U_WZNCSPT@WzNaturalCubicSplineDyn@@V?$allocator@U_WZNCSPT@WzNaturalCubicSplineDyn@@@std@@@std@@KAXXZ 100447ce f   effectbody.obj
 0001:000437ce       __ehhandler$?_Xlen@?$vector@USt_EffLODParam@@V?$allocator@USt_EffLODParam@@@std@@@std@@KAXXZ 100447ce f   effectbody.obj
 0001:000437ce       __ehhandler$?_Xlen@?$vector@PAUsEffectTexture@CEffectManager@@V?$allocator@PAUsEffectTexture@CEffectManager@@@std@@@std@@KAXXZ 100447ce f   effectbody.obj
 0001:000437ce       __ehhandler$?_Xlen@?$vector@U_List_position@?$_Hash@V?$_Hmap_traits@PAXPAVCEffectBody@@V?$hash_compare@PAXU?$less@PAX@std@@@stdext@@V?$allocator@U?$pair@QAXPAVCEffectBody@@@std@@@std@@$0A@@stdext@@@stdext@@V?$allocator@U_List_position@?$_Hash@V?$_Hmap_traits@PAXPAVCEffectBody@@V?$hash_compare@PAXU?$less@PAX@std@@@stdext@@V?$allocator@U?$pair@QAXPAVCEffectBody@@@std@@@std@@$0A@@stdext@@@stdext@@@std@@@std@@KAXXZ 100447ce f   effectbody.obj
 0001:000437ce       __ehhandler$?_Xlen@?$vector@U_List_position@?$_Hash@V?$_Hmap_traits@KPAUSt_BodyCreate@@V?$hash_compare@KU?$less@K@std@@@stdext@@V?$allocator@U?$pair@$$CBKPAUSt_BodyCreate@@@std@@@std@@$0A@@stdext@@@stdext@@V?$allocator@U_List_position@?$_Hash@V?$_Hmap_traits@KPAUSt_BodyCreate@@V?$hash_compare@KU?$less@K@std@@@stdext@@V?$allocator@U?$pair@$$CBKPAUSt_BodyCreate@@@std@@@std@@$0A@@stdext@@@stdext@@@std@@@std@@KAXXZ 100447ce f   effectbody.obj
 0001:000437ce       __ehhandler$?_Xlen@?$vector@USt_AutoCtlParam@@V?$allocator@USt_AutoCtlParam@@@std@@@std@@KAXXZ 100447ce f   effectbody.obj
 0001:000437ce       __ehhandler$?_Xlen@?$vector@PAXV?$allocator@PAX@std@@@std@@KAXXZ 100447ce f   effectbody.obj
 0001:000437ce       __ehhandler$?_Xlen@?$vector@U_List_position@?$_Hash@V?$_Hmap_traits@KV?$basic_string@DU?$char_traits@D@std@@V?$allocator@D@2@@std@@V?$hash_compare@KU?$less@K@std@@@stdext@@V?$allocator@U?$pair@$$CBKV?$basic_string@DU?$char_traits@D@std@@V?$allocator@D@2@@std@@@std@@@2@$0A@@stdext@@@stdext@@V?$allocator@U_List_position@?$_Hash@V?$_Hmap_traits@KV?$basic_string@DU?$char_traits@D@std@@V?$allocator@D@2@@std@@V?$hash_compare@KU?$less@K@std@@@stdext@@V?$allocator@U?$pair@$$CBKV?$basic_string@DU?$char_traits@D@std@@V?$allocator@D@2@@std@@@std@@@2@$0A@@stdext@@@stdext@@@std@@@std@@KAXXZ 100447ce f   effectbody.obj
 0001:000437ce       __ehhandler$?_Xlen@?$vector@PAUSt_SoundInfo@@V?$allocator@PAUSt_SoundInfo@@@std@@@std@@KAXXZ 100447ce f   effectbody.obj
 0001:000437ec       __unwindfunclet$?_Xlen@_String_base@std@@SAXXZ$0 100447ec f   libcpmt:string.obj
 0001:000437ec       __unwindfunclet$?_Xran@_String_base@std@@SAXXZ$0 100447ec f   libcpmt:string.obj
 0001:000437f4       __ehhandler$?_Xlen@_String_base@std@@SAXXZ 100447f4 f   libcpmt:string.obj
 0001:000437f4       __ehhandler$?_Xran@_String_base@std@@SAXXZ 100447f4 f   libcpmt:string.obj
 0001:0004380f       __ehhandler$?CallUnexpected@@YAXPBU_s_ESTypeList@@@Z 1004480f f   LIBCMT:frame.obj
 0001:0004382a       __unwindfunclet$?Initialize@WzLogSystem@WzLog@@QAEXXZ$0 1004482a f   ProgramCommonLibForEngine_p:wzlogsystem.obj
 0001:00043837       __ehhandler$?Initialize@WzLogSystem@WzLog@@QAEXXZ 10044837 f   ProgramCommonLibForEngine_p:wzlogsystem.obj
 0001:0004385f       __unwindfunclet$?InitializeWzLogSystem@@YAXXZ$0 1004485f f   ProgramCommonLibForEngine_p:wzlogsystem.obj
 0001:00043869       __ehhandler$?InitializeWzLogSystem@@YAXXZ 10044869 f   ProgramCommonLibForEngine_p:wzlogsystem.obj
 0001:00043884       __unwindfunclet$??0CDiscAccess@@QAE@XZ$0 10044884 f   ProgramCommonLibForEngine_p:discaccess.obj
 0001:00043892       __unwindfunclet$??0CDiscAccess@@QAE@XZ$1 10044892 f   ProgramCommonLibForEngine_p:discaccess.obj
 0001:000438a0       __ehhandler$??0CDiscAccess@@QAE@XZ 100448a0 f   ProgramCommonLibForEngine_p:discaccess.obj
 0001:000438bb       __unwindfunclet$??1CDiscAccess@@QAE@XZ$0 100448bb f   ProgramCommonLibForEngine_p:discaccess.obj
 0001:000438c9       __unwindfunclet$??1CDiscAccess@@QAE@XZ$1 100448c9 f   ProgramCommonLibForEngine_p:discaccess.obj
 0001:000438d7       __ehhandler$??1CDiscAccess@@QAE@XZ 100448d7 f   ProgramCommonLibForEngine_p:discaccess.obj
 0001:000438f2       __unwindfunclet$?OpenDisc_Hard@CDiscAccess@@QAEHKPBD@Z$0 100448f2 f   ProgramCommonLibForEngine_p:discaccess.obj
 0001:000438fa       __ehhandler$?OpenDisc_Hard@CDiscAccess@@QAEHKPBD@Z 100448fa f   ProgramCommonLibForEngine_p:discaccess.obj
 0001:00043915       __unwindfunclet$?OpenDisc_Packer@CDiscAccess@@QAEHKPBD0W4ENUM_OPEN_PACKER_TYPE@@@Z$0 10044915 f   ProgramCommonLibForEngine_p:discaccess.obj
 0001:0004391d       __unwindfunclet$?OpenDisc_Packer@CDiscAccess@@QAEHKPBD0W4ENUM_OPEN_PACKER_TYPE@@@Z$1 1004491d f   ProgramCommonLibForEngine_p:discaccess.obj
 0001:00043927       __ehhandler$?OpenDisc_Packer@CDiscAccess@@QAEHKPBD0W4ENUM_OPEN_PACKER_TYPE@@@Z 10044927 f   ProgramCommonLibForEngine_p:discaccess.obj
 0001:00043942       __unwindfunclet$?CloseDisc@CDiscAccess@@QAEXK@Z$0 10044942 f   ProgramCommonLibForEngine_p:discaccess.obj
 0001:0004394a       __ehhandler$?CloseDisc@CDiscAccess@@QAEXK@Z 1004494a f   ProgramCommonLibForEngine_p:discaccess.obj
 0001:00043965       __unwindfunclet$?SetActiveDisc@CDiscAccess@@QAEHK@Z$0 10044965 f   ProgramCommonLibForEngine_p:discaccess.obj
 0001:0004396d       __ehhandler$?SetActiveDisc@CDiscAccess@@QAEHK@Z 1004496d f   ProgramCommonLibForEngine_p:discaccess.obj
 0001:00043988       __unwindfunclet$?OpenFile@CDiscAccess@@QAEPAXKPBDKKW4ENUM_OPEN_DISPOSITION@@@Z$0 10044988 f   ProgramCommonLibForEngine_p:discaccess.obj
 0001:00043990       __ehhandler$?OpenFile@CDiscAccess@@QAEPAXKPBDKKW4ENUM_OPEN_DISPOSITION@@@Z 10044990 f   ProgramCommonLibForEngine_p:discaccess.obj
 0001:000439b8       __unwindfunclet$?CloseFile@CDiscAccess@@QAEHPAX@Z$0 100449b8 f   ProgramCommonLibForEngine_p:discaccess.obj
 0001:000439c0       __ehhandler$?CloseFile@CDiscAccess@@QAEHPAX@Z 100449c0 f   ProgramCommonLibForEngine_p:discaccess.obj
 0001:000439db       __unwindfunclet$?SeekFile@CDiscAccess@@QAEKPAXJW4ENUM_SEEK_ORIGIN@@@Z$0 100449db f   ProgramCommonLibForEngine_p:discaccess.obj
 0001:000439e3       __ehhandler$?SeekFile@CDiscAccess@@QAEKPAXJW4ENUM_SEEK_ORIGIN@@@Z 100449e3 f   ProgramCommonLibForEngine_p:discaccess.obj
 0001:000439fe       __unwindfunclet$?ReadFile@CDiscAccess@@QAEKPAX0K@Z$0 100449fe f   ProgramCommonLibForEngine_p:discaccess.obj
 0001:00043a06       __ehhandler$?ReadFile@CDiscAccess@@QAEKPAX0K@Z 10044a06 f   ProgramCommonLibForEngine_p:discaccess.obj
 0001:00043a21       __unwindfunclet$?WriteFile@CDiscAccess@@QAEKPAXPBXK@Z$0 10044a21 f   ProgramCommonLibForEngine_p:discaccess.obj
 0001:00043a29       __ehhandler$?WriteFile@CDiscAccess@@QAEKPAXPBXK@Z 10044a29 f   ProgramCommonLibForEngine_p:discaccess.obj
 0001:00043a44       __unwindfunclet$?FileExists@CDiscAccess@@QAEHKPBD@Z$0 10044a44 f   ProgramCommonLibForEngine_p:discaccess.obj
 0001:00043a4c       __ehhandler$?FileExists@CDiscAccess@@QAEHKPBD@Z 10044a4c f   ProgramCommonLibForEngine_p:discaccess.obj
 0001:00043a74       __unwindfunclet$?GetFileSize@CDiscAccess@@QAEKPAX@Z$0 10044a74 f   ProgramCommonLibForEngine_p:discaccess.obj
 0001:00043a7c       __ehhandler$?GetFileSize@CDiscAccess@@QAEKPAX@Z 10044a7c f   ProgramCommonLibForEngine_p:discaccess.obj
 0001:00043a97       __unwindfunclet$?GetFileInformationByHandle@CDiscAccess@@QAEHPAXPAUSt_FileInformation@@@Z$0 10044a97 f   ProgramCommonLibForEngine_p:discaccess.obj
 0001:00043a9f       __ehhandler$?GetFileInformationByHandle@CDiscAccess@@QAEHPAXPAUSt_FileInformation@@@Z 10044a9f f   ProgramCommonLibForEngine_p:discaccess.obj
 0001:00043ac7       __unwindfunclet$?CopyFileA@CDiscAccess@@QAEHKPBD0@Z$0 10044ac7 f   ProgramCommonLibForEngine_p:discaccess.obj
 0001:00043acf       __ehhandler$?CopyFileA@CDiscAccess@@QAEHKPBD0@Z 10044acf f   ProgramCommonLibForEngine_p:discaccess.obj
 0001:00043af7       __unwindfunclet$?DeleteFileA@CDiscAccess@@QAEHKPBD@Z$0 10044af7 f   ProgramCommonLibForEngine_p:discaccess.obj
 0001:00043aff       __ehhandler$?DeleteFileA@CDiscAccess@@QAEHKPBD@Z 10044aff f   ProgramCommonLibForEngine_p:discaccess.obj
 0001:00043b27       __unwindfunclet$?CreateDirectoryA@CDiscAccess@@QAEHKPBD@Z$0 10044b27 f   ProgramCommonLibForEngine_p:discaccess.obj
 0001:00043b2f       __ehhandler$?CreateDirectoryA@CDiscAccess@@QAEHKPBD@Z 10044b2f f   ProgramCommonLibForEngine_p:discaccess.obj
 0001:00043b57       __unwindfunclet$?RemoveDirectoryA@CDiscAccess@@QAEHKPBD@Z$0 10044b57 f   ProgramCommonLibForEngine_p:discaccess.obj
 0001:00043b5f       __ehhandler$?RemoveDirectoryA@CDiscAccess@@QAEHKPBD@Z 10044b5f f   ProgramCommonLibForEngine_p:discaccess.obj
 0001:00043b87       __unwindfunclet$??0?$CWzHandleManager@PAVCEffectBody@@@@QAE@XZ$0 10044b87 f   ProgramCommonLibForEngine_p:discaccess.obj
 0001:00043b87       __unwindfunclet$??0?$CWzHandleManager@USt_DAFileInfo@@@@QAE@XZ$0 10044b87 f   ProgramCommonLibForEngine_p:discaccess.obj
 0001:00043b92       __unwindfunclet$??0?$CWzHandleManager@PAVCEffectBody@@@@QAE@XZ$1 10044b92 f   ProgramCommonLibForEngine_p:discaccess.obj
 0001:00043b92       __unwindfunclet$??0?$CWzHandleManager@USt_DAFileInfo@@@@QAE@XZ$1 10044b92 f   ProgramCommonLibForEngine_p:discaccess.obj
 0001:00043b9d       __unwindfunclet$??0?$CWzHandleManager@PAVCEffectBody@@@@QAE@XZ$2 10044b9d f   ProgramCommonLibForEngine_p:discaccess.obj
 0001:00043b9d       __unwindfunclet$??0?$CWzHandleManager@USt_DAFileInfo@@@@QAE@XZ$2 10044b9d f   ProgramCommonLibForEngine_p:discaccess.obj
 0001:00043ba8       __ehhandler$??0?$CWzHandleManager@USt_DAFileInfo@@@@QAE@XZ 10044ba8 f   ProgramCommonLibForEngine_p:discaccess.obj
 0001:00043ba8       __ehhandler$??0?$CWzHandleManager@PAVCEffectBody@@@@QAE@XZ 10044ba8 f   ProgramCommonLibForEngine_p:discaccess.obj
 0001:00043bc3       __unwindfunclet$?CreateDiscAccess@CScriptRead@@AAEXXZ$0 10044bc3 f   ProgramCommonLibForEngine_p:scriptread.obj
 0001:00043bcd       __ehhandler$?CreateDiscAccess@CScriptRead@@AAEXXZ 10044bcd f   ProgramCommonLibForEngine_p:scriptread.obj
 0001:00043be8       __unwindfunclet$??1WzNaturalCubicSplineDyn@@QAE@XZ$0 10044be8 f   Common_p:wznaturalcubicsplinedyn.obj
 0001:00043bf3       __unwindfunclet$??1WzNaturalCubicSplineDyn@@QAE@XZ$1 10044bf3 f   Common_p:wznaturalcubicsplinedyn.obj
 0001:00043bfb       __ehhandler$??1WzNaturalCubicSplineDyn@@QAE@XZ 10044bfb f   Common_p:wznaturalcubicsplinedyn.obj
 0001:00043c20       ??__Eg_effDbgInfo@@YAXXZ   10044c20 f   effectmanager.obj
 0001:00043c36       ??__Eg_cSplineX@@YAXXZ     10044c36 f   eelementflatchain.obj
 0001:00043c50       ??__Eg_cSplineY@@YAXXZ     10044c50 f   eelementflatchain.obj
 0001:00043c6a       ??__Eg_cSplineZ@@YAXXZ     10044c6a f   eelementflatchain.obj
 0001:00043c84       ??__Eg_cSpline2X@@YAXXZ    10044c84 f   eelementflatchain.obj
 0001:00043c9e       ??__Eg_cSpline2Y@@YAXXZ    10044c9e f   eelementflatchain.obj
 0001:00043cb8       ??__Eg_cSpline2Z@@YAXXZ    10044cb8 f   eelementflatchain.obj
 0001:00043ce0       ??__Eautofree@@YAXXZ       10044ce0 f   wzFilePacker_static:wzFilePacker.obj
 0001:00043cf0       ??__Fg_cSplineX@@YAXXZ     10044cf0 f   eelementflatchain.obj
 0001:00043cff       ??__Fg_cSplineY@@YAXXZ     10044cff f   eelementflatchain.obj
 0001:00043d0e       ??__Fg_cSplineZ@@YAXXZ     10044d0e f   eelementflatchain.obj
 0001:00043d1d       ??__Fg_cSpline2X@@YAXXZ    10044d1d f   eelementflatchain.obj
 0001:00043d2c       ??__Fg_cSpline2Y@@YAXXZ    10044d2c f   eelementflatchain.obj
 0001:00043d3b       ??__Fg_cSpline2Z@@YAXXZ    10044d3b f   eelementflatchain.obj
 0001:00043d4a       ??__Fnomem@?5???2@YAPAXI@Z@YAXXZ 10044d4a f   LIBCMT:new.obj
 0001:00043d60       ??__Fautofree@@YAXXZ       10044d60 f   wzFilePacker_static:wzFilePacker.obj

 Exports

  ordinal    name

        1    ?AddAutoLvlCtlParam@CEffectManager@@QAEXHH@Z (public: void __thiscall CEffectManager::AddAutoLvlCtlParam(int,int))
        2    ?AddAutoRateCtlParam@CEffectManager@@QAEXHH@Z (public: void __thiscall CEffectManager::AddAutoRateCtlParam(int,int))
        3    ?AddEffectInfo@CEffectManager@@QAE_NK@Z (public: bool __thiscall CEffectManager::AddEffectInfo(unsigned long))
        4    ?AddEffectLODParam@CEffectManager@@QAEXMH@Z (public: void __thiscall CEffectManager::AddEffectLODParam(float,int))
        5    ?ClearAutoLvlCtlParams@CEffectManager@@QAEXXZ (public: void __thiscall CEffectManager::ClearAutoLvlCtlParams(void))
        6    ?ClearAutoRateCtlParams@CEffectManager@@QAEXXZ (public: void __thiscall CEffectManager::ClearAutoRateCtlParams(void))
        7    ?ClearEffectLODParams@CEffectManager@@QAEXXZ (public: void __thiscall CEffectManager::ClearEffectLODParams(void))
        8    ?ClearSoundInfos@CEffectManager@@QAEXXZ (public: void __thiscall CEffectManager::ClearSoundInfos(void))
        9    ?Create@CEffectManager@@QAE_NPAVCDrawBase@@PAVCWorldBase@@@Z (public: bool __thiscall CEffectManager::Create(class CDrawBase *,class CWorldBase *))
       10    ?CreateEffect@CEffectManager@@QAEPAXKABUWzVector@@00H@Z (public: void * __thiscall CEffectManager::CreateEffect(unsigned long,struct WzVector const &,struct WzVector const &,struct WzVector const &,int))
       11    ?CreateEffect@CEffectManager@@QAEPAXKABUWzVector@@0H@Z (public: void * __thiscall CEffectManager::CreateEffect(unsigned long,struct WzVector const &,struct WzVector const &,int))
       12    ?CreateEffect@CEffectManager@@QAEPAXKABUWzVector@@H@Z (public: void * __thiscall CEffectManager::CreateEffect(unsigned long,struct WzVector const &,int))
       13    ?CreateSelectedElements@CEffectManager@@QAEPAXKABUWzVector@@PAV?$list@HV?$allocator@H@std@@@std@@@Z (public: void * __thiscall CEffectManager::CreateSelectedElements(unsigned long,struct WzVector const &,class std::list<int,class std::allocator<int> > *))
       14    ?DeleteEleInfo@CEffectManager@@QAEXPAUSt_Ele_Node@@@Z (public: void __thiscall CEffectManager::DeleteEleInfo(struct St_Ele_Node *))
       15    ?Destroy@CEffectManager@@QAEXXZ (public: void __thiscall CEffectManager::Destroy(void))
       16    ?DestroyAllEffect@CEffectManager@@QAEXXZ (public: void __thiscall CEffectManager::DestroyAllEffect(void))
       17    ?GetEffectBodyMap@CEffectManager@@QAEAAV?$hash_map@PAXPAVCEffectBody@@V?$hash_compare@PAXU?$less@PAX@std@@@stdext@@V?$allocator@U?$pair@QAXPAVCEffectBody@@@std@@@std@@@stdext@@XZ (public: class stdext::hash_map<void *,class CEffectBody *,class stdext::hash_compare<void *,struct std::less<void *> >,class std::allocator<struct std::pair<void * const,class CEffectBody *> > > & __thiscall CEffectManager::GetEffectBodyMap(void))
       18    ?GetEffectInfo@CEffectManager@@QAEPAUSt_BodyCreate@@K@Z (public: struct St_BodyCreate * __thiscall CEffectManager::GetEffectInfo(unsigned long))
       19    ?GetEffectPtrHandle@CEffectManager@@QAEPAVCEffectBody@@PAX@Z (public: class CEffectBody * __thiscall CEffectManager::GetEffectPtrHandle(void *))
       20    ?IsRenderEffect@CEffectManager@@QAE_NXZ (public: bool __thiscall CEffectManager::IsRenderEffect(void))
       21    ?Load@CEffectManager@@QAEPAUSt_BodyCreate@@PAXK@Z (public: struct St_BodyCreate * __thiscall CEffectManager::Load(void *,unsigned long))
       22    ?Load@CEffectManager@@QAEPAUSt_BodyCreate@@PBDK@Z (public: struct St_BodyCreate * __thiscall CEffectManager::Load(char const *,unsigned long))
       23    ?LoadEffectFromFile@CEffectManager@@QAE_NPBD0W4EENUM_LOAD_TYPE@@H@Z (public: bool __thiscall CEffectManager::LoadEffectFromFile(char const *,char const *,enum EENUM_LOAD_TYPE,int))
       24    ?LoadEleInfo@CEffectManager@@QAEPAUSt_Ele_Node@@PAX@Z (public: struct St_Ele_Node * __thiscall CEffectManager::LoadEleInfo(void *))
       25    ?LoadMeshFiles@CEffectManager@@QAE_NPBD0W4EENUM_LOAD_TYPE@@@Z (public: bool __thiscall CEffectManager::LoadMeshFiles(char const *,char const *,enum EENUM_LOAD_TYPE))
       26    ?LoadTextureFiles@CEffectManager@@QAE_NPBD0W4EENUM_LOAD_TYPE@@@Z (public: bool __thiscall CEffectManager::LoadTextureFiles(char const *,char const *,enum EENUM_LOAD_TYPE))
       27    ?Move@CEffectManager@@QAEXK@Z (public: void __thiscall CEffectManager::Move(unsigned long))
       28    ?RegisterEffectInfo@CEffectManager@@QAEXPBUSt_BodyCreate@@@Z (public: void __thiscall CEffectManager::RegisterEffectInfo(struct St_BodyCreate const *))
       29    ?ReleaseAllEffectInfo@CEffectManager@@QAEXXZ (public: void __thiscall CEffectManager::ReleaseAllEffectInfo(void))
       30    ?ReleaseAtEffectInfo@CEffectManager@@QAEXK@Z (public: void __thiscall CEffectManager::ReleaseAtEffectInfo(unsigned long))
       31    ?ReleaseEffectTexture@CEffectManager@@QAEXXZ (public: void __thiscall CEffectManager::ReleaseEffectTexture(void))
       32    ?RemoveEffectPtr@CEffectManager@@QAEXPAX@Z (public: void __thiscall CEffectManager::RemoveEffectPtr(void *))
       33    ?Render@CEffectManager@@QAEXXZ (public: void __thiscall CEffectManager::Render(void))
       34    ?Save@CEffectManager@@QAE_NPAXK@Z (public: bool __thiscall CEffectManager::Save(void *,unsigned long))
       35    ?Save@CEffectManager@@QAE_NPBDK@Z (public: bool __thiscall CEffectManager::Save(char const *,unsigned long))
       36    ?SaveEleInfo@CEffectManager@@QAEXPAXPAUSt_Ele_Node@@@Z (public: void __thiscall CEffectManager::SaveEleInfo(void *,struct St_Ele_Node *))
       37    ?SetAllElementTargetPos@CEffectBody@@QAEXABUWzVector@@@Z (public: void __thiscall CEffectBody::SetAllElementTargetPos(struct WzVector const &))
       38    ?SetLifeInfo@CEElementFlatChain@@QAEXKK@Z (public: void __thiscall CEElementFlatChain::SetLifeInfo(unsigned long,unsigned long))
       39    ?SetRenderEffect@CEffectManager@@QAEX_N@Z (public: void __thiscall CEffectManager::SetRenderEffect(bool))
       40    ?SetTailNum@CEElementFlatChain@@QAEXH@Z (public: void __thiscall CEElementFlatChain::SetTailNum(int))
       41    ?ShrinkMemoryPool@CEffectManager@@QAEXXZ (public: void __thiscall CEffectManager::ShrinkMemoryPool(void))
       42    ?UnLoadEffectFromFile@CEffectManager@@QAEXPBD@Z (public: void __thiscall CEffectManager::UnLoadEffectFromFile(char const *))
       43    ?g_effDbgInfo@@3USt_EffDbgInfo@@A (struct St_EffDbgInfo g_effDbgInfo)
       44    ?wvRot@?1??CreateEffect@CEffectManager@@QAEPAXKABUWzVector@@0H@Z@4U3@A (struct WzVector `public: void * __thiscall CEffectManager::CreateEffect(unsigned long,struct WzVector const &,struct WzVector const &,int)'::`2'::wvRot)
       45    ?wvRot@?1??CreateEffect@CEffectManager@@QAEPAXKABUWzVector@@H@Z@4U3@A (struct WzVector `public: void * __thiscall CEffectManager::CreateEffect(unsigned long,struct WzVector const &,int)'::`2'::wvRot)
       46    ?wvScale@?1??CreateEffect@CEffectManager@@QAEPAXKABUWzVector@@H@Z@4U3@A (struct WzVector `public: void * __thiscall CEffectManager::CreateEffect(unsigned long,struct WzVector const &,int)'::`2'::wvScale)
       47    _Func_ContactEffect
               exported name: Func_ContactEffect
